
================================================================================

Section Cross References

    NAND_DevConfig.obj(i.NFI_GPIO_Setting) refers to gpio.obj(i.GPIO_ReturnMode) for GPIO_ReturnMode
    NAND_DevConfig.obj(.data) refers to nand_mtd_fdm50.obj(i.single_Page_Read) for single_Page_Read
    NAND_DevConfig.obj(.data) refers to nand_mtd_fdm50.obj(i.single_Page_Read) for single_Page_Read
    NAND_DevConfig.obj(.data) refers to nand_mtd_fdm50.obj(i.single_Page_Read) for single_Page_Read
    NAND_DevConfig.obj(.data) refers to nand_mtd_fdm50.obj(i.single_Page_Read) for single_Page_Read
    NAND_DevConfig.obj(.data) refers to nand_mtd_fdm50.obj(i.single_Page_Read) for single_Page_Read
    bl_BOOTARM.obj(STACK_POOL_INTSRAM) refers (Special) to bl_Cache.obj(EXT_BOOTLOADER_CODE) for CacheInit
    bl_BOOTARM.obj(STACK_POOL_INTSRAM) refers (Special) to bl_Main.obj(EXT_BOOTLOADER_CODE) for FactoryProcedure
    bl_BOOTARM.obj(STACK_POOL_INTSRAM) refers (Special) to bl_Main.obj(INTERNCODE) for BootAndHandOver
    bl_BOOTARM.obj(DUMMY_POOL) refers (Special) to bl_Cache.obj(EXT_BOOTLOADER_CODE) for CacheInit
    bl_BOOTARM.obj(DUMMY_POOL) refers (Special) to bl_Main.obj(EXT_BOOTLOADER_CODE) for FactoryProcedure
    bl_BOOTARM.obj(DUMMY_POOL) refers (Special) to bl_Main.obj(INTERNCODE) for BootAndHandOver
    bl_BOOTARM.obj(C$$code) refers to bl_BOOTARM.obj(STACK_POOL_INTSRAM) for SPV_Stack_Pool
    bl_BOOTARM.obj(C$$code) refers to bl_BOOTARM.obj(DUMMY_POOL) for DUMMY_END
    bl_BOOTARM.obj(C$$code) refers to bl_Main.obj(i.INT_Version_Check) for INT_Version_Check
    bl_BOOTARM.obj(C$$code) refers to bl_Init.obj(i.Init_DTLB) for Init_DTLB
    bl_BOOTARM.obj(C$$code) refers to bl_regioninit.obj(RegionInit) for INT_InitEMIInitCode
    bl_BOOTARM.obj(C$$code) refers to bl_Init.obj(EMIINITCODE) for SetPLLEMI
    bl_BOOTARM.obj(C$$code) refers to custom_emi.obj(i.custom_InitDRAM) for custom_InitDRAM
    bl_BOOTARM.obj(C$$code) refers to bl_ImageLoader.obj(i.PreserveExtBootloaderHeader) for PreserveExtBootloaderHeader
    bl_BOOTARM.obj(C$$code) refers to bl_Init.obj(i.GenerateRandomSeed) for GenerateRandomSeed
    bl_BOOTARM.obj(C$$code) refers to bl_Init.obj(i.Init) for Init
    bl_BOOTARM.obj(C$$code) refers to bl_ImageLoader.obj(i.LoadExtBootloader) for LoadExtBootloader
    bl_BOOTARM.obj(C$$code) refers to bl_Main.obj(i.VerifyExtBootloader) for VerifyExtBootloader
    bl_BOOTARM.obj(C$$code) refers to bl_Main.obj(EXT_BOOTLOADER_CODE) for ExtBootloader
    bl_BOOTARM.obj(C$$code) refers (Special) to bl_Cache.obj(EXT_BOOTLOADER_CODE) for CacheInit
    bl_BOOTARM.obj(C$$code) refers (Special) to bl_Main.obj(EXT_BOOTLOADER_CODE) for FactoryProcedure
    bl_BOOTARM.obj(C$$code) refers (Special) to bl_Main.obj(INTERNCODE) for BootAndHandOver
    bl_BOOTARM.obj(SHARECODE) refers (Special) to bl_Cache.obj(EXT_BOOTLOADER_CODE) for CacheInit
    bl_BOOTARM.obj(SHARECODE) refers (Special) to bl_Main.obj(EXT_BOOTLOADER_CODE) for FactoryProcedure
    bl_BOOTARM.obj(SHARECODE) refers (Special) to bl_Main.obj(INTERNCODE) for BootAndHandOver
    bl_BOOTARM.obj(INTERNCODE) refers (Special) to bl_Cache.obj(EXT_BOOTLOADER_CODE) for CacheInit
    bl_BOOTARM.obj(INTERNCODE) refers (Special) to bl_Main.obj(EXT_BOOTLOADER_CODE) for FactoryProcedure
    bl_BOOTARM.obj(INTERNCODE) refers (Special) to bl_Main.obj(INTERNCODE) for BootAndHandOver
    bl_Cache.obj(EXT_BOOTLOADER_CODE) refers to cache.obj(INTERNCODE) for CodeCacheClearAllSetting
    bl_Cache.obj(EXT_BOOTLOADER_CODE) refers to cache.obj(INTERNCODE) for MPUClearAllSetting
    bl_Cache.obj(EXT_BOOTLOADER_CODE) refers to cache.obj(i.CodeCacheGetChannel) for CodeCacheGetChannel
    bl_Cache.obj(EXT_BOOTLOADER_CODE) refers to cache.obj(INTERNCODE) for CodeCacheSetting
    bl_Cache.obj(EXT_BOOTLOADER_CODE) refers to cache.obj(INTERNCODE) for CodeCacheConfig
    bl_DBGPRINT.obj(i.itof) refers to rtsdiv10.o(.text) for __rt_sdiv10
    bl_DBGPRINT.obj(i.itof) refers to bl_DBGPRINT.obj(.bss) for .bss$2
    bl_DBGPRINT.obj(i.dbg_print) refers to llcmpge.o(.text) for _ll_cmpge
    bl_DBGPRINT.obj(i.dbg_print) refers to llneg.o(.text) for _ll_neg
    bl_DBGPRINT.obj(i.dbg_print) refers to dfltll_clz.o(x$fpl$dfltll) for _ll_sto_d
    bl_DBGPRINT.obj(i.dbg_print) refers to dgeqf.o(x$fpl$dgeqf) for _dcmpge
    bl_DBGPRINT.obj(i.dbg_print) refers to bl_DBGPRINT.obj(i.itoa) for itoa
    bl_DBGPRINT.obj(i.dbg_print) refers to llsubls.o(.text) for _ll_subls
    bl_DBGPRINT.obj(i.dbg_print) refers to llmullu.o(.text) for _ll_mullu
    bl_DBGPRINT.obj(i.dbg_print) refers to bl_DBGPRINT.obj(i.itof) for itof
    bl_DBGPRINT.obj(i.dbg_print) refers to bl_UART.obj(i.PutUARTByte) for PutUARTByte
    bl_DBGPRINT.obj(i.dbg_print) refers to bl_DBGPRINT.obj(.bss) for .bss$2
    bl_DBGPRINT.obj(i.itoa) refers to rt_sdiv.o(.text) for __rt_sdiv
    bl_DBGPRINT.obj(i.itoa) refers to bl_DBGPRINT.obj(.bss) for .bss$2
    bl_DBGPRINT.obj(i.itoa) refers to bl_DBGPRINT.obj(.constdata) for .constdata$1
    bl_Init.obj(i.WaitFor32KStable) refers to l1_interface.obj(i.HW_TDMA_Start) for HW_TDMA_Start
    bl_Init.obj(i.WaitFor32KStable) refers to l1_interface.obj(i.HW_wait_32k_start) for HW_wait_32k_start
    bl_Init.obj(EMIINITCODE) refers to bl_Init.obj(i.WacthDogRestart) for WacthDogRestart
    bl_Init.obj(EMIINITCODE) refers to bl_Init.obj(EMIINITCODE) for INT_SetPLL
    bl_Init.obj(EMIINITCODE) refers to custom_emi.obj(EMIINITCODE) for custom_setEMI
    bl_Init.obj(EMIINITCODE) refers to custom_emi.obj(EMIINITCODE) for custom_setAdvEMI
    bl_Init.obj(EMIINITCODE) refers to bl_Main.obj(HEAD_BL) for g_ExtBootloaderInfo
    bl_Init.obj(i.CheckPoint) refers to bl_Init.obj(i.startGPTTImer3) for startGPTTImer3
    bl_Init.obj(i.CheckPoint) refers to bl_Init.obj(.data) for .data$0
    bl_Init.obj(i.Init) refers to bl_Init.obj(i.WacthDogRestart) for WacthDogRestart
    bl_Init.obj(i.Init) refers to bl_Init.obj(i.WaitFor32KStable) for WaitFor32KStable
    bl_Init.obj(i.Init) refers to bl_UART.obj(i.uart_init) for uart_init
    bl_Init.obj(i.Init) refers to bl_Init.obj(i.DriverInit) for DriverInit
    bl_Init.obj(i.Init) refers to bl_DBGPRINT.obj(i.dbg_print) for dbg_print
    bl_Init.obj(i.Init) refers to bl_Main.obj(HEAD_BL) for g_ExtBootloaderInfo
    bl_Init.obj(i.Init) refers to bl_Main.obj(.bss) for g_randomSeed
    bl_Init.obj(i.Init) refers to bl_Init.obj(.constdata) for .constdata$1
    bl_Init.obj(EXT_BOOTLOADER_CODE) refers to gpio.obj(i.GPIO_ModeSetup) for GPIO_ModeSetup
    bl_Init.obj(EXT_BOOTLOADER_CODE) refers to gpio.obj(i.GPIO_InitIO) for GPIO_InitIO
    bl_Init.obj(EXT_BOOTLOADER_CODE) refers to gpio.obj(i.GPIO_PullenSetup) for GPIO_PullenSetup
    bl_Init.obj(EXT_BOOTLOADER_CODE) refers to gpio.obj(i.GPIO_PullSelSetup) for GPIO_PullSelSetup
    bl_Init.obj(EXT_BOOTLOADER_CODE) refers to gpio_var.obj(.constdata) for gpio_usbdl_pin
    bl_Init.obj(EXT_BOOTLOADER_CODE) refers to bl_Init.obj(EXT_BOOTLOADER_CODE) for InitUSBDLGPIO
    bl_Init.obj(EXT_BOOTLOADER_CODE) refers to custom_blconfig.obj(i.custom_ROM_baseaddr) for custom_ROM_baseaddr
    bl_Init.obj(EXT_BOOTLOADER_CODE) refers to custom_blconfig.obj(i.custom_RAM_baseaddr) for custom_RAM_baseaddr
    bl_Init.obj(EXT_BOOTLOADER_CODE) refers to SSS_secure_shared.obj(COMMON_CODE) for SST_Get_MAUI_Feature_Combination
    bl_Init.obj(EXT_BOOTLOADER_CODE) refers to bl_Main.obj(.bss) for g_mauiFeatureCombination
    bl_Init.obj(EXT_BOOTLOADER_CODE) refers to custom_blconfig.obj(i.custom_ROM_baseaddr) for custom_ROM_baseaddr
    bl_Init.obj(EXT_BOOTLOADER_CODE) refers to custom_blconfig.obj(i.custom_RAM_baseaddr) for custom_RAM_baseaddr
    bl_Init.obj(EXT_BOOTLOADER_CODE) refers to SSS_secure_shared.obj(COMMON_CODE) for SST_Get_MAUI_Paired_Version
    bl_Init.obj(EXT_BOOTLOADER_CODE) refers to bl_DBGPRINT.obj(i.dbg_print) for dbg_print
    bl_Init.obj(EXT_BOOTLOADER_CODE) refers to bl_Main.obj(HEAD_BL) for g_ExtBootloaderInfo
    bl_Init.obj(EXT_BOOTLOADER_CODE) refers to bl_Init.obj(.constdata) for .constdata$1
    bl_Main.obj(i.INT_Version_Check) refers to bl_Main.obj(i.INT_Version_Check_PutUARTByte) for INT_Version_Check_PutUARTByte
    bl_Main.obj(EXT_BOOTLOADER_CODE) refers to gpio.obj(i.GPIO_ReadIO) for GPIO_ReadIO
    bl_Main.obj(EXT_BOOTLOADER_CODE) refers to gpio_var.obj(.constdata) for gpio_usbdl_pin
    bl_Main.obj(EXT_BOOTLOADER_CODE) refers to bl_Init.obj(i.isGPTTImer3Started) for isGPTTImer3Started
    bl_Main.obj(EXT_BOOTLOADER_CODE) refers to bl_Init.obj(i.startGPTTImer3) for startGPTTImer3
    bl_Main.obj(EXT_BOOTLOADER_CODE) refers to bl_Init.obj(i.getGPTTImer3Value) for getGPTTImer3Value
    bl_Main.obj(EXT_BOOTLOADER_CODE) refers to bl_Main.obj(.bss) for .bss$2
    bl_Main.obj(EXT_BOOTLOADER_CODE) refers to custom_blconfig.obj(.constdata) for usbdlauto_timeout
    bl_Main.obj(EXT_BOOTLOADER_CODE) refers to bl_Main.obj(.data) for .data$0
    bl_Main.obj(EXT_BOOTLOADER_CODE) refers to custom_blconfig.obj(.constdata) for usbdlauto_timeout
    bl_Main.obj(EXT_BOOTLOADER_CODE) refers to bl_Main.obj(.bss) for .bss$2
    bl_Main.obj(EXT_BOOTLOADER_CODE) refers to bl_Init.obj(i.getGPTTImer3Value) for getGPTTImer3Value
    bl_Main.obj(EXT_BOOTLOADER_CODE) refers to custom_blconfig.obj(.constdata) for usbdlauto_timeout
    bl_Main.obj(EXT_BOOTLOADER_CODE) refers to bl_Main.obj(.bss) for .bss$2
    bl_Main.obj(EXT_BOOTLOADER_CODE) refers to bl_Main.obj(.data) for .data$0
    bl_Main.obj(EXT_BOOTLOADER_CODE) refers to bl_Main.obj(EXT_BOOTLOADER_CODE) for USBDLGPIO_Enabled
    bl_Main.obj(EXT_BOOTLOADER_CODE) refers to usbdl_usbacm_adap.obj(i.USBDLKey_Pressed) for USBDLKey_Pressed
    bl_Main.obj(EXT_BOOTLOADER_CODE) refers to bl_Main.obj(EXT_BOOTLOADER_CODE) for USBDL_Stop_Timer
    bl_Main.obj(EXT_BOOTLOADER_CODE) refers to usbdl_pmu.obj(i.USBDL_Cable_IN) for USBDL_Cable_IN
    bl_Main.obj(EXT_BOOTLOADER_CODE) refers to bl_Main.obj(EXT_BOOTLOADER_CODE) for USBDL_Start_Timer
    bl_Main.obj(EXT_BOOTLOADER_CODE) refers to bl_Main.obj(EXT_BOOTLOADER_CODE) for USBDL_Is_Timeout
    bl_Main.obj(EXT_BOOTLOADER_CODE) refers to gpio_var.obj(.constdata) for gpio_usbdl_pin
    bl_Main.obj(EXT_BOOTLOADER_CODE) refers to bl_Main.obj(.bss) for .bss$2
    bl_Main.obj(EXT_BOOTLOADER_CODE) refers to custom_blconfig.obj(.constdata) for usbdlkey_position
    bl_Main.obj(EXT_BOOTLOADER_CODE) refers to custom_blconfig.obj(.constdata) for usbdlauto_timeout
    bl_Main.obj(EXT_BOOTLOADER_CODE) refers to usbdl_usbacm_adap.obj(i.USBDL_Update_USB_Download_Mode) for USBDL_Update_USB_Download_Mode
    bl_Main.obj(EXT_BOOTLOADER_CODE) refers to bl_DBGPRINT.obj(i.dbg_print) for dbg_print
    bl_Main.obj(EXT_BOOTLOADER_CODE) refers to usbdl_usbacm_adap.obj(i.USBDL_UART_Init) for USBDL_UART_Init
    bl_Main.obj(EXT_BOOTLOADER_CODE) refers to usbdl_usbacm_adap.obj(i.USBDL_Is_USB_Download_Mode) for USBDL_Is_USB_Download_Mode
    bl_Main.obj(EXT_BOOTLOADER_CODE) refers to usbdl_usbacm_adap.obj(i.USBDL_CheckStartCmd) for USBDL_CheckStartCmd
    bl_Main.obj(EXT_BOOTLOADER_CODE) refers to bl_Main.obj(EXT_BOOTLOADER_CODE) for USBDL_Is_Timeout
    bl_Main.obj(EXT_BOOTLOADER_CODE) refers to usbdl_usbacm_adap.obj(i.USBDL_Release) for USBDL_Release
    bl_Main.obj(EXT_BOOTLOADER_CODE) refers to bl_Init.obj(i.WatchDogResetAll) for WatchDogResetAll
    bl_Main.obj(EXT_BOOTLOADER_CODE) refers to bl_Main.obj(EXT_BOOTLOADER_CODE) for USBDL_Stop_Timer
    bl_Main.obj(EXT_BOOTLOADER_CODE) refers to bl_FactoryConn.obj(i.Connect_FactoryTool) for Connect_FactoryTool
    bl_Main.obj(EXT_BOOTLOADER_CODE) refers to bl_Main.obj(.bss) for .bss$2
    bl_Main.obj(EXT_BOOTLOADER_CODE) refers to bl_Main.obj(.constdata) for .constdata$1
    bl_Main.obj(EXT_BOOTLOADER_CODE) refers to lib_init.o(.text) for __rt_lib_init
    bl_Main.obj(EXT_BOOTLOADER_CODE) refers to bl_Init.obj(i.WacthDogRestart) for WacthDogRestart
    bl_Main.obj(EXT_BOOTLOADER_CODE) refers to bl_UART.obj(i.uart_init) for uart_init
    bl_Main.obj(EXT_BOOTLOADER_CODE) refers to bl_Main.obj(EXT_BOOTLOADER_CODE) for USBDL_Main
    bl_Main.obj(EXT_BOOTLOADER_CODE) refers to bl_Main.obj(.bss) for .bss$2
    bl_Main.obj(EXT_BOOTLOADER_CODE) refers to bl_Main.obj(HEAD_BL) for HEAD_BL$5
    bl_Main.obj(INTERNCODE) refers to bl_UART.obj(i.CheckUARTSendEnd) for CheckUARTSendEnd
    bl_Main.obj(INTERNCODE) refers to bl_BOOTARM.obj(SHARECODE) for JumpCmd
    bl_Main.obj(INTERNCODE) refers to bl_ImageLoader.obj(EXT_BOOTLOADER_CODE) for NorFlashBooting
    bl_Main.obj(INTERNCODE) refers to custom_blconfig.obj(i.custom_ROM_baseaddr) for custom_ROM_baseaddr
    bl_Main.obj(INTERNCODE) refers to custom_blconfig.obj(i.custom_RAM_baseaddr) for custom_RAM_baseaddr
    bl_Main.obj(INTERNCODE) refers to bl_Cache.obj(EXT_BOOTLOADER_CODE) for CacheDeinit
    bl_Main.obj(INTERNCODE) refers to bl_DBGPRINT.obj(i.dbg_print) for dbg_print
    bl_Main.obj(INTERNCODE) refers to bl_Main.obj(INTERNCODE) for jump_cmd
    bl_Main.obj(INTERNCODE) refers to bl_Main.obj(.bss) for .bss$2
    bl_Main.obj(INTERNCODE) refers to bl_Main.obj(.constdata) for .constdata$1
    bl_Main.obj(INTERNCODE) refers to bl_Secure.obj(.bss) for g_Bl_Secure_Test
    bl_Main.obj(EXT_BOOTLOADER_CODE) refers to bl_DBGPRINT.obj(i.dbg_print) for dbg_print
    bl_Main.obj(EXT_BOOTLOADER_CODE) refers to bl_regioninit.obj(EXT_BOOTLOADER_CODE) for InitRegionsExt
    bl_Main.obj(EXT_BOOTLOADER_CODE) refers to bl_Init.obj(EXT_BOOTLOADER_CODE) for InitExt
    bl_Main.obj(EXT_BOOTLOADER_CODE) refers to bl_Init.obj(EXT_BOOTLOADER_CODE) for GetFeatureCombination
    bl_Main.obj(EXT_BOOTLOADER_CODE) refers to bl_Init.obj(EXT_BOOTLOADER_CODE) for CheckPairedVersion
    bl_Main.obj(EXT_BOOTLOADER_CODE) refers to bl_Main.obj(EXT_BOOTLOADER_CODE) for FactoryProcedure
    bl_Main.obj(EXT_BOOTLOADER_CODE) refers to bl_Cache.obj(EXT_BOOTLOADER_CODE) for CacheInit
    bl_Main.obj(EXT_BOOTLOADER_CODE) refers to bl_Main.obj(INTERNCODE) for BootAndHandOver
    bl_Main.obj(EXT_BOOTLOADER_CODE) refers to bl_verno.obj(.constdata) for BootLDVerno
    bl_Main.obj(EXT_BOOTLOADER_CODE) refers to bl_Main.obj(.constdata) for .constdata$1
    bl_Main.obj(EXT_BOOTLOADER_CODE) refers to bl_Main.obj(.bss) for .bss$2
    bl_Main.obj(EXT_BOOTLOADER_CODE) refers to bl_ImageLoader.obj(BL_INFO_NOR) for BL_Shared_info
    bl_UART.obj(i.uart_init) refers to bl_UART.obj(.data) for UART_Baud_Table
    bl_portingfunc.obj(i.kal_assert_fail) refers to bl_DBGPRINT.obj(i.dbg_print) for dbg_print
    bl_portingfunc.obj(i.kal_assert_fail) refers to bl_portingfunc.obj(.constdata) for .constdata$1
    cache.obj(i.MPUGetChannel) refers to bl_portingfunc.obj(i.SaveAndSetIRQMask) for SaveAndSetIRQMask
    cache.obj(i.MPUGetChannel) refers to bl_portingfunc.obj(i.RestoreIRQMask) for RestoreIRQMask
    cache.obj(i.MPUGetChannel) refers to cache.obj(.bss) for .bss$2
    cache.obj(i.MPUFreeChannel) refers to bl_portingfunc.obj(i.kal_assert_fail) for kal_assert_fail
    cache.obj(i.MPUFreeChannel) refers to bl_portingfunc.obj(i.SaveAndSetIRQMask) for SaveAndSetIRQMask
    cache.obj(i.MPUFreeChannel) refers to bl_portingfunc.obj(i.RestoreIRQMask) for RestoreIRQMask
    cache.obj(i.MPUFreeChannel) refers to cache.obj(.constdata) for .constdata$1
    cache.obj(i.MPUFreeChannel) refers to cache.obj(.bss) for .bss$2
    cache.obj(i.CodeCacheGetChannel) refers to bl_portingfunc.obj(i.SaveAndSetIRQMask) for SaveAndSetIRQMask
    cache.obj(i.CodeCacheGetChannel) refers to bl_portingfunc.obj(i.RestoreIRQMask) for RestoreIRQMask
    cache.obj(i.CodeCacheGetChannel) refers to cache.obj(.bss) for .bss$2
    cache.obj(i.CodeCacheFreeChannel) refers to bl_portingfunc.obj(i.kal_assert_fail) for kal_assert_fail
    cache.obj(i.CodeCacheFreeChannel) refers to bl_portingfunc.obj(i.SaveAndSetIRQMask) for SaveAndSetIRQMask
    cache.obj(i.CodeCacheFreeChannel) refers to bl_portingfunc.obj(i.RestoreIRQMask) for RestoreIRQMask
    cache.obj(i.CodeCacheFreeChannel) refers to cache.obj(.constdata) for .constdata$1
    cache.obj(i.CodeCacheFreeChannel) refers to cache.obj(.bss) for .bss$2
    cache.obj(INTERNCODE) refers to bl_portingfunc.obj(i.SaveAndSetIRQMask) for SaveAndSetIRQMask
    cache.obj(INTERNCODE) refers to bl_portingfunc.obj(i.RestoreIRQMask) for RestoreIRQMask
    cache.obj(INTERNCODE) refers to bl_portingfunc.obj(i.kal_assert_fail) for kal_assert_fail
    cache.obj(INTERNCODE) refers to bl_portingfunc.obj(i.SaveAndSetIRQMask) for SaveAndSetIRQMask
    cache.obj(INTERNCODE) refers to bl_portingfunc.obj(i.RestoreIRQMask) for RestoreIRQMask
    cache.obj(INTERNCODE) refers to cache.obj(.constdata) for .constdata$1
    cache.obj(INTERNCODE) refers to cache.obj(.bss) for .bss$2
    cache.obj(INTERNCODE) refers to bl_portingfunc.obj(i.kal_assert_fail) for kal_assert_fail
    cache.obj(INTERNCODE) refers to bl_portingfunc.obj(i.SaveAndSetIRQMask) for SaveAndSetIRQMask
    cache.obj(INTERNCODE) refers to bl_portingfunc.obj(i.RestoreIRQMask) for RestoreIRQMask
    cache.obj(INTERNCODE) refers to cache.obj(.constdata) for .constdata$1
    cache.obj(INTERNCODE) refers to cache.obj(.bss) for .bss$2
    cache.obj(i.query_is_l1cache_cacheable) refers to bl_portingfunc.obj(i.SaveAndSetIRQMask) for SaveAndSetIRQMask
    cache.obj(i.query_is_l1cache_cacheable) refers to bl_portingfunc.obj(i.RestoreIRQMask) for RestoreIRQMask
    cache.obj(i.query_is_l1cache_cacheable) refers to cache.obj(.constdata) for .constdata$1
    cache.obj(i.dynamic_switch_cacheable_region) refers to bl_portingfunc.obj(i.kal_assert_fail) for kal_assert_fail
    cache.obj(i.dynamic_switch_cacheable_region) refers to cache.obj(i.CodeCacheGetChannel) for CodeCacheGetChannel
    cache.obj(i.dynamic_switch_cacheable_region) refers to cache.obj(INTERNCODE) for CodeCacheSetting
    cache.obj(i.dynamic_switch_cacheable_region) refers to cache.obj(i.query_is_l1cache_cacheable) for query_is_l1cache_cacheable
    cache.obj(i.dynamic_switch_cacheable_region) refers to bl_portingfunc.obj(i.SaveAndSetIRQMask) for SaveAndSetIRQMask
    cache.obj(i.dynamic_switch_cacheable_region) refers to bl_portingfunc.obj(i.RestoreIRQMask) for RestoreIRQMask
    cache.obj(i.dynamic_switch_cacheable_region) refers to cache.obj(.constdata) for .constdata$1
    cache.obj(i.dynamic_switch_cacheable_region) refers to cache.obj(.bss) for .bss$2
    cache.obj(i.free_all_channels) refers to bl_portingfunc.obj(i.SaveAndSetIRQMask) for SaveAndSetIRQMask
    cache.obj(i.free_all_channels) refers to bl_portingfunc.obj(i.RestoreIRQMask) for RestoreIRQMask
    cache.obj(i.free_all_channels) refers to cache.obj(.constdata) for .constdata$1
    cache.obj(i.free_all_channels) refers to cache.obj(.bss) for .bss$2
    cache.obj(INTERNCODE) refers to cache.obj(INTERNCODE) for CodeCacheClearAllSetting
    cache.obj(INTERNCODE) refers to cache.obj(INTERNCODE) for MPUClearAllSetting
    cache.obj(i.CustomizedCacheInit) refers to cache.obj(i.SetupMPUbyROMSegment) for SetupMPUbyROMSegment
    cache.obj(i.CustomizedCacheInit) refers to bl_Cache.obj(EXT_BOOTLOADER_CODE) for SetupMPUonTCM
    cache.obj(i.CustomizedCacheInit) refers to cache.obj(i.dynamic_switch_cacheable_region) for dynamic_switch_cacheable_region
    cache.obj(i.CustomizedCacheInit) refers to bl_Cache.obj(EXT_BOOTLOADER_CODE) for SetupMPUCacheByFeature
    cache.obj(i.CustomizedCacheInit) refers to cache.obj(INTERNCODE) for CodeCacheConfig
    cache.obj(i.SetupMPUbyROMSegment) refers to bl_portingfunc.obj(i.kal_assert_fail) for kal_assert_fail
    cache.obj(i.SetupMPUbyROMSegment) refers to cache.obj(i.MPUGetChannel) for MPUGetChannel
    cache.obj(i.SetupMPUbyROMSegment) refers to cache.obj(INTERNCODE) for MPUSetting
    cache.obj(i.SetupMPUbyROMSegment) refers to cache.obj(.constdata) for .constdata$1
    custom_emi.obj(EMIINITCODE) refers to custom_emi.obj(.constdata) for .constdata$1
    custom_emi.obj(EMIINITCODE) refers to custom_emi.obj(.constdata) for .constdata$1
    custom_emi.obj(EMIINITCODE) refers to custom_emi.obj(.data) for psram_compare_pattern
    custom_emi.obj(INTSRAM_ROCODE) refers to custom_emi.obj(.bss) for .bss$2
    custom_emi.obj(INTSRAM_ROCODE) refers to custom_emi.obj(.constdata) for .constdata$1
    custom_emi.obj(INTSRAM_ROCODE) refers to custom_emi.obj(.data) for psram_compare_pattern
    gpio.obj(i.GPIO_ModeSetup) refers to bl_portingfunc.obj(i.SaveAndSetIRQMask) for SaveAndSetIRQMask
    gpio.obj(i.GPIO_ModeSetup) refers to bl_portingfunc.obj(i.RestoreIRQMask) for RestoreIRQMask
    gpio.obj(i.GPIO_ModeSetup) refers to gpio_drv.obj(.bss) for gpio_debug_enable
    gpio.obj(i.GPIO_ModeSetup) refers to gpio_setting.obj(.data) for gpio_check_for_write
    gpio.obj(i.GPIO_ModeSetup) refers to gpio_setting.obj(.data) for gpio_check_for_read
    gpio.obj(i.GPIO_ModeSetup_FAST) refers to gpio_drv.obj(.bss) for gpio_debug_enable
    gpio.obj(i.GPIO_ModeSetup_FAST) refers to gpio_setting.obj(.data) for gpio_check_for_write
    gpio.obj(i.GPIO_ModeSetup_FAST) refers to gpio_setting.obj(.data) for gpio_check_for_read
    gpio.obj(i.GPIO_InitIO) refers to gpio_drv.obj(.bss) for gpio_debug_enable
    gpio.obj(i.GPIO_InitIO) refers to gpio_setting.obj(.data) for gpio_check_for_write
    gpio.obj(i.GPIO_InitIO) refers to gpio_setting.obj(.data) for gpio_check_for_read
    gpio.obj(i.GPIO_ReadIO) refers to gpio_drv.obj(.bss) for gpio_debug_enable
    gpio.obj(i.GPIO_ReadIO) refers to gpio_setting.obj(.data) for gpio_check_for_read
    gpio.obj(i.GPIO_WriteIO) refers to gpio_drv.obj(.bss) for gpio_debug_enable
    gpio.obj(i.GPIO_WriteIO) refers to gpio_setting.obj(.data) for gpio_check_for_write
    gpio.obj(i.GPIO_WriteIO_Force) refers to bl_portingfunc.obj(i.kal_assert_fail) for kal_assert_fail
    gpio.obj(i.GPIO_WriteIO_Force) refers to gpio_drv.obj(.bss) for gpio_debug_enable
    gpio.obj(i.GPIO_WriteIO_Force) refers to gpio.obj(.constdata) for .constdata$1
    gpio.obj(i.GPIO_Check_MultiPins) refers to gpio.obj(i.GPIO_ReturnMode) for GPIO_ReturnMode
    gpio.obj(i.GPIO_Check_MultiPins) refers to gpio.obj(i.GPIO_ReturnDir) for GPIO_ReturnDir
    gpio.obj(i.GPIO_Check_MultiPins) refers to bl_portingfunc.obj(i.kal_assert_fail) for kal_assert_fail
    gpio.obj(i.GPIO_Check_MultiPins) refers to gpio.obj(.constdata) for .constdata$1
    gpio_drv.obj(i.GPIO_init) refers to gpio_setting.obj(i.GPIO_setting_init) for GPIO_setting_init
    keypad_def.obj(i.keypad_GetFunc) refers to keypad_def.obj(.constdata) for .constdata$1
    keypad_def.obj(i.keypad_Get_Data) refers to keypad_def.obj(.constdata) for .constdata$1
    keypad_def.obj(.constdata) refers to keypad_def.obj(i.keypad_Get_Data) for keypad_Get_Data
    l1_interface.obj(i.HW_TDMA_Enable_CTIRQ1) refers to l1_interface.obj(i.HW_TDMA_Start) for HW_TDMA_Start
    nand_dal.obj(i.init_multiProgram) refers to memset.o(.text) for memset
    nand_dal.obj(i.init_multiProgram) refers to bl_DBGPRINT.obj(i.dbg_print) for dbg_print
    nand_dal.obj(i.init_multiProgram) refers to nand_dal.obj(.bss) for .bss$2
    nand_dal.obj(i.init_multiProgram) refers to nand_dal.obj(.constdata) for .constdata$1
    nand_dal.obj(i.init_multiProgram) refers to rt_udiv.o(.text) for __rt_udiv
    nand_dal.obj(i.init_multiErase) refers to memset.o(.text) for memset
    nand_dal.obj(i.init_multiErase) refers to bl_DBGPRINT.obj(i.dbg_print) for dbg_print
    nand_dal.obj(i.init_multiErase) refers to nand_dal.obj(.bss) for .bss$2
    nand_dal.obj(i.init_multiErase) refers to nand_dal.obj(.constdata) for .constdata$1
    nand_dal.obj(i.init_CE_interleave) refers to nand_dal.obj(.bss) for .bss$2
    nand_dal.obj(i.DAL_init) refers to nand_mtd_fdm50.obj(i.get_MTD_lock) for get_MTD_lock
    nand_dal.obj(i.DAL_init) refers to memset.o(.text) for memset
    nand_dal.obj(i.DAL_init) refers to nand_mtd_fdm50.obj(i.MTD_MountDevice) for MTD_MountDevice
    nand_dal.obj(i.DAL_init) refers to nand_mtd_fdm50.obj(i.free_MTD_lock) for free_MTD_lock
    nand_dal.obj(i.DAL_init) refers to bl_DBGPRINT.obj(i.dbg_print) for dbg_print
    nand_dal.obj(i.DAL_init) refers to memcmp.o(.text) for memcmp
    nand_dal.obj(i.DAL_init) refers to nand_dal.obj(i.init_multiProgram) for init_multiProgram
    nand_dal.obj(i.DAL_init) refers to nand_dal.obj(i.init_multiErase) for init_multiErase
    nand_dal.obj(i.DAL_init) refers to nand_dal.obj(i.init_CE_interleave) for init_CE_interleave
    nand_dal.obj(i.DAL_init) refers to rt_udiv.o(.text) for __rt_udiv
    nand_dal.obj(i.DAL_init) refers to nand_dal.obj(.bss) for .bss$2
    nand_dal.obj(i.DAL_init) refers to nand_dal.obj(.constdata) for .constdata$1
    nand_dal.obj(i.DAL_ShutDown) refers to nand_mtd_fdm50.obj(i.get_MTD_lock) for get_MTD_lock
    nand_dal.obj(i.DAL_ShutDown) refers to nand_mtd_fdm50.obj(i.MTD_ShutDown) for MTD_ShutDown
    nand_dal.obj(i.DAL_ShutDown) refers to nand_mtd_fdm50.obj(i.free_MTD_lock) for free_MTD_lock
    nand_dal.obj(i.DAL_FDM_Flash_Info_Init) refers to nand_mtd_fdm50.obj(i.get_MTD_lock) for get_MTD_lock
    nand_dal.obj(i.DAL_FDM_Flash_Info_Init) refers to rt_udiv.o(.text) for __rt_udiv
    nand_dal.obj(i.DAL_FDM_Flash_Info_Init) refers to nand_mtd_fdm50.obj(i.free_MTD_lock) for free_MTD_lock
    nand_dal.obj(i.DAL_FDM_Flash_Info_Init) refers to nand_dal.obj(.bss) for .bss$2
    nand_dal.obj(i.DAL_FDM_Flash_Info_Init) refers to nand_mtd_fdm50.obj(i.samsung_twoPlane_Program) for samsung_twoPlane_Program
    nand_dal.obj(i.readMapCache) refers to rt_udiv.o(.text) for __rt_udiv
    nand_dal.obj(i.readMapCache) refers to nand_dal.obj(.bss) for .bss$2
    nand_dal.obj(i.writeMapCache) refers to rt_udiv.o(.text) for __rt_udiv
    nand_dal.obj(i.writeMapCache) refers to nand_dal.obj(.bss) for .bss$2
    nand_dal.obj(i.addressMap) refers to nand_dal.obj(i.readMapCache) for readMapCache
    nand_dal.obj(i.addressMap) refers to rt_udiv.o(.text) for __rt_udiv
    nand_dal.obj(i.addressMap) refers to bl_DBGPRINT.obj(i.dbg_print) for dbg_print
    nand_dal.obj(i.addressMap) refers to nand_dal.obj(i.writeMapCache) for writeMapCache
    nand_dal.obj(i.addressMap) refers to nand_dal.obj(.bss) for .bss$2
    nand_dal.obj(i.addressMap) refers to nand_dal.obj(.constdata) for .constdata$1
    nand_dal.obj(i.DAL_ProgramPage) refers to nand_mtd_fdm50.obj(i.get_MTD_lock) for get_MTD_lock
    nand_dal.obj(i.DAL_ProgramPage) refers to nand_mtd_fdm50.obj(i.free_MTD_lock) for free_MTD_lock
    nand_dal.obj(i.DAL_ProgramPage) refers to memset.o(.text) for memset
    nand_dal.obj(i.DAL_ProgramPage) refers to rt_udiv.o(.text) for __rt_udiv
    nand_dal.obj(i.DAL_ProgramPage) refers to nand_dal.obj(i.addressMap) for addressMap
    nand_dal.obj(i.DAL_ProgramPage) refers to nand_dal.obj(.bss) for .bss$2
    nand_dal.obj(i.DAL_ProgramPage) refers to nand_mtd_fdm50.obj(.bss) for Mtd_para
    nand_dal.obj(i.DAL_ProgramPage) refers to nand_mtd_fdm50.obj(i.MTD_CE_Interleave_CacheProgram) for MTD_CE_Interleave_CacheProgram
    nand_dal.obj(i.DAL_ProgramPage) refers to nand_mtd_fdm50.obj(i.MTD_CE_Interleave_Program) for MTD_CE_Interleave_Program
    nand_dal.obj(i.DAL_ProgramPage) refers to nand_mtd_fdm50.obj(i.MTD_CacheProgram) for MTD_CacheProgram
    nand_dal.obj(i.DAL_ProgramPage) refers to nand_mtd_fdm50.obj(i.MTD_Program) for MTD_Program
    nand_dal.obj(i.DAL_ReadPage) refers to nand_mtd_fdm50.obj(i.get_MTD_lock) for get_MTD_lock
    nand_dal.obj(i.DAL_ReadPage) refers to nand_mtd_fdm50.obj(i.free_MTD_lock) for free_MTD_lock
    nand_dal.obj(i.DAL_ReadPage) refers to memset.o(.text) for memset
    nand_dal.obj(i.DAL_ReadPage) refers to nand_dal.obj(i.addressMap) for addressMap
    nand_dal.obj(i.DAL_ReadPage) refers to rt_udiv.o(.text) for __rt_udiv
    nand_dal.obj(i.DAL_ReadPage) refers to nand_dal.obj(.bss) for .bss$2
    nand_dal.obj(i.DAL_ReadPage) refers to nand_mtd_fdm50.obj(.bss) for Mtd_para
    nand_dal.obj(i.DAL_ReadPage) refers to nand_mtd_fdm50.obj(i.MTD_Read) for MTD_Read
    nand_dal.obj(i.DAL_CopyPage) refers to nand_mtd_fdm50.obj(i.get_MTD_lock) for get_MTD_lock
    nand_dal.obj(i.DAL_CopyPage) refers to rt_udiv.o(.text) for __rt_udiv
    nand_dal.obj(i.DAL_CopyPage) refers to nand_mtd_fdm50.obj(i.free_MTD_lock) for free_MTD_lock
    nand_dal.obj(i.DAL_CopyPage) refers to memset.o(.text) for memset
    nand_dal.obj(i.DAL_CopyPage) refers to memcpy.o(.text) for memcpy
    nand_dal.obj(i.DAL_CopyPage) refers to nand_dal.obj(i.addressMap) for addressMap
    nand_dal.obj(i.DAL_CopyPage) refers to nand_mtd_fdm50.obj(i.MTD_Read) for MTD_Read
    nand_dal.obj(i.DAL_CopyPage) refers to nand_dal.obj(.bss) for .bss$2
    nand_dal.obj(i.DAL_CopyPage) refers to nand_mtd_fdm50.obj(.bss) for Mtd_para
    nand_dal.obj(i.DAL_CopyPage) refers to nand_mtd_fdm50.obj(i.MTD_CE_Interleave_CacheProgram) for MTD_CE_Interleave_CacheProgram
    nand_dal.obj(i.DAL_CopyPage) refers to nand_mtd_fdm50.obj(i.MTD_CE_Interleave_Program) for MTD_CE_Interleave_Program
    nand_dal.obj(i.DAL_CopyPage) refers to nand_mtd_fdm50.obj(i.MTD_CacheProgram) for MTD_CacheProgram
    nand_dal.obj(i.DAL_CopyPage) refers to nand_mtd_fdm50.obj(i.MTD_Program) for MTD_Program
    nand_dal.obj(i.DAL_EraseBlock) refers to nand_mtd_fdm50.obj(i.get_MTD_lock) for get_MTD_lock
    nand_dal.obj(i.DAL_EraseBlock) refers to nand_mtd_fdm50.obj(i.free_MTD_lock) for free_MTD_lock
    nand_dal.obj(i.DAL_EraseBlock) refers to memset.o(.text) for memset
    nand_dal.obj(i.DAL_EraseBlock) refers to nand_dal.obj(i.addressMap) for addressMap
    nand_dal.obj(i.DAL_EraseBlock) refers to rt_udiv.o(.text) for __rt_udiv
    nand_dal.obj(i.DAL_EraseBlock) refers to nand_dal.obj(.bss) for .bss$2
    nand_dal.obj(i.DAL_EraseBlock) refers to nand_mtd_fdm50.obj(.bss) for Mtd_para
    nand_dal.obj(i.DAL_EraseBlock) refers to nand_mtd_fdm50.obj(i.MTD_Erase) for MTD_Erase
    nand_dal.obj(i.DAL_MarkBlockBad) refers to nand_mtd_fdm50.obj(i.get_MTD_lock) for get_MTD_lock
    nand_dal.obj(i.DAL_MarkBlockBad) refers to nand_mtd_fdm50.obj(i.free_MTD_lock) for free_MTD_lock
    nand_dal.obj(i.DAL_MarkBlockBad) refers to memset.o(.text) for memset
    nand_dal.obj(i.DAL_MarkBlockBad) refers to nand_dal.obj(i.addressMap) for addressMap
    nand_dal.obj(i.DAL_MarkBlockBad) refers to nand_mtd_fdm50.obj(i.MTD_Erase) for MTD_Erase
    nand_dal.obj(i.DAL_MarkBlockBad) refers to nand_mtd_fdm50.obj(i.MTD_Read) for MTD_Read
    nand_dal.obj(i.DAL_MarkBlockBad) refers to nand_mtd_fdm50.obj(i.MTD_MarkBlockBad) for MTD_MarkBlockBad
    nand_dal.obj(i.DAL_MarkBlockBad) refers to nand_dal.obj(.bss) for .bss$2
    nand_dal.obj(i.DAL_MarkBlockBad) refers to nand_mtd_fdm50.obj(.bss) for Mtd_para
    nand_dal.obj(i.DAL_CheckBadBlock) refers to nand_mtd_fdm50.obj(i.get_MTD_lock) for get_MTD_lock
    nand_dal.obj(i.DAL_CheckBadBlock) refers to nand_mtd_fdm50.obj(i.free_MTD_lock) for free_MTD_lock
    nand_dal.obj(i.DAL_CheckBadBlock) refers to memset.o(.text) for memset
    nand_dal.obj(i.DAL_CheckBadBlock) refers to nand_dal.obj(i.addressMap) for addressMap
    nand_dal.obj(i.DAL_CheckBadBlock) refers to nand_mtd_fdm50.obj(i.MTD_CheckBlockBad) for MTD_CheckBlockBad
    nand_dal.obj(i.DAL_CheckBadBlock) refers to nand_dal.obj(.bss) for .bss$2
    nand_dal.obj(i.DAL_CheckBadBlock) refers to nand_mtd_fdm50.obj(.bss) for Mtd_para
    nand_dal.obj(i.DAL_CheckBadBlock) refers to nand_dal.obj(.constdata) for .constdata$1
    nand_dal.obj(i.IsGoodBlock) refers to nand_dal.obj(.bss) for .bss$2
    nand_dal.obj(i.IsGoodBlock) refers to nand_dal.obj(.constdata) for .constdata$1
    nand_dal.obj(i.DAL_NAND_Reset) refers to nand_mtd_fdm50.obj(i.get_MTD_lock) for get_MTD_lock
    nand_dal.obj(i.DAL_NAND_Reset) refers to nand_mtd_fdm50.obj(i.MTD_NAND_Reset) for MTD_NAND_Reset
    nand_dal.obj(i.DAL_NAND_Reset) refers to nand_mtd_fdm50.obj(i.free_MTD_lock) for free_MTD_lock
    nand_dal.obj(i.DAL_NAND_Reset) refers to nand_dal.obj(.bss) for .bss$2
    nand_dal.obj(i.DAL_NAND_Reset) refers to nand_mtd_fdm50.obj(.bss) for Mtd_para
    nand_dal.obj(i.DAL_GetFDMData) refers to nand_dal.obj(.bss) for .bss$2
    nand_dal.obj(i.DAL_SetFDMData) refers to memset.o(.text) for memset
    nand_dal.obj(i.DAL_SetFDMData) refers to nand_dal.obj(.bss) for .bss$2
    nand_dal.obj(i.NANDsanitycheck_Factory) refers to nand_dal.obj(i.DAL_init) for DAL_init
    nand_dal.obj(i.NANDsanitycheck_Factory) refers to nand_dal.obj(i.DAL_FDM_Flash_Info_Init) for DAL_FDM_Flash_Info_Init
    nand_dal.obj(i.NANDsanitycheck_Factory) refers to nand_dal.obj(.bss) for .bss$2
    nand_dal.obj(i.DAL_GetDeviceInfo) refers to memcpy.o(.text) for memcpy
    nand_dal.obj(i.DAL_GetDeviceInfo) refers to memset.o(.text) for memset
    nand_dal.obj(i.DAL_GetDeviceInfo) refers to nand_dal.obj(.bss) for .bss$2
    nand_dal.obj(i.DAL_GetDeviceIDInfo) refers to nand_dal.obj(.bss) for .bss$2
    nand_mtd_fdm50.obj(i.read_status) refers to nand_mtd_fdm50.obj(i.NFI_OP_RESET) for NFI_OP_RESET
    nand_mtd_fdm50.obj(i.NFI_Correct) refers to nand_dal.obj(.bss) for Flash_Info
    nand_mtd_fdm50.obj(i.readfifo) refers to nand_mtd_fdm50.obj(i.NFI_Correct) for NFI_Correct
    nand_mtd_fdm50.obj(i.readfifo) refers to nand_dal.obj(.bss) for Flash_Info
    nand_mtd_fdm50.obj(i.readfifo) refers to nand_mtd_fdm50.obj(.bss) for .bss$2
    nand_mtd_fdm50.obj(i.ID_Table_OrderCheck) refers to nand_dal.obj(.constdata) for ZEROBIT
    nand_mtd_fdm50.obj(i.ID_Table_OrderCheck) refers to NAND_DevConfig.obj(.constdata) for NAND_ID_Table
    nand_mtd_fdm50.obj(i.FlashAttrib_AutoDetect) refers to memset.o(.text) for memset
    nand_mtd_fdm50.obj(i.FlashAttrib_AutoDetect) refers to nand_mtd_fdm50.obj(i.FlashSetAttrib_By2ndID) for FlashSetAttrib_By2ndID
    nand_mtd_fdm50.obj(i.FlashAttrib_AutoDetect) refers to memcpy.o(.text) for memcpy
    nand_mtd_fdm50.obj(i.FlashAttrib_AutoDetect) refers to rt_sdiv.o(.text) for __rt_sdiv
    nand_mtd_fdm50.obj(i.FlashAttrib_AutoDetect) refers to nand_mtd_fdm50.obj(.constdata) for .constdata$1
    nand_mtd_fdm50.obj(i.FlashAttrib_AutoDetect) refers to NAND_DevConfig.obj(.data) for Default_ID_Table
    nand_mtd_fdm50.obj(i.FlashAttrib_AutoDetect) refers to NAND_DevConfig.obj(.constdata) for ID_2K_Mask
    nand_mtd_fdm50.obj(i.FlashAttrib_AutoDetect) refers to NAND_DevConfig.obj(.constdata) for ID_512_Mask
    nand_mtd_fdm50.obj(i.FlashAttrib_AutoDetect) refers to NAND_DevConfig.obj(.data) for TOSHIBA_SUB_DRIVER
    nand_mtd_fdm50.obj(i.FlashAttrib_AutoDetect) refers to NAND_DevConfig.obj(.data) for MICRON_SUB_DRIVER
    nand_mtd_fdm50.obj(i.FlashAttrib_AutoDetect) refers to NAND_DevConfig.obj(.data) for SAMSUNG_SINGLE_CACHE_SUB_DRIVER
    nand_mtd_fdm50.obj(i.FlashAttrib_AutoDetect) refers to NAND_DevConfig.obj(.data) for SAMSUNG_SUB_DRIVER
    nand_mtd_fdm50.obj(i.FlashAttrib_AutoDetect) refers to NAND_DevConfig.obj(.data) for HYNIX_ST_SUB_DRIVER
    nand_mtd_fdm50.obj(i.InitializeMTDData) refers to nand_mtd_fdm50.obj(i.NFI_OP_RESET) for NFI_OP_RESET
    nand_mtd_fdm50.obj(i.InitializeMTDData) refers to nand_mtd_fdm50.obj(i.nAND_RESET) for nAND_RESET
    nand_mtd_fdm50.obj(i.InitializeMTDData) refers to memset.o(.text) for memset
    nand_mtd_fdm50.obj(i.InitializeMTDData) refers to nand_mtd_fdm50.obj(i.FlashAttrib_AutoDetect) for FlashAttrib_AutoDetect
    nand_mtd_fdm50.obj(i.InitializeMTDData) refers to bl_DBGPRINT.obj(i.dbg_print) for dbg_print
    nand_mtd_fdm50.obj(i.InitializeMTDData) refers to rt_udiv.o(.text) for __rt_udiv
    nand_mtd_fdm50.obj(i.InitializeMTDData) refers to nand_dal.obj(.bss) for Flash_Info
    nand_mtd_fdm50.obj(i.InitializeMTDData) refers to nand_mtd_fdm50.obj(.constdata) for .constdata$1
    nand_mtd_fdm50.obj(i.InitializeMTDData) refers to NAND_DevConfig.obj(.constdata) for NAND_ID_Table
    nand_mtd_fdm50.obj(i.InitializeMTDData) refers to NAND_DevConfig.obj(.data) for Default_ID_Table
    nand_mtd_fdm50.obj(i.InitializeMTDData) refers to nand_mtd_fdm50.obj(.data) for .data$0
    nand_mtd_fdm50.obj(i.single_Page_Program) refers to nand_mtd_fdm50.obj(i.NFI_OP_RESET) for NFI_OP_RESET
    nand_mtd_fdm50.obj(i.single_Page_Program) refers to nand_mtd_fdm50.obj(i.NFI_Pointer) for NFI_Pointer
    nand_mtd_fdm50.obj(i.single_Page_Program) refers to nand_mtd_fdm50.obj(i.send_command_add_data) for send_command_add_data
    nand_mtd_fdm50.obj(i.single_Page_Program) refers to nand_mtd_fdm50.obj(i.read_status) for read_status
    nand_mtd_fdm50.obj(i.single_Page_Program) refers to nand_mtd_fdm50.obj(i.nAND_RESET) for nAND_RESET
    nand_mtd_fdm50.obj(i.single_Page_Program) refers to nand_mtd_fdm50.obj(.bss) for .bss$2
    nand_mtd_fdm50.obj(i.single_Page_Program) refers to nand_dal.obj(.bss) for Flash_Info
    nand_mtd_fdm50.obj(i.single_Page_CacheProgram) refers to nand_mtd_fdm50.obj(i.NFI_OP_RESET) for NFI_OP_RESET
    nand_mtd_fdm50.obj(i.single_Page_CacheProgram) refers to nand_mtd_fdm50.obj(i.NFI_Pointer) for NFI_Pointer
    nand_mtd_fdm50.obj(i.single_Page_CacheProgram) refers to nand_mtd_fdm50.obj(i.send_command_add_data) for send_command_add_data
    nand_mtd_fdm50.obj(i.single_Page_CacheProgram) refers to nand_mtd_fdm50.obj(i.read_status) for read_status
    nand_mtd_fdm50.obj(i.single_Page_CacheProgram) refers to nand_mtd_fdm50.obj(i.nAND_RESET) for nAND_RESET
    nand_mtd_fdm50.obj(i.single_Page_CacheProgram) refers to nand_mtd_fdm50.obj(.bss) for .bss$2
    nand_mtd_fdm50.obj(i.single_Page_CacheProgram) refers to nand_dal.obj(.bss) for Flash_Info
    nand_mtd_fdm50.obj(i.single_Page_Read) refers to nand_mtd_fdm50.obj(i.NFI_OP_RESET) for NFI_OP_RESET
    nand_mtd_fdm50.obj(i.single_Page_Read) refers to nand_mtd_fdm50.obj(i.NFI_Pointer) for NFI_Pointer
    nand_mtd_fdm50.obj(i.single_Page_Read) refers to nand_mtd_fdm50.obj(i.send_command_add) for send_command_add
    nand_mtd_fdm50.obj(i.single_Page_Read) refers to nand_mtd_fdm50.obj(i.read_status) for read_status
    nand_mtd_fdm50.obj(i.single_Page_Read) refers to nand_mtd_fdm50.obj(i.readfifo) for readfifo
    nand_mtd_fdm50.obj(i.single_Page_Read) refers to nand_mtd_fdm50.obj(i.nAND_RESET) for nAND_RESET
    nand_mtd_fdm50.obj(i.single_Page_Read) refers to nand_mtd_fdm50.obj(.bss) for .bss$2
    nand_mtd_fdm50.obj(i.single_Page_Read) refers to nand_dal.obj(.bss) for Flash_Info
    nand_mtd_fdm50.obj(i.single_Block_Erase) refers to nand_mtd_fdm50.obj(i.NFI_OP_RESET) for NFI_OP_RESET
    nand_mtd_fdm50.obj(i.single_Block_Erase) refers to nand_mtd_fdm50.obj(i.NFI_Pointer) for NFI_Pointer
    nand_mtd_fdm50.obj(i.single_Block_Erase) refers to nand_mtd_fdm50.obj(i.send_command_add) for send_command_add
    nand_mtd_fdm50.obj(i.single_Block_Erase) refers to nand_mtd_fdm50.obj(i.read_status) for read_status
    nand_mtd_fdm50.obj(i.single_Block_Erase) refers to nand_mtd_fdm50.obj(i.nAND_RESET) for nAND_RESET
    nand_mtd_fdm50.obj(i.single_Block_Erase) refers to nand_mtd_fdm50.obj(.bss) for .bss$2
    nand_mtd_fdm50.obj(i.single_Block_Erase) refers to nand_dal.obj(.bss) for Flash_Info
    nand_mtd_fdm50.obj(i.toshiba_twoPlane_Program) refers to nand_mtd_fdm50.obj(i.NFI_OP_RESET) for NFI_OP_RESET
    nand_mtd_fdm50.obj(i.toshiba_twoPlane_Program) refers to nand_mtd_fdm50.obj(i.send_command_add_data) for send_command_add_data
    nand_mtd_fdm50.obj(i.toshiba_twoPlane_Program) refers to nand_mtd_fdm50.obj(i.read_status) for read_status
    nand_mtd_fdm50.obj(i.toshiba_twoPlane_Program) refers to nand_mtd_fdm50.obj(i.nAND_RESET) for nAND_RESET
    nand_mtd_fdm50.obj(i.toshiba_twoPlane_Program) refers to nand_mtd_fdm50.obj(.bss) for .bss$2
    nand_mtd_fdm50.obj(i.toshiba_twoPlane_Program) refers to nand_dal.obj(.bss) for Flash_Info
    nand_mtd_fdm50.obj(i.toshiba_twoPlane_Erase) refers to nand_mtd_fdm50.obj(i.NFI_OP_RESET) for NFI_OP_RESET
    nand_mtd_fdm50.obj(i.toshiba_twoPlane_Erase) refers to nand_mtd_fdm50.obj(i.send_command_add) for send_command_add
    nand_mtd_fdm50.obj(i.toshiba_twoPlane_Erase) refers to nand_mtd_fdm50.obj(i.read_status) for read_status
    nand_mtd_fdm50.obj(i.toshiba_twoPlane_Erase) refers to nand_mtd_fdm50.obj(i.nAND_RESET) for nAND_RESET
    nand_mtd_fdm50.obj(i.toshiba_twoPlane_Erase) refers to nand_mtd_fdm50.obj(.bss) for .bss$2
    nand_mtd_fdm50.obj(i.toshiba_fourPlane_Program) refers to nand_mtd_fdm50.obj(i.NFI_OP_RESET) for NFI_OP_RESET
    nand_mtd_fdm50.obj(i.toshiba_fourPlane_Program) refers to nand_mtd_fdm50.obj(i.NFI_Pointer) for NFI_Pointer
    nand_mtd_fdm50.obj(i.toshiba_fourPlane_Program) refers to nand_mtd_fdm50.obj(i.send_command_add_data) for send_command_add_data
    nand_mtd_fdm50.obj(i.toshiba_fourPlane_Program) refers to nand_mtd_fdm50.obj(i.read_status) for read_status
    nand_mtd_fdm50.obj(i.toshiba_fourPlane_Program) refers to nand_mtd_fdm50.obj(i.nAND_RESET) for nAND_RESET
    nand_mtd_fdm50.obj(i.toshiba_fourPlane_Program) refers to nand_mtd_fdm50.obj(.bss) for .bss$2
    nand_mtd_fdm50.obj(i.toshiba_fourPlane_Program) refers to nand_dal.obj(.bss) for Flash_Info
    nand_mtd_fdm50.obj(i.toshiba_fourPlane_Erase) refers to nand_mtd_fdm50.obj(i.NFI_OP_RESET) for NFI_OP_RESET
    nand_mtd_fdm50.obj(i.toshiba_fourPlane_Erase) refers to nand_mtd_fdm50.obj(i.send_command_add) for send_command_add
    nand_mtd_fdm50.obj(i.toshiba_fourPlane_Erase) refers to nand_mtd_fdm50.obj(i.read_status) for read_status
    nand_mtd_fdm50.obj(i.toshiba_fourPlane_Erase) refers to nand_mtd_fdm50.obj(i.nAND_RESET) for nAND_RESET
    nand_mtd_fdm50.obj(i.toshiba_fourPlane_Erase) refers to nand_mtd_fdm50.obj(.bss) for .bss$2
    nand_mtd_fdm50.obj(i.toshiba_fourPlane_Erase) refers to nand_dal.obj(.bss) for Flash_Info
    nand_mtd_fdm50.obj(i.toshiba_twoPlane_CacheProgram) refers to nand_mtd_fdm50.obj(i.NFI_OP_RESET) for NFI_OP_RESET
    nand_mtd_fdm50.obj(i.toshiba_twoPlane_CacheProgram) refers to nand_mtd_fdm50.obj(i.send_command_add_data) for send_command_add_data
    nand_mtd_fdm50.obj(i.toshiba_twoPlane_CacheProgram) refers to nand_mtd_fdm50.obj(i.read_status) for read_status
    nand_mtd_fdm50.obj(i.toshiba_twoPlane_CacheProgram) refers to nand_mtd_fdm50.obj(i.nAND_RESET) for nAND_RESET
    nand_mtd_fdm50.obj(i.toshiba_twoPlane_CacheProgram) refers to nand_mtd_fdm50.obj(.bss) for .bss$2
    nand_mtd_fdm50.obj(i.toshiba_twoPlane_CacheProgram) refers to nand_dal.obj(.bss) for Flash_Info
    nand_mtd_fdm50.obj(i.toshiba_fourPlane_CacheProgram) refers to nand_mtd_fdm50.obj(i.NFI_OP_RESET) for NFI_OP_RESET
    nand_mtd_fdm50.obj(i.toshiba_fourPlane_CacheProgram) refers to nand_mtd_fdm50.obj(i.send_command_add_data) for send_command_add_data
    nand_mtd_fdm50.obj(i.toshiba_fourPlane_CacheProgram) refers to nand_mtd_fdm50.obj(i.read_status) for read_status
    nand_mtd_fdm50.obj(i.toshiba_fourPlane_CacheProgram) refers to nand_mtd_fdm50.obj(i.nAND_RESET) for nAND_RESET
    nand_mtd_fdm50.obj(i.toshiba_fourPlane_CacheProgram) refers to nand_mtd_fdm50.obj(.bss) for .bss$2
    nand_mtd_fdm50.obj(i.toshiba_fourPlane_CacheProgram) refers to nand_dal.obj(.bss) for Flash_Info
    nand_mtd_fdm50.obj(i.samsung_twoPlane_Program) refers to nand_mtd_fdm50.obj(i.NFI_OP_RESET) for NFI_OP_RESET
    nand_mtd_fdm50.obj(i.samsung_twoPlane_Program) refers to nand_mtd_fdm50.obj(i.send_command_add_data) for send_command_add_data
    nand_mtd_fdm50.obj(i.samsung_twoPlane_Program) refers to nand_mtd_fdm50.obj(i.read_status) for read_status
    nand_mtd_fdm50.obj(i.samsung_twoPlane_Program) refers to nand_mtd_fdm50.obj(i.nAND_RESET) for nAND_RESET
    nand_mtd_fdm50.obj(i.samsung_twoPlane_Program) refers to nand_mtd_fdm50.obj(i.single_Page_Program) for single_Page_Program
    nand_mtd_fdm50.obj(i.samsung_twoPlane_Program) refers to nand_dal.obj(.bss) for Flash_Info
    nand_mtd_fdm50.obj(i.samsung_twoPlane_Program) refers to nand_mtd_fdm50.obj(.bss) for .bss$2
    nand_mtd_fdm50.obj(i.samsung_twoPlane_Erase) refers to nand_mtd_fdm50.obj(i.NFI_OP_RESET) for NFI_OP_RESET
    nand_mtd_fdm50.obj(i.samsung_twoPlane_Erase) refers to nand_mtd_fdm50.obj(i.send_command_add) for send_command_add
    nand_mtd_fdm50.obj(i.samsung_twoPlane_Erase) refers to nand_mtd_fdm50.obj(i.read_status) for read_status
    nand_mtd_fdm50.obj(i.samsung_twoPlane_Erase) refers to nand_mtd_fdm50.obj(i.single_Block_Erase) for single_Block_Erase
    nand_mtd_fdm50.obj(i.samsung_twoPlane_Erase) refers to nand_mtd_fdm50.obj(i.nAND_RESET) for nAND_RESET
    nand_mtd_fdm50.obj(i.samsung_twoPlane_Erase) refers to nand_dal.obj(.bss) for Flash_Info
    nand_mtd_fdm50.obj(i.samsung_twoPlane_Erase) refers to nand_mtd_fdm50.obj(.bss) for .bss$2
    nand_mtd_fdm50.obj(i.samsung_twoDie_Program) refers to nand_mtd_fdm50.obj(i.single_Page_Program) for single_Page_Program
    nand_mtd_fdm50.obj(i.samsung_twoDie_Program) refers to nand_mtd_fdm50.obj(i.read_status) for read_status
    nand_mtd_fdm50.obj(i.samsung_twoDie_Program) refers to nand_dal.obj(.bss) for Flash_Info
    nand_mtd_fdm50.obj(i.samsung_twoDie_Program) refers to nand_mtd_fdm50.obj(.bss) for .bss$2
    nand_mtd_fdm50.obj(i.samsung_twoDie_Erase) refers to nand_mtd_fdm50.obj(i.single_Block_Erase) for single_Block_Erase
    nand_mtd_fdm50.obj(i.samsung_twoDie_Erase) refers to nand_mtd_fdm50.obj(i.read_status) for read_status
    nand_mtd_fdm50.obj(i.samsung_twoDie_Erase) refers to nand_mtd_fdm50.obj(.bss) for .bss$2
    nand_mtd_fdm50.obj(i.samsung_twoDie_twoPlane_Program) refers to nand_mtd_fdm50.obj(i.samsung_twoPlane_Program) for samsung_twoPlane_Program
    nand_mtd_fdm50.obj(i.samsung_twoDie_twoPlane_Program) refers to nand_dal.obj(.bss) for Flash_Info
    nand_mtd_fdm50.obj(i.samsung_twoDie_twoPlane_Erase) refers to nand_mtd_fdm50.obj(i.samsung_twoPlane_Erase) for samsung_twoPlane_Erase
    nand_mtd_fdm50.obj(i.micron_twoPlane_Program) refers to nand_mtd_fdm50.obj(i.NFI_OP_RESET) for NFI_OP_RESET
    nand_mtd_fdm50.obj(i.micron_twoPlane_Program) refers to nand_mtd_fdm50.obj(i.send_command_add_data) for send_command_add_data
    nand_mtd_fdm50.obj(i.micron_twoPlane_Program) refers to nand_mtd_fdm50.obj(i.read_status) for read_status
    nand_mtd_fdm50.obj(i.micron_twoPlane_Program) refers to nand_mtd_fdm50.obj(i.nAND_RESET) for nAND_RESET
    nand_mtd_fdm50.obj(i.micron_twoPlane_Program) refers to nand_mtd_fdm50.obj(.bss) for .bss$2
    nand_mtd_fdm50.obj(i.micron_twoPlane_Program) refers to nand_dal.obj(.bss) for Flash_Info
    nand_mtd_fdm50.obj(i.micron_twoPlane_Erase) refers to nand_mtd_fdm50.obj(i.NFI_OP_RESET) for NFI_OP_RESET
    nand_mtd_fdm50.obj(i.micron_twoPlane_Erase) refers to nand_mtd_fdm50.obj(i.send_command_add) for send_command_add
    nand_mtd_fdm50.obj(i.micron_twoPlane_Erase) refers to nand_mtd_fdm50.obj(i.read_status) for read_status
    nand_mtd_fdm50.obj(i.micron_twoPlane_Erase) refers to nand_mtd_fdm50.obj(i.nAND_RESET) for nAND_RESET
    nand_mtd_fdm50.obj(i.micron_twoPlane_Erase) refers to nand_mtd_fdm50.obj(.bss) for .bss$2
    nand_mtd_fdm50.obj(i.micron_twoPlane_CacheProgram) refers to nand_mtd_fdm50.obj(i.NFI_OP_RESET) for NFI_OP_RESET
    nand_mtd_fdm50.obj(i.micron_twoPlane_CacheProgram) refers to nand_mtd_fdm50.obj(i.send_command_add_data) for send_command_add_data
    nand_mtd_fdm50.obj(i.micron_twoPlane_CacheProgram) refers to nand_mtd_fdm50.obj(i.read_status) for read_status
    nand_mtd_fdm50.obj(i.micron_twoPlane_CacheProgram) refers to nand_mtd_fdm50.obj(i.nAND_RESET) for nAND_RESET
    nand_mtd_fdm50.obj(i.micron_twoPlane_CacheProgram) refers to nand_mtd_fdm50.obj(.bss) for .bss$2
    nand_mtd_fdm50.obj(i.micron_twoPlane_CacheProgram) refers to nand_dal.obj(.bss) for Flash_Info
    nand_mtd_fdm50.obj(i.micron_twoDie_Program) refers to nand_mtd_fdm50.obj(i.single_Page_Program) for single_Page_Program
    nand_mtd_fdm50.obj(i.micron_twoDie_Program) refers to nand_mtd_fdm50.obj(i.read_status) for read_status
    nand_mtd_fdm50.obj(i.micron_twoDie_Program) refers to nand_dal.obj(.bss) for Flash_Info
    nand_mtd_fdm50.obj(i.micron_twoDie_Program) refers to nand_mtd_fdm50.obj(.bss) for .bss$2
    nand_mtd_fdm50.obj(i.micron_twoDie_Erase) refers to nand_mtd_fdm50.obj(i.single_Block_Erase) for single_Block_Erase
    nand_mtd_fdm50.obj(i.micron_twoDie_Erase) refers to nand_mtd_fdm50.obj(i.read_status) for read_status
    nand_mtd_fdm50.obj(i.micron_twoDie_Erase) refers to nand_mtd_fdm50.obj(.bss) for .bss$2
    nand_mtd_fdm50.obj(i.micron_twoDie_twoPlane_Program) refers to nand_mtd_fdm50.obj(i.micron_twoPlane_Program) for micron_twoPlane_Program
    nand_mtd_fdm50.obj(i.micron_twoDie_twoPlane_Program) refers to nand_dal.obj(.bss) for Flash_Info
    nand_mtd_fdm50.obj(i.micron_twoDie_twoPlane_Erase) refers to nand_mtd_fdm50.obj(i.micron_twoPlane_Erase) for micron_twoPlane_Erase
    nand_mtd_fdm50.obj(i.micron_twoDie_CacheProgram) refers to nand_mtd_fdm50.obj(i.single_Page_CacheProgram) for single_Page_CacheProgram
    nand_mtd_fdm50.obj(i.micron_twoDie_CacheProgram) refers to nand_dal.obj(.bss) for Flash_Info
    nand_mtd_fdm50.obj(i.micron_twoDie_twoPlane_CacheProgram) refers to nand_mtd_fdm50.obj(i.micron_twoPlane_CacheProgram) for micron_twoPlane_CacheProgram
    nand_mtd_fdm50.obj(i.micron_twoDie_twoPlane_CacheProgram) refers to nand_mtd_fdm50.obj(i.micron_twoPlane_Program) for micron_twoPlane_Program
    nand_mtd_fdm50.obj(i.micron_twoDie_twoPlane_CacheProgram) refers to nand_dal.obj(.bss) for Flash_Info
    nand_mtd_fdm50.obj(i.samsung_OTPAccess) refers to nand_mtd_fdm50.obj(i.NFI_OP_RESET) for NFI_OP_RESET
    nand_mtd_fdm50.obj(i.samsung_OTPAccess) refers to nand_mtd_fdm50.obj(i.send_command_add) for send_command_add
    nand_mtd_fdm50.obj(i.samsung_OTPAccess) refers to nand_mtd_fdm50.obj(i.readfifo) for readfifo
    nand_mtd_fdm50.obj(i.samsung_OTPAccess) refers to nand_mtd_fdm50.obj(i.send_command_add_data) for send_command_add_data
    nand_mtd_fdm50.obj(i.samsung_OTPAccess) refers to nand_mtd_fdm50.obj(i.read_status) for read_status
    nand_mtd_fdm50.obj(i.samsung_OTPAccess) refers to nand_mtd_fdm50.obj(i.nAND_RESET) for nAND_RESET
    nand_mtd_fdm50.obj(i.samsung_OTPAccess) refers to nand_dal.obj(.bss) for Flash_Info
    nand_mtd_fdm50.obj(i.samsung_OTPAccess) refers to nand_mtd_fdm50.obj(.bss) for .bss$2
    nand_mtd_fdm50.obj(i.samsung_OTPAccess) refers to nand_mtd_fdm50.obj(.constdata) for .constdata$1
    nand_mtd_fdm50.obj(i.samsung_OTPQueryLength) refers to nand_dal.obj(.bss) for Flash_Info
    nand_mtd_fdm50.obj(i.MTD_MountDevice) refers to NAND_DevConfig.obj(i.NFI_GPIO_Setting) for NFI_GPIO_Setting
    nand_mtd_fdm50.obj(i.MTD_MountDevice) refers to nand_mtd_fdm50.obj(i.NFI_OP_RESET) for NFI_OP_RESET
    nand_mtd_fdm50.obj(i.MTD_MountDevice) refers to nand_mtd_fdm50.obj(i.InitializeMTDData) for InitializeMTDData
    nand_mtd_fdm50.obj(i.MTD_MountDevice) refers to nand_mtd_fdm50.obj(.bss) for .bss$2
    nand_mtd_fdm50.obj(i.MTD_MountDevice) refers to nand_mtd_fdm50.obj(.data) for .data$0
    nand_mtd_fdm50.obj(i.MTD_MountDevice) refers to nand_dal.obj(.bss) for Flash_Info
    nand_mtd_fdm50.obj(i.MTD_CE_Interleave_Program) refers to nand_mtd_fdm50.obj(i.NFI_OP_RESET) for NFI_OP_RESET
    nand_mtd_fdm50.obj(i.MTD_CE_Interleave_Program) refers to nand_dal.obj(.bss) for Flash_Info
    nand_mtd_fdm50.obj(i.MTD_CE_Interleave_CacheProgram) refers to rt_udiv.o(.text) for __rt_udiv
    nand_mtd_fdm50.obj(i.MTD_CE_Interleave_CacheProgram) refers to nand_mtd_fdm50.obj(i.NFI_OP_RESET) for NFI_OP_RESET
    nand_mtd_fdm50.obj(i.MTD_CE_Interleave_CacheProgram) refers to nand_dal.obj(.bss) for Flash_Info
    nand_mtd_fdm50.obj(i.MTD_Program) refers to nand_mtd_fdm50.obj(i.NFI_OP_RESET) for NFI_OP_RESET
    nand_mtd_fdm50.obj(i.MTD_Program) refers to nand_dal.obj(.bss) for Flash_Info
    nand_mtd_fdm50.obj(i.MTD_CacheProgram) refers to rt_udiv.o(.text) for __rt_udiv
    nand_mtd_fdm50.obj(i.MTD_CacheProgram) refers to nand_mtd_fdm50.obj(i.NFI_OP_RESET) for NFI_OP_RESET
    nand_mtd_fdm50.obj(i.MTD_CacheProgram) refers to nand_dal.obj(.bss) for Flash_Info
    nand_mtd_fdm50.obj(i.MTD_Read) refers to nand_mtd_fdm50.obj(i.single_Page_Read) for single_Page_Read
    nand_mtd_fdm50.obj(i.MTD_Read) refers to nand_dal.obj(.bss) for Flash_Info
    nand_mtd_fdm50.obj(i.MTD_Erase) refers to nand_mtd_fdm50.obj(i.NFI_OP_RESET) for NFI_OP_RESET
    nand_mtd_fdm50.obj(i.MTD_Erase) refers to nand_dal.obj(.bss) for Flash_Info
    nand_mtd_fdm50.obj(i.MTD_MarkBlockBad) refers to nand_mtd_fdm50.obj(i.single_Page_Program) for single_Page_Program
    nand_mtd_fdm50.obj(i.MTD_MarkBlockBad) refers to nand_mtd_fdm50.obj(i.NFI_OP_RESET) for NFI_OP_RESET
    nand_mtd_fdm50.obj(i.MTD_MarkBlockBad) refers to nand_dal.obj(.bss) for Flash_Info
    nand_mtd_fdm50.obj(i.MTD_CheckBlockBad) refers to nand_mtd_fdm50.obj(i.single_Page_Read) for single_Page_Read
    nand_mtd_fdm50.obj(i.MTD_CheckBlockBad) refers to nand_mtd_fdm50.obj(i.NFI_OP_RESET) for NFI_OP_RESET
    nand_mtd_fdm50.obj(i.MTD_CheckBlockBad) refers to nand_dal.obj(.bss) for Flash_Info
    nand_mtd_fdm50.obj(i.MTD_CheckBlockBad) refers to nand_dal.obj(.constdata) for ZEROBIT
    nand_mtd_fdm50.obj(i.MTD_NAND_Reset) refers to nand_mtd_fdm50.obj(i.NFI_OP_RESET) for NFI_OP_RESET
    nand_mtd_fdm50.obj(i.MTD_NAND_Reset) refers to nand_mtd_fdm50.obj(i.nAND_RESET) for nAND_RESET
    nand_mtd_fdm50.obj(i.nfi_lisr) refers to bl_DBGPRINT.obj(i.dbg_print) for dbg_print
    nand_mtd_fdm50.obj(i.nfi_lisr) refers to nand_mtd_fdm50.obj(.constdata) for .constdata$1
    nand_mtd_fdm50.obj(i.nfi_hisr) refers to bl_DBGPRINT.obj(i.dbg_print) for dbg_print
    nand_mtd_fdm50.obj(i.nfi_hisr) refers to nand_mtd_fdm50.obj(.constdata) for .constdata$1
    nand_mtd_fdm50.obj(i.NFI_DMA_Callback) refers to bl_DBGPRINT.obj(i.dbg_print) for dbg_print
    nand_mtd_fdm50.obj(i.NFI_DMA_Callback) refers to nand_mtd_fdm50.obj(.constdata) for .constdata$1
    usb_custom.obj(i.USB_GetDeviceParam) refers to usb_custom.obj(.constdata) for .constdata$1
    usb_custom.obj(i.USB_GetMsParam) refers to usb_custom.obj(.constdata) for .constdata$1
    usb_custom.obj(i.USB_GetAcmParam) refers to usb_custom.obj(.constdata) for .constdata$1
    usb_custom.obj(i.USB_GetVideoParam) refers to usb_custom.obj(.constdata) for .constdata$1
    usb_custom.obj(i.USB_GetCustomFunc) refers to usb_custom.obj(.constdata) for .constdata$1
    usb_custom.obj(i.USB_PowerControl) refers to usbdl_pmu.obj(i.pmu6253_vusb_enable) for pmu6253_vusb_enable
    usb_custom.obj(.constdata) refers to usb_custom.obj(.constdata) for USB_MANUFACTURER_STRING
    usb_custom.obj(.constdata) refers to usb_custom.obj(.constdata) for USB_PRODUCT_STRING
    usb_custom.obj(.constdata) refers to usb_custom.obj(.constdata) for INQUIRE_DATA
    usb_custom.obj(.constdata) refers to usb_custom.obj(.constdata) for USB_MS_INTERFACE_STRING
    usb_custom.obj(.constdata) refers to usb_custom.obj(.constdata) for USB_ACM_COMM_INTERFACE_STRING
    usb_custom.obj(.constdata) refers to usb_custom.obj(.constdata) for USB_ACM_DATA_INTERFACE_STRING
    usb_custom.obj(.constdata) refers to usb_custom.obj(.constdata) for USB_VIDEO_VC_INTERFACE_STRING
    usb_custom.obj(.constdata) refers to usb_custom.obj(.constdata) for USB_VIDEO_CT_INTERFACE_STRING
    usb_custom.obj(.constdata) refers to usb_custom.obj(.constdata) for USB_VIDEO_OUTPUT_INTERFACE_STRING
    usb_custom.obj(.constdata) refers to usb_custom.obj(.constdata) for USB_VIDEO_PU_INTERFACE_STRING
    usb_custom.obj(.constdata) refers to usb_custom.obj(.constdata) for USB_VIDEO_VS_INTERFACE_STRING
    usb_custom.obj(.constdata) refers to usb_custom.obj(i.USB_GetDeviceParam) for USB_GetDeviceParam
    usb_custom.obj(.constdata) refers to usb_custom.obj(i.USB_GetMsParam) for USB_GetMsParam
    usb_custom.obj(.constdata) refers to usb_custom.obj(i.USB_GetAcmParam) for USB_GetAcmParam
    usb_custom.obj(.constdata) refers to usb_custom.obj(i.USB_GetVideoParam) for USB_GetVideoParam
    usbdl_usb.obj(i.USB_Init_Device_Status) refers to memset.o(.text) for memset
    usbdl_usb.obj(i.USB_Init_Device_Status) refers to usbdl_usb.obj(.bss) for .bss$2
    usbdl_usb.obj(i.USB_Register_EP0_RxHdlr) refers to usbdl_usb.obj(.bss) for .bss$2
    usbdl_usb.obj(i.USB_Generate_EP0Data) refers to usbdl_usb.obj(.bss) for .bss$2
    usbdl_usb.obj(i.USB_Init) refers to usbdl_usb_drv.obj(i.USB_Init_Drv_Info) for USB_Init_Drv_Info
    usbdl_usb.obj(i.USB_Init) refers to usbdl_usb.obj(i.USB_Init_Device_Status) for USB_Init_Device_Status
    usbdl_usb.obj(i.USB_Init) refers to usbdl_usbacm_drv.obj(i.USB_Init_Acm_Status) for USB_Init_Acm_Status
    usbdl_usb.obj(i.USB_Init) refers to usbdl_usb_drv.obj(i.USB_Register_Drv_Info) for USB_Register_Drv_Info
    usbdl_usb.obj(i.USB_Init) refers to usbdl_usb_resource.obj(i.USB_Software_Create) for USB_Software_Create
    usbdl_usb.obj(i.USB_Init) refers to usbdl_usb_drv.obj(i.USB_Reset_Drv) for USB_Reset_Drv
    usbdl_usb.obj(i.USB_Init) refers to usbdl_usb_drv.obj(i.USB_Initialize_Drv) for USB_Initialize_Drv
    usbdl_usb.obj(i.USB_Init) refers to usbdl_usb.obj(i.USB_Initialize) for USB_Initialize
    usbdl_usb.obj(i.USB_Init) refers to usbdl_usb_drv.obj(i.USB_Set_DP_Pull_High) for USB_Set_DP_Pull_High
    usbdl_usb.obj(i.USB_Init) refers to usbdl_usb_resource.obj(i.USB_Software_Init) for USB_Software_Init
    usbdl_usb.obj(i.USB_Init) refers to usbdl_usb.obj(.bss) for .bss$2
    usbdl_usb.obj(i.USB_Init) refers to usbdl_usb.obj(i.USB_Reset) for USB_Reset
    usbdl_usb.obj(i.USB_Init) refers to usbdl_usb.obj(i.USB_Endpoint0_Hdlr) for USB_Endpoint0_Hdlr
    usbdl_usb.obj(i.USB_Initialize) refers to usbdl_usb_resource.obj(i.USB_Software_Speed_Init) for USB_Software_Speed_Init
    usbdl_usb.obj(i.USB_Initialize) refers to usbdl_usb_drv.obj(i.USB_Reset_FIFO) for USB_Reset_FIFO
    usbdl_usb.obj(i.USB_Initialize) refers to usbdl_usb_drv.obj(i.USB_TxEPInit) for USB_TxEPInit
    usbdl_usb.obj(i.USB_Initialize) refers to usbdl_usb_drv.obj(i.USB_RxEPInit) for USB_RxEPInit
    usbdl_usb.obj(i.USB_Initialize) refers to usbdl_usb_resource.obj(i.USB_Software_Init) for USB_Software_Init
    usbdl_usb.obj(i.USB_Initialize) refers to usbdl_usb.obj(.bss) for .bss$2
    usbdl_usb.obj(i.USB_Endpoint0_Hdlr) refers to usbdl_usb_drv.obj(i.USB_Get_EP0_Status) for USB_Get_EP0_Status
    usbdl_usb.obj(i.USB_Endpoint0_Hdlr) refers to usbdl_usb_drv.obj(i.USB_Update_EP0_State) for USB_Update_EP0_State
    usbdl_usb.obj(i.USB_Endpoint0_Hdlr) refers to usbdl_usb_drv.obj(i.USB_EP0_Pkt_Len) for USB_EP0_Pkt_Len
    usbdl_usb.obj(i.USB_Endpoint0_Hdlr) refers to bl_portingfunc.obj(i.kal_assert_fail) for kal_assert_fail
    usbdl_usb.obj(i.USB_Endpoint0_Hdlr) refers to usbdl_usb_drv.obj(i.USB_SetAddress) for USB_SetAddress
    usbdl_usb.obj(i.USB_Endpoint0_Hdlr) refers to usbdl_usb.obj(i.USB_Endpoint0_Idle) for USB_Endpoint0_Idle
    usbdl_usb.obj(i.USB_Endpoint0_Hdlr) refers to usbdl_usb.obj(i.USB_Endpoint0_Tx) for USB_Endpoint0_Tx
    usbdl_usb.obj(i.USB_Endpoint0_Hdlr) refers to usbdl_usb.obj(.bss) for .bss$2
    usbdl_usb.obj(i.USB_Endpoint0_Hdlr) refers to usbdl_usb.obj(.constdata) for .constdata$1
    usbdl_usb.obj(i.USB_Reset) refers to usbdl_usb_drv.obj(i.USB_ResetDrv_Info) for USB_ResetDrv_Info
    usbdl_usb.obj(i.USB_Reset) refers to usbdl_usb_drv.obj(i.USB_Initialize_Drv) for USB_Initialize_Drv
    usbdl_usb.obj(i.USB_Reset) refers to usbdl_usb.obj(i.USB_Initialize) for USB_Initialize
    usbdl_usb.obj(i.USB_Reset) refers to usbdl_usb.obj(.bss) for .bss$2
    usbdl_usb.obj(i.USB_Endpoint0_Tx) refers to usbdl_usb_drv.obj(i.USB_EPFIFOWrite) for USB_EPFIFOWrite
    usbdl_usb.obj(i.USB_Endpoint0_Tx) refers to usbdl_usb_drv.obj(i.USB_Update_EP0_State) for USB_Update_EP0_State
    usbdl_usb.obj(i.USB_Endpoint0_Tx) refers to usbdl_usb.obj(.bss) for .bss$2
    usbdl_usb.obj(i.USB_Endpoint0_Idle) refers to usbdl_usb_drv.obj(i.USB_EPFIFORead) for USB_EPFIFORead
    usbdl_usb.obj(i.USB_Endpoint0_Idle) refers to usbdl_usb.obj(i.USB_Stdcmd) for USB_Stdcmd
    usbdl_usb.obj(i.USB_Endpoint0_Idle) refers to usbdl_usb_drv.obj(i.USB_Update_EP0_State) for USB_Update_EP0_State
    usbdl_usb.obj(i.USB_Endpoint0_Idle) refers to usbdl_usb.obj(.bss) for .bss$2
    usbdl_usb.obj(i.USB_Stdcmd) refers to usbdl_debug_tool.obj(i.drv_get_current_time) for drv_get_current_time
    usbdl_usb.obj(i.USB_Stdcmd) refers to usbdl_debug_tool.obj(i.USB_Dbg_Trace) for USB_Dbg_Trace
    usbdl_usb.obj(i.USB_Stdcmd) refers to usbdl_usb_drv.obj(i.USB_SetAddress) for USB_SetAddress
    usbdl_usb.obj(i.USB_Stdcmd) refers to usbdl_usb.obj(i.USB_Cmd_GetDescriptor) for USB_Cmd_GetDescriptor
    usbdl_usb.obj(i.USB_Stdcmd) refers to usbdl_usb.obj(i.USB_Generate_EP0Data) for USB_Generate_EP0Data
    usbdl_usb.obj(i.USB_Stdcmd) refers to usbdl_usb.obj(i.USB_Cmd_SetFeature) for USB_Cmd_SetFeature
    usbdl_usb.obj(i.USB_Stdcmd) refers to usbdl_usb.obj(i.USB_Cmd_GetStatus) for USB_Cmd_GetStatus
    usbdl_usb.obj(i.USB_Stdcmd) refers to usbdl_usb_drv.obj(i.USB_Update_EP0_State) for USB_Update_EP0_State
    usbdl_usb.obj(i.USB_Stdcmd) refers to usbdl_usb.obj(.bss) for .bss$2
    usbdl_usb.obj(i.USB_Cmd_GetStatus) refers to usbdl_usb_drv.obj(i.USB_Get_EP_Stall_Status) for USB_Get_EP_Stall_Status
    usbdl_usb.obj(i.USB_Cmd_GetStatus) refers to usbdl_usb.obj(i.USB_Generate_EP0Data) for USB_Generate_EP0Data
    usbdl_usb.obj(i.USB_Cmd_GetStatus) refers to usbdl_usb.obj(.bss) for .bss$2
    usbdl_usb.obj(i.USB_Cmd_SetFeature) refers to usbdl_usb_drv.obj(i.USB_CtrlEPStall) for USB_CtrlEPStall
    usbdl_usb.obj(i.USB_Cmd_SetFeature) refers to usbdl_usb.obj(.bss) for .bss$2
    usbdl_usb.obj(i.USB_Cmd_GetDescriptor) refers to usbdl_usb_resource.obj(i.USB_Software_Speed_Init) for USB_Software_Speed_Init
    usbdl_usb.obj(i.USB_Cmd_GetDescriptor) refers to usbdl_usb.obj(i.USB_Generate_EP0Data) for USB_Generate_EP0Data
    usbdl_usb.obj(i.USB_Cmd_GetDescriptor) refers to usbdl_usb.obj(.bss) for .bss$2
    usbdl_usb_drv.obj(i.USB_Init_Drv_Info) refers to usbdl_usb_drv.obj(.bss) for .bss$2
    usbdl_usb_drv.obj(i.USB_ResetDrv_Info) refers to usbdl_usb_drv.obj(.bss) for .bss$2
    usbdl_usb_drv.obj(i.USB_Register_Drv_Info) refers to usbdl_usb_drv.obj(i.USB_EP_Check) for USB_EP_Check
    usbdl_usb_drv.obj(i.USB_Register_Drv_Info) refers to usbdl_usb_drv.obj(.bss) for .bss$2
    usbdl_usb_drv.obj(i.USB_Get_EP_Stall_Status) refers to usbdl_usb_drv.obj(i.USB_EP_Check) for USB_EP_Check
    usbdl_usb_drv.obj(i.USB_Get_EP_Stall_Status) refers to usbdl_usb_drv.obj(.bss) for .bss$2
    usbdl_usb_drv.obj(i.USB_PDNDisable) refers to bl_portingfunc.obj(i.SaveAndSetIRQMask) for SaveAndSetIRQMask
    usbdl_usb_drv.obj(i.USB_PDNDisable) refers to bl_portingfunc.obj(i.RestoreIRQMask) for RestoreIRQMask
    usbdl_usb_drv.obj(i.USB_PDNDisable) refers to usbdl_usb_drv.obj(.bss) for .bss$2
    usbdl_usb_drv.obj(i.USBDL_USBPowerON) refers to usbdl_usb_drv.obj(i.USB_PDNDisable) for USB_PDNDisable
    usbdl_usb_drv.obj(i.USBDL_USBPowerON) refers to usb_custom.obj(i.USB_PowerControl) for USB_PowerControl
    usbdl_usb_drv.obj(i.USBDL_USBPowerON) refers to usbdl_usb_drv.obj(i.USB_UART_Share) for USB_UART_Share
    usbdl_usb_drv.obj(i.USB_Reset_Drv) refers to usbdl_usb_drv.obj(i.USB_High_Speed_Enable) for USB_High_Speed_Enable
    usbdl_usb_drv.obj(i.USB_Initialize_Drv) refers to usbdl_usb_drv.obj(i.USB_EnSysIntr) for USB_EnSysIntr
    usbdl_usb_drv.obj(i.USB_Initialize_Drv) refers to usbdl_usb_drv.obj(i.USB_EP0En) for USB_EP0En
    usbdl_usb_drv.obj(i.USB_TxEPInit) refers to bl_portingfunc.obj(i.kal_assert_fail) for kal_assert_fail
    usbdl_usb_drv.obj(i.USB_TxEPInit) refers to usbdl_usb_drv.obj(.constdata) for .constdata$1
    usbdl_usb_drv.obj(i.USB_TxEPInit) refers to usbdl_usb_drv.obj(.data) for .data$0
    usbdl_usb_drv.obj(i.USB_RxEPInit) refers to bl_portingfunc.obj(i.kal_assert_fail) for kal_assert_fail
    usbdl_usb_drv.obj(i.USB_RxEPInit) refers to usbdl_usb_drv.obj(.constdata) for .constdata$1
    usbdl_usb_drv.obj(i.USB_RxEPInit) refers to usbdl_usb_drv.obj(.data) for .data$0
    usbdl_usb_drv.obj(i.USB_TxEPEn) refers to bl_portingfunc.obj(i.kal_assert_fail) for kal_assert_fail
    usbdl_usb_drv.obj(i.USB_TxEPEn) refers to usbdl_usb_drv.obj(.constdata) for .constdata$1
    usbdl_usb_drv.obj(i.USB_RxEPEn) refers to bl_portingfunc.obj(i.kal_assert_fail) for kal_assert_fail
    usbdl_usb_drv.obj(i.USB_RxEPEn) refers to usbdl_usb_drv.obj(.constdata) for .constdata$1
    usbdl_usb_drv.obj(i.USB_EPFIFORead_Shift) refers to bl_portingfunc.obj(i.kal_assert_fail) for kal_assert_fail
    usbdl_usb_drv.obj(i.USB_EPFIFORead_Shift) refers to usbdl_usb_drv.obj(.constdata) for .constdata$1
    usbdl_usb_drv.obj(i.USB_EPFIFORead) refers to usbdl_usb_drv.obj(i.USB_EPFIFORead_Shift) for USB_EPFIFORead_Shift
    usbdl_usb_drv.obj(i.USB_EPFIFOWrite) refers to bl_portingfunc.obj(i.kal_assert_fail) for kal_assert_fail
    usbdl_usb_drv.obj(i.USB_EPFIFOWrite) refers to usbdl_usb_drv.obj(.constdata) for .constdata$1
    usbdl_usb_drv.obj(i.USB_CtrlEPStall) refers to usbdl_usb_drv.obj(i.USB_EP_Check) for USB_EP_Check
    usbdl_usb_drv.obj(i.USB_CtrlEPStall) refers to usbdl_usb_drv.obj(.bss) for .bss$2
    usbdl_usb_drv.obj(i.USB_EP_Bulk_Tx_Ready) refers to usbdl_usb_drv.obj(i.USB_EP_Check) for USB_EP_Check
    usbdl_usb_drv.obj(i.USB_EP_Bulk_Tx_Ready) refers to bl_portingfunc.obj(i.kal_assert_fail) for kal_assert_fail
    usbdl_usb_drv.obj(i.USB_EP_Bulk_Tx_Ready) refers to usbdl_usb_drv.obj(.constdata) for .constdata$1
    usbdl_usb_drv.obj(i.USB_EP_Rx_Pkt_Len) refers to usbdl_usb_drv.obj(i.USB_EP_Check) for USB_EP_Check
    usbdl_usb_drv.obj(i.USB_EP_Bulk_Rx_Ready) refers to usbdl_usb_drv.obj(i.USB_EP_Check) for USB_EP_Check
    usbdl_usb_drv.obj(i.USB_Is_EP_Bulk_Tx_Empty) refers to usbdl_usb_drv.obj(i.USB_EP_Check) for USB_EP_Check
    usbdl_usb_drv.obj(i.USB_Charger_Detect_Init) refers to usbdl_usb_drv.obj(i.USB_UART_Share) for USB_UART_Share
    usbdl_usb_drv.obj(i.USB_Reset_FIFO) refers to usbdl_usb_drv.obj(.data) for .data$0
    usbdl_usb_drv.obj(i.USB_HISR) refers to bl_portingfunc.obj(i.kal_assert_fail) for kal_assert_fail
    usbdl_usb_drv.obj(i.USB_HISR) refers to usbdl_usb_drv.obj(i.USB_Is_High_Speed) for USB_Is_High_Speed
    usbdl_usb_drv.obj(i.USB_HISR) refers to usbdl_usb_drv.obj(.bss) for .bss$2
    usbdl_usb_drv.obj(i.USB_HISR) refers to usbdl_usb_drv.obj(.constdata) for .constdata$1
    usbdl_usb_drv.obj(i.USB_EP_Check) refers to bl_portingfunc.obj(i.kal_assert_fail) for kal_assert_fail
    usbdl_usb_drv.obj(i.USB_EP_Check) refers to usbdl_usb_drv.obj(.constdata) for .constdata$1
    usbdl_usb_resource.obj(i.USB_Register_CreateFunc) refers to bl_portingfunc.obj(i.kal_assert_fail) for kal_assert_fail
    usbdl_usb_resource.obj(i.USB_Register_CreateFunc) refers to usbdl_usb_resource.obj(.bss) for .bss$2
    usbdl_usb_resource.obj(i.USB_Register_CreateFunc) refers to usbdl_usb_resource.obj(.constdata) for .constdata$1
    usbdl_usb_resource.obj(i.USB_Register_Device_Code) refers to bl_portingfunc.obj(i.kal_assert_fail) for kal_assert_fail
    usbdl_usb_resource.obj(i.USB_Register_Device_Code) refers to usbdl_usb_resource.obj(.bss) for .bss$2
    usbdl_usb_resource.obj(i.USB_Register_Device_Code) refers to usbdl_usb_resource.obj(.constdata) for .constdata$1
    usbdl_usb_resource.obj(i.USB_DeRegister_CreateFunc) refers to usbdl_usb_resource.obj(.bss) for .bss$2
    usbdl_usb_resource.obj(i.USB_DeRegister_Device_Code) refers to usbdl_usb_resource.obj(.bss) for .bss$2
    usbdl_usb_resource.obj(i.USB_Get_Intr_Ep) refers to bl_portingfunc.obj(i.kal_assert_fail) for kal_assert_fail
    usbdl_usb_resource.obj(i.USB_Get_Intr_Ep) refers to usbdl_usb.obj(.bss) for gUsbDevice
    usbdl_usb_resource.obj(i.USB_Get_Intr_Ep) refers to usbdl_usb_resource.obj(.constdata) for .constdata$1
    usbdl_usb_resource.obj(i.USB_Get_Bulk_Tx_Ep) refers to bl_portingfunc.obj(i.kal_assert_fail) for kal_assert_fail
    usbdl_usb_resource.obj(i.USB_Get_Bulk_Tx_Ep) refers to usbdl_usb.obj(.bss) for gUsbDevice
    usbdl_usb_resource.obj(i.USB_Get_Bulk_Tx_Ep) refers to usbdl_usb_resource.obj(.constdata) for .constdata$1
    usbdl_usb_resource.obj(i.USB_Get_Bulk_Rx_Ep) refers to bl_portingfunc.obj(i.kal_assert_fail) for kal_assert_fail
    usbdl_usb_resource.obj(i.USB_Get_Bulk_Rx_Ep) refers to usbdl_usb.obj(.bss) for gUsbDevice
    usbdl_usb_resource.obj(i.USB_Get_Bulk_Rx_Ep) refers to usbdl_usb_resource.obj(.constdata) for .constdata$1
    usbdl_usb_resource.obj(i.USB_Get_Interface_Number) refers to bl_portingfunc.obj(i.kal_assert_fail) for kal_assert_fail
    usbdl_usb_resource.obj(i.USB_Get_Interface_Number) refers to usbdl_usb.obj(.bss) for gUsbDevice
    usbdl_usb_resource.obj(i.USB_Get_Interface_Number) refers to usbdl_usb_resource.obj(.constdata) for .constdata$1
    usbdl_usb_resource.obj(i.USB_Get_String_Number) refers to bl_portingfunc.obj(i.kal_assert_fail) for kal_assert_fail
    usbdl_usb_resource.obj(i.USB_Get_String_Number) refers to usbdl_usb.obj(.bss) for gUsbDevice
    usbdl_usb_resource.obj(i.USB_Get_String_Number) refers to usbdl_usb_resource.obj(.constdata) for .constdata$1
    usbdl_usb_resource.obj(i.USB_Software_Speed_Init) refers to bl_portingfunc.obj(i.kal_assert_fail) for kal_assert_fail
    usbdl_usb_resource.obj(i.USB_Software_Speed_Init) refers to memcpy.o(.text) for memcpy
    usbdl_usb_resource.obj(i.USB_Software_Speed_Init) refers to usbdl_usb_resource.obj(.bss) for .bss$2
    usbdl_usb_resource.obj(i.USB_Software_Speed_Init) refers to usbdl_usb_resource.obj(.constdata) for .constdata$1
    usbdl_usb_resource.obj(i.USB_Software_Speed_Init) refers to usbdl_usb.obj(.bss) for gUsbDevice
    usbdl_usb_resource.obj(i.USB_Software_Create) refers to usbdl_usb_resource.obj(i.USB_Get_String_Number) for USB_Get_String_Number
    usbdl_usb_resource.obj(i.USB_Software_Create) refers to bl_portingfunc.obj(i.kal_assert_fail) for kal_assert_fail
    usbdl_usb_resource.obj(i.USB_Software_Create) refers to usbdl_usb_resource.obj(i.USB_Software_Speed_Init) for USB_Software_Speed_Init
    usbdl_usb_resource.obj(i.USB_Software_Create) refers to usbdl_usb.obj(.bss) for gUsbDevice
    usbdl_usb_resource.obj(i.USB_Software_Create) refers to usbdl_usb_resource.obj(.constdata) for .constdata$1
    usbdl_usb_resource.obj(i.USB_Software_Create) refers to usbdl_usb_resource.obj(.bss) for .bss$2
    usbdl_usb_resource.obj(i.USB_Software_Init) refers to bl_portingfunc.obj(i.kal_assert_fail) for kal_assert_fail
    usbdl_usb_resource.obj(i.USB_Software_Init) refers to usbdl_usb_resource.obj(.bss) for .bss$2
    usbdl_usb_resource.obj(i.USB_Software_Init) refers to usbdl_usb_resource.obj(.constdata) for .constdata$1
    usbdl_usbacm_adap.obj(i.keypad_customize_init) refers to keypad_def.obj(i.keypad_GetFunc) for keypad_GetFunc
    usbdl_usbacm_adap.obj(i.keypad_customize_init) refers to usbdl_usbacm_adap.obj(.bss) for .bss$2
    usbdl_usbacm_adap.obj(i.USBDLKey_Pressed) refers to keypad_def.obj(i.keypad_GetFunc) for keypad_GetFunc
    usbdl_usbacm_adap.obj(i.USBDLKey_Pressed) refers to bl_portingfunc.obj(i.kal_assert_fail) for kal_assert_fail
    usbdl_usbacm_adap.obj(i.USBDLKey_Pressed) refers to usbdl_usbacm_adap.obj(.data) for .data$0
    usbdl_usbacm_adap.obj(i.USBDLKey_Pressed) refers to usbdl_usbacm_adap.obj(.bss) for .bss$2
    usbdl_usbacm_adap.obj(i.USBDLKey_Pressed) refers to custom_blconfig.obj(.constdata) for usbdlkey_position
    usbdl_usbacm_adap.obj(i.USBDLKey_Pressed) refers to usbdl_usbacm_adap.obj(.constdata) for .constdata$1
    usbdl_usbacm_adap.obj(i.USBDL_Update_USB_Download_Mode) refers to bl_Main.obj(EXT_BOOTLOADER_CODE) for USBDL_Ready_To_Enter_DLMode
    usbdl_usbacm_adap.obj(i.USBDL_Update_USB_Download_Mode) refers to usbdl_usbacm_adap.obj(.bss) for .bss$2
    usbdl_usbacm_adap.obj(i.USBDL_Update_USB_Download_Mode) refers to usbdl_usb.obj(.bss) for gUsbDevice
    usbdl_usbacm_adap.obj(i.USBDL_Is_USB_Download_Mode) refers to usbdl_usbacm_adap.obj(.bss) for .bss$2
    usbdl_usbacm_adap.obj(i.USBDL_hwInit) refers to gpio_drv.obj(i.GPIO_init) for GPIO_init
    usbdl_usbacm_adap.obj(i.USBDL_hwInit) refers to usbdl_usb_drv.obj(i.USBDL_USBPowerON) for USBDL_USBPowerON
    usbdl_usbacm_adap.obj(i.USBDL_ACMInit) refers to usb_custom.obj(i.USB_GetCustomFunc) for USB_GetCustomFunc
    usbdl_usbacm_adap.obj(i.USBDL_ACMInit) refers to usbdl_usb_resource.obj(i.USB_Register_CreateFunc) for USB_Register_CreateFunc
    usbdl_usbacm_adap.obj(i.USBDL_ACMInit) refers to usbdl_usb_resource.obj(i.USB_Register_Device_Code) for USB_Register_Device_Code
    usbdl_usbacm_adap.obj(i.USBDL_ACMInit) refers to usbdl_usb.obj(i.USB_Init) for USB_Init
    usbdl_usbacm_adap.obj(i.USBDL_ACMInit) refers to usbdl_usb.obj(.bss) for gUsbDevice
    usbdl_usbacm_adap.obj(i.USBDL_ACMInit) refers to usbdl_usbacm_drv.obj(.bss) for g_UsbACM
    usbdl_usbacm_adap.obj(i.USBDL_ACMInit) refers to usbdl_usbacm_drv.obj(i.USB_Acm_DataIf_Speed_Reset) for USB_Acm_DataIf_Speed_Reset
    usbdl_usbacm_adap.obj(i.USBDL_ACMInit) refers to usbdl_usbacm_drv.obj(i.USB_Acm_DataIf_Reset) for USB_Acm_DataIf_Reset
    usbdl_usbacm_adap.obj(i.USBDL_ACMInit) refers to usbdl_usbacm_drv.obj(i.USB_Acm_DataIf_Create) for USB_Acm_DataIf_Create
    usbdl_usbacm_adap.obj(i.USBDL_ACMInit) refers to usbdl_usbacm_adap.obj(.constdata) for .constdata$1
    usbdl_usbacm_adap.obj(i.USBDL_ACMInit) refers to usbdl_usbacm_drv.obj(i.USB_Acm_CommIf_Speed_Reset) for USB_Acm_CommIf_Speed_Reset
    usbdl_usbacm_adap.obj(i.USBDL_ACMInit) refers to usbdl_usbacm_drv.obj(i.USB_Acm_CommIf_Reset) for USB_Acm_CommIf_Reset
    usbdl_usbacm_adap.obj(i.USBDL_ACMInit) refers to usbdl_usbacm_drv.obj(i.USB_Acm_CommIf_Create) for USB_Acm_CommIf_Create
    usbdl_usbacm_adap.obj(i.USBDL_UART_Init) refers to usbdl_usbacm_adap.obj(i.USBDL_hwInit) for USBDL_hwInit
    usbdl_usbacm_adap.obj(i.USBDL_UART_Init) refers to bl_Init.obj(EXT_BOOTLOADER_CODE) for InitUSBDLGPIO
    usbdl_usbacm_adap.obj(i.USBDL_UART_Init) refers to usbdl_usbacm_adap.obj(i.USBDL_ACMInit) for USBDL_ACMInit
    usbdl_usbacm_adap.obj(i.USBDL_UART_Init) refers to usbdl_usb_drv.obj(i.USB_HISR) for USB_HISR
    usbdl_usbacm_adap.obj(i.USBDL_UART_Init) refers to usbdl_usbacm_adap.obj(i.USBDL_Update_USB_Download_Mode) for USBDL_Update_USB_Download_Mode
    usbdl_usbacm_adap.obj(i.USBDL_UART_Init) refers to usbdl_usb_drv.obj(i.USB_TxEPEn) for USB_TxEPEn
    usbdl_usbacm_adap.obj(i.USBDL_UART_Init) refers to usbdl_usb_drv.obj(i.USB_RxEPEn) for USB_RxEPEn
    usbdl_usbacm_adap.obj(i.USBDL_UART_Init) refers to usbdl_usb.obj(.bss) for gUsbDevice
    usbdl_usbacm_adap.obj(i.USBDL_UART_Init) refers to usbdl_usbacm_adap.obj(.bss) for .bss$2
    usbdl_usbacm_adap.obj(i.USBDL_UART_Init) refers to usbdl_usbacm_drv.obj(.bss) for g_UsbACM
    usbdl_usbacm_adap.obj(i.USBDL_Release) refers to usbdl_usb_drv.obj(i.USB_UART_Share) for USB_UART_Share
    usbdl_usbacm_adap.obj(i.USBDL_Release) refers to usbdl_usbacm_drv.obj(i.USB_Release_Acm_Status) for USB_Release_Acm_Status
    usbdl_usbacm_adap.obj(i.USBDL_Release) refers to usbdl_usb_resource.obj(i.USB_DeRegister_CreateFunc) for USB_DeRegister_CreateFunc
    usbdl_usbacm_adap.obj(i.USBDL_Release) refers to usbdl_usb_resource.obj(i.USB_DeRegister_Device_Code) for USB_DeRegister_Device_Code
    usbdl_usbacm_adap.obj(i.USBDL_Release) refers to usbdl_usb_drv.obj(i.USBDL_USBPowerON) for USBDL_USBPowerON
    usbdl_usbacm_adap.obj(i.USBDL_Release) refers to usbdl_usbacm_adap.obj(.bss) for .bss$2
    usbdl_usbacm_adap.obj(i.USB_Charger_Detect) refers to usbdl_usb_drv.obj(i.USB_Charger_Detect_Init) for USB_Charger_Detect_Init
    usbdl_usbacm_adap.obj(i.USB_Charger_Detect) refers to usbdl_usb_drv.obj(i.USB_Detect_Is_Charger_In) for USB_Detect_Is_Charger_In
    usbdl_usbacm_adap.obj(i.USB_Charger_Detect) refers to usbdl_usb_drv.obj(i.USB_Charger_Detect_Release) for USB_Charger_Detect_Release
    usbdl_usbacm_adap.obj(i.USBDL_PutUARTByte_Ext) refers to bl_Main.obj(EXT_BOOTLOADER_CODE) for USBDL_Is_Timeout
    usbdl_usbacm_adap.obj(i.USBDL_PutUARTByte_Ext) refers to usbdl_usb_drv.obj(i.USB_Is_High_Speed) for USB_Is_High_Speed
    usbdl_usbacm_adap.obj(i.USBDL_PutUARTByte_Ext) refers to usbdl_usb_drv.obj(i.USB_EPFIFOWrite) for USB_EPFIFOWrite
    usbdl_usbacm_adap.obj(i.USBDL_PutUARTByte_Ext) refers to usbdl_usb_drv.obj(i.USB_EP_Bulk_Tx_Ready) for USB_EP_Bulk_Tx_Ready
    usbdl_usbacm_adap.obj(i.USBDL_PutUARTByte_Ext) refers to usbdl_usb_drv.obj(i.USB_HISR) for USB_HISR
    usbdl_usbacm_adap.obj(i.USBDL_PutUARTByte_Ext) refers to usbdl_usb.obj(.bss) for gUsbDevice
    usbdl_usbacm_adap.obj(i.USBDL_PutUARTByte_Ext) refers to usbdl_usbacm_adap.obj(.bss) for .bss$2
    usbdl_usbacm_adap.obj(i.USBDL_PutUARTByte_Ext) refers to usbdl_usbacm_drv.obj(.bss) for g_UsbACM
    usbdl_usbacm_adap.obj(i.USBDL_PutUARTByte) refers to usbdl_usbacm_adap.obj(i.USBDL_PutUARTByte_Ext) for USBDL_PutUARTByte_Ext
    usbdl_usbacm_adap.obj(i.USBDL_PutUARTByte_Complete_Ext) refers to bl_Main.obj(EXT_BOOTLOADER_CODE) for USBDL_Is_Timeout
    usbdl_usbacm_adap.obj(i.USBDL_PutUARTByte_Complete_Ext) refers to usbdl_usb_drv.obj(i.USB_EPFIFOWrite) for USB_EPFIFOWrite
    usbdl_usbacm_adap.obj(i.USBDL_PutUARTByte_Complete_Ext) refers to usbdl_usb_drv.obj(i.USB_EP_Bulk_Tx_Ready) for USB_EP_Bulk_Tx_Ready
    usbdl_usbacm_adap.obj(i.USBDL_PutUARTByte_Complete_Ext) refers to usbdl_usb_drv.obj(i.USB_HISR) for USB_HISR
    usbdl_usbacm_adap.obj(i.USBDL_PutUARTByte_Complete_Ext) refers to usbdl_usb.obj(.bss) for gUsbDevice
    usbdl_usbacm_adap.obj(i.USBDL_PutUARTByte_Complete_Ext) refers to usbdl_usbacm_adap.obj(.bss) for .bss$2
    usbdl_usbacm_adap.obj(i.USBDL_PutUARTByte_Complete_Ext) refers to usbdl_usbacm_drv.obj(.bss) for g_UsbACM
    usbdl_usbacm_adap.obj(i.USBDL_PutUARTByte_Complete) refers to usbdl_usbacm_adap.obj(i.USBDL_PutUARTByte_Complete_Ext) for USBDL_PutUARTByte_Complete_Ext
    usbdl_usbacm_adap.obj(i.USBDL_GetUARTByte_Ext) refers to bl_Main.obj(EXT_BOOTLOADER_CODE) for USBDL_Is_Timeout
    usbdl_usbacm_adap.obj(i.USBDL_GetUARTByte_Ext) refers to usbdl_usb_drv.obj(i.USB_HISR) for USB_HISR
    usbdl_usbacm_adap.obj(i.USBDL_GetUARTByte_Ext) refers to usbdl_usbacm_adap.obj(.bss) for .bss$2
    usbdl_usbacm_adap.obj(i.USBDL_GetUARTByte) refers to usbdl_usbacm_adap.obj(i.USBDL_GetUARTByte_Ext) for USBDL_GetUARTByte_Ext
    usbdl_usbacm_adap.obj(i.USBDL_CheckStartCmd) refers to usbdl_usbacm_adap.obj(i.USBDL_GetUARTByte_Ext) for USBDL_GetUARTByte_Ext
    usbdl_usbacm_adap.obj(i.USBDL_CheckStartCmd) refers to usbdl_usbacm_adap.obj(i.USBDL_PutUARTByte_Ext) for USBDL_PutUARTByte_Ext
    usbdl_usbacm_adap.obj(i.USBDL_CheckStartCmd) refers to usbdl_usbacm_adap.obj(i.USBDL_PutUARTByte_Complete_Ext) for USBDL_PutUARTByte_Complete_Ext
    usbdl_usbacm_adap.obj(i.USBDL_CheckStartCmd) refers to bl_Main.obj(EXT_BOOTLOADER_CODE) for USBDL_Is_Timeout
    usbdl_usbacm_adap.obj(i.USBDL_CheckStartCmd) refers to usbdl_usbacm_adap.obj(.constdata) for .constdata$1
    usbdl_usbacm_adap.obj(i.USBDL_USB_Config_Init) refers to usbdl_usbacm_adap.obj(i.USBDL_ACMInit) for USBDL_ACMInit
    usbdl_usbacm_adap.obj(i.USBDL_USB_Config_Init) refers to usbdl_usbacm_drv.obj(.bss) for g_UsbACM
    usbdl_usbacm_adap.obj(i.USBDL_USB_Config_Init) refers to usbdl_usb.obj(.bss) for gUsbDevice
    usbdl_usbacm_adap.obj(i.USBDL_USB_Config_Init) refers to usbdl_usbacm_adap.obj(.bss) for .bss$2
    usbdl_usbacm_drv.obj(i.USB_Acm_CommIf_Create) refers to usbdl_usb_resource.obj(i.USB_Get_Interface_Number) for USB_Get_Interface_Number
    usbdl_usbacm_drv.obj(i.USB_Acm_CommIf_Create) refers to usbdl_usb_resource.obj(i.USB_Get_Intr_Ep) for USB_Get_Intr_Ep
    usbdl_usbacm_drv.obj(i.USB_Acm_CommIf_Create) refers to usbdl_usb_resource.obj(i.USB_Get_String_Number) for USB_Get_String_Number
    usbdl_usbacm_drv.obj(i.USB_Acm_CommIf_Create) refers to usbdl_usb_drv.obj(i.USB_Register_Drv_Info) for USB_Register_Drv_Info
    usbdl_usbacm_drv.obj(i.USB_Acm_CommIf_Create) refers to usbdl_usbacm_drv.obj(.bss) for .bss$2
    usbdl_usbacm_drv.obj(i.USB_Acm_CommIf_Create) refers to usbdl_usbacm_drv.obj(i.USB_Acm_Ep0_Command) for USB_Acm_Ep0_Command
    usbdl_usbacm_drv.obj(i.USB_Acm_CommIf_Reset) refers to usbdl_usbacm_drv.obj(.bss) for .bss$2
    usbdl_usbacm_drv.obj(i.USB_Acm_CommIf_Speed_Reset) refers to usbdl_usbacm_drv.obj(.bss) for .bss$2
    usbdl_usbacm_drv.obj(i.USB_Acm_DataIf_Create) refers to usbdl_usb_resource.obj(i.USB_Get_Interface_Number) for USB_Get_Interface_Number
    usbdl_usbacm_drv.obj(i.USB_Acm_DataIf_Create) refers to usbdl_usb_resource.obj(i.USB_Get_Bulk_Tx_Ep) for USB_Get_Bulk_Tx_Ep
    usbdl_usbacm_drv.obj(i.USB_Acm_DataIf_Create) refers to usbdl_usb_resource.obj(i.USB_Get_Bulk_Rx_Ep) for USB_Get_Bulk_Rx_Ep
    usbdl_usbacm_drv.obj(i.USB_Acm_DataIf_Create) refers to usbdl_usb_resource.obj(i.USB_Get_String_Number) for USB_Get_String_Number
    usbdl_usbacm_drv.obj(i.USB_Acm_DataIf_Create) refers to usbdl_usb_drv.obj(i.USB_Register_Drv_Info) for USB_Register_Drv_Info
    usbdl_usbacm_drv.obj(i.USB_Acm_DataIf_Create) refers to usbdl_usbacm_drv.obj(.bss) for .bss$2
    usbdl_usbacm_drv.obj(i.USB_Acm_DataIf_Create) refers to usbdl_usbacm_drv.obj(i.USB_Acm_BulkIn_Hdr) for USB_Acm_BulkIn_Hdr
    usbdl_usbacm_drv.obj(i.USB_Acm_DataIf_Create) refers to usbdl_usbacm_drv.obj(i.USB_Acm_BulkIn_Reset) for USB_Acm_BulkIn_Reset
    usbdl_usbacm_drv.obj(i.USB_Acm_DataIf_Create) refers to usbdl_usbacm_drv.obj(i.USB_Acm_BulkOut_Hdr) for USB_Acm_BulkOut_Hdr
    usbdl_usbacm_drv.obj(i.USB_Acm_DataIf_Create) refers to usbdl_usbacm_drv.obj(i.USB_Acm_BulkOut_Reset) for USB_Acm_BulkOut_Reset
    usbdl_usbacm_drv.obj(i.USB_Acm_DataIf_Reset) refers to usbdl_usb_drv.obj(i.USB_TxEPEn) for USB_TxEPEn
    usbdl_usbacm_drv.obj(i.USB_Acm_DataIf_Reset) refers to usbdl_usb_drv.obj(i.USB_RxEPEn) for USB_RxEPEn
    usbdl_usbacm_drv.obj(i.USB_Acm_DataIf_Reset) refers to usbdl_usbacm_drv.obj(.bss) for .bss$2
    usbdl_usbacm_drv.obj(i.USB_Acm_DataIf_Speed_Reset) refers to usbdl_usb_drv.obj(i.USB_Is_High_Speed) for USB_Is_High_Speed
    usbdl_usbacm_drv.obj(i.USB_Acm_DataIf_Speed_Reset) refers to usbdl_usbacm_drv.obj(.bss) for .bss$2
    usbdl_usbacm_drv.obj(i.USB_Init_Acm_Status) refers to usbdl_usbacm_drv.obj(.bss) for .bss$2
    usbdl_usbacm_drv.obj(i.USB_Release_Acm_Status) refers to usbdl_usbacm_drv.obj(.bss) for .bss$2
    usbdl_usbacm_drv.obj(i.USB_Acm_Ep0_Command) refers to usbdl_usb.obj(i.USB_Register_EP0_RxHdlr) for USB_Register_EP0_RxHdlr
    usbdl_usbacm_drv.obj(i.USB_Acm_Ep0_Command) refers to usbdl_usb.obj(i.USB_Generate_EP0Data) for USB_Generate_EP0Data
    usbdl_usbacm_drv.obj(i.USB_Acm_Ep0_Command) refers to usbdl_usb_drv.obj(i.USB_Update_EP0_State) for USB_Update_EP0_State
    usbdl_usbacm_drv.obj(i.USB_Acm_Ep0_Command) refers to usbdl_usb.obj(.bss) for gUsbDevice
    usbdl_usbacm_drv.obj(i.USB_Acm_Ep0_Command) refers to usbdl_usbacm_drv.obj(i.USB_Acm_Ep0_SetLineCoding) for USB_Acm_Ep0_SetLineCoding
    usbdl_usbacm_drv.obj(i.USB_Acm_Ep0_Command) refers to usbdl_usbacm_drv.obj(.bss) for .bss$2
    usbdl_usbacm_drv.obj(i.USB_Acm_BulkOut_Reset) refers to usbdl_usbacm_drv.obj(.bss) for .bss$2
    usbdl_usbacm_drv.obj(i.USB_Acm_BulkOut_Reset) refers to usbdl_usbacm_adap.obj(.bss) for usbacm_rx_buf
    usbdl_usbacm_drv.obj(i.USB_Acm_BulkOut_Hdr) refers to usbdl_usb_drv.obj(i.USB_EP_Rx_Pkt_Len) for USB_EP_Rx_Pkt_Len
    usbdl_usbacm_drv.obj(i.USB_Acm_BulkOut_Hdr) refers to usbdl_usb_drv.obj(i.USB_EPFIFORead) for USB_EPFIFORead
    usbdl_usbacm_drv.obj(i.USB_Acm_BulkOut_Hdr) refers to usbdl_usb_drv.obj(i.USB_EP_Bulk_Rx_Ready) for USB_EP_Bulk_Rx_Ready
    usbdl_usbacm_drv.obj(i.USB_Acm_BulkOut_Hdr) refers to usbdl_usbacm_adap.obj(.bss) for usbacm_rx_buf
    usbdl_usbacm_drv.obj(i.USB_Acm_BulkOut_Hdr) refers to usbdl_usbacm_drv.obj(.bss) for .bss$2
    usbdl_usbacm_drv.obj(i.USB_Acm_BulkIn_Reset) refers to usbdl_usbacm_drv.obj(.bss) for .bss$2
    usbdl_usbacm_drv.obj(i.USB_Acm_BulkIn_Reset) refers to usbdl_usbacm_adap.obj(.bss) for usbacm_tx_buf
    usbdl_usbacm_drv.obj(i.USB_Acm_BulkIn_Hdr) refers to usbdl_usbacm_drv.obj(.bss) for .bss$2
    usbdl_usbacm_drv.obj(i.USB_Acm_Ep0_SetLineCoding) refers to usbdl_usb_drv.obj(i.USB_EP0_Pkt_Len) for USB_EP0_Pkt_Len
    usbdl_usbacm_drv.obj(i.USB_Acm_Ep0_SetLineCoding) refers to usbdl_usb_drv.obj(i.USB_EPFIFORead) for USB_EPFIFORead
    usbdl_usbacm_drv.obj(i.USB_Acm_Ep0_SetLineCoding) refers to usbdl_usbacm_drv.obj(i.USB2UART_LineCoding2DCB) for USB2UART_LineCoding2DCB
    usbdl_usbacm_drv.obj(i.USB_Acm_Ep0_SetLineCoding) refers to usbdl_usb_drv.obj(i.USB_Update_EP0_State) for USB_Update_EP0_State
    usbdl_usbacm_drv.obj(i.USB_Acm_Ep0_SetLineCoding) refers to usbdl_usbacm_drv.obj(.bss) for .bss$2
    usbdl_usbacm_drv.obj(i.USB_Acm_Ep0_SetLineCoding) refers to usbdl_usb.obj(.bss) for gUsbDevice
    SSS_secure_shared.obj(FAST_CODE) refers to rt_udiv.o(.text) for __rt_udiv
    SSS_secure_shared.obj(FAST_CODE) refers to bl_portingfunc.obj(i.kal_assert_fail) for kal_assert_fail
    SSS_secure_shared.obj(FAST_CODE) refers to SSS_secure_shared.obj(.constdata) for .constdata$1
    SSS_secure_shared.obj(INIT_CODE) refers to SSS_interface.obj(INIT_CODE) for g_SST_CHE_base_init
    SSS_secure_shared.obj(INIT_CODE) refers to SSS_interface.obj(INIT_CODE) for g_SST_CONFIG_base_init
    SSS_secure_shared.obj(COMMON_CODE) refers to SSS_interface.obj(.constdata) for g_SST_CONFIG_base
    SSS_secure_shared.obj(COMMON_CODE) refers to SSS_interface.obj(.constdata) for g_SST_EFUSE_base
    SSS_secure_shared.obj(COMMON_CODE) refers to SSS_interface.obj(.constdata) for g_EFUSE_VER
    SSS_secure_shared.obj(COMMON_CODE) refers to SSS_interface.obj(.constdata) for g_SST_CONFIG_base
    SSS_secure_shared.obj(COMMON_CODE) refers to SSS_interface.obj(.constdata) for g_SST_CONFIG_base
    SSS_secure_shared.obj(COMMON_CODE) refers to bl_portingfunc.obj(i.kal_assert_fail) for kal_assert_fail
    SSS_secure_shared.obj(COMMON_CODE) refers to SSS_secure_shared.obj(COMMON_CODE) for SST_Secure_HW_Init
    SSS_secure_shared.obj(COMMON_CODE) refers to SSS_secure_shared.obj(COMMON_CODE) for SST_Secure_HW_DeInit
    SSS_secure_shared.obj(COMMON_CODE) refers to SSS_interface.obj(.constdata) for g_SST_CHE_base
    SSS_secure_shared.obj(COMMON_CODE) refers to SSS_secure_shared.obj(.constdata) for .constdata$1
    SSS_secure_shared.obj(COMMON_CODE) refers to SSS_interface.obj(.constdata) for g_SST_BootROM_version
    SSS_secure_shared.obj(COMMON_CODE) refers to SSS_secure_shared.obj(COMMON_CODE) for SST_Secure_Algo_With_Level
    SSS_secure_shared.obj(COMMON_CODE) refers to SSS_secure_shared.obj(COMMON_CODE) for SST_Secure_Get_SwOtp
    SSS_secure_shared.obj(COMMON_CODE) refers to SSS_secure_shared.obj(COMMON_CODE) for SST_Secure_Algo_With_Level
    SSS_secure_shared.obj(COMMON_CODE) refers to rt_memcpy.o(.text) for __rt_memcpy
    SSS_secure_shared.obj(COMMON_CODE) refers to SSS_interface.obj(.constdata) for g_SST_BootROM_version
    SSS_secure_shared.obj(COMMON_CODE) refers to SSS_secure_shared.obj(COMMON_CODE) for SST_Secure_Get_SwOtp
    SSS_secure_shared.obj(COMMON_CODE) refers to SSS_secure_shared.obj(COMMON_CODE) for SST_Secure_Algo_With_Level
    SSS_secure_shared.obj(COMMON_CODE) refers to rt_memcpy.o(.text) for __rt_memcpy
    SSS_secure_shared.obj(COMMON_CODE) refers to SSS_interface.obj(.constdata) for g_SST_BootROM_version
    SSS_secure_shared.obj(COMMON_CODE) refers to md5_engine.obj(i.CHE_md5_init) for CHE_md5_init
    SSS_secure_shared.obj(COMMON_CODE) refers to md5_engine.obj(i.CHE_md5_append) for CHE_md5_append
    SSS_secure_shared.obj(COMMON_CODE) refers to md5_engine.obj(i.CHE_md5_finish) for CHE_md5_finish
    SSS_secure_shared.obj(COMMON_CODE) refers to SSS_secure_shared.obj(COMMON_CODE) for SST_Secure_HW_Init
    SSS_secure_shared.obj(COMMON_CODE) refers to sha1_hw.obj(i.SEJ_sha1) for SEJ_sha1
    SSS_secure_shared.obj(COMMON_CODE) refers to SSS_secure_shared.obj(COMMON_CODE) for SST_Secure_HW_DeInit
    SSS_secure_shared.obj(COMMON_CODE) refers to sha1_sw.obj(i.Sha1_SW_init) for Sha1_SW_init
    SSS_secure_shared.obj(COMMON_CODE) refers to sha1_sw.obj(i.Sha1_SW_append) for Sha1_SW_append
    SSS_secure_shared.obj(COMMON_CODE) refers to sha1_sw.obj(i.Sha1_SW_finish) for Sha1_SW_finish
    SSS_secure_shared.obj(COMMON_CODE) refers to memcmp.o(.text) for memcmp
    SSS_secure_shared.obj(COMMON_CODE) refers to SSS_interface.obj(.constdata) for g_SST_HW_HASH
    SSS_secure_shared.obj(COMMON_CODE) refers to md5_engine.obj(i.CHE_md5_init) for CHE_md5_init
    SSS_secure_shared.obj(COMMON_CODE) refers to md5_engine.obj(i.CHE_md5_append) for CHE_md5_append
    SSS_secure_shared.obj(COMMON_CODE) refers to md5_engine.obj(i.CHE_md5_finish) for CHE_md5_finish
    SSS_secure_shared.obj(COMMON_CODE) refers to sha1_engine.obj(i.CHE_sha1_Init) for CHE_sha1_Init
    SSS_secure_shared.obj(COMMON_CODE) refers to sha1_engine.obj(i.CHE_sha1_append) for CHE_sha1_append
    SSS_secure_shared.obj(COMMON_CODE) refers to sha1_engine.obj(i.CHE_sha1_finish) for CHE_sha1_finish
    SSS_secure_shared.obj(COMMON_CODE) refers to rt_memcpy.o(.text) for __rt_memcpy
    SSS_secure_shared.obj(COMMON_CODE) refers to memcmp.o(.text) for memcmp
    SSS_secure_shared.obj(COMMON_CODE) refers to SSS_secure_shared.obj(COMMON_CODE) for SST_Secure_GetHashLen
    SSS_secure_shared.obj(COMMON_CODE) refers to custom_flash.obj(i.custom_get_NORFLASH_Base) for custom_get_NORFLASH_Base
    SSS_secure_shared.obj(COMMON_CODE) refers to SSS_secure_shared.obj(COMMON_CODE) for SST_Secure_Compare_Hash
    SSS_secure_shared.obj(COMMON_CODE) refers to SSS_secure_shared.obj(.constdata) for .constdata$1
    SSS_secure_shared.obj(COMMON_CODE) refers to SSS_secure_shared.obj(.bss) for .bss$2
    SSS_secure_shared.obj(COMMON_CODE) refers to memcmp.o(.text) for memcmp
    SSS_secure_shared.obj(COMMON_CODE) refers to SSS_secure_shared.obj(COMMON_CODE) for SST_Secure_GetHashLen
    SSS_secure_shared.obj(COMMON_CODE) refers to custom_flash.obj(i.custom_get_NORFLASH_Base) for custom_get_NORFLASH_Base
    SSS_secure_shared.obj(COMMON_CODE) refers to SSS_secure_shared.obj(COMMON_CODE) for SST_Secure_Compare_Hash
    SSS_secure_shared.obj(COMMON_CODE) refers to SSS_secure_shared.obj(.constdata) for .constdata$1
    SSS_secure_shared.obj(COMMON_CODE) refers to SSS_secure_shared.obj(.bss) for .bss$2
    SSS_secure_shared.obj(COMMON_CODE) refers to SSS_secure_shared.obj(COMMON_CODE) for SST_Is_Secure_BB
    SSS_secure_shared.obj(COMMON_CODE) refers to SSS_secure_shared.obj(COMMON_CODE) for SST_Secure_Get_SwOtp
    SSS_secure_shared.obj(COMMON_CODE) refers to strlen.o(.text) for strlen
    SSS_secure_shared.obj(COMMON_CODE) refers to strncmp.o(.text) for strncmp
    SSS_secure_shared.obj(COMMON_CODE) refers to SSS_secure_shared.obj(COMMON_CODE) for SST_Secure_Decrypt_MAC
    SSS_secure_shared.obj(COMMON_CODE) refers to SSS_secure_shared.obj(COMMON_CODE) for SST_Secure_CheckSecInfo
    SSS_secure_shared.obj(COMMON_CODE) refers to SSS_secure_shared.obj(COMMON_CODE) for SST_Secure_Check_Primary_MAUI
    SSS_secure_shared.obj(COMMON_CODE) refers to SSS_secure_shared.obj(INIT_CODE) for SST_DTLB_Config
    SSS_secure_shared.obj(COMMON_CODE) refers to SSS_interface.obj(.constdata) for g_SST_SecureNFB
    SSS_secure_shared.obj(COMMON_CODE) refers to SSS_interface.obj(.constdata) for g_SST_UAoffset
    SSS_secure_shared.obj(COMMON_CODE) refers to SSS_interface.obj(.constdata) for g_SST_INTSRAM_base
    SSS_secure_shared.obj(COMMON_CODE) refers to rt_udiv.o(.text) for __rt_udiv
    SSS_secure_shared.obj(COMMON_CODE) refers to SSS_interface.obj(.constdata) for g_SST_SWOTP
    SSS_secure_shared.obj(COMMON_CODE) refers to SSS_interface.obj(.constdata) for g_SST_RTC_base
    SSS_secure_shared.obj(COMMON_CODE) refers to SSS_secure_shared.obj(COMMON_CODE) for SST_Is_Secure_BB
    SSS_secure_shared.obj(COMMON_CODE) refers to SSS_secure_shared.obj(COMMON_CODE) for SST_Secure_Decrypt_MAC
    SSS_secure_shared.obj(COMMON_CODE) refers to SSS_secure_shared.obj(COMMON_CODE) for SST_Secure_CheckSecInfo
    SSS_secure_shared.obj(COMMON_CODE) refers to SSS_secure.obj(i.SST_Secure_Decrease_MAC_Index) for SST_Secure_Decrease_MAC_Index
    SSS_secure_shared.obj(COMMON_CODE) refers to SSS_secure_shared.obj(COMMON_CODE) for SST_Secure_Get_MAC_Index
    SSS_secure_shared.obj(COMMON_CODE) refers to rt_udiv.o(.text) for __rt_udiv
    SSS_secure_shared.obj(COMMON_CODE) refers to SSS_secure_shared.obj(COMMON_CODE) for SST_Secure_Compare_Hash
    SSS_secure_shared.obj(COMMON_CODE) refers to SSS_secure.obj(i.SST_Secure_Increase_MAC_Index) for SST_Secure_Increase_MAC_Index
    SSS_secure_shared.obj(COMMON_CODE) refers to SSS_interface.obj(.constdata) for g_SST_SecurePlatform
    SSS_secure_shared.obj(COMMON_CODE) refers to SSS_interface.obj(.constdata) for g_SST_REMAPPING_ADDR
    SSS_secure_shared.obj(COMMON_CODE) refers to SSS_interface.obj(.constdata) for g_SST_SecureRO
    SSS_secure_shared.obj(COMMON_CODE) refers to SSS_secure_shared.obj(COMMON_CODE) for SST_Secure_Algo
    SSS_secure_shared.obj(COMMON_CODE) refers to bl_portingfunc.obj(i.kal_assert_fail) for kal_assert_fail
    SSS_secure_shared.obj(COMMON_CODE) refers to SSS_secure_shared.obj(COMMON_CODE) for SST_Is_Secure_BB
    SSS_secure_shared.obj(COMMON_CODE) refers to SSS_secure_shared.obj(COMMON_CODE) for SST_Secure_Decrypt_MAC
    SSS_secure_shared.obj(COMMON_CODE) refers to SSS_secure_shared.obj(COMMON_CODE) for SST_Secure_CheckSecInfo
    SSS_secure_shared.obj(COMMON_CODE) refers to SSS_secure_shared.obj(COMMON_CODE) for SST_Secure_Compare_Hash
    SSS_secure_shared.obj(COMMON_CODE) refers to SSS_secure_shared.obj(COMMON_CODE) for SST_Decrypt_Secure_RO
    SSS_secure_shared.obj(COMMON_CODE) refers to SSS_interface.obj(.constdata) for g_SST_SecureRO
    SSS_secure_shared.obj(COMMON_CODE) refers to SSS_interface.obj(.constdata) for g_SST_REMAPPING_ADDR
    SSS_secure_shared.obj(COMMON_CODE) refers to SSS_secure_shared.obj(.constdata) for .constdata$1
    SSS_secure_shared.obj(COMMON_CODE) refers to SSS_interface.obj(.constdata) for g_SST_NFB
    SSS_secure_shared.obj(COMMON_CODE) refers to SSS_interface.obj(.constdata) for g_FOTA_MAC_Offset
    SSS_secure_shared.obj(COMMON_CODE) refers to SSS_secure_shared.obj(FAST_CODE) for SST_Search_Secinfo_Tag
    SSS_secure_shared.obj(COMMON_CODE) refers to SSS_secure_shared.obj(COMMON_CODE) for SST_Secure_Decrypt_MAC
    SSS_secure_shared.obj(COMMON_CODE) refers to SSS_secure_shared.obj(COMMON_CODE) for SST_Secure_CheckSecInfo
    SSS_secure_shared.obj(COMMON_CODE) refers to SSS_interface.obj(.constdata) for g_SST_REMAPPING_ADDR
    SSS_secure_shared.obj(COMMON_CODE) refers to SSS_interface.obj(.constdata) for g_SST_REMAPPING_ADDR
    SSS_secure_shared.obj(COMMON_CODE) refers to SSS_secure_shared.obj(.constdata) for .constdata$1
    SSS_secure_shared.obj(COMMON_CODE) refers to SSS_secure_shared.obj(COMMON_CODE) for SST_Get_MAUI_Rom_Info
    SSS_secure_shared.obj(COMMON_CODE) refers to rt_memcpy.o(.text) for __rt_memcpy
    SSS_secure_shared.obj(COMMON_CODE) refers to SSS_secure_shared.obj(COMMON_CODE) for SST_Get_MAUI_Rom_Info
    SSS_secure_shared.obj(COMMON_CODE) refers to SSS_secure_shared.obj(COMMON_CODE) for SST_Get_MAUI_Rom_Info
    SSS_secure_shared.obj(COMMON_CODE) refers to SSS_secure_shared.obj(COMMON_CODE) for SST_Is_Secure_BB
    SSS_secure_shared.obj(COMMON_CODE) refers to SSS_secure_shared.obj(COMMON_CODE) for SST_Secure_Get_SwOtp
    SSS_secure_shared.obj(COMMON_CODE) refers to SSS_secure_shared.obj(COMMON_CODE) for SST_Secure_Algo_With_Level
    SSS_secure_shared.obj(COMMON_CODE) refers to SSS_secure_shared.obj(COMMON_CODE) for SST_Secure_Compare_Hash
    SSS_secure_shared.obj(COMMON_CODE) refers to SSS_interface.obj(.constdata) for g_SST_SecurePlatform
    SSS_secure_shared.obj(COMMON_CODE) refers to SSS_interface.obj(.constdata) for g_SST_SWOTP
    SSS_secure_shared.obj(COMMON_CODE) refers to SSS_interface.obj(.constdata) for g_SST_SecureNFB
    SSS_secure_shared.obj(COMMON_CODE) refers to SSS_interface.obj(.constdata) for g_SST_BootROM_version
    SSS_secure_shared.obj(COMMON_CODE) refers to SSS_interface.obj(.constdata) for g_SST_INTSRAM_base
    SSS_secure_shared.obj(COMMON_CODE) refers to SSS_interface.obj(.constdata) for g_SST_FOTA
    SSS_secure_shared.obj(COMMON_CODE) refers to SSS_interface.obj(.constdata) for g_SST_SecureNFB
    SSS_secure_shared.obj(COMMON_CODE) refers to bl_Secure.obj(.bss) for g_nfb_secure_ro_addr
    SSS_secure_shared.obj(COMMON_CODE) refers to bl_portingfunc.obj(i.kal_assert_fail) for kal_assert_fail
    SSS_secure_shared.obj(COMMON_CODE) refers to sha1_engine.obj(i.CHE_sha1_Init) for CHE_sha1_Init
    SSS_secure_shared.obj(COMMON_CODE) refers to sha1_engine.obj(i.CHE_sha1_append) for CHE_sha1_append
    SSS_secure_shared.obj(COMMON_CODE) refers to sha1_engine.obj(i.CHE_sha1_finish) for CHE_sha1_finish
    SSS_secure_shared.obj(COMMON_CODE) refers to SSS_secure_shared.obj(.constdata) for .constdata$1
    SSS_secure_shared.obj(COMMON_CODE) refers to SSS_interface.obj(.constdata) for g_SST_CONFIG_base
    SSS_secure_shared.obj(COMMON_CODE) refers to bl_portingfunc.obj(i.kal_assert_fail) for kal_assert_fail
    SSS_secure_shared.obj(COMMON_CODE) refers to SSS_interface.obj(.constdata) for g_SST_CHE_base
    SSS_secure_shared.obj(COMMON_CODE) refers to SSS_secure_shared.obj(.constdata) for .constdata$1
    SSS_secure_shared.obj(COMMON_CODE) refers to SSS_secure_shared.obj(COMMON_CODE) for SST_Secure_Compare_Hash
    bl_FactoryConn.obj(i.GetData) refers to usbdl_usbacm_adap.obj(i.USBDL_GetUARTByte) for USBDL_GetUARTByte
    bl_FactoryConn.obj(i.PutData) refers to usbdl_usbacm_adap.obj(i.USBDL_PutUARTByte) for USBDL_PutUARTByte
    bl_FactoryConn.obj(i.Get16Data) refers to usbdl_usbacm_adap.obj(i.USBDL_GetUARTByte) for USBDL_GetUARTByte
    bl_FactoryConn.obj(i.Put16Data) refers to usbdl_usbacm_adap.obj(i.USBDL_PutUARTByte) for USBDL_PutUARTByte
    bl_FactoryConn.obj(i.writeCMD) refers to bl_FactoryConn.obj(i.GetData) for GetData
    bl_FactoryConn.obj(i.writeCMD) refers to bl_FactoryConn.obj(i.PutData) for PutData
    bl_FactoryConn.obj(i.writeCMD) refers to usbdl_usbacm_adap.obj(i.USBDL_PutUARTByte_Complete) for USBDL_PutUARTByte_Complete
    bl_FactoryConn.obj(i.writeCMD) refers to bl_FactoryConn.obj(i.Get16Data) for Get16Data
    bl_FactoryConn.obj(i.writeCMD) refers to bl_FactoryConn.obj(i.Put16Data) for Put16Data
    bl_FactoryConn.obj(i.readCMD) refers to bl_FactoryConn.obj(i.GetData) for GetData
    bl_FactoryConn.obj(i.readCMD) refers to bl_FactoryConn.obj(i.PutData) for PutData
    bl_FactoryConn.obj(i.readCMD) refers to usbdl_usbacm_adap.obj(i.USBDL_PutUARTByte_Complete) for USBDL_PutUARTByte_Complete
    bl_FactoryConn.obj(i.readCMD) refers to bl_FactoryConn.obj(i.Put16Data) for Put16Data
    bl_FactoryConn.obj(i.writeCMD_noecho) refers to bl_FactoryConn.obj(i.GetData) for GetData
    bl_FactoryConn.obj(i.writeCMD_noecho) refers to bl_FactoryConn.obj(i.PutData) for PutData
    bl_FactoryConn.obj(i.writeCMD_noecho) refers to usbdl_usbacm_adap.obj(i.USBDL_PutUARTByte_Complete) for USBDL_PutUARTByte_Complete
    bl_FactoryConn.obj(i.writeCMD_noecho) refers to bl_FactoryConn.obj(i.Get16Data) for Get16Data
    bl_FactoryConn.obj(i.writeCMD_32) refers to bl_FactoryConn.obj(i.GetData) for GetData
    bl_FactoryConn.obj(i.writeCMD_32) refers to bl_FactoryConn.obj(i.PutData) for PutData
    bl_FactoryConn.obj(i.writeCMD_32) refers to usbdl_usbacm_adap.obj(i.USBDL_PutUARTByte_Complete) for USBDL_PutUARTByte_Complete
    bl_FactoryConn.obj(i.readCMD_32) refers to bl_FactoryConn.obj(i.GetData) for GetData
    bl_FactoryConn.obj(i.readCMD_32) refers to bl_FactoryConn.obj(i.PutData) for PutData
    bl_FactoryConn.obj(i.readCMD_32) refers to usbdl_usbacm_adap.obj(i.USBDL_PutUARTByte_Complete) for USBDL_PutUARTByte_Complete
    bl_FactoryConn.obj(i.checksumCMD) refers to bl_FactoryConn.obj(i.GetData) for GetData
    bl_FactoryConn.obj(i.checksumCMD) refers to bl_FactoryConn.obj(i.PutData) for PutData
    bl_FactoryConn.obj(i.checksumCMD) refers to usbdl_usbacm_adap.obj(i.USBDL_PutUARTByte_Complete) for USBDL_PutUARTByte_Complete
    bl_FactoryConn.obj(i.checksumCMD) refers to bl_FactoryConn.obj(i.Put16Data) for Put16Data
    bl_FactoryConn.obj(i.getSWVersionCMD) refers to custom_blconfig.obj(i.custom_get_software_version) for custom_get_software_version
    bl_FactoryConn.obj(i.getSWVersionCMD) refers to usbdl_usbacm_adap.obj(i.USBDL_PutUARTByte) for USBDL_PutUARTByte
    bl_FactoryConn.obj(i.getSWVersionCMD) refers to usbdl_usbacm_adap.obj(i.USBDL_PutUARTByte_Complete) for USBDL_PutUARTByte_Complete
    bl_FactoryConn.obj(i.getBlRegionCMD) refers to bl_Main.obj(EXT_BOOTLOADER_CODE) for GetBootloaderRegion
    bl_FactoryConn.obj(i.getBlRegionCMD) refers to usbdl_usbacm_adap.obj(i.USBDL_PutUARTByte) for USBDL_PutUARTByte
    bl_FactoryConn.obj(i.getBlRegionCMD) refers to usbdl_usbacm_adap.obj(i.USBDL_PutUARTByte_Complete) for USBDL_PutUARTByte_Complete
    bl_FactoryConn.obj(i.jump_cmd2) refers to bl_FactoryConn.obj(i.GetData) for GetData
    bl_FactoryConn.obj(i.jump_cmd2) refers to bl_FactoryConn.obj(i.PutData) for PutData
    bl_FactoryConn.obj(i.jump_cmd2) refers to usbdl_usbacm_adap.obj(i.USBDL_PutUARTByte_Complete) for USBDL_PutUARTByte_Complete
    bl_FactoryConn.obj(i.jump_cmd2) refers to bl_Alg.obj(BL_ALGORITHM) for bl_Alg_SignatureVerify
    bl_FactoryConn.obj(i.jump_cmd2) refers to usbdl_usbacm_adap.obj(i.USBDL_PutUARTByte) for USBDL_PutUARTByte
    bl_FactoryConn.obj(i.jump_cmd2) refers to bl_portingfunc.obj(i.kal_assert_fail) for kal_assert_fail
    bl_FactoryConn.obj(i.jump_cmd2) refers to usbdl_usbacm_adap.obj(i.USBDL_CheckUARTSendEnd) for USBDL_CheckUARTSendEnd
    bl_FactoryConn.obj(i.jump_cmd2) refers to bl_portingfunc.obj(i.INT_DisableCacheOnEMI) for INT_DisableCacheOnEMI
    bl_FactoryConn.obj(i.jump_cmd2) refers to bl_Alg.obj(BL_ALGORITHM) for bl_Alg_Copy_Func_Tbl
    bl_FactoryConn.obj(i.jump_cmd2) refers to bl_BOOTARM.obj(SHARECODE) for JumpCmd
    bl_FactoryConn.obj(i.jump_cmd2) refers to SSS_interface.obj(.constdata) for g_SST_USBDownload4EndUser
    bl_FactoryConn.obj(i.jump_cmd2) refers to bl_Secure.obj(.bss) for g_BlFirstDownload
    bl_FactoryConn.obj(i.jump_cmd2) refers to bl_FactoryConn.obj(.constdata) for .constdata$1
    bl_FactoryConn.obj(i.waitBlReadyCMD) refers to custom_blconfig.obj(i.custom_check_valid_secro) for custom_check_valid_secro
    bl_FactoryConn.obj(i.waitBlReadyCMD) refers to usbdl_usbacm_adap.obj(i.USBDL_PutUARTByte) for USBDL_PutUARTByte
    bl_FactoryConn.obj(i.waitBlReadyCMD) refers to usbdl_usbacm_adap.obj(i.USBDL_PutUARTByte_Complete) for USBDL_PutUARTByte_Complete
    bl_FactoryConn.obj(i.waitBlReadyCMD) refers to bl_portingfunc.obj(i.kal_assert_fail) for kal_assert_fail
    bl_FactoryConn.obj(i.waitBlReadyCMD) refers to SSS_interface.obj(.constdata) for g_SST_USBDownload4EndUser
    bl_FactoryConn.obj(i.waitBlReadyCMD) refers to bl_FactoryConn.obj(.constdata) for .constdata$1
    bl_FactoryConn.obj(i.bl_Get_Secure_RO) refers to SSS_secure_shared.obj(FAST_CODE) for SST_Search_Secinfo_Tag
    bl_FactoryConn.obj(i.bl_Get_Secure_RO) refers to SSS_secure_shared.obj(COMMON_CODE) for SST_Get_Secinfo
    bl_FactoryConn.obj(i.bl_Get_Secure_RO) refers to SSS_secure_shared.obj(COMMON_CODE) for SST_Decrypt_Secure_RO
    bl_FactoryConn.obj(i.bl_Get_Secure_RO) refers to SSS_interface.obj(.constdata) for g_SST_SecureNFB
    bl_FactoryConn.obj(i.bl_Get_Secure_RO) refers to bl_Secure.obj(.bss) for g_nfb_secure_ro_addr
    bl_FactoryConn.obj(i.bl_Get_Secure_RO) refers to SSS_interface.obj(.constdata) for g_SST_REMAPPING_ADDR
    bl_FactoryConn.obj(i.bl_Get_Secure_RO) refers to custom_blconfig.obj(.constdata) for g_custom_secure_ro_addr
    bl_FactoryConn.obj(i.Connect_FactoryTool) refers to usbdl_usbacm_adap.obj(i.USBDL_GetUARTByte) for USBDL_GetUARTByte
    bl_FactoryConn.obj(i.Connect_FactoryTool) refers to custom_blconfig.obj(i.custom_check_valid_secro) for custom_check_valid_secro
    bl_FactoryConn.obj(i.Connect_FactoryTool) refers to SSS_secure_shared.obj(COMMON_CODE) for SST_Is_Secure_BB
    bl_FactoryConn.obj(i.Connect_FactoryTool) refers to usbdl_usbacm_adap.obj(i.USBDL_PutUARTByte) for USBDL_PutUARTByte
    bl_FactoryConn.obj(i.Connect_FactoryTool) refers to usbdl_usbacm_adap.obj(i.USBDL_PutUARTByte_Complete) for USBDL_PutUARTByte_Complete
    bl_FactoryConn.obj(i.Connect_FactoryTool) refers to bl_FactoryConn.obj(i.readCMD) for readCMD
    bl_FactoryConn.obj(i.Connect_FactoryTool) refers to bl_FactoryConn.obj(i.writeCMD_noecho) for writeCMD_noecho
    bl_FactoryConn.obj(i.Connect_FactoryTool) refers to bl_FactoryConn.obj(i.readCMD_32) for readCMD_32
    bl_FactoryConn.obj(i.Connect_FactoryTool) refers to bl_FactoryConn.obj(i.getBlRegionCMD) for getBlRegionCMD
    bl_FactoryConn.obj(i.Connect_FactoryTool) refers to bl_FactoryConn.obj(i.writeCMD) for writeCMD
    bl_FactoryConn.obj(i.Connect_FactoryTool) refers to bl_FactoryConn.obj(i.writeCMD_32) for writeCMD_32
    bl_FactoryConn.obj(i.Connect_FactoryTool) refers to bl_FactoryConn.obj(i.checksumCMD) for checksumCMD
    bl_FactoryConn.obj(i.Connect_FactoryTool) refers to bl_FactoryConn.obj(i.getSWVersionCMD) for getSWVersionCMD
    bl_FactoryConn.obj(i.Connect_FactoryTool) refers to bl_FactoryConn.obj(i.jump_cmd2) for jump_cmd2
    bl_FactoryConn.obj(i.Connect_FactoryTool) refers to bl_FactoryConn.obj(i.waitBlReadyCMD) for waitBlReadyCMD
    bl_FactoryConn.obj(i.Connect_FactoryTool) refers to SSS_interface.obj(.constdata) for g_SST_SecurePlatform
    bl_FactoryConn.obj(i.Connect_FactoryTool) refers to SSS_interface.obj(.constdata) for g_SST_BootROM_version
    bl_FactoryConn.obj(i.Connect_FactoryTool) refers to SSS_interface.obj(.constdata) for g_SST_USBDownload4EndUser
    bl_FactoryConn.obj(i.Connect_FactoryTool) refers to bl_Secure.obj(.bss) for g_BlFirstDownload
    bl_Secure.obj(INIT_CODE) refers to SSS_secure_shared.obj(INIT_CODE) for SST_DTLB_Config
    bl_Secure.obj(INIT_CODE) refers to bl_BOOTARM.obj(C$$code) for INT_Vectors
    bl_Secure.obj(INIT_CODE) refers to bl_Secure.obj(BL_SECINFO) for BL_SECINFO$7
    bl_Secure.obj(BL_SECINFO) refers to bl_Secure.obj(BL_SECURE_MAC_CONTENT) for g_BlSecureMAC
    md5_engine.obj(i.CHE_md5_append) refers to bl_portingfunc.obj(i.kal_assert_fail) for kal_assert_fail
    md5_engine.obj(i.CHE_md5_append) refers to rt_memcpy.o(.text) for __rt_memcpy
    md5_engine.obj(i.CHE_md5_append) refers to md5_engine.obj(i.CHE_md5_process) for CHE_md5_process
    md5_engine.obj(i.CHE_md5_append) refers to md5_engine.obj(.constdata) for .constdata$1
    md5_engine.obj(i.CHE_md5_finish) refers to md5_engine.obj(i.CHE_md5_append) for CHE_md5_append
    md5_engine.obj(i.CHE_md5_finish) refers to md5_engine.obj(.constdata) for .constdata$1
    md5_engine.obj(i.CHE_md5_process) refers to rt_memcpy.o(.text) for __rt_memcpy
    md5_engine.obj(i.CHE_md5_process) refers to md5_engine.obj(.constdata) for .constdata$1
    sha1_engine.obj(i.CHE_sha1_Init) refers to sha1_engine.obj(.bss) for .bss$2
    sha1_engine.obj(i.CHE_shaTransform) refers to sha1_engine.obj(.bss) for .bss$2
    sha1_engine.obj(i.CHE_sha1_append) refers to sha1_engine.obj(i.CHE_shaTransform) for CHE_shaTransform
    sha1_engine.obj(i.CHE_sha1_append) refers to sha1_engine.obj(.bss) for .bss$2
    sha1_engine.obj(i.CHE_shaStrUpdate) refers to strlen.o(.text) for strlen
    sha1_engine.obj(i.CHE_shaStrUpdate) refers to sha1_engine.obj(i.CHE_sha1_append) for CHE_sha1_append
    sha1_engine.obj(i.CHE_shapad) refers to sha1_engine.obj(.bss) for .bss$2
    sha1_engine.obj(i.CHE_shaBytes) refers to sha1_engine.obj(.bss) for .bss$2
    sha1_engine.obj(i.CHE_shaString) refers to rt_memcpy_w.o(.text) for __rt_memcpy_w
    sha1_engine.obj(i.CHE_shaString) refers to sha1_engine.obj(.constdata) for .constdata$1
    sha1_engine.obj(i.CHE_sha1_finish) refers to sha1_engine.obj(i.CHE_shapad) for CHE_shapad
    sha1_engine.obj(i.CHE_sha1_finish) refers to sha1_engine.obj(i.CHE_shaTransform) for CHE_shaTransform
    sha1_engine.obj(i.CHE_sha1_finish) refers to sha1_engine.obj(i.CHE_shaBytes) for CHE_shaBytes
    sha1_engine.obj(i.CHE_sha1_finish) refers to sha1_engine.obj(.bss) for .bss$2
    sha1_engine.obj(i.CHE_shaHash) refers to sha1_engine.obj(i.CHE_sha1_Init) for CHE_sha1_Init
    sha1_engine.obj(i.CHE_shaHash) refers to sha1_engine.obj(i.CHE_sha1_append) for CHE_sha1_append
    sha1_engine.obj(i.CHE_shaHash) refers to sha1_engine.obj(i.CHE_sha1_finish) for CHE_sha1_finish
    SSS_secure.obj(i.SST_Secure_Increase_MAC_Index) refers to rt_udiv.o(.text) for __rt_udiv
    SSS_secure.obj(i.SST_Secure_Increase_MAC_Index) refers to SSS_interface.obj(.constdata) for g_SST_SecureNFB
    SSS_secure.obj(i.SST_Secure_Increase_MAC_Index) refers to SSS_interface.obj(.constdata) for g_SST_SWOTP
    SSS_secure.obj(i.SST_Secure_Increase_MAC_Index) refers to SSS_interface.obj(.constdata) for g_SST_RTC_base
    SSS_secure.obj(i.SST_Secure_Decrease_MAC_Index) refers to rt_udiv.o(.text) for __rt_udiv
    SSS_secure.obj(i.SST_Secure_Decrease_MAC_Index) refers to SSS_interface.obj(.constdata) for g_SST_SecureNFB
    SSS_secure.obj(i.SST_Secure_Decrease_MAC_Index) refers to SSS_interface.obj(.constdata) for g_SST_SWOTP
    SSS_secure.obj(i.SST_Secure_Decrease_MAC_Index) refers to SSS_interface.obj(.constdata) for g_SST_RTC_base
    SSS_secure.obj(i.SST_VerifyNFBSecondaryImage) refers to SSS_secure_shared.obj(COMMON_CODE) for SST_Is_Secure_BB
    SSS_secure.obj(i.SST_VerifyNFBSecondaryImage) refers to SSS_secure_shared.obj(COMMON_CODE) for SST_Secure_Decrypt_MAC
    SSS_secure.obj(i.SST_VerifyNFBSecondaryImage) refers to SSS_secure_shared.obj(COMMON_CODE) for SST_Secure_Get_MAC_Index
    SSS_secure.obj(i.SST_VerifyNFBSecondaryImage) refers to SSS_secure_shared.obj(COMMON_CODE) for SST_Secure_Compare_Hash
    SSS_secure.obj(i.SST_VerifyNFBSecondaryImage) refers to bl_portingfunc.obj(i.kal_assert_fail) for kal_assert_fail
    SSS_secure.obj(i.SST_VerifyNFBSecondaryImage) refers to SSS_secure.obj(i.SST_Secure_Increase_MAC_Index) for SST_Secure_Increase_MAC_Index
    SSS_secure.obj(i.SST_VerifyNFBSecondaryImage) refers to SSS_interface.obj(.constdata) for g_SST_SecureNFB
    SSS_secure.obj(i.SST_VerifyNFBSecondaryImage) refers to SSS_interface.obj(.constdata) for g_SST_INTSRAM_base
    SSS_secure.obj(i.SST_VerifyNFBSecondaryImage) refers to SSS_secure.obj(.constdata) for .constdata$1
    SSS_secure.obj(i.SST_VerifyNFBSecondaryImage) refers to SSS_interface.obj(.constdata) for g_SST_SecureRO
    sha1_hw.obj(i.SEJ_sha1) refers to bl_portingfunc.obj(i.kal_assert_fail) for kal_assert_fail
    sha1_hw.obj(i.SEJ_sha1) refers to sha1_hw.obj(i.SEJ_sha1_mcu) for SEJ_sha1_mcu
    sha1_hw.obj(i.SEJ_sha1) refers to sha1_hw_asm.obj(SHARECODE) for SEJ_SHA1_LDM_64B
    sha1_hw.obj(i.SEJ_sha1) refers to sha1_hw.obj(i.SEJ_sha1_padding) for SEJ_sha1_padding
    sha1_hw.obj(i.SEJ_sha1) refers to sha1_hw.obj(.constdata) for .constdata$1
    sha1_hw.obj(i.SEJ_sha1) refers to SSS_interface.obj(.constdata) for g_SST_CHE_base
    sha1_hw.obj(i.SEJ_sha1_mcu) refers to SSS_interface.obj(.constdata) for g_SST_CHE_base
    sha1_hw.obj(i.SEJ_sha1_padding) refers to rt_memclr_w.o(.text) for __rt_memclr_w
    sha1_hw.obj(i.SEJ_sha1_padding) refers to llshl.o(.text) for _ll_shift_l
    sha1_hw.obj(i.SEJ_sha1_padding) refers to llushr.o(.text) for _ll_ushift_r
    sha1_hw.obj(i.SEJ_sha1_padding) refers to SSS_interface.obj(.constdata) for g_SST_CHE_base
    sha1_sw.obj(i.Sha1_SW_init) refers to sha1_sw.obj(.bss) for .bss$2
    sha1_sw.obj(i.Sha1_SW_append) refers to sha1_sw.obj(i.CHE_shaTransform) for CHE_shaTransform
    sha1_sw.obj(i.Sha1_SW_append) refers to sha1_sw.obj(.bss) for .bss$2
    sha1_sw.obj(i.Sha1_SW_finish) refers to sha1_sw.obj(i.CHE_shapad) for CHE_shapad
    sha1_sw.obj(i.Sha1_SW_finish) refers to sha1_sw.obj(i.CHE_shaTransform) for CHE_shaTransform
    sha1_sw.obj(i.Sha1_SW_finish) refers to sha1_sw.obj(.bss) for .bss$2
    sha1_sw.obj(i.CHE_shaTransform) refers to sha1_sw.obj(.bss) for .bss$2
    sha1_sw.obj(i.CHE_shapad) refers to sha1_sw.obj(.bss) for .bss$2
    lib_init.o(.text) refers to fpinit.o(x$fpl$fpinit) for _fp_init
    lib_init.o(.text) refers to libspace.o(.text) for __user_libspace
    llmullu.o(.text) refers to llmul3m.o(.text) for _ll_mul
    memcpy.o(.text) refers to rt_memcpy.o(.text) for __rt_memcpy
    memset.o(.text) refers to rt_memclr.o(.text) for _memset
    rt_memcpy.o(.text) refers to rt_memcpy_w.o(.text) for _memcpy_lastbytes
    rt_sdiv.o(.text) refers to rt_div0.o(.text) for __rt_div0
    rt_udiv.o(.text) refers to rt_div0.o(.text) for __rt_div0
    dfltll_clz.o(x$fpl$dfltll) refers (Special) to except.o(x$fpl$exception) for __fpl_exception
    dfltll_clz.o(x$fpl$dfltll) refers (Special) to rt_fp_status_addr.o(.text) for __rt_fp_status_addr
    dgeqf.o(x$fpl$dgeqf) refers to dcmpin.o(x$fpl$dcmpinfnan) for __fpl_dcmp_InfNaN
    libspace.o(.text) refers to libspace.o(.bss) for __libspace_start
    rt_div0.o(.text) refers to rt_raise.o(.text) for __rt_raise
    rt_fp_status_addr.o(.text) refers to libspace.o(.text) for __user_libspace
    rt_memclr.o(.text) refers to rt_memclr_w.o(.text) for _memset_w
    fpinit.o(x$fpl$fpinit) refers to rt_fp_status_addr.o(.text) for __rt_fp_status_addr
    dcmpin.o(x$fpl$dcmpinfnan) refers to except.o(x$fpl$exception) for __fpl_exception
    dcmpin.o(x$fpl$dcmpinfnan) refers to dcheck.o(x$fpl$dcheck) for __fpl_dcheck_NaN2
    except.o(x$fpl$exception) refers to rt_fp_status_addr.o(.text) for __rt_fp_status_addr
    except.o(x$fpl$exception) refers to trapv.o(x$fpl$trapveneer) for _fp_trapveneer
    except.o(x$fpl$exception) refers to retnan.o(x$fpl$retnan) for __fpl_return_NaN
    rt_raise.o(.text) refers to __raise.o(.text) for __raise
    rt_raise.o(.text) refers to sys_exit.o(.text) for _sys_exit
    dcheck.o(x$fpl$dcheck) refers to retnan.o(x$fpl$retnan) for __fpl_return_NaN
    dcheck.o(x$fpl$dcheck) refers to except.o(x$fpl$exception) for __fpl_exception
    retnan.o(x$fpl$retnan) refers to trapv.o(x$fpl$trapveneer) for __fpl_cmpreturn
    trapv.o(x$fpl$trapveneer) refers to _fptrap.o(.text) for _fp_trap
    trapv.o(x$fpl$trapveneer) refers to rt_fp_status_addr.o(.text) for __rt_fp_status_addr
    __raise.o(.text) refers to defsig.o(.text) for __default_signal_handler
    __raise.o(.text) refers to callvia.o(.text) for __call_via_r2
    _fptrap.o(.text) refers to rt_raise.o(.text) for __rt_raise
    sys_exit.o(.text) refers to use_semi.o(.text) for __I_use_semihosting_swi
    defsig.o(.text) refers to sys_wrch.o(.text) for _ttywrch
    defsig.o(.text) refers to defsig.o(.constdata) for .constdata$1
    sys_wrch.o(.text) refers (Special) to use_semi.o(.text) for __I_use_semihosting_swi
    nand_mtd_fdm50.obj(i.send_command_add_data) refers to nand_mtd_fdm50.obj(i.writefifo) for writefifo


================================================================================

Image Symbol Table

    Mapping Symbols

    Sym    Value        Execution Region

    $a     0x00000000   READ_ONLY
    $d     0x00000020   READ_ONLY
    $a     0x0000002c   READ_ONLY
    $d     0x000000ac   READ_ONLY
    $f     0x000000ac   READ_ONLY
    $a     0x000000b0   READ_ONLY
    $d     0x000000b8   READ_ONLY
    $f     0x000000b8   READ_ONLY
    $d     0x000000bc   READ_ONLY
    $t     0x00000400   READ_ONLY_TAIL
    $b     0x00000408   READ_ONLY_TAIL
    $b     0x00000412   READ_ONLY_TAIL
    $b     0x0000041e   READ_ONLY_TAIL
    $b     0x0000042a   READ_ONLY_TAIL
    $b     0x0000042e   READ_ONLY_TAIL
    $b     0x00000432   READ_ONLY_TAIL
    $b     0x0000043a   READ_ONLY_TAIL
    $b     0x00000440   READ_ONLY_TAIL
    $b     0x0000044c   READ_ONLY_TAIL
    $b     0x00000458   READ_ONLY_TAIL
    $b     0x00000462   READ_ONLY_TAIL
    $b     0x0000046c   READ_ONLY_TAIL
    $b     0x00000472   READ_ONLY_TAIL
    $b     0x00000476   READ_ONLY_TAIL
    $b     0x0000047a   READ_ONLY_TAIL
    $b     0x0000047e   READ_ONLY_TAIL
    $b     0x00000482   READ_ONLY_TAIL
    $b     0x00000486   READ_ONLY_TAIL
    $b     0x0000048a   READ_ONLY_TAIL
    $b     0x0000048e   READ_ONLY_TAIL
    $b     0x000004a0   READ_ONLY_TAIL
    $b     0x000004a4   READ_ONLY_TAIL
    $b     0x000004a8   READ_ONLY_TAIL
    $d     0x000004b2   READ_ONLY_TAIL
    $t     0x000004b8   READ_ONLY_TAIL
    $d     0x000004ba   READ_ONLY_TAIL
    $a     0x000004bc   READ_ONLY_TAIL
    $t     0x000004c8   READ_ONLY_TAIL
    $d     0x000004ca   READ_ONLY_TAIL
    $a     0x000004cc   READ_ONLY_TAIL
    $t     0x000004d4   READ_ONLY_TAIL
    $d     0x000004d6   READ_ONLY_TAIL
    $a     0x000004d8   READ_ONLY_TAIL
    $t     0x000004e4   READ_ONLY_TAIL
    $d     0x000004e6   READ_ONLY_TAIL
    $a     0x000004e8   READ_ONLY_TAIL
    $t     0x000004f4   READ_ONLY_TAIL
    $d     0x000004f6   READ_ONLY_TAIL
    $a     0x000004f8   READ_ONLY_TAIL
    $t     0x00000508   READ_ONLY_TAIL
    $d     0x0000050a   READ_ONLY_TAIL
    $a     0x0000050c   READ_ONLY_TAIL
    $t     0x0000052c   READ_ONLY_TAIL
    $d     0x0000052e   READ_ONLY_TAIL
    $a     0x00000530   READ_ONLY_TAIL
    $t     0x00000588   READ_ONLY_TAIL
    $d     0x0000058a   READ_ONLY_TAIL
    $a     0x0000058c   READ_ONLY_TAIL
    $t     0x00000640   READ_ONLY_TAIL
    $d     0x00000642   READ_ONLY_TAIL
    $a     0x00000644   READ_ONLY_TAIL
    $t     0x000006b0   READ_ONLY_TAIL
    $d     0x000006b2   READ_ONLY_TAIL
    $a     0x000006b4   READ_ONLY_TAIL
    $t     0x00000788   READ_ONLY_TAIL
    $d     0x0000078a   READ_ONLY_TAIL
    $a     0x0000078c   READ_ONLY_TAIL
    $t     0x000007cc   READ_ONLY_TAIL
    $d     0x000007ce   READ_ONLY_TAIL
    $a     0x000007d0   READ_ONLY_TAIL
    $d     0x000007d8   READ_ONLY_TAIL
    $t     0x000007dc   READ_ONLY_TAIL
    $d     0x000007de   READ_ONLY_TAIL
    $a     0x000007e0   READ_ONLY_TAIL
    $t     0x000007fc   READ_ONLY_TAIL
    $d     0x000007fe   READ_ONLY_TAIL
    $a     0x00000800   READ_ONLY_TAIL
    $t     0x0000080c   READ_ONLY_TAIL
    $d     0x0000080e   READ_ONLY_TAIL
    $a     0x00000810   READ_ONLY_TAIL
    $t     0x00000824   READ_ONLY_TAIL
    $d     0x00000826   READ_ONLY_TAIL
    $a     0x00000828   READ_ONLY_TAIL
    $t     0x0000086c   READ_ONLY_TAIL
    $d     0x0000086e   READ_ONLY_TAIL
    $a     0x00000870   READ_ONLY_TAIL
    $t     0x0000088c   READ_ONLY_TAIL
    $b     0x0000089a   READ_ONLY_TAIL
    $b     0x000008a8   READ_ONLY_TAIL
    $b     0x000008be   READ_ONLY_TAIL
    $d     0x000008c6   READ_ONLY_TAIL
    $t     0x000008d0   READ_ONLY_TAIL
    $b     0x000008e4   READ_ONLY_TAIL
    $b     0x00000902   READ_ONLY_TAIL
    $d     0x00000912   READ_ONLY_TAIL
    $t     0x00000914   READ_ONLY_TAIL
    $d     0x00000916   READ_ONLY_TAIL
    $a     0x00000918   READ_ONLY_TAIL
    $d     0x00000928   READ_ONLY_TAIL
    $f     0x00000928   READ_ONLY_TAIL
    $t     0x00000930   READ_ONLY_TAIL
    $b     0x0000099c   READ_ONLY_TAIL
    $b     0x000009aa   READ_ONLY_TAIL
    $b     0x000009be   READ_ONLY_TAIL
    $b     0x000009ca   READ_ONLY_TAIL
    $d     0x000009d6   READ_ONLY_TAIL
    $t     0x00000a58   READ_ONLY_TAIL
    $d     0x00000a5a   READ_ONLY_TAIL
    $a     0x00000a5c   READ_ONLY_TAIL
    $t     0x00000a60   READ_ONLY_TAIL
    $d     0x00000a72   READ_ONLY_TAIL
    $t     0x00000a74   READ_ONLY_TAIL
    $d     0x00000a76   READ_ONLY_TAIL
    $t     0x00000a78   READ_ONLY_TAIL
    $d     0x00000b32   READ_ONLY_TAIL
    $t     0x00000b4c   READ_ONLY_TAIL
    $d     0x00000b90   READ_ONLY_TAIL
    $t     0x00000b98   READ_ONLY_TAIL
    $b     0x00000b9c   READ_ONLY_TAIL
    $b     0x00000bba   READ_ONLY_TAIL
    $d     0x00000bce   READ_ONLY_TAIL
    $t     0x00000bd0   READ_ONLY_TAIL
    $b     0x00000bda   READ_ONLY_TAIL
    $b     0x00000bde   READ_ONLY_TAIL
    $b     0x00000bf6   READ_ONLY_TAIL
    $b     0x00000bfc   READ_ONLY_TAIL
    $b     0x00000c04   READ_ONLY_TAIL
    $d     0x00000c0a   READ_ONLY_TAIL
    $t     0x00000c14   READ_ONLY_TAIL
    $d     0x00000c16   READ_ONLY_TAIL
    $t     0x00000c18   READ_ONLY_TAIL
    $b     0x00000c26   READ_ONLY_TAIL
    $b     0x00000c2e   READ_ONLY_TAIL
    $b     0x00000c36   READ_ONLY_TAIL
    $b     0x00000c3e   READ_ONLY_TAIL
    $d     0x00000c44   READ_ONLY_TAIL
    $t     0x00000c48   READ_ONLY_TAIL
    $b     0x00000c4a   READ_ONLY_TAIL
    $b     0x00000c52   READ_ONLY_TAIL
    $b     0x00000c58   READ_ONLY_TAIL
    $b     0x00000c64   READ_ONLY_TAIL
    $d     0x00000c6a   READ_ONLY_TAIL
    $t     0x00000c70   READ_ONLY_TAIL
    $b     0x00000c72   READ_ONLY_TAIL
    $b     0x00000c78   READ_ONLY_TAIL
    $b     0x00000c82   READ_ONLY_TAIL
    $b     0x00000c98   READ_ONLY_TAIL
    $d     0x00000ca4   READ_ONLY_TAIL
    $t     0x00000cac   READ_ONLY_TAIL
    $b     0x00000cb2   READ_ONLY_TAIL
    $d     0x00000cc2   READ_ONLY_TAIL
    $t     0x00000cc8   READ_ONLY_TAIL
    $b     0x00000cda   READ_ONLY_TAIL
    $b     0x00000ce2   READ_ONLY_TAIL
    $b     0x00000cea   READ_ONLY_TAIL
    $d     0x00000cf4   READ_ONLY_TAIL
    $t     0x00000d00   READ_ONLY_TAIL
    $d     0x00000d10   READ_ONLY_TAIL
    $t     0x00000d18   READ_ONLY_TAIL
    $b     0x00000d34   READ_ONLY_TAIL
    $d     0x00000d5c   READ_ONLY_TAIL
    $t     0x00000d68   READ_ONLY_TAIL
    $b     0x00000d76   READ_ONLY_TAIL
    $b     0x00000d86   READ_ONLY_TAIL
    $b     0x00000d90   READ_ONLY_TAIL
    $b     0x00000da6   READ_ONLY_TAIL
    $b     0x00000dae   READ_ONLY_TAIL
    $b     0x00000db2   READ_ONLY_TAIL
    $d     0x00000dc4   READ_ONLY_TAIL
    $t     0x00000dd4   READ_ONLY_TAIL
    $b     0x00000dde   READ_ONLY_TAIL
    $b     0x00000de8   READ_ONLY_TAIL
    $b     0x00000dec   READ_ONLY_TAIL
    $b     0x00000df0   READ_ONLY_TAIL
    $b     0x00000df8   READ_ONLY_TAIL
    $b     0x00000e00   READ_ONLY_TAIL
    $b     0x00000e0c   READ_ONLY_TAIL
    $b     0x00000e12   READ_ONLY_TAIL
    $b     0x00000e1a   READ_ONLY_TAIL
    $b     0x00000e1e   READ_ONLY_TAIL
    $d     0x00000e24   READ_ONLY_TAIL
    $t     0x00000e30   READ_ONLY_TAIL
    $b     0x00000e36   READ_ONLY_TAIL
    $b     0x00000e4a   READ_ONLY_TAIL
    $b     0x00000e4e   READ_ONLY_TAIL
    $b     0x00000e52   READ_ONLY_TAIL
    $d     0x00000e58   READ_ONLY_TAIL
    $t     0x00000e60   READ_ONLY_TAIL
    $b     0x00000e66   READ_ONLY_TAIL
    $b     0x00000e6e   READ_ONLY_TAIL
    $b     0x00000e72   READ_ONLY_TAIL
    $b     0x00000e76   READ_ONLY_TAIL
    $b     0x00000e7a   READ_ONLY_TAIL
    $b     0x00000e7e   READ_ONLY_TAIL
    $b     0x00000e8c   READ_ONLY_TAIL
    $b     0x00000ea0   READ_ONLY_TAIL
    $b     0x00000ea4   READ_ONLY_TAIL
    $b     0x00000eae   READ_ONLY_TAIL
    $d     0x00000eb4   READ_ONLY_TAIL
    $t     0x00000ec8   READ_ONLY_TAIL
    $a     0x00000ecc   READ_ONLY_TAIL
    $d     0x00001100   READ_ONLY_TAIL
    $a     0x000011c8   READ_ONLY_TAIL
    $d     0x000011d0   READ_ONLY_TAIL
    $f     0x000011d0   READ_ONLY_TAIL
    $a     0x000011d4   READ_ONLY_TAIL
    $d     0x000011dc   READ_ONLY_TAIL
    $f     0x000011dc   READ_ONLY_TAIL
    $a     0x000011e0   READ_ONLY_TAIL
    $d     0x000011e8   READ_ONLY_TAIL
    $f     0x000011e8   READ_ONLY_TAIL
    $a     0x000011ec   READ_ONLY_TAIL
    $d     0x000011f4   READ_ONLY_TAIL
    $f     0x000011f4   READ_ONLY_TAIL
    $a     0x000011f8   READ_ONLY_TAIL
    $d     0x00001200   READ_ONLY_TAIL
    $f     0x00001200   READ_ONLY_TAIL
    $a     0x00001204   READ_ONLY_TAIL
    $d     0x0000120c   READ_ONLY_TAIL
    $f     0x0000120c   READ_ONLY_TAIL
    $a     0x00001210   READ_ONLY_TAIL
    $d     0x00001218   READ_ONLY_TAIL
    $f     0x00001218   READ_ONLY_TAIL
    $a     0x0000121c   READ_ONLY_TAIL
    $d     0x00001224   READ_ONLY_TAIL
    $f     0x00001224   READ_ONLY_TAIL
    $a     0x00001228   READ_ONLY_TAIL
    $d     0x00001230   READ_ONLY_TAIL
    $f     0x00001230   READ_ONLY_TAIL
    $a     0x00001234   READ_ONLY_TAIL
    $d     0x0000123c   READ_ONLY_TAIL
    $f     0x0000123c   READ_ONLY_TAIL
    $a     0x00001240   READ_ONLY_TAIL
    $d     0x00001248   READ_ONLY_TAIL
    $f     0x00001248   READ_ONLY_TAIL
    $a     0x0000124c   READ_ONLY_TAIL
    $d     0x00001250   READ_ONLY_TAIL
    $f     0x00001250   READ_ONLY_TAIL
    $t     0x00001254   READ_ONLY_TAIL
    $b     0x00001258   READ_ONLY_TAIL
    $b     0x0000127a   READ_ONLY_TAIL
    $b     0x0000128e   READ_ONLY_TAIL
    $d     0x00001296   READ_ONLY_TAIL
    $t     0x0000129c   READ_ONLY_TAIL
    $b     0x000012aa   READ_ONLY_TAIL
    $b     0x000012bc   READ_ONLY_TAIL
    $b     0x000012d2   READ_ONLY_TAIL
    $b     0x000012e0   READ_ONLY_TAIL
    $b     0x000012f0   READ_ONLY_TAIL
    $b     0x000012fa   READ_ONLY_TAIL
    $b     0x00001312   READ_ONLY_TAIL
    $b     0x00001320   READ_ONLY_TAIL
    $b     0x00001330   READ_ONLY_TAIL
    $b     0x0000133e   READ_ONLY_TAIL
    $b     0x00001348   READ_ONLY_TAIL
    $b     0x0000134e   READ_ONLY_TAIL
    $b     0x00001354   READ_ONLY_TAIL
    $b     0x0000135a   READ_ONLY_TAIL
    $b     0x00001360   READ_ONLY_TAIL
    $b     0x00001366   READ_ONLY_TAIL
    $d     0x0000136c   READ_ONLY_TAIL
    $t     0x0000137c   READ_ONLY_TAIL
    $d     0x00001384   READ_ONLY_TAIL
    $t     0x00001388   READ_ONLY_TAIL
    $d     0x000013ea   READ_ONLY_TAIL
    $t     0x00001400   READ_ONLY_TAIL
    $b     0x00001436   READ_ONLY_TAIL
    $b     0x0000145a   READ_ONLY_TAIL
    $d     0x00001460   READ_ONLY_TAIL
    $t     0x00001474   READ_ONLY_TAIL
    $d     0x000014b4   READ_ONLY_TAIL
    $t     0x000014bc   READ_ONLY_TAIL
    $d     0x000014fc   READ_ONLY_TAIL
    $t     0x00001504   READ_ONLY_TAIL
    $d     0x0000154e   READ_ONLY_TAIL
    $t     0x00001560   READ_ONLY_TAIL
    $b     0x00001562   READ_ONLY_TAIL
    $d     0x00001672   READ_ONLY_TAIL
    $t     0x000016a0   READ_ONLY_TAIL
    $d     0x000016bc   READ_ONLY_TAIL
    $t     0x000016c0   READ_ONLY_TAIL
    $b     0x000016c8   READ_ONLY_TAIL
    $d     0x000016e6   READ_ONLY_TAIL
    $t     0x000016e8   READ_ONLY_TAIL
    $b     0x000016f0   READ_ONLY_TAIL
    $d     0x0000170a   READ_ONLY_TAIL
    $t     0x0000170c   READ_ONLY_TAIL
    $d     0x00001714   READ_ONLY_TAIL
    $t     0x00001718   READ_ONLY_TAIL
    $d     0x00001760   READ_ONLY_TAIL
    $t     0x00001770   READ_ONLY_TAIL
    $b     0x000017f4   READ_ONLY_TAIL
    $b     0x000017fa   READ_ONLY_TAIL
    $b     0x00001800   READ_ONLY_TAIL
    $b     0x00001806   READ_ONLY_TAIL
    $b     0x0000180c   READ_ONLY_TAIL
    $b     0x00001812   READ_ONLY_TAIL
    $b     0x00001822   READ_ONLY_TAIL
    $b     0x0000182c   READ_ONLY_TAIL
    $b     0x00001832   READ_ONLY_TAIL
    $b     0x00001838   READ_ONLY_TAIL
    $b     0x0000183e   READ_ONLY_TAIL
    $b     0x00001844   READ_ONLY_TAIL
    $b     0x0000184a   READ_ONLY_TAIL
    $b     0x00001850   READ_ONLY_TAIL
    $b     0x00001856   READ_ONLY_TAIL
    $b     0x00001866   READ_ONLY_TAIL
    $b     0x00001870   READ_ONLY_TAIL
    $b     0x00001876   READ_ONLY_TAIL
    $b     0x0000187c   READ_ONLY_TAIL
    $b     0x00001882   READ_ONLY_TAIL
    $b     0x00001890   READ_ONLY_TAIL
    $d     0x00001898   READ_ONLY_TAIL
    $t     0x000018ac   READ_ONLY_TAIL
    $d     0x000018bc   READ_ONLY_TAIL
    $t     0x000018c0   READ_ONLY_TAIL
    $b     0x000018c4   READ_ONLY_TAIL
    $b     0x000018c8   READ_ONLY_TAIL
    $b     0x000018cc   READ_ONLY_TAIL
    $b     0x000018d0   READ_ONLY_TAIL
    $b     0x000018dc   READ_ONLY_TAIL
    $b     0x000018e8   READ_ONLY_TAIL
    $d     0x000018ee   READ_ONLY_TAIL
    $t     0x000018fc   READ_ONLY_TAIL
    $d     0x000018fe   READ_ONLY_TAIL
    $t     0x00001900   READ_ONLY_TAIL
    $d     0x00001906   READ_ONLY_TAIL
    $t     0x00001908   READ_ONLY_TAIL
    $b     0x0000191c   READ_ONLY_TAIL
    $b     0x00001940   READ_ONLY_TAIL
    $b     0x0000197c   READ_ONLY_TAIL
    $p     0x00001984   READ_ONLY_TAIL
    $b     0x000019f2   READ_ONLY_TAIL
    $d     0x00001a0a   READ_ONLY_TAIL
    $t     0x00001a24   READ_ONLY_TAIL
    $b     0x00001a28   READ_ONLY_TAIL
    $p     0x00001a2e   READ_ONLY_TAIL
    $b     0x00001a34   READ_ONLY_TAIL
    $p     0x00001a3a   READ_ONLY_TAIL
    $b     0x00001a48   READ_ONLY_TAIL
    $b     0x00001a56   READ_ONLY_TAIL
    $b     0x00001a64   READ_ONLY_TAIL
    $b     0x00001a76   READ_ONLY_TAIL
    $d     0x00001a7c   READ_ONLY_TAIL
    $f     0x00001a84   READ_ONLY_TAIL
    $f     0x00001a88   READ_ONLY_TAIL
    $f     0x00001a8c   READ_ONLY_TAIL
    $f     0x00001a94   READ_ONLY_TAIL
    $f     0x00001a98   READ_ONLY_TAIL
    $f     0x00001a9c   READ_ONLY_TAIL
    $t     0x00001aa0   READ_ONLY_TAIL
    $b     0x00001aae   READ_ONLY_TAIL
    $b     0x00001abc   READ_ONLY_TAIL
    $b     0x00001ac2   READ_ONLY_TAIL
    $b     0x00001ac6   READ_ONLY_TAIL
    $d     0x00001af6   READ_ONLY_TAIL
    $t     0x00001b00   READ_ONLY_TAIL
    $d     0x00001b02   READ_ONLY_TAIL
    $t     0x00001b04   READ_ONLY_TAIL
    $b     0x00001b08   READ_ONLY_TAIL
    $d     0x00001b0e   READ_ONLY_TAIL
    $t     0x00001b10   READ_ONLY_TAIL
    $b     0x00001b16   READ_ONLY_TAIL
    $b     0x00001b34   READ_ONLY_TAIL
    $b     0x00001b3c   READ_ONLY_TAIL
    $d     0x00001b56   READ_ONLY_TAIL
    $t     0x00001b60   READ_ONLY_TAIL
    $d     0x00001b66   READ_ONLY_TAIL
    $t     0x00001b6c   READ_ONLY_TAIL
    $b     0x00001b70   READ_ONLY_TAIL
    $d     0x00001b76   READ_ONLY_TAIL
    $t     0x00001b78   READ_ONLY_TAIL
    $b     0x00001b7c   READ_ONLY_TAIL
    $d     0x00001b82   READ_ONLY_TAIL
    $t     0x00001b84   READ_ONLY_TAIL
    $b     0x00001b8a   READ_ONLY_TAIL
    $b     0x00001bb6   READ_ONLY_TAIL
    $b     0x00001bbc   READ_ONLY_TAIL
    $b     0x00001bc4   READ_ONLY_TAIL
    $b     0x00001bcc   READ_ONLY_TAIL
    $d     0x00001bde   READ_ONLY_TAIL
    $t     0x00001bf0   READ_ONLY_TAIL
    $b     0x00001bf8   READ_ONLY_TAIL
    $b     0x00001c00   READ_ONLY_TAIL
    $b     0x00001c3c   READ_ONLY_TAIL
    $b     0x00001c42   READ_ONLY_TAIL
    $b     0x00001c48   READ_ONLY_TAIL
    $b     0x00001c50   READ_ONLY_TAIL
    $d     0x00001c64   READ_ONLY_TAIL
    $t     0x00001c74   READ_ONLY_TAIL
    $b     0x00001c78   READ_ONLY_TAIL
    $b     0x00001c7c   READ_ONLY_TAIL
    $b     0x00001c80   READ_ONLY_TAIL
    $b     0x00001c84   READ_ONLY_TAIL
    $b     0x00001c8a   READ_ONLY_TAIL
    $d     0x00001c96   READ_ONLY_TAIL
    $t     0x00001c9c   READ_ONLY_TAIL
    $b     0x00001cb0   READ_ONLY_TAIL
    $b     0x00001cb4   READ_ONLY_TAIL
    $b     0x00001cba   READ_ONLY_TAIL
    $b     0x00001cc4   READ_ONLY_TAIL
    $b     0x00001cd6   READ_ONLY_TAIL
    $b     0x00001d0c   READ_ONLY_TAIL
    $b     0x00001d1c   READ_ONLY_TAIL
    $d     0x00001d2c   READ_ONLY_TAIL
    $t     0x00001d48   READ_ONLY_TAIL
    $b     0x00001d52   READ_ONLY_TAIL
    $b     0x00001d62   READ_ONLY_TAIL
    $b     0x00001d68   READ_ONLY_TAIL
    $b     0x00001e26   READ_ONLY_TAIL
    $b     0x00001e2c   READ_ONLY_TAIL
    $d     0x00001e32   READ_ONLY_TAIL
    $t     0x00001e4c   READ_ONLY_TAIL
    $b     0x00001e4e   READ_ONLY_TAIL
    $d     0x00001e74   READ_ONLY_TAIL
    $t     0x00001e7c   READ_ONLY_TAIL
    $b     0x00001e7e   READ_ONLY_TAIL
    $b     0x00001e84   READ_ONLY_TAIL
    $d     0x00001e96   READ_ONLY_TAIL
    $t     0x00001e98   READ_ONLY_TAIL
    $d     0x00001ea0   READ_ONLY_TAIL
    $t     0x00001ea4   READ_ONLY_TAIL
    $d     0x00001eb4   READ_ONLY_TAIL
    $t     0x00001ebc   READ_ONLY_TAIL
    $b     0x00001ecc   READ_ONLY_TAIL
    $b     0x00001ede   READ_ONLY_TAIL
    $b     0x00001ee6   READ_ONLY_TAIL
    $d     0x00001eec   READ_ONLY_TAIL
    $t     0x00001ef4   READ_ONLY_TAIL
    $d     0x00001f04   READ_ONLY_TAIL
    $t     0x00001f0c   READ_ONLY_TAIL
    $b     0x00001f12   READ_ONLY_TAIL
    $b     0x00001f1c   READ_ONLY_TAIL
    $b     0x00001f58   READ_ONLY_TAIL
    $b     0x00001fb0   READ_ONLY_TAIL
    $d     0x00001fd8   READ_ONLY_TAIL
    $f     0x00001fdc   READ_ONLY_TAIL
    $t     0x00001fe0   READ_ONLY_TAIL
    $d     0x00001fea   READ_ONLY_TAIL
    $t     0x00001ff0   READ_ONLY_TAIL
    $d     0x00001ffe   READ_ONLY_TAIL
    $t     0x00002004   READ_ONLY_TAIL
    $b     0x0000200a   READ_ONLY_TAIL
    $b     0x0000201c   READ_ONLY_TAIL
    $b     0x00002024   READ_ONLY_TAIL
    $b     0x00002062   READ_ONLY_TAIL
    $b     0x00002072   READ_ONLY_TAIL
    $b     0x00002084   READ_ONLY_TAIL
    $d     0x000020c6   READ_ONLY_TAIL
    $f     0x000020cc   READ_ONLY_TAIL
    $f     0x000020d0   READ_ONLY_TAIL
    $f     0x000020d4   READ_ONLY_TAIL
    $f     0x000020d8   READ_ONLY_TAIL
    $t     0x000020dc   READ_ONLY_TAIL
    $b     0x000020f8   READ_ONLY_TAIL
    $b     0x00002108   READ_ONLY_TAIL
    $d     0x0000210e   READ_ONLY_TAIL
    $t     0x00002114   READ_ONLY_TAIL
    $b     0x00002116   READ_ONLY_TAIL
    $d     0x00002142   READ_ONLY_TAIL
    $t     0x00002148   READ_ONLY_TAIL
    $b     0x00002178   READ_ONLY_TAIL
    $b     0x00002186   READ_ONLY_TAIL
    $b     0x00002192   READ_ONLY_TAIL
    $d     0x00002198   READ_ONLY_TAIL
    $f     0x0000219c   READ_ONLY_TAIL
    $t     0x000021a4   READ_ONLY_TAIL
    $b     0x000021a6   READ_ONLY_TAIL
    $b     0x000021b8   READ_ONLY_TAIL
    $b     0x000021c2   READ_ONLY_TAIL
    $b     0x000021d2   READ_ONLY_TAIL
    $d     0x000021d8   READ_ONLY_TAIL
    $t     0x000021e0   READ_ONLY_TAIL
    $b     0x00002232   READ_ONLY_TAIL
    $b     0x0000224e   READ_ONLY_TAIL
    $d     0x0000225a   READ_ONLY_TAIL
    $t     0x00002260   READ_ONLY_TAIL
    $b     0x00002298   READ_ONLY_TAIL
    $b     0x000022a6   READ_ONLY_TAIL
    $d     0x000022b2   READ_ONLY_TAIL
    $t     0x000022bc   READ_ONLY_TAIL
    $b     0x00002310   READ_ONLY_TAIL
    $d     0x0000231c   READ_ONLY_TAIL
    $t     0x00002320   READ_ONLY_TAIL
    $b     0x0000232a   READ_ONLY_TAIL
    $d     0x0000237c   READ_ONLY_TAIL
    $t     0x00002384   READ_ONLY_TAIL
    $d     0x00002386   READ_ONLY_TAIL
    $t     0x00002388   READ_ONLY_TAIL
    $d     0x00002390   READ_ONLY_TAIL
    $t     0x00002394   READ_ONLY_TAIL
    $d     0x0000239c   READ_ONLY_TAIL
    $t     0x000023a0   READ_ONLY_TAIL
    $d     0x000023ae   READ_ONLY_TAIL
    $t     0x000023b0   READ_ONLY_TAIL
    $d     0x000023c6   READ_ONLY_TAIL
    $t     0x000023cc   READ_ONLY_TAIL
    $b     0x000023d0   READ_ONLY_TAIL
    $d     0x000023d6   READ_ONLY_TAIL
    $t     0x000023d8   READ_ONLY_TAIL
    $b     0x000023fa   READ_ONLY_TAIL
    $d     0x0000241e   READ_ONLY_TAIL
    $t     0x0000242c   READ_ONLY_TAIL
    $b     0x0000244e   READ_ONLY_TAIL
    $d     0x00002472   READ_ONLY_TAIL
    $t     0x00002480   READ_ONLY_TAIL
    $b     0x00002488   READ_ONLY_TAIL
    $d     0x0000249c   READ_ONLY_TAIL
    $t     0x000024a0   READ_ONLY_TAIL
    $b     0x000024a8   READ_ONLY_TAIL
    $b     0x000024ce   READ_ONLY_TAIL
    $d     0x000024dc   READ_ONLY_TAIL
    $t     0x000024e4   READ_ONLY_TAIL
    $b     0x00002514   READ_ONLY_TAIL
    $d     0x0000251a   READ_ONLY_TAIL
    $t     0x00002520   READ_ONLY_TAIL
    $b     0x0000252a   READ_ONLY_TAIL
    $d     0x00002540   READ_ONLY_TAIL
    $t     0x00002544   READ_ONLY_TAIL
    $d     0x00002556   READ_ONLY_TAIL
    $t     0x00002558   READ_ONLY_TAIL
    $b     0x00002560   READ_ONLY_TAIL
    $b     0x0000257c   READ_ONLY_TAIL
    $b     0x00002590   READ_ONLY_TAIL
    $b     0x0000259c   READ_ONLY_TAIL
    $p     0x000025bc   READ_ONLY_TAIL
    $b     0x000025d4   READ_ONLY_TAIL
    $b     0x000025ec   READ_ONLY_TAIL
    $b     0x000025f6   READ_ONLY_TAIL
    $b     0x000025fe   READ_ONLY_TAIL
    $b     0x00002608   READ_ONLY_TAIL
    $d     0x00002610   READ_ONLY_TAIL
    $t     0x0000261c   READ_ONLY_TAIL
    $b     0x0000262c   READ_ONLY_TAIL
    $p     0x00002666   READ_ONLY_TAIL
    $b     0x0000266c   READ_ONLY_TAIL
    $b     0x00002678   READ_ONLY_TAIL
    $d     0x0000267e   READ_ONLY_TAIL
    $t     0x00002684   READ_ONLY_TAIL
    $b     0x000026aa   READ_ONLY_TAIL
    $b     0x000026c8   READ_ONLY_TAIL
    $d     0x000026ce   READ_ONLY_TAIL
    $t     0x000026d4   READ_ONLY_TAIL
    $d     0x000026e8   READ_ONLY_TAIL
    $t     0x000026ec   READ_ONLY_TAIL
    $d     0x000026f0   READ_ONLY_TAIL
    $t     0x000026f4   READ_ONLY_TAIL
    $d     0x000026f8   READ_ONLY_TAIL
    $t     0x000026fc   READ_ONLY_TAIL
    $d     0x00002700   READ_ONLY_TAIL
    $t     0x00002704   READ_ONLY_TAIL
    $d     0x00002708   READ_ONLY_TAIL
    $t     0x0000270c   READ_ONLY_TAIL
    $d     0x00002710   READ_ONLY_TAIL
    $t     0x00002714   READ_ONLY_TAIL
    $b     0x00002744   READ_ONLY_TAIL
    $d     0x0000275a   READ_ONLY_TAIL
    $t     0x00002764   READ_ONLY_TAIL
    $b     0x00002794   READ_ONLY_TAIL
    $d     0x000027aa   READ_ONLY_TAIL
    $t     0x000027b4   READ_ONLY_TAIL
    $d     0x000027da   READ_ONLY_TAIL
    $t     0x000027dc   READ_ONLY_TAIL
    $b     0x000027e4   READ_ONLY_TAIL
    $d     0x000027fc   READ_ONLY_TAIL
    $t     0x00002804   READ_ONLY_TAIL
    $b     0x00002836   READ_ONLY_TAIL
    $d     0x0000284e   READ_ONLY_TAIL
    $t     0x00002858   READ_ONLY_TAIL
    $b     0x00002888   READ_ONLY_TAIL
    $d     0x00002898   READ_ONLY_TAIL
    $t     0x000028a0   READ_ONLY_TAIL
    $b     0x000028d2   READ_ONLY_TAIL
    $d     0x000028ec   READ_ONLY_TAIL
    $t     0x000028f4   READ_ONLY_TAIL
    $b     0x00002928   READ_ONLY_TAIL
    $p     0x0000292e   READ_ONLY_TAIL
    $b     0x0000293c   READ_ONLY_TAIL
    $b     0x0000296e   READ_ONLY_TAIL
    $p     0x00002974   READ_ONLY_TAIL
    $p     0x000029a0   READ_ONLY_TAIL
    $b     0x000029be   READ_ONLY_TAIL
    $p     0x00002a08   READ_ONLY_TAIL
    $b     0x00002a22   READ_ONLY_TAIL
    $d     0x00002a40   READ_ONLY_TAIL
    $t     0x00002a4c   READ_ONLY_TAIL
    $d     0x00002a66   READ_ONLY_TAIL
    $t     0x00002a68   READ_ONLY_TAIL
    $b     0x00002a6e   READ_ONLY_TAIL
    $b     0x00002a72   READ_ONLY_TAIL
    $b     0x00002a76   READ_ONLY_TAIL
    $b     0x00002a86   READ_ONLY_TAIL
    $b     0x00002a90   READ_ONLY_TAIL
    $b     0x00002a94   READ_ONLY_TAIL
    $b     0x00002a9c   READ_ONLY_TAIL
    $b     0x00002aa0   READ_ONLY_TAIL
    $b     0x00002aa4   READ_ONLY_TAIL
    $b     0x00002aaa   READ_ONLY_TAIL
    $b     0x00002ab0   READ_ONLY_TAIL
    $d     0x00002ab6   READ_ONLY_TAIL
    $f     0x00002abc   READ_ONLY_TAIL
    $f     0x00002ac0   READ_ONLY_TAIL
    $t     0x00002ac4   READ_ONLY_TAIL
    $d     0x00002ad4   READ_ONLY_TAIL
    $t     0x00002ad8   READ_ONLY_TAIL
    $b     0x00002ae6   READ_ONLY_TAIL
    $b     0x00002af6   READ_ONLY_TAIL
    $b     0x00002b12   READ_ONLY_TAIL
    $b     0x00002b2e   READ_ONLY_TAIL
    $b     0x00002b4a   READ_ONLY_TAIL
    $d     0x00002b8c   READ_ONLY_TAIL
    $t     0x00002b90   READ_ONLY_TAIL
    $d     0x00002bce   READ_ONLY_TAIL
    $t     0x00002bd4   READ_ONLY_TAIL
    $b     0x00002bd8   READ_ONLY_TAIL
    $b     0x00002bdc   READ_ONLY_TAIL
    $b     0x00002c14   READ_ONLY_TAIL
    $b     0x00002c4c   READ_ONLY_TAIL
    $b     0x00002c86   READ_ONLY_TAIL
    $b     0x00002cb4   READ_ONLY_TAIL
    $d     0x00002cba   READ_ONLY_TAIL
    $t     0x00002cc0   READ_ONLY_TAIL
    $b     0x00002cc8   READ_ONLY_TAIL
    $b     0x00002cda   READ_ONLY_TAIL
    $d     0x00002ce0   READ_ONLY_TAIL
    $t     0x00002ce4   READ_ONLY_TAIL
    $d     0x00002cf6   READ_ONLY_TAIL
    $t     0x00002cf8   READ_ONLY_TAIL
    $b     0x00002cfe   READ_ONLY_TAIL
    $b     0x00002d14   READ_ONLY_TAIL
    $d     0x00002d24   READ_ONLY_TAIL
    $t     0x00002d2c   READ_ONLY_TAIL
    $b     0x00002d2e   READ_ONLY_TAIL
    $b     0x00002d60   READ_ONLY_TAIL
    $d     0x00002d7e   READ_ONLY_TAIL
    $t     0x00002d88   READ_ONLY_TAIL
    $b     0x00002db0   READ_ONLY_TAIL
    $d     0x00002dc6   READ_ONLY_TAIL
    $t     0x00002dd0   READ_ONLY_TAIL
    $b     0x00002df8   READ_ONLY_TAIL
    $b     0x00002e0e   READ_ONLY_TAIL
    $d     0x00002e16   READ_ONLY_TAIL
    $t     0x00002e1c   READ_ONLY_TAIL
    $d     0x00002e22   READ_ONLY_TAIL
    $t     0x00002e28   READ_ONLY_TAIL
    $d     0x00002e38   READ_ONLY_TAIL
    $t     0x00002e3c   READ_ONLY_TAIL
    $b     0x00002e3e   READ_ONLY_TAIL
    $b     0x00002e42   READ_ONLY_TAIL
    $b     0x00002e46   READ_ONLY_TAIL
    $p     0x00002e64   READ_ONLY_TAIL
    $p     0x00002e84   READ_ONLY_TAIL
    $p     0x00002ea4   READ_ONLY_TAIL
    $d     0x00002eb4   READ_ONLY_TAIL
    $t     0x00002eb8   READ_ONLY_TAIL
    $d     0x00002ee0   READ_ONLY_TAIL
    $t     0x00002ee8   READ_ONLY_TAIL
    $b     0x00002f04   READ_ONLY_TAIL
    $d     0x00002f0a   READ_ONLY_TAIL
    $t     0x00002f10   READ_ONLY_TAIL
    $d     0x00002f18   READ_ONLY_TAIL
    $t     0x00002f1c   READ_ONLY_TAIL
    $b     0x00002f3c   READ_ONLY_TAIL
    $d     0x00002f68   READ_ONLY_TAIL
    $t     0x00002f6c   READ_ONLY_TAIL
    $b     0x00002f90   READ_ONLY_TAIL
    $b     0x00002fd8   READ_ONLY_TAIL
    $b     0x00002ffc   READ_ONLY_TAIL
    $d     0x00003004   READ_ONLY_TAIL
    $t     0x00003014   READ_ONLY_TAIL
    $d     0x0000303a   READ_ONLY_TAIL
    $t     0x0000303c   READ_ONLY_TAIL
    $b     0x0000304c   READ_ONLY_TAIL
    $b     0x00003080   READ_ONLY_TAIL
    $b     0x000030b0   READ_ONLY_TAIL
    $p     0x000030be   READ_ONLY_TAIL
    $b     0x000030e6   READ_ONLY_TAIL
    $b     0x00003128   READ_ONLY_TAIL
    $b     0x00003132   READ_ONLY_TAIL
    $b     0x000031ac   READ_ONLY_TAIL
    $b     0x000031bc   READ_ONLY_TAIL
    $d     0x000031c4   READ_ONLY_TAIL
    $t     0x000031d4   READ_ONLY_TAIL
    $b     0x000031fc   READ_ONLY_TAIL
    $p     0x00003212   READ_ONLY_TAIL
    $b     0x0000322e   READ_ONLY_TAIL
    $d     0x00003242   READ_ONLY_TAIL
    $t     0x0000324c   READ_ONLY_TAIL
    $p     0x0000326c   READ_ONLY_TAIL
    $b     0x00003284   READ_ONLY_TAIL
    $b     0x000032a2   READ_ONLY_TAIL
    $b     0x000032c4   READ_ONLY_TAIL
    $b     0x000032e6   READ_ONLY_TAIL
    $b     0x00003326   READ_ONLY_TAIL
    $d     0x0000332e   READ_ONLY_TAIL
    $t     0x00003340   READ_ONLY_TAIL
    $d     0x00003362   READ_ONLY_TAIL
    $b     0x0000337e   READ_ONLY_TAIL
    $t     0x0000337e   READ_ONLY_TAIL
    $b     0x0000338a   READ_ONLY_TAIL
    $b     0x000033b4   READ_ONLY_TAIL
    $b     0x000033c0   READ_ONLY_TAIL
    $b     0x000033cc   READ_ONLY_TAIL
    $b     0x000033d4   READ_ONLY_TAIL
    $b     0x000033da   READ_ONLY_TAIL
    $b     0x000033e6   READ_ONLY_TAIL
    $b     0x00003416   READ_ONLY_TAIL
    $b     0x00003422   READ_ONLY_TAIL
    $b     0x0000342e   READ_ONLY_TAIL
    $b     0x0000343a   READ_ONLY_TAIL
    $b     0x00003468   READ_ONLY_TAIL
    $b     0x00003474   READ_ONLY_TAIL
    $b     0x00003482   READ_ONLY_TAIL
    $b     0x00003488   READ_ONLY_TAIL
    $b     0x00003494   READ_ONLY_TAIL
    $b     0x0000349c   READ_ONLY_TAIL
    $b     0x000034a8   READ_ONLY_TAIL
    $b     0x000034b0   READ_ONLY_TAIL
    $b     0x000034b6   READ_ONLY_TAIL
    $b     0x000034c2   READ_ONLY_TAIL
    $b     0x000034ca   READ_ONLY_TAIL
    $b     0x000034e2   READ_ONLY_TAIL
    $b     0x000034ee   READ_ONLY_TAIL
    $b     0x000034fa   READ_ONLY_TAIL
    $d     0x00003500   READ_ONLY_TAIL
    $t     0x00003508   READ_ONLY_TAIL
    $b     0x00003528   READ_ONLY_TAIL
    $d     0x00003556   READ_ONLY_TAIL
    $t     0x0000355c   READ_ONLY_TAIL
    $b     0x00003582   READ_ONLY_TAIL
    $b     0x000035e0   READ_ONLY_TAIL
    $d     0x000035e8   READ_ONLY_TAIL
    $t     0x000035f8   READ_ONLY_TAIL
    $d     0x00003610   READ_ONLY_TAIL
    $t     0x00003614   READ_ONLY_TAIL
    $d     0x00003660   READ_ONLY_TAIL
    $t     0x00003668   READ_ONLY_TAIL
    $b     0x0000366a   READ_ONLY_TAIL
    $b     0x0000367a   READ_ONLY_TAIL
    $d     0x00003688   READ_ONLY_TAIL
    $t     0x00003690   READ_ONLY_TAIL
    $b     0x00003694   READ_ONLY_TAIL
    $b     0x0000369a   READ_ONLY_TAIL
    $b     0x0000369e   READ_ONLY_TAIL
    $b     0x000036a2   READ_ONLY_TAIL
    $b     0x000036a8   READ_ONLY_TAIL
    $b     0x000036ac   READ_ONLY_TAIL
    $b     0x000036c2   READ_ONLY_TAIL
    $b     0x000036c6   READ_ONLY_TAIL
    $d     0x000036d2   READ_ONLY_TAIL
    $t     0x000036d4   READ_ONLY_TAIL
    $d     0x000036da   READ_ONLY_TAIL
    $t     0x000036dc   READ_ONLY_TAIL
    $d     0x000036e0   READ_ONLY_TAIL
    $t     0x000036e4   READ_ONLY_TAIL
    $d     0x000036f2   READ_ONLY_TAIL
    $t     0x000036f8   READ_ONLY_TAIL
    $b     0x00003702   READ_ONLY_TAIL
    $b     0x00003710   READ_ONLY_TAIL
    $b     0x00003714   READ_ONLY_TAIL
    $b     0x00003720   READ_ONLY_TAIL
    $b     0x0000372a   READ_ONLY_TAIL
    $d     0x00003732   READ_ONLY_TAIL
    $t     0x00003734   READ_ONLY_TAIL
    $d     0x0000373e   READ_ONLY_TAIL
    $t     0x00003744   READ_ONLY_TAIL
    $b     0x0000374c   READ_ONLY_TAIL
    $b     0x00003756   READ_ONLY_TAIL
    $b     0x0000375a   READ_ONLY_TAIL
    $b     0x00003766   READ_ONLY_TAIL
    $b     0x0000376a   READ_ONLY_TAIL
    $d     0x0000378a   READ_ONLY_TAIL
    $t     0x00003790   READ_ONLY_TAIL
    $b     0x000037a8   READ_ONLY_TAIL
    $b     0x000037ae   READ_ONLY_TAIL
    $b     0x000037b2   READ_ONLY_TAIL
    $b     0x000037ba   READ_ONLY_TAIL
    $b     0x000037c0   READ_ONLY_TAIL
    $b     0x000037c4   READ_ONLY_TAIL
    $b     0x000037c8   READ_ONLY_TAIL
    $b     0x000037ce   READ_ONLY_TAIL
    $b     0x000037d2   READ_ONLY_TAIL
    $b     0x000037d6   READ_ONLY_TAIL
    $b     0x000037dc   READ_ONLY_TAIL
    $b     0x000037e0   READ_ONLY_TAIL
    $b     0x000037e4   READ_ONLY_TAIL
    $b     0x000037ea   READ_ONLY_TAIL
    $b     0x000037ee   READ_ONLY_TAIL
    $b     0x00003800   READ_ONLY_TAIL
    $b     0x0000380a   READ_ONLY_TAIL
    $b     0x0000380e   READ_ONLY_TAIL
    $b     0x0000382e   READ_ONLY_TAIL
    $b     0x00003836   READ_ONLY_TAIL
    $b     0x0000383a   READ_ONLY_TAIL
    $b     0x00003846   READ_ONLY_TAIL
    $b     0x0000384c   READ_ONLY_TAIL
    $b     0x00003850   READ_ONLY_TAIL
    $b     0x00003854   READ_ONLY_TAIL
    $b     0x00003858   READ_ONLY_TAIL
    $b     0x00003860   READ_ONLY_TAIL
    $b     0x00003866   READ_ONLY_TAIL
    $d     0x0000386e   READ_ONLY_TAIL
    $t     0x00003880   READ_ONLY_TAIL
    $d     0x00003884   READ_ONLY_TAIL
    $t     0x00003888   READ_ONLY_TAIL
    $d     0x0000388c   READ_ONLY_TAIL
    $t     0x00003890   READ_ONLY_TAIL
    $d     0x000038a2   READ_ONLY_TAIL
    $t     0x000038a8   READ_ONLY_TAIL
    $b     0x000038aa   READ_ONLY_TAIL
    $b     0x000038b0   READ_ONLY_TAIL
    $b     0x000038b4   READ_ONLY_TAIL
    $b     0x000038b8   READ_ONLY_TAIL
    $b     0x000038be   READ_ONLY_TAIL
    $b     0x000038c2   READ_ONLY_TAIL
    $b     0x000038ce   READ_ONLY_TAIL
    $b     0x000038d8   READ_ONLY_TAIL
    $d     0x000038de   READ_ONLY_TAIL
    $t     0x000038e0   READ_ONLY_TAIL
    $b     0x000038e2   READ_ONLY_TAIL
    $b     0x000038e8   READ_ONLY_TAIL
    $b     0x000038ec   READ_ONLY_TAIL
    $b     0x000038f0   READ_ONLY_TAIL
    $b     0x000038f6   READ_ONLY_TAIL
    $b     0x000038fa   READ_ONLY_TAIL
    $b     0x00003906   READ_ONLY_TAIL
    $b     0x00003910   READ_ONLY_TAIL
    $d     0x00003916   READ_ONLY_TAIL
    $t     0x00003918   READ_ONLY_TAIL
    $d     0x00003928   READ_ONLY_TAIL
    $t     0x0000392c   READ_ONLY_TAIL
    $b     0x00003936   READ_ONLY_TAIL
    $b     0x00003944   READ_ONLY_TAIL
    $b     0x00003948   READ_ONLY_TAIL
    $b     0x00003962   READ_ONLY_TAIL
    $b     0x0000396a   READ_ONLY_TAIL
    $b     0x0000396e   READ_ONLY_TAIL
    $d     0x00003974   READ_ONLY_TAIL
    $t     0x00003980   READ_ONLY_TAIL
    $b     0x00003982   READ_ONLY_TAIL
    $b     0x00003988   READ_ONLY_TAIL
    $b     0x0000398c   READ_ONLY_TAIL
    $b     0x00003990   READ_ONLY_TAIL
    $b     0x00003996   READ_ONLY_TAIL
    $b     0x0000399a   READ_ONLY_TAIL
    $b     0x000039a2   READ_ONLY_TAIL
    $b     0x000039a8   READ_ONLY_TAIL
    $b     0x000039b6   READ_ONLY_TAIL
    $b     0x000039be   READ_ONLY_TAIL
    $b     0x000039c4   READ_ONLY_TAIL
    $b     0x000039c8   READ_ONLY_TAIL
    $b     0x000039cc   READ_ONLY_TAIL
    $b     0x000039d2   READ_ONLY_TAIL
    $b     0x000039d6   READ_ONLY_TAIL
    $b     0x000039de   READ_ONLY_TAIL
    $b     0x000039e4   READ_ONLY_TAIL
    $b     0x000039f2   READ_ONLY_TAIL
    $b     0x000039fa   READ_ONLY_TAIL
    $b     0x00003a00   READ_ONLY_TAIL
    $b     0x00003a04   READ_ONLY_TAIL
    $b     0x00003a08   READ_ONLY_TAIL
    $b     0x00003a0e   READ_ONLY_TAIL
    $b     0x00003a12   READ_ONLY_TAIL
    $b     0x00003a1a   READ_ONLY_TAIL
    $b     0x00003a28   READ_ONLY_TAIL
    $d     0x00003a2e   READ_ONLY_TAIL
    $t     0x00003a30   READ_ONLY_TAIL
    $d     0x00003a32   READ_ONLY_TAIL
    $a     0x00003a34   READ_ONLY_TAIL
    $t     0x00003a74   READ_ONLY_TAIL
    $d     0x00003a76   READ_ONLY_TAIL
    $a     0x00003a78   READ_ONLY_TAIL
    $t     0x00003ae0   READ_ONLY_TAIL
    $d     0x00003ae2   READ_ONLY_TAIL
    $a     0x00003ae4   READ_ONLY_TAIL
    $t     0x00003aec   READ_ONLY_TAIL
    $d     0x00003aee   READ_ONLY_TAIL
    $a     0x00003af0   READ_ONLY_TAIL
    $t     0x00003b64   READ_ONLY_TAIL
    $d     0x00003b66   READ_ONLY_TAIL
    $a     0x00003b68   READ_ONLY_TAIL
    $d     0x00003be4   READ_ONLY_TAIL
    $t     0x00003be8   READ_ONLY_TAIL
    $d     0x00003bea   READ_ONLY_TAIL
    $a     0x00003bec   READ_ONLY_TAIL
    $d     0x00003d2c   READ_ONLY_TAIL
    $t     0x00003d50   READ_ONLY_TAIL
    $d     0x00003d52   READ_ONLY_TAIL
    $a     0x00003d54   READ_ONLY_TAIL
    $t     0x00003d6c   READ_ONLY_TAIL
    $d     0x00003d6e   READ_ONLY_TAIL
    $a     0x00003d70   READ_ONLY_TAIL
    $d     0x00003e00   READ_ONLY_TAIL
    $t     0x00003e08   READ_ONLY_TAIL
    $d     0x00003e0a   READ_ONLY_TAIL
    $a     0x00003e0c   READ_ONLY_TAIL
    $t     0x00003e30   READ_ONLY_TAIL
    $d     0x00003e32   READ_ONLY_TAIL
    $a     0x00003e34   READ_ONLY_TAIL
    $d     0x00003eb4   READ_ONLY_TAIL
    $f     0x000041f0   READ_ONLY_TAIL
    $d     0x00004244   READ_ONLY_TAIL
    $f     0x000042bc   READ_ONLY_TAIL
    $f     0x000042c0   READ_ONLY_TAIL
    $f     0x000042c4   READ_ONLY_TAIL
    $f     0x000042c8   READ_ONLY_TAIL
    $d     0x000042cc   READ_ONLY_TAIL
    $d     0x08000000   EXT_READ_WRITE
    $d     0x40000000   BL_INFO_NOR
    $t     0x40000080   EMIINIT_CODE
    $a     0x40000080   FAST_ALGORITHM
    $d     0x40000084   FAST_ALGORITHM
    $f     0x40000084   FAST_ALGORITHM
    $a     0x40000088   FAST_ALGORITHM
    $d     0x4000008c   FAST_ALGORITHM
    $f     0x4000008c   FAST_ALGORITHM
    $a     0x40000090   FAST_ALGORITHM
    $d     0x40000094   FAST_ALGORITHM
    $f     0x40000094   FAST_ALGORITHM
    $a     0x40000098   FAST_ALGORITHM
    $d     0x4000009c   FAST_ALGORITHM
    $f     0x4000009c   FAST_ALGORITHM
    $a     0x400000a0   FAST_ALGORITHM
    $d     0x400000a4   FAST_ALGORITHM
    $f     0x400000a4   FAST_ALGORITHM
    $a     0x400000a8   FAST_ALGORITHM
    $d     0x400000ac   FAST_ALGORITHM
    $f     0x400000ac   FAST_ALGORITHM
    $a     0x400000b0   FAST_ALGORITHM
    $d     0x400000b4   FAST_ALGORITHM
    $f     0x400000b4   FAST_ALGORITHM
    $a     0x400000b8   FAST_ALGORITHM
    $d     0x400000bc   FAST_ALGORITHM
    $f     0x400000bc   FAST_ALGORITHM
    $t     0x400000c0   FAST_ALGORITHM
    $d     0x400000dc   FAST_ALGORITHM
    $t     0x400000e4   FAST_ALGORITHM
    $d     0x400000ec   FAST_ALGORITHM
    $t     0x400000f0   FAST_ALGORITHM
    $d     0x40000100   FAST_ALGORITHM
    $t     0x40000104   FAST_ALGORITHM
    $d     0x40000106   FAST_ALGORITHM
    $t     0x40000108   FAST_ALGORITHM
    $d     0x4000011a   EMIINIT_CODE
    $t     0x4000013c   EMIINIT_CODE
    $b     0x4000013e   EMIINIT_CODE
    $b     0x4000014a   EMIINIT_CODE
    $b     0x4000014e   EMIINIT_CODE
    $b     0x40000150   FAST_ALGORITHM
    $b     0x40000154   EMIINIT_CODE
    $b     0x40000158   EMIINIT_CODE
    $b     0x4000015c   EMIINIT_CODE
    $d     0x40000162   EMIINIT_CODE
    $b     0x40000164   FAST_ALGORITHM
    $t     0x40000168   EMIINIT_CODE
    $b     0x40000170   FAST_ALGORITHM
    $b     0x40000178   FAST_ALGORITHM
    $b     0x40000184   FAST_ALGORITHM
    $d     0x400001ba   EMIINIT_CODE
    $t     0x400001cc   EMIINIT_CODE
    $b     0x400001f2   FAST_ALGORITHM
    $b     0x4000021a   FAST_ALGORITHM
    $b     0x40000220   FAST_ALGORITHM
    $b     0x40000228   FAST_ALGORITHM
    $b     0x40000254   FAST_ALGORITHM
    $d     0x4000026c   FAST_ALGORITHM
    $t     0x40000284   FAST_ALGORITHM
    $b     0x400002ae   FAST_ALGORITHM
    $d     0x400002e2   FAST_ALGORITHM
    $t     0x400002ec   FAST_ALGORITHM
    $b     0x400002fe   FAST_ALGORITHM
    $d     0x40000304   EMIINIT_CODE
    $d     0x40000324   FAST_ALGORITHM
    $t     0x40000328   FAST_ALGORITHM
    $a     0x40000330   EMIINIT_CODE
    $d     0x40000338   EMIINIT_CODE
    $f     0x40000338   EMIINIT_CODE
    $b     0x40000340   FAST_ALGORITHM
    $d     0x4000034c   FAST_ALGORITHM
    $t     0x40000354   FAST_ALGORITHM
    $d     0x40000394   FAST_ALGORITHM
    $t     0x4000060c   FAST_CODE
    $b     0x40000616   FAST_CODE
    $b     0x4000061c   FAST_CODE
    $d     0x40000622   FAST_CODE
    $t     0x40000628   FAST_CODE
    $b     0x40000638   FAST_CODE
    $b     0x4000063e   FAST_CODE
    $b     0x40000644   FAST_CODE
    $b     0x4000064c   FAST_CODE
    $b     0x40000658   FAST_CODE
    $b     0x4000065e   FAST_CODE
    $d     0x4000066a   FAST_CODE
    $t     0x40000678   FAST_CODE
    $b     0x4000067e   FAST_CODE
    $b     0x400006be   FAST_CODE
    $b     0x400006e6   FAST_CODE
    $b     0x4000070c   FAST_CODE
    $b     0x4000073a   FAST_CODE
    $b     0x40000764   FAST_CODE
    $b     0x40000772   FAST_CODE
    $d     0x4000077a   FAST_CODE
    $t     0x40000788   FAST_CODE
    $d     0x400007b4   FAST_CODE
    $t     0x400007bc   FAST_CODE
    $d     0x400007e8   FAST_CODE
    $a     0x400007f4   FAST_CODE
    $d     0x40000810   FAST_CODE
    $f     0x40000810   FAST_CODE
    $a     0x40000814   FAST_CODE
    $d     0x4000081c   FAST_CODE
    $f     0x4000081c   FAST_CODE
    $a     0x40000820   FAST_CODE
    $d     0x40000828   FAST_CODE
    $f     0x40000828   FAST_CODE
    $a     0x4000082c   FAST_CODE
    $d     0x40000834   FAST_CODE
    $f     0x40000834   FAST_CODE
    $d     0x4001cc00   READ_WRITE

    Local Symbols

    Symbol Name                              Value     Ov Type        Size  Object(Section)

    drv\src\NAND_DevConfig.c                 0x00000000   Number         0  NAND_DevConfig.obj ABSOLUTE
    sss\interface\src\SSS_interface.c        0x00000000   Number         0  SSS_interface.obj ABSOLUTE
    .constdata                               0x00003eb5   Data           0  SSS_interface.obj(.constdata)
    .constdata                               0x00003eb8   Data           0  SSS_interface.obj(.constdata)
    .constdata                               0x00003ec0   Data           0  SSS_interface.obj(.constdata)
    .constdata                               0x00003eb4   Data           0  SSS_interface.obj(.constdata)
    .constdata                               0x00003ec8   Data           0  SSS_interface.obj(.constdata)
    .constdata                               0x00003ec4   Data           0  SSS_interface.obj(.constdata)
    .constdata                               0x00003ebc   Data           0  SSS_interface.obj(.constdata)
    .constdata$42                            0x00003eb4   Data           0  SSS_interface.obj(.constdata)
    .constdata$52                            0x00003eb5   Data           0  SSS_interface.obj(.constdata)
    .constdata$107                           0x00003eb8   Data           0  SSS_interface.obj(.constdata)
    .constdata$112                           0x00003ebc   Data           0  SSS_interface.obj(.constdata)
    .constdata$122                           0x00003ec0   Data           0  SSS_interface.obj(.constdata)
    .constdata$137                           0x00003ec4   Data           0  SSS_interface.obj(.constdata)
    .constdata$152                           0x00003ec8   Data           0  SSS_interface.obj(.constdata)
    bootloader\src\bl_Alg.c                  0x00000000   Number         0  bl_Alg.obj ABSOLUTE
    BL_ALGORITHM                             0x00000a78   Thumb Code     0  bl_Alg.obj(BL_ALGORITHM)
    BL_ALGORITHM                             0x00000a74   Thumb Code     0  bl_Alg.obj(BL_ALGORITHM)
    C$debug_frame189                         0x00000000   Data           0  bl_Alg.obj(.debug_frame)
    C$debug_frame190                         0x0000003c   Data           0  bl_Alg.obj(.debug_frame)
    bootloader/src/bl_BOOTARM.s              0x00000000   Number         0  bl_BOOTARM.obj ABSOLUTE
    DUMMY_POOL                               0x0800003c   Data           4  bl_BOOTARM.obj(DUMMY_POOL)
    C$$code                                  0x00000000   ARM Code     164  bl_BOOTARM.obj(C$$code)
    <Anonymous Symbol>                       0x00000000   Data          96  bl_BOOTARM.obj(.debug_info)
    SHARECODE                                0x400007f0   Data          24  bl_BOOTARM.obj(SHARECODE)
    STACK_POOL_INTSRAM                       0x4001cc00   Data        4096  bl_BOOTARM.obj(STACK_POOL_INTSRAM)
    <Anonymous Symbol>                       0x00000000   Data         176  bl_BOOTARM.obj(.debug_line)
    <Anonymous Symbol>                       0x00000000   Data          12  bl_BOOTARM.obj(.debug_abbrev)
    BOOTROM_FLASH_REMAP                      0x00000002   Number         0  bl_BOOTARM.obj ABSOLUTE
    FLASH_SRAM_REMAP                         0x00000003   Number         0  bl_BOOTARM.obj ABSOLUTE
    Undefined_Handler                        0x00000004   ARM Code       0  bl_BOOTARM.obj(C$$code)
    SWIHandler                               0x00000008   ARM Code       0  bl_BOOTARM.obj(C$$code)
    Prefetch_Handler                         0x0000000c   ARM Code       0  bl_BOOTARM.obj(C$$code)
    Abort_Handler                            0x00000010   ARM Code       0  bl_BOOTARM.obj(C$$code)
    Mode_USR                                 0x00000010   Number         0  bl_BOOTARM.obj ABSOLUTE
    Mode_FIQ                                 0x00000011   Number         0  bl_BOOTARM.obj ABSOLUTE
    Mode_IRQ                                 0x00000012   Number         0  bl_BOOTARM.obj ABSOLUTE
    Mode_SVC                                 0x00000013   Number         0  bl_BOOTARM.obj ABSOLUTE
    SUP_MODE                                 0x00000013   Number         0  bl_BOOTARM.obj ABSOLUTE
    Reserved_vector                          0x00000014   ARM Code       0  bl_BOOTARM.obj(C$$code)
    Mode_ABT                                 0x00000017   Number         0  bl_BOOTARM.obj ABSOLUTE
    IrqHandler                               0x00000018   ARM Code       0  bl_BOOTARM.obj(C$$code)
    Mode_UNDEF                               0x0000001b   Number         0  bl_BOOTARM.obj ABSOLUTE
    FiqHandler                               0x0000001c   ARM Code       0  bl_BOOTARM.obj(C$$code)
    MODE_MASK                                0x0000001f   Number         0  bl_BOOTARM.obj ABSOLUTE
    Mode_SYS                                 0x0000001f   Number         0  bl_BOOTARM.obj ABSOLUTE
    BOOT_Stack_End                           0x00000020   Data           0  bl_BOOTARM.obj(C$$code)
    BOOT_Stack_Start                         0x00000024   Data           0  bl_BOOTARM.obj(C$$code)
    DUMMY_PTR                                0x00000028   Data           0  bl_BOOTARM.obj(C$$code)
    ResetHandler                             0x0000002c   ARM Code       0  bl_BOOTARM.obj(C$$code)
    F_BIT                                    0x00000040   Number         0  bl_BOOTARM.obj ABSOLUTE
    stack_fill_ff                            0x0000004c   ARM Code       0  bl_BOOTARM.obj(C$$code)
    I_BIT                                    0x00000080   Number         0  bl_BOOTARM.obj ABSOLUTE
    End_BootLoader                           0x000000a0   ARM Code       0  bl_BOOTARM.obj(C$$code)
    INT_BIT                                  0x000000c0   Number         0  bl_BOOTARM.obj ABSOLUTE
    LOCKOUT                                  0x000000c0   Number         0  bl_BOOTARM.obj ABSOLUTE
    LOCK_MSK                                 0x000000c0   Number         0  bl_BOOTARM.obj ABSOLUTE
    SPV_STACK_SIZE                           0x00001000   Number         0  bl_BOOTARM.obj ABSOLUTE
    DUMMY_END                                0x0800003c   Data           0  bl_BOOTARM.obj(DUMMY_POOL)
    EMI_BASE_REG                             0x400007f0   Data           0  bl_BOOTARM.obj(SHARECODE)
    SPV_Stack_Pool                           0x4001cc00   Data           0  bl_BOOTARM.obj(STACK_POOL_INTSRAM)
    bootloader\src\bl_Cache.c                0x00000000   Number         0  bl_Cache.obj ABSOLUTE
    EXT_BOOTLOADER_CODE                      0x00000be4   Thumb Code     0  bl_Cache.obj(EXT_BOOTLOADER_CODE)
    EXT_BOOTLOADER_CODE                      0x00000bd0   Thumb Code     0  bl_Cache.obj(EXT_BOOTLOADER_CODE)
    C$debug_frame192                         0x00000078   Data           0  bl_Cache.obj(.debug_frame)
    C$debug_frame193                         0x000000c4   Data           0  bl_Cache.obj(.debug_frame)
    bootloader\src\bl_DBGPRINT.c             0x00000000   Number         0  bl_DBGPRINT.obj ABSOLUTE
    i.itoa                                   0x40000284   Thumb Code     0  bl_DBGPRINT.obj(i.itoa)
    i.dbg_print                              0x4000010c   Thumb Code     0  bl_DBGPRINT.obj(i.dbg_print)
    i.itof                                   0x400002ec   Thumb Code     0  bl_DBGPRINT.obj(i.itof)
    .constdata                               0x4000039c   Data           0  bl_DBGPRINT.obj(.constdata)
    .bss                                     0x400003e0   Data           0  bl_DBGPRINT.obj(.bss)
    C$debug_frame190                         0x0000010c   Data           0  bl_DBGPRINT.obj(.debug_frame)
    C$debug_frame191                         0x0000015c   Data           0  bl_DBGPRINT.obj(.debug_frame)
    C$debug_frame192                         0x000001bc   Data           0  bl_DBGPRINT.obj(.debug_frame)
    itoa                                     0x40000284   Thumb Code    94  bl_DBGPRINT.obj(i.itoa)
    .constdata$1                             0x4000039c   Data           0  bl_DBGPRINT.obj(.constdata)
    .bss$2                                   0x400003e0   Data           0  bl_DBGPRINT.obj(.bss)
    rev@itoa_0                               0x400003e0   Data          21  bl_DBGPRINT.obj(.bss)
    rev@itof_0                               0x400003f5   Data          21  bl_DBGPRINT.obj(.bss)
    bootloader\src\bl_FOTA.c                 0x00000000   Number         0  bl_FOTA.obj ABSOLUTE
    bootloader\src\bl_ImageLoader.c          0x00000000   Number         0  bl_ImageLoader.obj ABSOLUTE
    i.PreserveExtBootloaderHeader            0x00001904   Thumb Code     0  bl_ImageLoader.obj(i.PreserveExtBootloaderHeader)
    EXT_BOOTLOADER_CODE                      0x00000c14   Thumb Code     0  bl_ImageLoader.obj(EXT_BOOTLOADER_CODE)
    BL_INFO_NOR                              0x40000000   Data           0  bl_ImageLoader.obj(BL_INFO_NOR)
    i.LoadExtBootloader                      0x00001900   Thumb Code     0  bl_ImageLoader.obj(i.LoadExtBootloader)
    C$debug_frame14                          0x00000210   Data           0  bl_ImageLoader.obj(.debug_frame)
    C$debug_frame15                          0x0000024c   Data           0  bl_ImageLoader.obj(.debug_frame)
    C$debug_frame16                          0x00000288   Data           0  bl_ImageLoader.obj(.debug_frame)
    BL_INFO_NOR$8                            0x40000000   Data           0  bl_ImageLoader.obj(BL_INFO_NOR)
    bootloader\src\bl_Init.c                 0x00000000   Number         0  bl_Init.obj ABSOLUTE
    EXT_BOOTLOADER_CODE                      0x00000c18   Thumb Code     0  bl_Init.obj(EXT_BOOTLOADER_CODE)
    i.Init                                   0x000018c0   Thumb Code     0  bl_Init.obj(i.Init)
    i.Init_DTLB                              0x000018fc   Thumb Code     0  bl_Init.obj(i.Init_DTLB)
    .constdata                               0x00003ecc   Data           0  bl_Init.obj(.constdata)
    EXT_BOOTLOADER_CODE                      0x00000c50   Thumb Code     0  bl_Init.obj(EXT_BOOTLOADER_CODE)
    i.WacthDogRestart                        0x00003658   Thumb Code     0  bl_Init.obj(i.WacthDogRestart)
    i.isGPTTImer3Started                     0x0000377c   Thumb Code     0  bl_Init.obj(i.isGPTTImer3Started)
    EXT_BOOTLOADER_CODE                      0x00000c70   Thumb Code     0  bl_Init.obj(EXT_BOOTLOADER_CODE)
    i.WatchDogResetAll                       0x00003680   Thumb Code     0  bl_Init.obj(i.WatchDogResetAll)
    EMIINITCODE                              0x4000013c   Thumb Code     0  bl_Init.obj(EMIINITCODE)
    i.startGPTTImer3                         0x00003918   Thumb Code     0  bl_Init.obj(i.startGPTTImer3)
    i.getGPTTImer3Value                      0x00003734   Thumb Code     0  bl_Init.obj(i.getGPTTImer3Value)
    EMIINITCODE                              0x40000080   Thumb Code     0  bl_Init.obj(EMIINITCODE)
    EXT_BOOTLOADER_CODE                      0x00000c48   Thumb Code     0  bl_Init.obj(EXT_BOOTLOADER_CODE)
    i.DriverInit                             0x0000137c   Thumb Code     0  bl_Init.obj(i.DriverInit)
    i.WaitFor32KStable                       0x00003668   Thumb Code     0  bl_Init.obj(i.WaitFor32KStable)
    i.GenerateRandomSeed                     0x000016a0   Thumb Code     0  bl_Init.obj(i.GenerateRandomSeed)
    C$debug_frame12                          0x000002c4   Data           0  bl_Init.obj(.debug_frame)
    C$debug_frame14                          0x00000314   Data           0  bl_Init.obj(.debug_frame)
    C$debug_frame16                          0x00000350   Data           0  bl_Init.obj(.debug_frame)
    C$debug_frame17                          0x0000038c   Data           0  bl_Init.obj(.debug_frame)
    C$debug_frame18                          0x000003d8   Data           0  bl_Init.obj(.debug_frame)
    C$debug_frame19                          0x00000414   Data           0  bl_Init.obj(.debug_frame)
    C$debug_frame21                          0x00000450   Data           0  bl_Init.obj(.debug_frame)
    C$debug_frame23                          0x0000048c   Data           0  bl_Init.obj(.debug_frame)
    C$debug_frame24                          0x000004c8   Data           0  bl_Init.obj(.debug_frame)
    C$debug_frame26                          0x00000518   Data           0  bl_Init.obj(.debug_frame)
    C$debug_frame27                          0x00000564   Data           0  bl_Init.obj(.debug_frame)
    C$debug_frame28                          0x000005b0   Data           0  bl_Init.obj(.debug_frame)
    C$debug_frame29                          0x000005fc   Data           0  bl_Init.obj(.debug_frame)
    C$debug_frame30                          0x00000648   Data           0  bl_Init.obj(.debug_frame)
    C$debug_frame31                          0x00000698   Data           0  bl_Init.obj(.debug_frame)
    C$debug_frame32                          0x000006d4   Data           0  bl_Init.obj(.debug_frame)
    .constdata$1                             0x00003ecc   Data           0  bl_Init.obj(.constdata)
    bootloader\src\bl_Main.c                 0x00000000   Number         0  bl_Main.obj ABSOLUTE
    EXT_BOOTLOADER_CODE                      0x00000d18   Thumb Code     0  bl_Main.obj(EXT_BOOTLOADER_CODE)
    HEAD_BL                                  0x000000bc   Data           0  bl_Main.obj(HEAD_BL)
    EXT_BOOTLOADER_CODE                      0x00000d00   Thumb Code     0  bl_Main.obj(EXT_BOOTLOADER_CODE)
    i.INT_Version_Check_PutUARTByte          0x000018ac   Thumb Code     0  bl_Main.obj(i.INT_Version_Check_PutUARTByte)
    INTERNCODE                               0x40000628   Thumb Code     0  bl_Main.obj(INTERNCODE)
    EXT_BOOTLOADER_CODE                      0x00000e30   Thumb Code     0  bl_Main.obj(EXT_BOOTLOADER_CODE)
    EXT_BOOTLOADER_CODE                      0x00000cc8   Thumb Code     0  bl_Main.obj(EXT_BOOTLOADER_CODE)
    .data                                    0x08000000   Data           0  bl_Main.obj(.data)
    .constdata                               0x00003f00   Data           0  bl_Main.obj(.constdata)
    EXT_BOOTLOADER_CODE                      0x00000cac   Thumb Code     0  bl_Main.obj(EXT_BOOTLOADER_CODE)
    EXT_BOOTLOADER_CODE                      0x00000ec8   Thumb Code     0  bl_Main.obj(EXT_BOOTLOADER_CODE)
    EXT_BOOTLOADER_CODE                      0x00000dd4   Thumb Code     0  bl_Main.obj(EXT_BOOTLOADER_CODE)
    i.INT_Version_Check                      0x00001770   Thumb Code     0  bl_Main.obj(i.INT_Version_Check)
    EXT_BOOTLOADER_CODE                      0x00000e60   Thumb Code     0  bl_Main.obj(EXT_BOOTLOADER_CODE)
    INTERNCODE                               0x4000060c   Thumb Code     0  bl_Main.obj(INTERNCODE)
    .bss                                     0x08000040   Data           0  bl_Main.obj(.bss)
    EXT_BOOTLOADER_CODE                      0x00000d68   Thumb Code     0  bl_Main.obj(EXT_BOOTLOADER_CODE)
    i.VerifyExtBootloader                    0x00003654   Thumb Code     0  bl_Main.obj(i.VerifyExtBootloader)
    HEAD_BL$5                                0x000000bc   Data           0  bl_Main.obj(HEAD_BL)
    C$debug_frame21                          0x00000720   Data           0  bl_Main.obj(.debug_frame)
    C$debug_frame22                          0x0000075c   Data           0  bl_Main.obj(.debug_frame)
    C$debug_frame23                          0x000007b0   Data           0  bl_Main.obj(.debug_frame)
    C$debug_frame24                          0x000007ec   Data           0  bl_Main.obj(.debug_frame)
    C$debug_frame25                          0x0000083c   Data           0  bl_Main.obj(.debug_frame)
    C$debug_frame26                          0x00000888   Data           0  bl_Main.obj(.debug_frame)
    C$debug_frame27                          0x000008c4   Data           0  bl_Main.obj(.debug_frame)
    C$debug_frame28                          0x0000091c   Data           0  bl_Main.obj(.debug_frame)
    C$debug_frame29                          0x0000096c   Data           0  bl_Main.obj(.debug_frame)
    C$debug_frame30                          0x000009c4   Data           0  bl_Main.obj(.debug_frame)
    C$debug_frame31                          0x00000a10   Data           0  bl_Main.obj(.debug_frame)
    C$debug_frame32                          0x00000a5c   Data           0  bl_Main.obj(.debug_frame)
    C$debug_frame33                          0x00000aa8   Data           0  bl_Main.obj(.debug_frame)
    C$debug_frame34                          0x00000af4   Data           0  bl_Main.obj(.debug_frame)
    .constdata$1                             0x00003f00   Data           0  bl_Main.obj(.constdata)
    .data$0                                  0x08000000   Data           0  bl_Main.obj(.data)
    usbdl_timer_start                        0x08000000   Data           2  bl_Main.obj(.data)
    .bss$2                                   0x08000040   Data           0  bl_Main.obj(.bss)
    usbdl_timer_state                        0x08000042   Data           1  bl_Main.obj(.bss)
    explicitUSBDL@USBDL_Ready_To_Enter_DLMode_0 0x08000043   Data           1  bl_Main.obj(.bss)
    boot_config                              0x08000044   Data           2  bl_Main.obj(.bss)
    bootloader\src\bl_NFI.c                  0x00000000   Number         0  bl_NFI.obj ABSOLUTE
    bootloader\src\bl_NFI_V3.c               0x00000000   Number         0  bl_NFI_V3.obj ABSOLUTE
    bootloader\src\bl_UART.c                 0x00000000   Number         0  bl_UART.obj ABSOLUTE
    i.uart_init                              0x40000354   Thumb Code     0  bl_UART.obj(i.uart_init)
    i.CheckUARTSendEnd                       0x400000c0   Thumb Code     0  bl_UART.obj(i.CheckUARTSendEnd)
    .data                                    0x08000002   Data           0  bl_UART.obj(.data)
    i.PutUARTByte                            0x400000f0   Thumb Code     0  bl_UART.obj(i.PutUARTByte)
    C$debug_frame192                         0x00000b30   Data           0  bl_UART.obj(.debug_frame)
    C$debug_frame193                         0x00000b6c   Data           0  bl_UART.obj(.debug_frame)
    C$debug_frame194                         0x00000ba8   Data           0  bl_UART.obj(.debug_frame)
    .data$0                                  0x08000002   Data           0  bl_UART.obj(.data)
    bootloader\src\bl_portingfunc.c          0x00000000   Number         0  bl_portingfunc.obj ABSOLUTE
    i.kal_assert_fail                        0x40000328   Thumb Code     0  bl_portingfunc.obj(i.kal_assert_fail)
    i.SaveAndSetIRQMask                      0x40000108   Thumb Code     0  bl_portingfunc.obj(i.SaveAndSetIRQMask)
    i.INT_DisableCacheOnEMI                  0x400000e4   Thumb Code     0  bl_portingfunc.obj(i.INT_DisableCacheOnEMI)
    i.RestoreIRQMask                         0x40000104   Thumb Code     0  bl_portingfunc.obj(i.RestoreIRQMask)
    .constdata                               0x400003a4   Data           0  bl_portingfunc.obj(.constdata)
    C$debug_frame188                         0x00000be4   Data           0  bl_portingfunc.obj(.debug_frame)
    C$debug_frame189                         0x00000c20   Data           0  bl_portingfunc.obj(.debug_frame)
    C$debug_frame190                         0x00000c5c   Data           0  bl_portingfunc.obj(.debug_frame)
    C$debug_frame192                         0x00000c98   Data           0  bl_portingfunc.obj(.debug_frame)
    .constdata$1                             0x400003a4   Data           0  bl_portingfunc.obj(.constdata)
    bootloader/src/bl_regioninit.s           0x00000000   Number         0  bl_regioninit.obj ABSOLUTE
    <Anonymous Symbol>                       0x0000000c   Data          12  bl_regioninit.obj(.debug_abbrev)
    <Anonymous Symbol>                       0x000000b0   Data         172  bl_regioninit.obj(.debug_line)
    EXT_BOOTLOADER_CODE                      0x00000ecc   ARM Code       8  bl_regioninit.obj(EXT_BOOTLOADER_CODE)
    RegionInit                               0x00000ed4   ARM Code     756  bl_regioninit.obj(RegionInit)
    <Anonymous Symbol>                       0x00000060   Data         100  bl_regioninit.obj(.debug_info)
    copy                                     0x00001010   ARM Code       0  bl_regioninit.obj(RegionInit)
    copy_region                              0x00001024   ARM Code       0  bl_regioninit.obj(RegionInit)
    backward_copy                            0x00001044   ARM Code       0  bl_regioninit.obj(RegionInit)
    zi_init                                  0x00001058   ARM Code       0  bl_regioninit.obj(RegionInit)
    bootloader\src\bl_verno.c                0x00000000   Number         0  bl_verno.obj ABSOLUTE
    .constdata                               0x00003fcc   Data           0  bl_verno.obj(.constdata)
    .constdata$46                            0x00003fcc   Data           0  bl_verno.obj(.constdata)
    init\src\cache.c                         0x00000000   Number         0  cache.obj ABSOLUTE
    INTERNCODE                               0x400006c4   Thumb Code     0  cache.obj(INTERNCODE)
    INTERNCODE                               0x40000788   Thumb Code     0  cache.obj(INTERNCODE)
    .constdata                               0x00003fd4   Data           0  cache.obj(.constdata)
    i.CodeCacheGetChannel                    0x00001254   Thumb Code     0  cache.obj(i.CodeCacheGetChannel)
    INTERNCODE                               0x40000678   Thumb Code     0  cache.obj(INTERNCODE)
    .bss                                     0x08000050   Data           0  cache.obj(.bss)
    INTERNCODE                               0x400007bc   Thumb Code     0  cache.obj(INTERNCODE)
    C$debug_frame210                         0x00000ce4   Data           0  cache.obj(.debug_frame)
    C$debug_frame212                         0x00000d3c   Data           0  cache.obj(.debug_frame)
    C$debug_frame213                         0x00000d8c   Data           0  cache.obj(.debug_frame)
    C$debug_frame214                         0x00000de8   Data           0  cache.obj(.debug_frame)
    C$debug_frame216                         0x00000e34   Data           0  cache.obj(.debug_frame)
    .constdata$1                             0x00003fd4   Data           0  cache.obj(.constdata)
    CACHE_CHANNEL_OFFSET_TABLE               0x00003fd4   Data          60  cache.obj(.constdata)
    .bss$2                                   0x08000050   Data           0  cache.obj(.bss)
    MPUChannelStatus                         0x08000050   Data           2  cache.obj(.bss)
    CodeCacheChannelStatus                   0x08000052   Data           2  cache.obj(.bss)
    init/src/cp15.s                          0x00000000   Number         0  cp15.obj ABSOLUTE
    custom\system\NOLLEC53_09B_PMWY_BB\custom_blconfig.c 0x00000000   Number         0  custom_blconfig.obj ABSOLUTE
    i.custom_ROM_baseaddr                    0x000036dc   Thumb Code     0  custom_blconfig.obj(i.custom_ROM_baseaddr)
    .constdata                               0x000041d0   Data           0  custom_blconfig.obj(.constdata)
    i.custom_get_software_version            0x000036e8   Thumb Code     0  custom_blconfig.obj(i.custom_get_software_version)
    i.custom_RAM_baseaddr                    0x000036d4   Thumb Code     0  custom_blconfig.obj(i.custom_RAM_baseaddr)
    .constdata                               0x000041d2   Data           0  custom_blconfig.obj(.constdata)
    i.custom_check_valid_secro               0x000036e4   Thumb Code     0  custom_blconfig.obj(i.custom_check_valid_secro)
    C$debug_frame200                         0x00000e80   Data           0  custom_blconfig.obj(.debug_frame)
    C$debug_frame201                         0x00000ebc   Data           0  custom_blconfig.obj(.debug_frame)
    C$debug_frame202                         0x00000ef8   Data           0  custom_blconfig.obj(.debug_frame)
    C$debug_frame203                         0x00000f34   Data           0  custom_blconfig.obj(.debug_frame)
    .constdata$41                            0x000041d0   Data           0  custom_blconfig.obj(.constdata)
    .constdata$46                            0x000041d2   Data           0  custom_blconfig.obj(.constdata)
    custom\system\NOLLEC53_09B_PMWY_BB\custom_emi.c 0x00000000   Number         0  custom_emi.obj ABSOLUTE
    .data                                    0x08000018   Data           0  custom_emi.obj(.data)
    i.custom_InitDRAM                        0x000036cc   Thumb Code     0  custom_emi.obj(i.custom_InitDRAM)
    EMIINITCODE                              0x40000168   Thumb Code     0  custom_emi.obj(EMIINITCODE)
    SECOND_PART                              0x000049a4   Data           0  custom_emi.obj(SECOND_PART)
    .constdata                               0x000041d4   Data           0  custom_emi.obj(.constdata)
    EMIINITCODE                              0x400001cc   Thumb Code     0  custom_emi.obj(EMIINITCODE)
    C$debug_frame210                         0x00000f70   Data           0  custom_emi.obj(.debug_frame)
    C$debug_frame211                         0x00000fbc   Data           0  custom_emi.obj(.debug_frame)
    C$debug_frame212                         0x00000ff8   Data           0  custom_emi.obj(.debug_frame)
    .constdata$1                             0x000041d4   Data           0  custom_emi.obj(.constdata)
    nor_compare_pattern                      0x000041d8   Data           4  custom_emi.obj(.constdata)
    SECOND_PART$50                           0x000049a4   Data           0  custom_emi.obj(SECOND_PART)
    .data$0                                  0x08000018   Data           0  custom_emi.obj(.data)
    custom\system\NOLLEC53_09B_PMWY_BB\custom_flash.c 0x00000000   Number         0  custom_flash.obj ABSOLUTE
    drv\src\gpio.c                           0x00000000   Number         0  gpio.obj ABSOLUTE
    i.GPIO_InitIO                            0x00001388   Thumb Code     0  gpio.obj(i.GPIO_InitIO)
    i.GPIO_PullenSetup                       0x000014bc   Thumb Code     0  gpio.obj(i.GPIO_PullenSetup)
    i.GPIO_PullSelSetup                      0x00001474   Thumb Code     0  gpio.obj(i.GPIO_PullSelSetup)
    i.GPIO_ModeSetup                         0x00001400   Thumb Code     0  gpio.obj(i.GPIO_ModeSetup)
    i.GPIO_ReadIO                            0x00001504   Thumb Code     0  gpio.obj(i.GPIO_ReadIO)
    C$debug_frame214                         0x0000104c   Data           0  gpio.obj(.debug_frame)
    C$debug_frame217                         0x0000109c   Data           0  gpio.obj(.debug_frame)
    C$debug_frame219                         0x000010d8   Data           0  gpio.obj(.debug_frame)
    C$debug_frame220                         0x00001114   Data           0  gpio.obj(.debug_frame)
    C$debug_frame221                         0x00001168   Data           0  gpio.obj(.debug_frame)
    custom\drv\misc_drv\NOLLEC53_09B_PMWY_BB\gpio_drv.c 0x00000000   Number         0  gpio_drv.obj ABSOLUTE
    i.GPIO_init                              0x00001560   Thumb Code     0  gpio_drv.obj(i.GPIO_init)
    .bss                                     0x08000054   Data           0  gpio_drv.obj(.bss)
    C$debug_frame214                         0x000011b8   Data           0  gpio_drv.obj(.debug_frame)
    .bss$42                                  0x08000054   Data           0  gpio_drv.obj(.bss)
    custom\drv\common_drv\gpio_setting.c     0x00000000   Number         0  gpio_setting.obj ABSOLUTE
    i.GPIO_setting_init                      0x00001568   Thumb Code     0  gpio_setting.obj(i.GPIO_setting_init)
    .data                                    0x08000028   Data           0  gpio_setting.obj(.data)
    .data                                    0x0800001c   Data           0  gpio_setting.obj(.data)
    C$debug_frame216                         0x00001204   Data           0  gpio_setting.obj(.debug_frame)
    .data$45                                 0x0800001c   Data           0  gpio_setting.obj(.data)
    .data$50                                 0x08000028   Data           0  gpio_setting.obj(.data)
    custom\drv\misc_drv\NOLLEC53_09B_PMWY_BB\codegen\gpio_var.c 0x00000000   Number         0  gpio_var.obj ABSOLUTE
    .constdata                               0x000041ec   Data           0  gpio_var.obj(.constdata)
    .constdata$116                           0x000041ec   Data           0  gpio_var.obj(.constdata)
    custom\drv\misc_drv\NOLLEC53_09B_PMWY_BB\keypad_def.c 0x00000000   Number         0  keypad_def.obj ABSOLUTE
    i.keypad_GetFunc                         0x00003880   Thumb Code     0  keypad_def.obj(i.keypad_GetFunc)
    i.keypad_Get_Data                        0x00003888   Thumb Code     0  keypad_def.obj(i.keypad_Get_Data)
    .constdata                               0x000041f0   Data           0  keypad_def.obj(.constdata)
    C$debug_frame219                         0x00001240   Data           0  keypad_def.obj(.debug_frame)
    C$debug_frame220                         0x0000127c   Data           0  keypad_def.obj(.debug_frame)
    .constdata$1                             0x000041f0   Data           0  keypad_def.obj(.constdata)
    interface\l1interface\l1_interface.c     0x00000000   Number         0  l1_interface.obj ABSOLUTE
    i.HW_wait_32k_start                      0x00001718   Thumb Code     0  l1_interface.obj(i.HW_wait_32k_start)
    i.HW_TDMA_Start                          0x0000170c   Thumb Code     0  l1_interface.obj(i.HW_TDMA_Start)
    C$debug_frame195                         0x000012b8   Data           0  l1_interface.obj(.debug_frame)
    C$debug_frame197                         0x000012f4   Data           0  l1_interface.obj(.debug_frame)
    drv\src\nand_dal.c                       0x00000000   Number         0  nand_dal.obj ABSOLUTE
    drv\src\nand_mtd_fdm50.c                 0x00000000   Number         0  nand_mtd_fdm50.obj ABSOLUTE
    custom\drv\common_drv\pwic_cust.c        0x00000000   Number         0  pwic_cust.obj ABSOLUTE
    custom\drv\misc_drv\NOLLEC53_09B_PMWY_BB\usb_custom.c 0x00000000   Number         0  usb_custom.obj ABSOLUTE
    .constdata                               0x0000431c   Data           0  usb_custom.obj(.constdata)
    .constdata                               0x000042cc   Data           0  usb_custom.obj(.constdata)
    .constdata                               0x000043aa   Data           0  usb_custom.obj(.constdata)
    .constdata                               0x000042f8   Data           0  usb_custom.obj(.constdata)
    .constdata                               0x00004338   Data           0  usb_custom.obj(.constdata)
    .constdata                               0x000043d0   Data           0  usb_custom.obj(.constdata)
    .constdata                               0x00004384   Data           0  usb_custom.obj(.constdata)
    .constdata                               0x000042e6   Data           0  usb_custom.obj(.constdata)
    i.USB_GetVideoParam                      0x0000270c   Thumb Code     0  usb_custom.obj(i.USB_GetVideoParam)
    .constdata                               0x0000435e   Data           0  usb_custom.obj(.constdata)
    i.USB_PowerControl                       0x00002d2c   Thumb Code     0  usb_custom.obj(i.USB_PowerControl)
    i.USB_GetAcmParam                        0x000026ec   Thumb Code     0  usb_custom.obj(i.USB_GetAcmParam)
    .constdata                               0x00004244   Data           0  usb_custom.obj(.constdata)
    .constdata                               0x000043fe   Data           0  usb_custom.obj(.constdata)
    i.USB_GetCustomFunc                      0x000026f4   Thumb Code     0  usb_custom.obj(i.USB_GetCustomFunc)
    .constdata                               0x00004424   Data           0  usb_custom.obj(.constdata)
    i.USB_GetDeviceParam                     0x000026fc   Thumb Code     0  usb_custom.obj(i.USB_GetDeviceParam)
    i.USB_GetMsParam                         0x00002704   Thumb Code     0  usb_custom.obj(i.USB_GetMsParam)
    C$debug_frame229                         0x00001348   Data           0  usb_custom.obj(.debug_frame)
    C$debug_frame230                         0x00001384   Data           0  usb_custom.obj(.debug_frame)
    C$debug_frame231                         0x000013c0   Data           0  usb_custom.obj(.debug_frame)
    C$debug_frame232                         0x000013fc   Data           0  usb_custom.obj(.debug_frame)
    C$debug_frame233                         0x00001438   Data           0  usb_custom.obj(.debug_frame)
    C$debug_frame234                         0x00001474   Data           0  usb_custom.obj(.debug_frame)
    .constdata$1                             0x00004244   Data           0  usb_custom.obj(.constdata)
    usb_device_param                         0x00004244   Data          20  usb_custom.obj(.constdata)
    usb_ms_param                             0x00004258   Data          20  usb_custom.obj(.constdata)
    usb_acm_param                            0x0000426c   Data          36  usb_custom.obj(.constdata)
    usb_video_param                          0x00004290   Data          44  usb_custom.obj(.constdata)
    USB_CustomFunc                           0x000042bc   Data          16  usb_custom.obj(.constdata)
    .constdata$41                            0x000042cc   Data           0  usb_custom.obj(.constdata)
    USB_MANUFACTURER_STRING                  0x000042cc   Data          26  usb_custom.obj(.constdata)
    .constdata$46                            0x000042e6   Data           0  usb_custom.obj(.constdata)
    USB_PRODUCT_STRING                       0x000042e6   Data          16  usb_custom.obj(.constdata)
    .constdata$51                            0x000042f8   Data           0  usb_custom.obj(.constdata)
    .constdata$56                            0x0000431c   Data           0  usb_custom.obj(.constdata)
    USB_MS_INTERFACE_STRING                  0x0000431c   Data          28  usb_custom.obj(.constdata)
    .constdata$61                            0x00004338   Data           0  usb_custom.obj(.constdata)
    USB_ACM_COMM_INTERFACE_STRING            0x00004338   Data          38  usb_custom.obj(.constdata)
    .constdata$66                            0x0000435e   Data           0  usb_custom.obj(.constdata)
    USB_ACM_DATA_INTERFACE_STRING            0x0000435e   Data          38  usb_custom.obj(.constdata)
    .constdata$71                            0x00004384   Data           0  usb_custom.obj(.constdata)
    USB_VIDEO_VC_INTERFACE_STRING            0x00004384   Data          38  usb_custom.obj(.constdata)
    .constdata$76                            0x000043aa   Data           0  usb_custom.obj(.constdata)
    USB_VIDEO_CT_INTERFACE_STRING            0x000043aa   Data          38  usb_custom.obj(.constdata)
    .constdata$81                            0x000043d0   Data           0  usb_custom.obj(.constdata)
    USB_VIDEO_OUTPUT_INTERFACE_STRING        0x000043d0   Data          46  usb_custom.obj(.constdata)
    .constdata$86                            0x000043fe   Data           0  usb_custom.obj(.constdata)
    USB_VIDEO_PU_INTERFACE_STRING            0x000043fe   Data          38  usb_custom.obj(.constdata)
    .constdata$91                            0x00004424   Data           0  usb_custom.obj(.constdata)
    USB_VIDEO_VS_INTERFACE_STRING            0x00004424   Data          38  usb_custom.obj(.constdata)
    bootloader\src\usbdl_b2spi.c             0x00000000   Number         0  usbdl_b2spi.obj ABSOLUTE
    bootloader\src\usbdl_debug_tool.c        0x00000000   Number         0  usbdl_debug_tool.obj ABSOLUTE
    i.drv_get_current_time                   0x000036ec   Thumb Code     0  usbdl_debug_tool.obj(i.drv_get_current_time)
    i.USB_Dbg_Trace                          0x00002384   Thumb Code     0  usbdl_debug_tool.obj(i.USB_Dbg_Trace)
    C$debug_frame210                         0x000014c0   Data           0  usbdl_debug_tool.obj(.debug_frame)
    C$debug_frame211                         0x000014fc   Data           0  usbdl_debug_tool.obj(.debug_frame)
    bootloader\src\usbdl_pmic6318.c          0x00000000   Number         0  usbdl_pmic6318.obj ABSOLUTE
    bootloader\src\usbdl_pmic6326.c          0x00000000   Number         0  usbdl_pmic6326.obj ABSOLUTE
    bootloader\src\usbdl_pmu.c               0x00000000   Number         0  usbdl_pmu.obj ABSOLUTE
    i.pmu6253_vusb_enable                    0x00003890   Thumb Code     0  usbdl_pmu.obj(i.pmu6253_vusb_enable)
    i.USBDL_Cable_IN                         0x00001aa0   Thumb Code     0  usbdl_pmu.obj(i.USBDL_Cable_IN)
    C$debug_frame219                         0x00001538   Data           0  usbdl_pmu.obj(.debug_frame)
    C$debug_frame220                         0x00001574   Data           0  usbdl_pmu.obj(.debug_frame)
    bootloader\src\usbdl_usb.c               0x00000000   Number         0  usbdl_usb.obj ABSOLUTE
    i.USB_Init                               0x00002a68   Thumb Code     0  usbdl_usb.obj(i.USB_Init)
    i.USB_Initialize                         0x00002bd4   Thumb Code     0  usbdl_usb.obj(i.USB_Initialize)
    i.USB_Endpoint0_Hdlr                     0x00002558   Thumb Code     0  usbdl_usb.obj(i.USB_Endpoint0_Hdlr)
    i.USB_Generate_EP0Data                   0x000026d4   Thumb Code     0  usbdl_usb.obj(i.USB_Generate_EP0Data)
    i.USB_Endpoint0_Idle                     0x0000261c   Thumb Code     0  usbdl_usb.obj(i.USB_Endpoint0_Idle)
    .bss                                     0x08000058   Data           0  usbdl_usb.obj(.bss)
    i.USB_Reset                              0x00002e3c   Thumb Code     0  usbdl_usb.obj(i.USB_Reset)
    i.USB_Cmd_GetDescriptor                  0x000021e0   Thumb Code     0  usbdl_usb.obj(i.USB_Cmd_GetDescriptor)
    i.USB_Init_Device_Status                 0x00002ad8   Thumb Code     0  usbdl_usb.obj(i.USB_Init_Device_Status)
    i.USB_Stdcmd                             0x00003340   Thumb Code     0  usbdl_usb.obj(i.USB_Stdcmd)
    i.USB_Cmd_SetFeature                     0x000022bc   Thumb Code     0  usbdl_usb.obj(i.USB_Cmd_SetFeature)
    i.USB_Cmd_GetStatus                      0x00002260   Thumb Code     0  usbdl_usb.obj(i.USB_Cmd_GetStatus)
    i.USB_Register_EP0_RxHdlr                0x00002e1c   Thumb Code     0  usbdl_usb.obj(i.USB_Register_EP0_RxHdlr)
    i.USB_Endpoint0_Tx                       0x00002684   Thumb Code     0  usbdl_usb.obj(i.USB_Endpoint0_Tx)
    .constdata                               0x0000444c   Data           0  usbdl_usb.obj(.constdata)
    C$debug_frame225                         0x000015b0   Data           0  usbdl_usb.obj(.debug_frame)
    C$debug_frame226                         0x00001600   Data           0  usbdl_usb.obj(.debug_frame)
    C$debug_frame227                         0x0000163c   Data           0  usbdl_usb.obj(.debug_frame)
    C$debug_frame228                         0x00001678   Data           0  usbdl_usb.obj(.debug_frame)
    C$debug_frame229                         0x000016c8   Data           0  usbdl_usb.obj(.debug_frame)
    C$debug_frame230                         0x0000171c   Data           0  usbdl_usb.obj(.debug_frame)
    C$debug_frame231                         0x00001774   Data           0  usbdl_usb.obj(.debug_frame)
    C$debug_frame232                         0x000017c4   Data           0  usbdl_usb.obj(.debug_frame)
    C$debug_frame233                         0x00001818   Data           0  usbdl_usb.obj(.debug_frame)
    C$debug_frame234                         0x00001878   Data           0  usbdl_usb.obj(.debug_frame)
    C$debug_frame235                         0x000018cc   Data           0  usbdl_usb.obj(.debug_frame)
    C$debug_frame236                         0x00001920   Data           0  usbdl_usb.obj(.debug_frame)
    C$debug_frame237                         0x0000196c   Data           0  usbdl_usb.obj(.debug_frame)
    USB_Cmd_GetDescriptor                    0x000021e0   Thumb Code   122  usbdl_usb.obj(i.USB_Cmd_GetDescriptor)
    USB_Cmd_GetStatus                        0x00002260   Thumb Code    82  usbdl_usb.obj(i.USB_Cmd_GetStatus)
    USB_Cmd_SetFeature                       0x000022bc   Thumb Code    96  usbdl_usb.obj(i.USB_Cmd_SetFeature)
    USB_Endpoint0_Hdlr                       0x00002558   Thumb Code   184  usbdl_usb.obj(i.USB_Endpoint0_Hdlr)
    USB_Endpoint0_Idle                       0x0000261c   Thumb Code    98  usbdl_usb.obj(i.USB_Endpoint0_Idle)
    USB_Endpoint0_Tx                         0x00002684   Thumb Code    74  usbdl_usb.obj(i.USB_Endpoint0_Tx)
    USB_Initialize                           0x00002bd4   Thumb Code   230  usbdl_usb.obj(i.USB_Initialize)
    USB_Reset                                0x00002e3c   Thumb Code   120  usbdl_usb.obj(i.USB_Reset)
    USB_Stdcmd                               0x00003340   Thumb Code   448  usbdl_usb.obj(i.USB_Stdcmd)
    .constdata$1                             0x0000444c   Data           0  usbdl_usb.obj(.constdata)
    .bss$2                                   0x08000058   Data           0  usbdl_usb.obj(.bss)
    status@USB_Cmd_GetStatus_0               0x08000058   Data           2  usbdl_usb.obj(.bss)
    bootloader\src\usbdl_usb_drv.c           0x00000000   Number         0  usbdl_usb_drv.obj ABSOLUTE
    i.USB_Get_EP0_Status                     0x000027b4   Thumb Code     0  usbdl_usb_drv.obj(i.USB_Get_EP0_Status)
    .bss                                     0x080001b0   Data           0  usbdl_usb_drv.obj(.bss)
    i.USB_Register_Drv_Info                  0x00002dd0   Thumb Code     0  usbdl_usb_drv.obj(i.USB_Register_Drv_Info)
    i.USB_Init_Drv_Info                      0x00002b90   Thumb Code     0  usbdl_usb_drv.obj(i.USB_Init_Drv_Info)
    i.USB_TxEPEn                             0x00003508   Thumb Code     0  usbdl_usb_drv.obj(i.USB_TxEPEn)
    i.USB_Reset_FIFO                         0x00002f10   Thumb Code     0  usbdl_usb_drv.obj(i.USB_Reset_FIFO)
    i.USB_CtrlEPStall                        0x00002320   Thumb Code     0  usbdl_usb_drv.obj(i.USB_CtrlEPStall)
    i.USB_EP_Check                           0x000024e4   Thumb Code     0  usbdl_usb_drv.obj(i.USB_EP_Check)
    i.USB_EP_Bulk_Rx_Ready                   0x00002480   Thumb Code     0  usbdl_usb_drv.obj(i.USB_EP_Bulk_Rx_Ready)
    i.USB_RxEPInit                           0x00002f6c   Thumb Code     0  usbdl_usb_drv.obj(i.USB_RxEPInit)
    i.USB_EPFIFOWrite                        0x0000242c   Thumb Code     0  usbdl_usb_drv.obj(i.USB_EPFIFOWrite)
    i.USB_EPFIFORead                         0x000023cc   Thumb Code     0  usbdl_usb_drv.obj(i.USB_EPFIFORead)
    i.USB_RxEPEn                             0x00002f1c   Thumb Code     0  usbdl_usb_drv.obj(i.USB_RxEPEn)
    i.USB_HISR                               0x000028f4   Thumb Code     0  usbdl_usb_drv.obj(i.USB_HISR)
    i.USB_Get_EP_Stall_Status                0x000027dc   Thumb Code     0  usbdl_usb_drv.obj(i.USB_Get_EP_Stall_Status)
    i.USB_EP_Bulk_Tx_Ready                   0x000024a0   Thumb Code     0  usbdl_usb_drv.obj(i.USB_EP_Bulk_Tx_Ready)
    i.USB_UART_Share                         0x000035f8   Thumb Code     0  usbdl_usb_drv.obj(i.USB_UART_Share)
    .data                                    0x08000034   Data           0  usbdl_usb_drv.obj(.data)
    i.USB_TxEPInit                           0x0000355c   Thumb Code     0  usbdl_usb_drv.obj(i.USB_TxEPInit)
    i.USBDL_USBPowerON                       0x00001d48   Thumb Code     0  usbdl_usb_drv.obj(i.USBDL_USBPowerON)
    i.USB_High_Speed_Enable                  0x00002a4c   Thumb Code     0  usbdl_usb_drv.obj(i.USB_High_Speed_Enable)
    i.USB_Set_DP_Pull_High                   0x00003020   Thumb Code     0  usbdl_usb_drv.obj(i.USB_Set_DP_Pull_High)
    i.USB_EP_Rx_Pkt_Len                      0x00002520   Thumb Code     0  usbdl_usb_drv.obj(i.USB_EP_Rx_Pkt_Len)
    i.USB_Update_EP0_State                   0x00003614   Thumb Code     0  usbdl_usb_drv.obj(i.USB_Update_EP0_State)
    i.USB_Reset_Drv                          0x00002ee8   Thumb Code     0  usbdl_usb_drv.obj(i.USB_Reset_Drv)
    i.USB_EnSysIntr                          0x00002544   Thumb Code     0  usbdl_usb_drv.obj(i.USB_EnSysIntr)
    i.USB_PDNDisable                         0x00002cf8   Thumb Code     0  usbdl_usb_drv.obj(i.USB_PDNDisable)
    i.USB_EPFIFORead_Shift                   0x000023d8   Thumb Code     0  usbdl_usb_drv.obj(i.USB_EPFIFORead_Shift)
    i.USB_EP0En                              0x000023a0   Thumb Code     0  usbdl_usb_drv.obj(i.USB_EP0En)
    i.USB_EP0_Pkt_Len                        0x000023b0   Thumb Code     0  usbdl_usb_drv.obj(i.USB_EP0_Pkt_Len)
    i.USB_ResetDrv_Info                      0x00002eb8   Thumb Code     0  usbdl_usb_drv.obj(i.USB_ResetDrv_Info)
    i.USB_SetAddress                         0x00003014   Thumb Code     0  usbdl_usb_drv.obj(i.USB_SetAddress)
    i.USB_Initialize_Drv                     0x00002cc0   Thumb Code     0  usbdl_usb_drv.obj(i.USB_Initialize_Drv)
    .constdata                               0x0000446c   Data           0  usbdl_usb_drv.obj(.constdata)
    i.USB_Is_High_Speed                      0x00002ce4   Thumb Code     0  usbdl_usb_drv.obj(i.USB_Is_High_Speed)
    C$debug_frame219                         0x000019c0   Data           0  usbdl_usb_drv.obj(.debug_frame)
    C$debug_frame220                         0x00001a0c   Data           0  usbdl_usb_drv.obj(.debug_frame)
    C$debug_frame221                         0x00001a48   Data           0  usbdl_usb_drv.obj(.debug_frame)
    C$debug_frame222                         0x00001ab0   Data           0  usbdl_usb_drv.obj(.debug_frame)
    C$debug_frame224                         0x00001b08   Data           0  usbdl_usb_drv.obj(.debug_frame)
    C$debug_frame225                         0x00001b58   Data           0  usbdl_usb_drv.obj(.debug_frame)
    C$debug_frame226                         0x00001b94   Data           0  usbdl_usb_drv.obj(.debug_frame)
    C$debug_frame227                         0x00001be8   Data           0  usbdl_usb_drv.obj(.debug_frame)
    C$debug_frame228                         0x00001c24   Data           0  usbdl_usb_drv.obj(.debug_frame)
    C$debug_frame229                         0x00001c60   Data           0  usbdl_usb_drv.obj(.debug_frame)
    C$debug_frame230                         0x00001ca8   Data           0  usbdl_usb_drv.obj(.debug_frame)
    C$debug_frame231                         0x00001ce4   Data           0  usbdl_usb_drv.obj(.debug_frame)
    C$debug_frame232                         0x00001d20   Data           0  usbdl_usb_drv.obj(.debug_frame)
    C$debug_frame233                         0x00001d68   Data           0  usbdl_usb_drv.obj(.debug_frame)
    C$debug_frame235                         0x00001da4   Data           0  usbdl_usb_drv.obj(.debug_frame)
    C$debug_frame236                         0x00001e00   Data           0  usbdl_usb_drv.obj(.debug_frame)
    C$debug_frame237                         0x00001e5c   Data           0  usbdl_usb_drv.obj(.debug_frame)
    C$debug_frame238                         0x00001eac   Data           0  usbdl_usb_drv.obj(.debug_frame)
    C$debug_frame239                         0x00001efc   Data           0  usbdl_usb_drv.obj(.debug_frame)
    C$debug_frame240                         0x00001f4c   Data           0  usbdl_usb_drv.obj(.debug_frame)
    C$debug_frame241                         0x00001f98   Data           0  usbdl_usb_drv.obj(.debug_frame)
    C$debug_frame242                         0x00001fe8   Data           0  usbdl_usb_drv.obj(.debug_frame)
    C$debug_frame243                         0x00002040   Data           0  usbdl_usb_drv.obj(.debug_frame)
    C$debug_frame244                         0x00002094   Data           0  usbdl_usb_drv.obj(.debug_frame)
    C$debug_frame245                         0x000020e0   Data           0  usbdl_usb_drv.obj(.debug_frame)
    C$debug_frame246                         0x0000211c   Data           0  usbdl_usb_drv.obj(.debug_frame)
    C$debug_frame247                         0x0000216c   Data           0  usbdl_usb_drv.obj(.debug_frame)
    C$debug_frame248                         0x000021bc   Data           0  usbdl_usb_drv.obj(.debug_frame)
    C$debug_frame252                         0x00002208   Data           0  usbdl_usb_drv.obj(.debug_frame)
    C$debug_frame256                         0x00002244   Data           0  usbdl_usb_drv.obj(.debug_frame)
    C$debug_frame257                         0x00002280   Data           0  usbdl_usb_drv.obj(.debug_frame)
    C$debug_frame258                         0x000022dc   Data           0  usbdl_usb_drv.obj(.debug_frame)
    USB_EP_Check                             0x000024e4   Thumb Code    54  usbdl_usb_drv.obj(i.USB_EP_Check)
    .constdata$1                             0x0000446c   Data           0  usbdl_usb_drv.obj(.constdata)
    .data$0                                  0x08000034   Data           0  usbdl_usb_drv.obj(.data)
    g_FIFOadd                                0x08000034   Data           4  usbdl_usb_drv.obj(.data)
    .bss$2                                   0x080001b0   Data           0  usbdl_usb_drv.obj(.bss)
    g_usb_pdn_owner                          0x080001b0   Data           4  usbdl_usb_drv.obj(.bss)
    bootloader\src\usbdl_usb_resource.c      0x00000000   Number         0  usbdl_usb_resource.obj ABSOLUTE
    i.USB_Get_Bulk_Rx_Ep                     0x00002714   Thumb Code     0  usbdl_usb_resource.obj(i.USB_Get_Bulk_Rx_Ep)
    i.USB_Register_CreateFunc                0x00002d34   Thumb Code     0  usbdl_usb_resource.obj(i.USB_Register_CreateFunc)
    i.USB_Software_Init                      0x000031d4   Thumb Code     0  usbdl_usb_resource.obj(i.USB_Software_Init)
    i.USB_Get_Interface_Number               0x00002804   Thumb Code     0  usbdl_usb_resource.obj(i.USB_Get_Interface_Number)
    i.USB_Get_Bulk_Tx_Ep                     0x00002764   Thumb Code     0  usbdl_usb_resource.obj(i.USB_Get_Bulk_Tx_Ep)
    i.USB_DeRegister_CreateFunc              0x00002388   Thumb Code     0  usbdl_usb_resource.obj(i.USB_DeRegister_CreateFunc)
    i.USB_Register_Device_Code               0x00002d88   Thumb Code     0  usbdl_usb_resource.obj(i.USB_Register_Device_Code)
    i.USB_Software_Create                    0x0000303c   Thumb Code     0  usbdl_usb_resource.obj(i.USB_Software_Create)
    i.USB_DeRegister_Device_Code             0x00002394   Thumb Code     0  usbdl_usb_resource.obj(i.USB_DeRegister_Device_Code)
    i.USB_Get_Intr_Ep                        0x00002858   Thumb Code     0  usbdl_usb_resource.obj(i.USB_Get_Intr_Ep)
    i.USB_Get_String_Number                  0x000028a0   Thumb Code     0  usbdl_usb_resource.obj(i.USB_Get_String_Number)
    i.USB_Software_Speed_Init                0x0000324c   Thumb Code     0  usbdl_usb_resource.obj(i.USB_Software_Speed_Init)
    .constdata                               0x00004490   Data           0  usbdl_usb_resource.obj(.constdata)
    .bss                                     0x08000218   Data           0  usbdl_usb_resource.obj(.bss)
    C$debug_frame216                         0x00002328   Data           0  usbdl_usb_resource.obj(.debug_frame)
    C$debug_frame217                         0x00002384   Data           0  usbdl_usb_resource.obj(.debug_frame)
    C$debug_frame218                         0x000023e0   Data           0  usbdl_usb_resource.obj(.debug_frame)
    C$debug_frame219                         0x0000241c   Data           0  usbdl_usb_resource.obj(.debug_frame)
    C$debug_frame220                         0x00002458   Data           0  usbdl_usb_resource.obj(.debug_frame)
    C$debug_frame221                         0x000024ac   Data           0  usbdl_usb_resource.obj(.debug_frame)
    C$debug_frame222                         0x00002500   Data           0  usbdl_usb_resource.obj(.debug_frame)
    C$debug_frame223                         0x00002554   Data           0  usbdl_usb_resource.obj(.debug_frame)
    C$debug_frame224                         0x000025a8   Data           0  usbdl_usb_resource.obj(.debug_frame)
    C$debug_frame225                         0x000025fc   Data           0  usbdl_usb_resource.obj(.debug_frame)
    C$debug_frame226                         0x00002658   Data           0  usbdl_usb_resource.obj(.debug_frame)
    C$debug_frame227                         0x000026b4   Data           0  usbdl_usb_resource.obj(.debug_frame)
    .constdata$1                             0x00004490   Data           0  usbdl_usb_resource.obj(.constdata)
    USB_Language_String                      0x00004490   Data           4  usbdl_usb_resource.obj(.constdata)
    .bss$2                                   0x08000218   Data           0  usbdl_usb_resource.obj(.bss)
    usb_ifcreate_number                      0x08000218   Data           1  usbdl_usb_resource.obj(.bss)
    usb_device_code                          0x0800021a   Data           8  usbdl_usb_resource.obj(.bss)
    usb_ifcreate_tbl                         0x08000224   Data          32  usbdl_usb_resource.obj(.bss)
    usb_conf_desc                            0x08000244   Data          67  usbdl_usb_resource.obj(.bss)
    bootloader\src\usbdl_usbacm_adap.c       0x00000000   Number         0  usbdl_usbacm_adap.obj ABSOLUTE
    i.USBDL_GetUARTByte_Ext                  0x00001b10   Thumb Code     0  usbdl_usbacm_adap.obj(i.USBDL_GetUARTByte_Ext)
    i.USBDL_CheckUARTSendEnd                 0x00001b00   Thumb Code     0  usbdl_usbacm_adap.obj(i.USBDL_CheckUARTSendEnd)
    i.USBDL_GetUARTByte                      0x00001b04   Thumb Code     0  usbdl_usbacm_adap.obj(i.USBDL_GetUARTByte)
    i.USBDL_Is_USB_Download_Mode             0x00001b60   Thumb Code     0  usbdl_usbacm_adap.obj(i.USBDL_Is_USB_Download_Mode)
    i.USBDL_Release                          0x00001c74   Thumb Code     0  usbdl_usbacm_adap.obj(i.USBDL_Release)
    i.USBDL_CheckStartCmd                    0x00001aa4   Thumb Code     0  usbdl_usbacm_adap.obj(i.USBDL_CheckStartCmd)
    .data                                    0x08000038   Data           0  usbdl_usbacm_adap.obj(.data)
    .bss                                     0x08000288   Data           0  usbdl_usbacm_adap.obj(.bss)
    i.USBDL_ACMInit                          0x00001a24   Thumb Code     0  usbdl_usbacm_adap.obj(i.USBDL_ACMInit)
    i.USBDL_PutUARTByte_Complete             0x00001b78   Thumb Code     0  usbdl_usbacm_adap.obj(i.USBDL_PutUARTByte_Complete)
    i.USBDL_UART_Init                        0x00001c9c   Thumb Code     0  usbdl_usbacm_adap.obj(i.USBDL_UART_Init)
    i.USBDL_Update_USB_Download_Mode         0x00001e4c   Thumb Code     0  usbdl_usbacm_adap.obj(i.USBDL_Update_USB_Download_Mode)
    i.USBDL_PutUARTByte_Ext                  0x00001bf0   Thumb Code     0  usbdl_usbacm_adap.obj(i.USBDL_PutUARTByte_Ext)
    i.USBDL_PutUARTByte_Complete_Ext         0x00001b84   Thumb Code     0  usbdl_usbacm_adap.obj(i.USBDL_PutUARTByte_Complete_Ext)
    i.USBDL_hwInit                           0x00001e7c   Thumb Code     0  usbdl_usbacm_adap.obj(i.USBDL_hwInit)
    i.USBDL_PutUARTByte                      0x00001b6c   Thumb Code     0  usbdl_usbacm_adap.obj(i.USBDL_PutUARTByte)
    i.USBDLKey_Pressed                       0x00001964   Thumb Code     0  usbdl_usbacm_adap.obj(i.USBDLKey_Pressed)
    .constdata                               0x0000457c   Data           0  usbdl_usbacm_adap.obj(.constdata)
    C$debug_frame240                         0x00002710   Data           0  usbdl_usbacm_adap.obj(.debug_frame)
    C$debug_frame241                         0x0000276c   Data           0  usbdl_usbacm_adap.obj(.debug_frame)
    C$debug_frame242                         0x000027bc   Data           0  usbdl_usbacm_adap.obj(.debug_frame)
    C$debug_frame243                         0x000027f8   Data           0  usbdl_usbacm_adap.obj(.debug_frame)
    C$debug_frame244                         0x00002844   Data           0  usbdl_usbacm_adap.obj(.debug_frame)
    C$debug_frame245                         0x00002894   Data           0  usbdl_usbacm_adap.obj(.debug_frame)
    C$debug_frame246                         0x000028e8   Data           0  usbdl_usbacm_adap.obj(.debug_frame)
    C$debug_frame248                         0x00002934   Data           0  usbdl_usbacm_adap.obj(.debug_frame)
    C$debug_frame249                         0x00002988   Data           0  usbdl_usbacm_adap.obj(.debug_frame)
    C$debug_frame250                         0x000029d4   Data           0  usbdl_usbacm_adap.obj(.debug_frame)
    C$debug_frame251                         0x00002a28   Data           0  usbdl_usbacm_adap.obj(.debug_frame)
    C$debug_frame252                         0x00002a74   Data           0  usbdl_usbacm_adap.obj(.debug_frame)
    C$debug_frame253                         0x00002acc   Data           0  usbdl_usbacm_adap.obj(.debug_frame)
    C$debug_frame254                         0x00002b18   Data           0  usbdl_usbacm_adap.obj(.debug_frame)
    C$debug_frame255                         0x00002b6c   Data           0  usbdl_usbacm_adap.obj(.debug_frame)
    .constdata$1                             0x0000457c   Data           0  usbdl_usbacm_adap.obj(.constdata)
    startcmd_len                             0x0000457c   Data           1  usbdl_usbacm_adap.obj(.constdata)
    startcmd                                 0x0000457d   Data           4  usbdl_usbacm_adap.obj(.constdata)
    .data$0                                  0x08000038   Data           0  usbdl_usbacm_adap.obj(.data)
    first@USBDLKey_Pressed_0                 0x08000038   Data           1  usbdl_usbacm_adap.obj(.data)
    .bss$2                                   0x08000288   Data           0  usbdl_usbacm_adap.obj(.bss)
    USBDL_Mode                               0x08000288   Data           1  usbdl_usbacm_adap.obj(.bss)
    index@USBDL_GetUARTByte_Ext_0            0x0800028c   Data           4  usbdl_usbacm_adap.obj(.bss)
    bootloader\src\usbdl_usbacm_drv.c        0x00000000   Number         0  usbdl_usbacm_drv.obj ABSOLUTE
    i.USB_Acm_DataIf_Reset                   0x000020dc   Thumb Code     0  usbdl_usbacm_drv.obj(i.USB_Acm_DataIf_Reset)
    i.USB_Acm_DataIf_Create                  0x00002004   Thumb Code     0  usbdl_usbacm_drv.obj(i.USB_Acm_DataIf_Create)
    i.USB_Acm_CommIf_Create                  0x00001f0c   Thumb Code     0  usbdl_usbacm_drv.obj(i.USB_Acm_CommIf_Create)
    i.USB_Acm_BulkIn_Reset                   0x00001ea4   Thumb Code     0  usbdl_usbacm_drv.obj(i.USB_Acm_BulkIn_Reset)
    i.USB_Acm_DataIf_Speed_Reset             0x00002114   Thumb Code     0  usbdl_usbacm_drv.obj(i.USB_Acm_DataIf_Speed_Reset)
    i.USB_Acm_CommIf_Speed_Reset             0x00001ff0   Thumb Code     0  usbdl_usbacm_drv.obj(i.USB_Acm_CommIf_Speed_Reset)
    i.USB_Acm_Ep0_SetLineCoding              0x000021a4   Thumb Code     0  usbdl_usbacm_drv.obj(i.USB_Acm_Ep0_SetLineCoding)
    i.USB_Acm_BulkOut_Reset                  0x00001ef4   Thumb Code     0  usbdl_usbacm_drv.obj(i.USB_Acm_BulkOut_Reset)
    i.USB_Acm_CommIf_Reset                   0x00001fe0   Thumb Code     0  usbdl_usbacm_drv.obj(i.USB_Acm_CommIf_Reset)
    i.USB_Release_Acm_Status                 0x00002e28   Thumb Code     0  usbdl_usbacm_drv.obj(i.USB_Release_Acm_Status)
    i.USB_Acm_BulkOut_Hdr                    0x00001ebc   Thumb Code     0  usbdl_usbacm_drv.obj(i.USB_Acm_BulkOut_Hdr)
    .bss                                     0x080006a0   Data           0  usbdl_usbacm_drv.obj(.bss)
    i.USB_Init_Acm_Status                    0x00002ac4   Thumb Code     0  usbdl_usbacm_drv.obj(i.USB_Init_Acm_Status)
    i.USB2UART_LineCoding2DCB                0x00001950   Thumb Code     0  usbdl_usbacm_drv.obj(i.USB2UART_LineCoding2DCB)
    i.USB_Acm_BulkIn_Hdr                     0x00001e98   Thumb Code     0  usbdl_usbacm_drv.obj(i.USB_Acm_BulkIn_Hdr)
    i.USB_Acm_Ep0_Command                    0x00002148   Thumb Code     0  usbdl_usbacm_drv.obj(i.USB_Acm_Ep0_Command)
    USB_Acm_BulkIn_Hdr                       0x00001e98   Thumb Code     8  usbdl_usbacm_drv.obj(i.USB_Acm_BulkIn_Hdr)
    USB_Acm_BulkIn_Reset                     0x00001ea4   Thumb Code    16  usbdl_usbacm_drv.obj(i.USB_Acm_BulkIn_Reset)
    USB_Acm_BulkOut_Hdr                      0x00001ebc   Thumb Code    48  usbdl_usbacm_drv.obj(i.USB_Acm_BulkOut_Hdr)
    USB_Acm_BulkOut_Reset                    0x00001ef4   Thumb Code    16  usbdl_usbacm_drv.obj(i.USB_Acm_BulkOut_Reset)
    USB_Acm_Ep0_Command                      0x00002148   Thumb Code    80  usbdl_usbacm_drv.obj(i.USB_Acm_Ep0_Command)
    USB_Acm_Ep0_SetLineCoding                0x000021a4   Thumb Code    52  usbdl_usbacm_drv.obj(i.USB_Acm_Ep0_SetLineCoding)
    C$debug_frame225                         0x00002ba8   Data           0  usbdl_usbacm_drv.obj(.debug_frame)
    C$debug_frame227                         0x00002be4   Data           0  usbdl_usbacm_drv.obj(.debug_frame)
    C$debug_frame228                         0x00002c38   Data           0  usbdl_usbacm_drv.obj(.debug_frame)
    C$debug_frame229                         0x00002c74   Data           0  usbdl_usbacm_drv.obj(.debug_frame)
    C$debug_frame230                         0x00002cb0   Data           0  usbdl_usbacm_drv.obj(.debug_frame)
    C$debug_frame231                         0x00002d04   Data           0  usbdl_usbacm_drv.obj(.debug_frame)
    C$debug_frame232                         0x00002d50   Data           0  usbdl_usbacm_drv.obj(.debug_frame)
    C$debug_frame233                         0x00002da0   Data           0  usbdl_usbacm_drv.obj(.debug_frame)
    C$debug_frame234                         0x00002ddc   Data           0  usbdl_usbacm_drv.obj(.debug_frame)
    C$debug_frame235                         0x00002e18   Data           0  usbdl_usbacm_drv.obj(.debug_frame)
    C$debug_frame236                         0x00002e68   Data           0  usbdl_usbacm_drv.obj(.debug_frame)
    C$debug_frame237                         0x00002ea4   Data           0  usbdl_usbacm_drv.obj(.debug_frame)
    C$debug_frame238                         0x00002ef4   Data           0  usbdl_usbacm_drv.obj(.debug_frame)
    C$debug_frame239                         0x00002f30   Data           0  usbdl_usbacm_drv.obj(.debug_frame)
    C$debug_frame240                         0x00002f6c   Data           0  usbdl_usbacm_drv.obj(.debug_frame)
    .bss$2                                   0x080006a0   Data           0  usbdl_usbacm_drv.obj(.bss)
    sss\components\src\SSS_secure_shared.c   0x00000000   Number         0  SSS_secure_shared.obj ABSOLUTE
    COMMON_CODE                              0x00000b4c   Thumb Code     0  SSS_secure_shared.obj(COMMON_CODE)
    COMMON_CODE                              0x00000b98   Thumb Code     0  SSS_secure_shared.obj(COMMON_CODE)
    .constdata                               0x000045c4   Data           0  SSS_secure_shared.obj(.constdata)
    COMMON_CODE                              0x00000bb8   Thumb Code     0  SSS_secure_shared.obj(COMMON_CODE)
    COMMON_CODE                              0x00000a7c   Thumb Code     0  SSS_secure_shared.obj(COMMON_CODE)
    C$debug_loc1380                          0x00000000   Data           0  SSS_secure_shared.obj(.debug_loc)
    C$debug_pubnames1198                     0x00000000   Data           0  SSS_secure_shared.obj(.debug_pubnames)
    C$debug_abbrev0                          0x00000018   Data           0  SSS_secure_shared.obj(.debug_abbrev)
    C$debug_pubnames1324                     0x00000028   Data           0  SSS_secure_shared.obj(.debug_pubnames)
    C$debug_pubnames1336                     0x00000054   Data           0  SSS_secure_shared.obj(.debug_pubnames)
    C$debug_loc1488                          0x00000060   Data           0  SSS_secure_shared.obj(.debug_loc)
    C$debug_pubnames1342                     0x0000008c   Data           0  SSS_secure_shared.obj(.debug_pubnames)
    C$debug_pubnames1378                     0x000000c0   Data           0  SSS_secure_shared.obj(.debug_pubnames)
    C$debug_info507                          0x000000c4   Data           0  SSS_secure_shared.obj(.debug_info)
    C$debug_pubnames1486                     0x000000e8   Data           0  SSS_secure_shared.obj(.debug_pubnames)
    C$debug_pubnames1498                     0x00000114   Data           0  SSS_secure_shared.obj(.debug_pubnames)
    C$debug_loc1500                          0x00000124   Data           0  SSS_secure_shared.obj(.debug_loc)
    C$debug_pubnames1504                     0x0000014c   Data           0  SSS_secure_shared.obj(.debug_pubnames)
    C$debug_line1376                         0x0000015c   Data           0  SSS_secure_shared.obj(.debug_line)
    C$debug_pubnames508                      0x00000180   Data           0  SSS_secure_shared.obj(.debug_pubnames)
    C$debug_loc1506                          0x000001d0   Data           0  SSS_secure_shared.obj(.debug_loc)
    C$debug_line1484                         0x000001e4   Data           0  SSS_secure_shared.obj(.debug_line)
    C$debug_line1496                         0x00000264   Data           0  SSS_secure_shared.obj(.debug_line)
    C$debug_pubnames1168                     0x00000268   Data           0  SSS_secure_shared.obj(.debug_pubnames)
    C$debug_info1197                         0x00000280   Data           0  SSS_secure_shared.obj(.debug_info)
    C$debug_line1502                         0x000002d0   Data           0  SSS_secure_shared.obj(.debug_line)
    C$debug_info3                            0x00000374   Data           0  SSS_secure_shared.obj(.debug_info)
    C$debug_info1323                         0x0000063c   Data           0  SSS_secure_shared.obj(.debug_info)
    C$debug_pubnames4                        0x0000063c   Data           0  SSS_secure_shared.obj(.debug_pubnames)
    C$debug_info1167                         0x00000738   Data           0  SSS_secure_shared.obj(.debug_info)
    C$debug_info1335                         0x000016d4   Data           0  SSS_secure_shared.obj(.debug_info)
    C$debug_info1341                         0x000017f0   Data           0  SSS_secure_shared.obj(.debug_info)
    C$debug_info1377                         0x000018e8   Data           0  SSS_secure_shared.obj(.debug_info)
    C$debug_info1485                         0x00001a3c   Data           0  SSS_secure_shared.obj(.debug_info)
    C$debug_info1497                         0x00001b88   Data           0  SSS_secure_shared.obj(.debug_info)
    C$debug_info1503                         0x00001c50   Data           0  SSS_secure_shared.obj(.debug_info)
    C$debug_frame1381                        0x00002fb8   Data           0  SSS_secure_shared.obj(.debug_frame)
    C$debug_frame1489                        0x0000300c   Data           0  SSS_secure_shared.obj(.debug_frame)
    C$debug_frame1501                        0x00003058   Data           0  SSS_secure_shared.obj(.debug_frame)
    C$debug_frame1507                        0x000030a8   Data           0  SSS_secure_shared.obj(.debug_frame)
    .constdata$1                             0x000045c4   Data           0  SSS_secure_shared.obj(.constdata)
    Setting1                                 0x000045dc   Data          16  SSS_secure_shared.obj(.constdata)
    Setting2                                 0x000045ec   Data          16  SSS_secure_shared.obj(.constdata)
    Setting3                                 0x000045fc   Data          24  SSS_secure_shared.obj(.constdata)
    Setting4                                 0x00004614   Data          24  SSS_secure_shared.obj(.constdata)
    Setting5                                 0x0000462c   Data          40  SSS_secure_shared.obj(.constdata)
    Setting6                                 0x00004654   Data          40  SSS_secure_shared.obj(.constdata)
    Setting7                                 0x0000467c   Data          32  SSS_secure_shared.obj(.constdata)
    Setting8                                 0x0000469c   Data          32  SSS_secure_shared.obj(.constdata)
    Setting9                                 0x000046bc   Data          32  SSS_secure_shared.obj(.constdata)
    sss\components\src\bl_FactoryConn.c      0x00000000   Number         0  bl_FactoryConn.obj ABSOLUTE
    i.getSWVersionCMD                        0x00003744   Thumb Code     0  bl_FactoryConn.obj(i.getSWVersionCMD)
    i.GetData                                0x000016e8   Thumb Code     0  bl_FactoryConn.obj(i.GetData)
    i.waitBlReadyCMD                         0x0000392c   Thumb Code     0  bl_FactoryConn.obj(i.waitBlReadyCMD)
    i.writeCMD                               0x00003980   Thumb Code     0  bl_FactoryConn.obj(i.writeCMD)
    i.readCMD_32                             0x000038e0   Thumb Code     0  bl_FactoryConn.obj(i.readCMD_32)
    i.Get16Data                              0x000016c0   Thumb Code     0  bl_FactoryConn.obj(i.Get16Data)
    i.readCMD                                0x000038a8   Thumb Code     0  bl_FactoryConn.obj(i.readCMD)
    i.jump_cmd2                              0x00003790   Thumb Code     0  bl_FactoryConn.obj(i.jump_cmd2)
    i.writeCMD_32                            0x000039bc   Thumb Code     0  bl_FactoryConn.obj(i.writeCMD_32)
    i.Connect_FactoryTool                    0x0000129c   Thumb Code     0  bl_FactoryConn.obj(i.Connect_FactoryTool)
    .constdata                               0x0000483c   Data           0  bl_FactoryConn.obj(.constdata)
    i.Put16Data                              0x00001908   Thumb Code     0  bl_FactoryConn.obj(i.Put16Data)
    i.PutData                                0x0000192c   Thumb Code     0  bl_FactoryConn.obj(i.PutData)
    i.getBlRegionCMD                         0x000036f8   Thumb Code     0  bl_FactoryConn.obj(i.getBlRegionCMD)
    i.writeCMD_noecho                        0x000039f8   Thumb Code     0  bl_FactoryConn.obj(i.writeCMD_noecho)
    i.checksumCMD                            0x00003690   Thumb Code     0  bl_FactoryConn.obj(i.checksumCMD)
    C$debug_abbrev0                          0x00000018   Data           0  SSS_secure_shared.obj(.debug_abbrev)
    C$debug_info9                            0x000000c4   Data           0  SSS_secure_shared.obj(.debug_info)
    C$debug_pubnames10                       0x00000180   Data           0  SSS_secure_shared.obj(.debug_pubnames)
    C$debug_loc1344                          0x00000260   Data           0  bl_FactoryConn.obj(.debug_loc)
    C$debug_pubnames1228                     0x00000268   Data           0  SSS_secure_shared.obj(.debug_pubnames)
    C$debug_loc1350                          0x000002ec   Data           0  bl_FactoryConn.obj(.debug_loc)
    C$debug_line1340                         0x00000338   Data           0  bl_FactoryConn.obj(.debug_line)
    C$debug_loc1356                          0x0000035c   Data           0  bl_FactoryConn.obj(.debug_loc)
    C$debug_line1346                         0x000003b0   Data           0  bl_FactoryConn.obj(.debug_line)
    C$debug_loc1362                          0x000003e8   Data           0  bl_FactoryConn.obj(.debug_loc)
    C$debug_line1352                         0x0000041c   Data           0  bl_FactoryConn.obj(.debug_line)
    C$debug_loc1368                          0x00000458   Data           0  bl_FactoryConn.obj(.debug_loc)
    C$debug_line1358                         0x00000494   Data           0  bl_FactoryConn.obj(.debug_line)
    C$debug_line1364                         0x000004fc   Data           0  bl_FactoryConn.obj(.debug_line)
    C$debug_loc1374                          0x00000500   Data           0  bl_FactoryConn.obj(.debug_loc)
    C$debug_line1370                         0x00000578   Data           0  bl_FactoryConn.obj(.debug_line)
    C$debug_loc1380                          0x00000580   Data           0  bl_FactoryConn.obj(.debug_loc)
    C$debug_line1376                         0x000005f0   Data           0  bl_FactoryConn.obj(.debug_line)
    C$debug_loc1386                          0x00000628   Data           0  bl_FactoryConn.obj(.debug_loc)
    C$debug_line1382                         0x0000066c   Data           0  bl_FactoryConn.obj(.debug_line)
    C$debug_loc1392                          0x000006d0   Data           0  bl_FactoryConn.obj(.debug_loc)
    C$debug_line1388                         0x000006e8   Data           0  bl_FactoryConn.obj(.debug_line)
    C$debug_info1227                         0x00000738   Data           0  SSS_secure_shared.obj(.debug_info)
    C$debug_loc1398                          0x00000750   Data           0  bl_FactoryConn.obj(.debug_loc)
    C$debug_line1394                         0x00000760   Data           0  bl_FactoryConn.obj(.debug_line)
    C$debug_pubnames1246                     0x0000076c   Data           0  bl_FactoryConn.obj(.debug_pubnames)
    C$debug_pubnames1252                     0x0000078c   Data           0  bl_FactoryConn.obj(.debug_pubnames)
    C$debug_pubnames1258                     0x000007ac   Data           0  bl_FactoryConn.obj(.debug_pubnames)
    C$debug_pubnames1264                     0x000007cc   Data           0  bl_FactoryConn.obj(.debug_pubnames)
    C$debug_line1400                         0x000007d8   Data           0  bl_FactoryConn.obj(.debug_line)
    C$debug_pubnames1270                     0x000007ec   Data           0  bl_FactoryConn.obj(.debug_pubnames)
    C$debug_loc1404                          0x000007f8   Data           0  bl_FactoryConn.obj(.debug_loc)
    C$debug_pubnames1276                     0x0000080c   Data           0  bl_FactoryConn.obj(.debug_pubnames)
    C$debug_pubnames1282                     0x0000082c   Data           0  bl_FactoryConn.obj(.debug_pubnames)
    C$debug_line1406                         0x00000850   Data           0  bl_FactoryConn.obj(.debug_line)
    C$debug_pubnames1288                     0x00000854   Data           0  bl_FactoryConn.obj(.debug_pubnames)
    C$debug_pubnames1294                     0x00000878   Data           0  bl_FactoryConn.obj(.debug_pubnames)
    C$debug_loc1410                          0x00000888   Data           0  bl_FactoryConn.obj(.debug_loc)
    C$debug_pubnames1300                     0x0000089c   Data           0  bl_FactoryConn.obj(.debug_pubnames)
    C$debug_line1412                         0x000008c0   Data           0  bl_FactoryConn.obj(.debug_line)
    C$debug_pubnames1306                     0x000008c0   Data           0  bl_FactoryConn.obj(.debug_pubnames)
    C$debug_pubnames1312                     0x000008e8   Data           0  bl_FactoryConn.obj(.debug_pubnames)
    C$debug_loc1416                          0x000008fc   Data           0  bl_FactoryConn.obj(.debug_loc)
    C$debug_pubnames1318                     0x00000910   Data           0  bl_FactoryConn.obj(.debug_pubnames)
    C$debug_pubnames1324                     0x00000930   Data           0  bl_FactoryConn.obj(.debug_pubnames)
    C$debug_pubnames1336                     0x00000958   Data           0  bl_FactoryConn.obj(.debug_pubnames)
    C$debug_line1418                         0x00000978   Data           0  bl_FactoryConn.obj(.debug_line)
    C$debug_pubnames1342                     0x00000984   Data           0  bl_FactoryConn.obj(.debug_pubnames)
    C$debug_pubnames1348                     0x000009a4   Data           0  bl_FactoryConn.obj(.debug_pubnames)
    C$debug_pubnames1354                     0x000009c4   Data           0  bl_FactoryConn.obj(.debug_pubnames)
    C$debug_line1430                         0x000009e0   Data           0  bl_FactoryConn.obj(.debug_line)
    C$debug_pubnames1360                     0x000009e4   Data           0  bl_FactoryConn.obj(.debug_pubnames)
    C$debug_pubnames1366                     0x00000a04   Data           0  bl_FactoryConn.obj(.debug_pubnames)
    C$debug_pubnames1372                     0x00000a24   Data           0  bl_FactoryConn.obj(.debug_pubnames)
    C$debug_pubnames1378                     0x00000a44   Data           0  bl_FactoryConn.obj(.debug_pubnames)
    C$debug_pubnames1384                     0x00000a6c   Data           0  bl_FactoryConn.obj(.debug_pubnames)
    C$debug_pubnames1390                     0x00000a90   Data           0  bl_FactoryConn.obj(.debug_pubnames)
    C$debug_pubnames1396                     0x00000ab4   Data           0  bl_FactoryConn.obj(.debug_pubnames)
    C$debug_loc1422                          0x00000ad0   Data           0  bl_FactoryConn.obj(.debug_loc)
    C$debug_pubnames1402                     0x00000ad8   Data           0  bl_FactoryConn.obj(.debug_pubnames)
    C$debug_pubnames1408                     0x00000b00   Data           0  bl_FactoryConn.obj(.debug_pubnames)
    C$debug_loc1434                          0x00000b04   Data           0  bl_FactoryConn.obj(.debug_loc)
    C$debug_pubnames1414                     0x00000b28   Data           0  bl_FactoryConn.obj(.debug_pubnames)
    C$debug_pubnames1420                     0x00000b48   Data           0  bl_FactoryConn.obj(.debug_pubnames)
    C$debug_pubnames1432                     0x00000b70   Data           0  bl_FactoryConn.obj(.debug_pubnames)
    C$debug_info1245                         0x00001d0c   Data           0  bl_FactoryConn.obj(.debug_info)
    C$debug_info1251                         0x00001df0   Data           0  bl_FactoryConn.obj(.debug_info)
    C$debug_info1257                         0x00001e94   Data           0  bl_FactoryConn.obj(.debug_info)
    C$debug_info1263                         0x00001f7c   Data           0  bl_FactoryConn.obj(.debug_info)
    C$debug_info1269                         0x00002020   Data           0  bl_FactoryConn.obj(.debug_info)
    C$debug_info1275                         0x0000212c   Data           0  bl_FactoryConn.obj(.debug_info)
    C$debug_info1281                         0x0000220c   Data           0  bl_FactoryConn.obj(.debug_info)
    C$debug_info1287                         0x00002318   Data           0  bl_FactoryConn.obj(.debug_info)
    C$debug_info1293                         0x00002420   Data           0  bl_FactoryConn.obj(.debug_info)
    C$debug_info1299                         0x00002504   Data           0  bl_FactoryConn.obj(.debug_info)
    C$debug_info1305                         0x000025f8   Data           0  bl_FactoryConn.obj(.debug_info)
    C$debug_info1311                         0x000026d4   Data           0  bl_FactoryConn.obj(.debug_info)
    C$debug_info1317                         0x000027f0   Data           0  bl_FactoryConn.obj(.debug_info)
    C$debug_info1323                         0x000029e0   Data           0  bl_FactoryConn.obj(.debug_info)
    C$debug_info1335                         0x00002aa4   Data           0  bl_FactoryConn.obj(.debug_info)
    C$debug_info1341                         0x00002c18   Data           0  bl_FactoryConn.obj(.debug_info)
    C$debug_info1347                         0x00002cf4   Data           0  bl_FactoryConn.obj(.debug_info)
    C$debug_info1353                         0x00002dac   Data           0  bl_FactoryConn.obj(.debug_info)
    C$debug_info1359                         0x00002e88   Data           0  bl_FactoryConn.obj(.debug_info)
    C$debug_info1365                         0x00002f40   Data           0  bl_FactoryConn.obj(.debug_info)
    C$debug_info1371                         0x00003034   Data           0  bl_FactoryConn.obj(.debug_info)
    C$debug_frame1345                        0x000030f4   Data           0  bl_FactoryConn.obj(.debug_frame)
    C$debug_info1377                         0x00003100   Data           0  bl_FactoryConn.obj(.debug_info)
    C$debug_frame1351                        0x00003144   Data           0  bl_FactoryConn.obj(.debug_frame)
    C$debug_frame1357                        0x00003194   Data           0  bl_FactoryConn.obj(.debug_frame)
    C$debug_frame1363                        0x000031e4   Data           0  bl_FactoryConn.obj(.debug_frame)
    C$debug_info1383                         0x000031e8   Data           0  bl_FactoryConn.obj(.debug_info)
    C$debug_frame1369                        0x00003234   Data           0  bl_FactoryConn.obj(.debug_frame)
    C$debug_frame1375                        0x00003288   Data           0  bl_FactoryConn.obj(.debug_frame)
    C$debug_info1389                         0x000032d0   Data           0  bl_FactoryConn.obj(.debug_info)
    C$debug_frame1381                        0x000032d8   Data           0  bl_FactoryConn.obj(.debug_frame)
    C$debug_frame1387                        0x00003328   Data           0  bl_FactoryConn.obj(.debug_frame)
    C$debug_frame1393                        0x0000337c   Data           0  bl_FactoryConn.obj(.debug_frame)
    C$debug_info1395                         0x0000339c   Data           0  bl_FactoryConn.obj(.debug_info)
    C$debug_frame1399                        0x000033cc   Data           0  bl_FactoryConn.obj(.debug_frame)
    C$debug_frame1405                        0x0000341c   Data           0  bl_FactoryConn.obj(.debug_frame)
    C$debug_frame1411                        0x00003474   Data           0  bl_FactoryConn.obj(.debug_frame)
    C$debug_info1401                         0x00003474   Data           0  bl_FactoryConn.obj(.debug_info)
    C$debug_frame1417                        0x000034c8   Data           0  bl_FactoryConn.obj(.debug_frame)
    C$debug_frame1423                        0x00003524   Data           0  bl_FactoryConn.obj(.debug_frame)
    C$debug_info1407                         0x00003538   Data           0  bl_FactoryConn.obj(.debug_info)
    C$debug_frame1435                        0x00003570   Data           0  bl_FactoryConn.obj(.debug_frame)
    C$debug_info1413                         0x00003618   Data           0  bl_FactoryConn.obj(.debug_info)
    C$debug_info1419                         0x000037c0   Data           0  bl_FactoryConn.obj(.debug_info)
    C$debug_info1431                         0x000038a0   Data           0  bl_FactoryConn.obj(.debug_info)
    .constdata$1                             0x0000483c   Data           0  bl_FactoryConn.obj(.constdata)
    sss\components\src\bl_Secure.c           0x00000000   Number         0  bl_Secure.obj ABSOLUTE
    .bss                                     0x08000738   Data           0  bl_Secure.obj(.bss)
    .bss                                     0x0800073c   Data           0  bl_Secure.obj(.bss)
    C$debug_abbrev0                          0x00000018   Data           0  SSS_secure_shared.obj(.debug_abbrev)
    C$debug_info9                            0x000000c4   Data           0  SSS_secure_shared.obj(.debug_info)
    C$debug_pubnames10                       0x00000180   Data           0  SSS_secure_shared.obj(.debug_pubnames)
    C$debug_pubnames16                       0x00000268   Data           0  SSS_secure_shared.obj(.debug_pubnames)
    C$debug_info15                           0x00000738   Data           0  SSS_secure_shared.obj(.debug_info)
    C$debug_pubnames4                        0x00000b9c   Data           0  bl_Secure.obj(.debug_pubnames)
    C$debug_info3                            0x00003a28   Data           0  bl_Secure.obj(.debug_info)
    .bss$20                                  0x08000738   Data           0  bl_Secure.obj(.bss)
    .bss$30                                  0x0800073c   Data           0  bl_Secure.obj(.bss)
    dp_engine\che\src\md5_engine.c           0x00000000   Number         0  md5_engine.obj ABSOLUTE
    dp_engine\che\src\sha1_engine.c          0x00000000   Number         0  sha1_engine.obj ABSOLUTE
    sss\components\src\SSS_secure.c          0x00000000   Number         0  SSS_secure.obj ABSOLUTE
    C$debug_abbrev0                          0x00000018   Data           0  SSS_secure_shared.obj(.debug_abbrev)
    C$debug_info507                          0x000000c4   Data           0  SSS_secure_shared.obj(.debug_info)
    C$debug_pubnames508                      0x00000180   Data           0  SSS_secure_shared.obj(.debug_pubnames)
    C$debug_pubnames1162                     0x00000268   Data           0  SSS_secure_shared.obj(.debug_pubnames)
    C$debug_info1161                         0x00000738   Data           0  SSS_secure_shared.obj(.debug_info)
    sss\components\src\sha1_hw.c             0x00000000   Number         0  sha1_hw.obj ABSOLUTE
    C$debug_abbrev0                          0x00000018   Data           0  SSS_secure_shared.obj(.debug_abbrev)
    C$debug_info513                          0x000000c4   Data           0  SSS_secure_shared.obj(.debug_info)
    C$debug_pubnames514                      0x00000180   Data           0  SSS_secure_shared.obj(.debug_pubnames)
    C$debug_pubnames1174                     0x00000268   Data           0  SSS_secure_shared.obj(.debug_pubnames)
    C$debug_info1173                         0x00000738   Data           0  SSS_secure_shared.obj(.debug_info)
    sss\components\src\sha1_sw.c             0x00000000   Number         0  sha1_sw.obj ABSOLUTE
    C$debug_abbrev0                          0x00000018   Data           0  SSS_secure_shared.obj(.debug_abbrev)
    C$debug_info507                          0x000000c4   Data           0  SSS_secure_shared.obj(.debug_info)
    C$debug_pubnames508                      0x00000180   Data           0  SSS_secure_shared.obj(.debug_pubnames)
    sss/components/src/sha1_hw_asm.s         0x00000000   Number         0  sha1_hw_asm.obj ABSOLUTE
    ../../armsys.c                           0x00000000   Number         0  lib_init.o ABSOLUTE
    .text                                    0x00000400   Thumb Code     0  lib_init.o(.text)
    C$debug_frame18                          0x000035c4   Data           0  lib_init.o(.debug_frame)
    ../../longlong.s                         0x00000000   Number         0  llcmpge.o ABSOLUTE
    <Anonymous Symbol>                       0x0000364c   Data          68  llcmpge.o(.debug_frame)
    .text                                    0x000004b8   Thumb Code    16  llcmpge.o(.text)
    ../../longlong.s                         0x00000000   Number         0  llmullu.o ABSOLUTE
    <Anonymous Symbol>                       0x00003690   Data          60  llmullu.o(.debug_frame)
    .text                                    0x000004c8   Thumb Code    12  llmullu.o(.text)
    ../../longlong.s                         0x00000000   Number         0  llneg.o ABSOLUTE
    .text                                    0x000004d4   Thumb Code    16  llneg.o(.text)
    <Anonymous Symbol>                       0x000036cc   Data          68  llneg.o(.debug_frame)
    ../../longlong.s                         0x00000000   Number         0  llshl.o ABSOLUTE
    ../../longlong.s                         0x00000000   Number         0  llsubls.o ABSOLUTE
    <Anonymous Symbol>                       0x00003710   Data          68  llsubls.o(.debug_frame)
    .text                                    0x000004e4   Thumb Code    16  llsubls.o(.text)
    ../../longlong.s                         0x00000000   Number         0  llushr.o ABSOLUTE
    ../../string.c                           0x00000000   Number         0  memcmp.o ABSOLUTE
    ../../memcpset.s                         0x00000000   Number         0  memcpy.o ABSOLUTE
    <Anonymous Symbol>                       0x00003754   Data          76  memcpy.o(.debug_frame)
    .text                                    0x000004f4   Thumb Code    20  memcpy.o(.text)
    ../../memcpset.s                         0x00000000   Number         0  memset.o ABSOLUTE
    <Anonymous Symbol>                       0x000037a0   Data          76  memset.o(.debug_frame)
    .text                                    0x00000508   Thumb Code    36  memset.o(.text)
    ../../memcpset.s                         0x00000000   Number         0  rt_memclr_w.o ABSOLUTE
    <Anonymous Symbol>                       0x000037ec   Data          84  rt_memclr_w.o(.debug_frame)
    .text                                    0x0000052c   Thumb Code    92  rt_memclr_w.o(.text)
    _loop                                    0x00000548   ARM Code       0  rt_memclr_w.o(.text)
    ../../memcpset.s                         0x00000000   Number         0  rt_memcpy.o ABSOLUTE
    .text                                    0x00000588   Thumb Code   184  rt_memcpy.o(.text)
    <Anonymous Symbol>                       0x00003840   Data          60  rt_memcpy.o(.debug_frame)
    _memcpy_dest_aligned                     0x000005c0   ARM Code       0  rt_memcpy.o(.text)
    _memcpy_src1_loop                        0x000005e0   ARM Code       0  rt_memcpy.o(.text)
    _memcpy_src2_loop                        0x00000600   ARM Code       0  rt_memcpy.o(.text)
    _memcpy_src3_loop                        0x00000620   ARM Code       0  rt_memcpy.o(.text)
    ../../memcpset.s                         0x00000000   Number         0  rt_memcpy_w.o ABSOLUTE
    .text                                    0x00000640   Thumb Code   112  rt_memcpy_w.o(.text)
    <Anonymous Symbol>                       0x0000387c   Data          84  rt_memcpy_w.o(.debug_frame)
    _memcpy_aligned_loop                     0x00000650   ARM Code       0  rt_memcpy_w.o(.text)
    _memcpy_small                            0x00000668   ARM Code       0  rt_memcpy_w.o(.text)
    ../../division.s                         0x00000000   Number         0  rt_sdiv.o ABSOLUTE
    <Anonymous Symbol>                       0x000038d0   Data          68  rt_sdiv.o(.debug_frame)
    .text                                    0x000006b0   Thumb Code   216  rt_sdiv.o(.text)
    ../../division.s                         0x00000000   Number         0  rt_udiv.o ABSOLUTE
    ../../division.s                         0x00000000   Number         0  rtsdiv10.o ABSOLUTE
    <Anonymous Symbol>                       0x00003914   Data          68  rtsdiv10.o(.debug_frame)
    .text                                    0x00000788   Thumb Code    68  rtsdiv10.o(.text)
    ../../string.c                           0x00000000   Number         0  strlen.o ABSOLUTE
    ../../string.c                           0x00000000   Number         0  strncmp.o ABSOLUTE
    ../../dfltll.s                           0x00000000   Number         0  dfltll_clz.o ABSOLUTE
    x$fpl$dfltll                             0x00003ae0   Thumb Code   132  dfltll_clz.o(x$fpl$dfltll)
    <Anonymous Symbol>                       0x00003958   Data          92  dfltll_clz.o(.debug_frame)
    dfltll_normalise                         0x00003b04   ARM Code       0  dfltll_clz.o(x$fpl$dfltll)
    ../../dgeqf.s                            0x00000000   Number         0  dgeqf.o ABSOLUTE
    x$fpl$dgeqf                              0x00003b64   Thumb Code   132  dgeqf.o(x$fpl$dgeqf)
    <Anonymous Symbol>                       0x000039b4   Data          96  dgeqf.o(.debug_frame)
    _dcmpge_check_NaNInf_pos                 0x00003b88   ARM Code       0  dgeqf.o(x$fpl$dgeqf)
    _dcmpge_negative                         0x00003ba0   ARM Code       0  dgeqf.o(x$fpl$dgeqf)
    _dcmpge_check_NaNInf_neg                 0x00003bc0   ARM Code       0  dgeqf.o(x$fpl$dgeqf)
    dcmpge_InfNaN                            0x00003bdc   ARM Code       0  dgeqf.o(x$fpl$dgeqf)
    ../../angel/sys.s                        0x00000000   Number         0  libspace.o ABSOLUTE
    <Anonymous Symbol>                       0x00003a14   Data          68  libspace.o(.debug_frame)
    .bss                                     0x08000740   Data          96  libspace.o(.bss)
    .text                                    0x000007cc   Thumb Code    16  libspace.o(.text)
    __libspace_start                         0x08000740   Data          96  libspace.o(.bss)
    ../../longlong.s                         0x00000000   Number         0  llmul3m.o ABSOLUTE
    <Anonymous Symbol>                       0x00003a58   Data          84  llmul3m.o(.debug_frame)
    .text                                    0x000007dc   Thumb Code    32  llmul3m.o(.text)
    ../../angel/rt.s                         0x00000000   Number         0  rt_div0.o ABSOLUTE
    <Anonymous Symbol>                       0x00003aac   Data          60  rt_div0.o(.debug_frame)
    .text                                    0x000007fc   Thumb Code    16  rt_div0.o(.text)
    ../../angel/rt.s                         0x00000000   Number         0  rt_fp_status_addr.o ABSOLUTE
    .text                                    0x0000080c   Thumb Code    24  rt_fp_status_addr.o(.text)
    <Anonymous Symbol>                       0x00003ae8   Data          80  rt_fp_status_addr.o(.debug_frame)
    ../../memcpset.s                         0x00000000   Number         0  rt_memclr.o ABSOLUTE
    .text                                    0x00000824   Thumb Code    72  rt_memclr.o(.text)
    <Anonymous Symbol>                       0x00003b38   Data          68  rt_memclr.o(.debug_frame)
    _Bytes                                   0x00000858   ARM Code       0  rt_memclr.o(.text)
    ../../fpinit.s                           0x00000000   Number         0  fpinit.o ABSOLUTE
    <Anonymous Symbol>                       0x00003b7c   Data          80  fpinit.o(.debug_frame)
    x$fpl$fpinit                             0x00003d50   Thumb Code    28  fpinit.o(x$fpl$fpinit)
    ../../dcmpin.s                           0x00000000   Number         0  dcmpin.o ABSOLUTE
    <Anonymous Symbol>                       0x00003bcc   Data          96  dcmpin.o(.debug_frame)
    x$fpl$dcmpinfnan                         0x00003a74   Thumb Code   108  dcmpin.o(x$fpl$dcmpinfnan)
    dcmp_neg                                 0x00003ab4   ARM Code       0  dcmpin.o(x$fpl$dcmpinfnan)
    dcmp_clear_v                             0x00003ac0   ARM Code       0  dcmpin.o(x$fpl$dcmpinfnan)
    dcmp_found_NaN                           0x00003ad0   ARM Code       0  dcmpin.o(x$fpl$dcmpinfnan)
    ../../except.s                           0x00000000   Number         0  except.o ABSOLUTE
    <Anonymous Symbol>                       0x00003c2c   Data         120  except.o(.debug_frame)
    x$fpl$exception                          0x00003be8   Thumb Code   360  except.o(x$fpl$exception)
    overflow                                 0x00003c84   ARM Code       0  except.o(x$fpl$exception)
    underflow                                0x00003c94   ARM Code       0  except.o(x$fpl$exception)
    divide_by_zero                           0x00003ca4   ARM Code       0  except.o(x$fpl$exception)
    inexact                                  0x00003cc0   ARM Code       0  except.o(x$fpl$exception)
    return_result                            0x00003cd0   ARM Code       0  except.o(x$fpl$exception)
    ovf_return                               0x00003cd8   ARM Code       0  except.o(x$fpl$exception)
    return_Inf                               0x00003ce4   ARM Code       0  except.o(x$fpl$exception)
    return_NaN                               0x00003d04   ARM Code       0  except.o(x$fpl$exception)
    prototype_double_Inf                     0x00003d2c   Data           0  except.o(x$fpl$exception)
    prototype_single_Inf                     0x00003d3c   Data           0  except.o(x$fpl$exception)
    prototype_double_NaN                     0x00003d44   Data           0  except.o(x$fpl$exception)
    prototype_single_NaN                     0x00003d4c   Data           0  except.o(x$fpl$exception)
    ../../angel/rt.s                         0x00000000   Number         0  rt_raise.o ABSOLUTE
    .text                                    0x0000086c   Thumb Code    32  rt_raise.o(.text)
    <Anonymous Symbol>                       0x00003ca4   Data          84  rt_raise.o(.debug_frame)
    ../../dcheck.s                           0x00000000   Number         0  dcheck.o ABSOLUTE
    <Anonymous Symbol>                       0x00003cf8   Data          84  dcheck.o(.debug_frame)
    x$fpl$dcheck                             0x00003a30   Thumb Code    68  dcheck.o(x$fpl$dcheck)
    dcheck_except                            0x00003a6c   ARM Code       0  dcheck.o(x$fpl$dcheck)
    ../../retnan.s                           0x00000000   Number         0  retnan.o ABSOLUTE
    <Anonymous Symbol>                       0x00003d4c   Data          92  retnan.o(.debug_frame)
    x$fpl$retnan                             0x00003d6c   Thumb Code   156  retnan.o(x$fpl$retnan)
    return_zero                              0x00003dc8   ARM Code       0  retnan.o(x$fpl$retnan)
    return_umaxint                           0x00003dd4   ARM Code       0  retnan.o(x$fpl$retnan)
    return_fpnan                             0x00003dec   ARM Code       0  retnan.o(x$fpl$retnan)
    ../../trapv.s                            0x00000000   Number         0  trapv.o ABSOLUTE
    x$fpl$trapveneer                         0x00003e08   Thumb Code   172  trapv.o(x$fpl$trapveneer)
    <Anonymous Symbol>                       0x00003da8   Data         132  trapv.o(.debug_frame)
    cmp_specflags_unordered                  0x00003e54   ARM Code       0  trapv.o(x$fpl$trapveneer)
    cmp_generic                              0x00003e60   ARM Code       0  trapv.o(x$fpl$trapveneer)
    cmp_boolean                              0x00003ea8   ARM Code       0  trapv.o(x$fpl$trapveneer)
    ../../signal.c                           0x00000000   Number         0  __raise.o ABSOLUTE
    .text                                    0x0000088c   Thumb Code     0  __raise.o(.text)
    C$debug_frame15                          0x00003e2c   Data           0  __raise.o(.debug_frame)
    ../../fenv.c                             0x00000000   Number         0  _fptrap.o ABSOLUTE
    .text                                    0x000008d0   Thumb Code     0  _fptrap.o(.text)
    C$debug_frame15                          0x00003e84   Data           0  _fptrap.o(.debug_frame)
    ../../angel/sys.s                        0x00000000   Number         0  sys_exit.o ABSOLUTE
    <Anonymous Symbol>                       0x00003ee4   Data          68  sys_exit.o(.debug_frame)
    .text                                    0x00000914   Thumb Code    28  sys_exit.o(.text)
    ../../unhosted.s                         0x00000000   Number         0  callvia.o ABSOLUTE
    .text                                    0x00000930   Thumb Code    16  callvia.o(.text)
    ../../signal.c                           0x00000000   Number         0  defsig.o ABSOLUTE
    .text                                    0x00000940   Thumb Code     0  defsig.o(.text)
    .constdata                               0x00004878   Data           0  defsig.o(.constdata)
    C$debug_frame15                          0x00003f28   Data           0  defsig.o(.debug_frame)
    .constdata$1                             0x00004878   Data           0  defsig.o(.constdata)
    messages@__default_signal_handler_0      0x00004878   Data          23  defsig.o(.constdata)
    ../../unhosted.s                         0x00000000   Number         0  sigdefs.o ABSOLUTE
    ../../angel/sys.s                        0x00000000   Number         0  use_semi.o ABSOLUTE
    <Anonymous Symbol>                       0x00003f7c   Data          68  use_semi.o(.debug_frame)
    .text                                    0x00000a58   Thumb Code     8  use_semi.o(.text)
    ../../angel/sysapp.c                     0x00000000   Number         0  sys_wrch.o ABSOLUTE
    .text                                    0x00000a60   Thumb Code     0  sys_wrch.o(.text)
    C$debug_frame14                          0x00003fc0   Data           0  sys_wrch.o(.debug_frame)

    Global Symbols

    Symbol Name                              Value     Ov Type        Size  Object(Section)

    BuildAttributes$$THUMB_ISAv2$M$E$P$PE$A:L22$X:L11$S22$IW$~STKCKD$~SHL$OSPACE$PRES8 0x00000000   Number         0  anon$$obj.o ABSOLUTE
    INT_Vectors                              0x00000000   ARM Code       0  bl_BOOTARM.obj(C$$code)
    Image$$BL_SECINFO$$Length                0x00000000   Number         0  anon$$obj.o ABSOLUTE
    Image$$BL_SECINFO$$ZI$$Length            0x00000000   Number         0  anon$$obj.o ABSOLUTE
    Image$$EMIINIT_CODE$$ZI$$Length          0x00000000   Number         0  anon$$obj.o ABSOLUTE
    Image$$FAST_CODE$$ZI$$Length             0x00000000   Number         0  anon$$obj.o ABSOLUTE
    Image$$READ_WRITE$$Length                0x00000000   Number         0  anon$$obj.o ABSOLUTE
    Image$$EXT_RAM$$Base                      - Undefined Weak Reference
    Image$$EXT_RAM$$Length                    - Undefined Weak Reference
    Image$$EXT_RAM$$ZI$$Base                  - Undefined Weak Reference
    Image$$EXT_RAM$$ZI$$Length                - Undefined Weak Reference
    Image$$READ_ONLY_SHARED$$Base             - Undefined Weak Reference
    Image$$READ_ONLY_SHARED$$Length           - Undefined Weak Reference
    Image$$READ_ONLY_SHARED$$ZI$$Base         - Undefined Weak Reference
    Image$$READ_ONLY_SHARED$$ZI$$Length       - Undefined Weak Reference
    Image$$READ_WRITE_SHARED$$Base            - Undefined Weak Reference
    Image$$READ_WRITE_SHARED$$Length          - Undefined Weak Reference
    Image$$READ_WRITE_SHARED$$ZI$$Base        - Undefined Weak Reference
    Image$$READ_WRITE_SHARED$$ZI$$Length      - Undefined Weak Reference
    Image$$READ_WRITE_SYS_RAM$$Base           - Undefined Weak Reference
    Image$$READ_WRITE_SYS_RAM$$Length         - Undefined Weak Reference
    Image$$READ_WRITE_SYS_RAM$$ZI$$Base       - Undefined Weak Reference
    Image$$READ_WRITE_SYS_RAM$$ZI$$Length     - Undefined Weak Reference
    Load$$EXT_RAM$$Base                       - Undefined Weak Reference
    Load$$READ_ONLY_SHARED$$Base              - Undefined Weak Reference
    Load$$READ_WRITE_SHARED$$Base             - Undefined Weak Reference
    Load$$READ_WRITE_SYS_RAM$$Base            - Undefined Weak Reference
    __Heap_DescSize                           - Undefined Weak Reference
    __alloca_initialize                       - Undefined Weak Reference
    __argv_alloc                              - Undefined Weak Reference
    __call_ctors()                            - Undefined Weak Reference
    __cpp_finalise                            - Undefined Weak Reference
    __cpp_initialise                          - Undefined Weak Reference
    __fpl_infinity                            - Undefined Weak Reference
    __rt_get_argv                             - Undefined Weak Reference
    __sigvec_lookup                           - Undefined Weak Reference
    _atexit_init                              - Undefined Weak Reference
    _clock_init                               - Undefined Weak Reference
    _fp_trap_big                              - Undefined Weak Reference
    _get_lc_collate                           - Undefined Weak Reference
    _get_lc_ctype                             - Undefined Weak Reference
    _get_lc_monetary                          - Undefined Weak Reference
    _get_lc_numeric                           - Undefined Weak Reference
    _get_lc_time                              - Undefined Weak Reference
    _getenv_init                              - Undefined Weak Reference
    _init_alloc                               - Undefined Weak Reference
    _init_user_alloc                          - Undefined Weak Reference
    _initio                                   - Undefined Weak Reference
    _rand_init                                - Undefined Weak Reference
    _signal_init                              - Undefined Weak Reference
    _terminate_user_alloc                     - Undefined Weak Reference
    _terminateio                              - Undefined Weak Reference
    Image$$EXT_READ_WRITE$$Length            0x00000040   Number         0  anon$$obj.o ABSOLUTE
    $Ven$AT$L$$SetPLLEMI                     0x000000a4   ARM Code       0  anon$$obj.o(Veneer$$Code)
    $Ven$AT$L$$ExtBootloader                 0x000000b0   ARM Code       0  anon$$obj.o(Veneer$$Code)
    g_ExtBootloaderInfo                      0x000000bc   Data          64  bl_Main.obj(HEAD_BL)
    Image$$FAST_ALGORITHM$$ZI$$Length        0x0000022c   Number         0  anon$$obj.o ABSOLUTE
    Image$$FAST_CODE$$Length                 0x0000022c   Number         0  anon$$obj.o ABSOLUTE
    Image$$EMIINIT_CODE$$Length              0x000002bc   Number         0  anon$$obj.o ABSOLUTE
    Image$$FAST_ALGORITHM$$Length            0x00000360   Number         0  anon$$obj.o ABSOLUTE
    Image$$BL_SECINFO$$Base                  0x00000400   Number         0  anon$$obj.o ABSOLUTE
    Image$$BL_SECINFO$$ZI$$Base              0x00000400   Number         0  anon$$obj.o ABSOLUTE
    Image$$READ_ONLY_TAIL$$Base              0x00000400   Number         0  anon$$obj.o ABSOLUTE
    Load$$BL_SECINFO$$Base                   0x00000400   Number         0  anon$$obj.o ABSOLUTE
    __rt_lib_init                            0x00000400   Thumb Code   158  lib_init.o(.text)
    __rt_lib_shutdown                        0x0000049e   Thumb Code    20  lib_init.o(.text)
    __16_ll_cmpge                            0x000004b8   Thumb Code    16  llcmpge.o(.text)
    _ll_cmpge                                0x000004bc   ARM Code       0  llcmpge.o(.text)
    __16_ll_mullu                            0x000004c8   Thumb Code    12  llmullu.o(.text)
    _ll_mullu                                0x000004cc   ARM Code       0  llmullu.o(.text)
    __16_ll_neg                              0x000004d4   Thumb Code    16  llneg.o(.text)
    _ll_neg                                  0x000004d8   ARM Code       0  llneg.o(.text)
    __16_ll_subls                            0x000004e4   Thumb Code    16  llsubls.o(.text)
    _ll_subls                                0x000004e8   ARM Code       0  llsubls.o(.text)
    memcpy                                   0x000004f4   Thumb Code    20  memcpy.o(.text)
    __32memcpy                               0x000004f8   ARM Code       0  memcpy.o(.text)
    memset                                   0x00000508   Thumb Code    36  memset.o(.text)
    __32memset                               0x0000050c   ARM Code       0  memset.o(.text)
    __16__rt_memclr_w                        0x0000052c   Thumb Code    92  rt_memclr_w.o(.text)
    __rt_memclr_w                            0x00000530   ARM Code       0  rt_memclr_w.o(.text)
    _memset_w                                0x00000534   ARM Code       0  rt_memclr_w.o(.text)
    __16__rt_memcpy                          0x00000588   Thumb Code   184  rt_memcpy.o(.text)
    __rt_memcpy                              0x0000058c   ARM Code       0  rt_memcpy.o(.text)
    __16__rt_memcpy_w                        0x00000640   Thumb Code   112  rt_memcpy_w.o(.text)
    __rt_memcpy_w                            0x00000644   ARM Code       0  rt_memcpy_w.o(.text)
    _memcpy_lastbytes                        0x00000690   ARM Code       0  rt_memcpy_w.o(.text)
    __16__rt_sdiv                            0x000006b0   Thumb Code   216  rt_sdiv.o(.text)
    __rt_sdiv                                0x000006b4   ARM Code       0  rt_sdiv.o(.text)
    Image$$EXT_READ_WRITE$$ZI$$Length        0x00000760   Number         0  anon$$obj.o ABSOLUTE
    __16__rt_sdiv10                          0x00000788   Thumb Code    68  rtsdiv10.o(.text)
    __rt_sdiv10                              0x0000078c   ARM Code       0  rtsdiv10.o(.text)
    __16__user_libspace                      0x000007cc   Thumb Code    12  libspace.o(.text)
    __user_libspace                          0x000007d0   ARM Code       0  libspace.o(.text)
    __16_ll_mul                              0x000007dc   Thumb Code    32  llmul3m.o(.text)
    _ll_mul                                  0x000007e0   ARM Code       0  llmul3m.o(.text)
    __16__rt_div0                            0x000007fc   Thumb Code    16  rt_div0.o(.text)
    __rt_div0                                0x00000800   ARM Code       0  rt_div0.o(.text)
    __16__rt_fp_status_addr                  0x0000080c   Thumb Code    24  rt_fp_status_addr.o(.text)
    __rt_fp_status_addr                      0x00000810   ARM Code       0  rt_fp_status_addr.o(.text)
    __16__rt_memclr                          0x00000824   Thumb Code    72  rt_memclr.o(.text)
    __rt_memclr                              0x00000828   ARM Code       0  rt_memclr.o(.text)
    _memset                                  0x0000082c   ARM Code       0  rt_memclr.o(.text)
    __rt_raise                               0x0000086c   Thumb Code    32  rt_raise.o(.text)
    __32__rt_raise                           0x00000870   ARM Code       0  rt_raise.o(.text)
    __raise                                  0x0000088c   Thumb Code    58  __raise.o(.text)
    _fp_trap                                 0x000008d0   Thumb Code    66  _fptrap.o(.text)
    __16_sys_exit                            0x00000914   Thumb Code    24  sys_exit.o(.text)
    _sys_exit                                0x00000918   ARM Code       0  sys_exit.o(.text)
    __call_via_r0                            0x00000930   Thumb Code     4  callvia.o(.text)
    __call_via_r1                            0x00000932   Thumb Code     4  callvia.o(.text)
    __call_via_r2                            0x00000934   Thumb Code     4  callvia.o(.text)
    __call_via_r3                            0x00000936   Thumb Code     4  callvia.o(.text)
    __call_via_r4                            0x00000938   Thumb Code     4  callvia.o(.text)
    __call_via_r5                            0x0000093a   Thumb Code     4  callvia.o(.text)
    __call_via_r6                            0x0000093c   Thumb Code     4  callvia.o(.text)
    __call_via_r7                            0x0000093e   Thumb Code     4  callvia.o(.text)
    __default_signal_handler                 0x00000940   Thumb Code   150  defsig.o(.text)
    __I_use_semihosting_swi                  0x00000a58   Thumb Code     8  use_semi.o(.text)
    __semihosting_swi_guard                  0x00000a58   Thumb Code     0  use_semi.o(.text)
    __32__I_use_semihosting_swi              0x00000a5c   ARM Code       0  use_semi.o(.text)
    _ttywrch                                 0x00000a60   Thumb Code    18  sys_wrch.o(.text)
    bl_Alg_Copy_Func_Tbl                     0x00000a74   Thumb Code     2  bl_Alg.obj(BL_ALGORITHM)
    bl_Alg_SignatureVerify                   0x00000a78   Thumb Code     4  bl_Alg.obj(BL_ALGORITHM)
    SST_Is_Secure_BB                         0x00000a7c   Thumb Code   182  SSS_secure_shared.obj(COMMON_CODE)
    SST_Get_MAUI_Rom_Info                    0x00000b4c   Thumb Code    68  SSS_secure_shared.obj(COMMON_CODE)
    SST_Get_MAUI_Feature_Combination         0x00000b98   Thumb Code    32  SSS_secure_shared.obj(COMMON_CODE)
    SST_Get_MAUI_Paired_Version              0x00000bb8   Thumb Code    22  SSS_secure_shared.obj(COMMON_CODE)
    CacheDeinit                              0x00000bd0   Thumb Code    20  bl_Cache.obj(EXT_BOOTLOADER_CODE)
    CacheInit                                0x00000be4   Thumb Code    38  bl_Cache.obj(EXT_BOOTLOADER_CODE)
    NorFlashBooting                          0x00000c14   Thumb Code     2  bl_ImageLoader.obj(EXT_BOOTLOADER_CODE)
    InitUSBDLGPIO                            0x00000c18   Thumb Code    44  bl_Init.obj(EXT_BOOTLOADER_CODE)
    InitExt                                  0x00000c48   Thumb Code     8  bl_Init.obj(EXT_BOOTLOADER_CODE)
    GetFeatureCombination                    0x00000c50   Thumb Code    26  bl_Init.obj(EXT_BOOTLOADER_CODE)
    CheckPairedVersion                       0x00000c70   Thumb Code    52  bl_Init.obj(EXT_BOOTLOADER_CODE)
    USBDLGPIO_Enabled                        0x00000cac   Thumb Code    22  bl_Main.obj(EXT_BOOTLOADER_CODE)
    USBDL_Start_Timer                        0x00000cc8   Thumb Code    44  bl_Main.obj(EXT_BOOTLOADER_CODE)
    USBDL_Stop_Timer                         0x00000d00   Thumb Code    16  bl_Main.obj(EXT_BOOTLOADER_CODE)
    USBDL_Is_Timeout                         0x00000d18   Thumb Code    68  bl_Main.obj(EXT_BOOTLOADER_CODE)
    USBDL_Ready_To_Enter_DLMode              0x00000d68   Thumb Code    92  bl_Main.obj(EXT_BOOTLOADER_CODE)
    USBDL_Main                               0x00000dd4   Thumb Code    80  bl_Main.obj(EXT_BOOTLOADER_CODE)
    FactoryProcedure                         0x00000e30   Thumb Code    40  bl_Main.obj(EXT_BOOTLOADER_CODE)
    ExtBootloader                            0x00000e60   Thumb Code    84  bl_Main.obj(EXT_BOOTLOADER_CODE)
    GetBootloaderRegion                      0x00000ec8   Thumb Code     4  bl_Main.obj(EXT_BOOTLOADER_CODE)
    InitRegionsExt                           0x00000ecc   ARM Code       0  bl_regioninit.obj(EXT_BOOTLOADER_CODE)
    InitRegions                              0x00000ed4   ARM Code       0  bl_regioninit.obj(RegionInit)
    Image$$READ_WRITE$$ZI$$Length            0x00001000   Number         0  anon$$obj.o ABSOLUTE
    INT_InitEMIInitCode                      0x0000106c   ARM Code       0  bl_regioninit.obj(RegionInit)
    INT_InitFastRegion                       0x000010a0   ARM Code       0  bl_regioninit.obj(RegionInit)
    $Ven$AT$L$$CodeCacheClearAllSetting      0x000011c8   ARM Code       0  anon$$obj.o(Veneer$$Code)
    $Ven$AT$L$$MPUClearAllSetting            0x000011d4   ARM Code       0  anon$$obj.o(Veneer$$Code)
    $Ven$AT$L$$CodeCacheSetting              0x000011e0   ARM Code       0  anon$$obj.o(Veneer$$Code)
    $Ven$AT$L$$CodeCacheConfig               0x000011ec   ARM Code       0  anon$$obj.o(Veneer$$Code)
    $Ven$AT$L$$dbg_print                     0x000011f8   ARM Code       0  anon$$obj.o(Veneer$$Code)
    $Ven$AT$L$$uart_init                     0x00001204   ARM Code       0  anon$$obj.o(Veneer$$Code)
    $Ven$AT$L$$BootAndHandOver               0x00001210   ARM Code       0  anon$$obj.o(Veneer$$Code)
    $Ven$AT$L$$SaveAndSetIRQMask             0x0000121c   ARM Code       0  anon$$obj.o(Veneer$$Code)
    $Ven$AT$L$$RestoreIRQMask                0x00001228   ARM Code       0  anon$$obj.o(Veneer$$Code)
    $Ven$AT$L$$kal_assert_fail               0x00001234   ARM Code       0  anon$$obj.o(Veneer$$Code)
    $Ven$AT$L$$INT_DisableCacheOnEMI         0x00001240   ARM Code       0  anon$$obj.o(Veneer$$Code)
    $Ven$AA$L$$JumpCmd                       0x0000124c   ARM Code       0  anon$$obj.o(Veneer$$Code)
    CodeCacheGetChannel                      0x00001254   Thumb Code    66  cache.obj(i.CodeCacheGetChannel)
    Connect_FactoryTool                      0x0000129c   Thumb Code   208  bl_FactoryConn.obj(i.Connect_FactoryTool)
    DriverInit                               0x0000137c   Thumb Code     8  bl_Init.obj(i.DriverInit)
    GPIO_InitIO                              0x00001388   Thumb Code    98  gpio.obj(i.GPIO_InitIO)
    GPIO_ModeSetup                           0x00001400   Thumb Code    96  gpio.obj(i.GPIO_ModeSetup)
    GPIO_PullSelSetup                        0x00001474   Thumb Code    64  gpio.obj(i.GPIO_PullSelSetup)
    GPIO_PullenSetup                         0x000014bc   Thumb Code    64  gpio.obj(i.GPIO_PullenSetup)
    GPIO_ReadIO                              0x00001504   Thumb Code    74  gpio.obj(i.GPIO_ReadIO)
    GPIO_init                                0x00001560   Thumb Code     8  gpio_drv.obj(i.GPIO_init)
    GPIO_setting_init                        0x00001568   Thumb Code   266  gpio_setting.obj(i.GPIO_setting_init)
    GenerateRandomSeed                       0x000016a0   Thumb Code    28  bl_Init.obj(i.GenerateRandomSeed)
    Get16Data                                0x000016c0   Thumb Code    38  bl_FactoryConn.obj(i.Get16Data)
    GetData                                  0x000016e8   Thumb Code    34  bl_FactoryConn.obj(i.GetData)
    HW_TDMA_Start                            0x0000170c   Thumb Code     8  l1_interface.obj(i.HW_TDMA_Start)
    HW_wait_32k_start                        0x00001718   Thumb Code    72  l1_interface.obj(i.HW_wait_32k_start)
    INT_Version_Check                        0x00001770   Thumb Code   296  bl_Main.obj(i.INT_Version_Check)
    INT_Version_Check_PutUARTByte            0x000018ac   Thumb Code    16  bl_Main.obj(i.INT_Version_Check_PutUARTByte)
    Init                                     0x000018c0   Thumb Code    46  bl_Init.obj(i.Init)
    Init_DTLB                                0x000018fc   Thumb Code     2  bl_Init.obj(i.Init_DTLB)
    LoadExtBootloader                        0x00001900   Thumb Code     4  bl_ImageLoader.obj(i.LoadExtBootloader)
    PreserveExtBootloaderHeader              0x00001904   Thumb Code     2  bl_ImageLoader.obj(i.PreserveExtBootloaderHeader)
    Put16Data                                0x00001908   Thumb Code    36  bl_FactoryConn.obj(i.Put16Data)
    PutData                                  0x0000192c   Thumb Code    36  bl_FactoryConn.obj(i.PutData)
    USB2UART_LineCoding2DCB                  0x00001950   Thumb Code    20  usbdl_usbacm_drv.obj(i.USB2UART_LineCoding2DCB)
    USBDLKey_Pressed                         0x00001964   Thumb Code   166  usbdl_usbacm_adap.obj(i.USBDLKey_Pressed)
    USBDL_ACMInit                            0x00001a24   Thumb Code    88  usbdl_usbacm_adap.obj(i.USBDL_ACMInit)
    USBDL_Cable_IN                           0x00001aa0   Thumb Code     4  usbdl_pmu.obj(i.USBDL_Cable_IN)
    USBDL_CheckStartCmd                      0x00001aa4   Thumb Code    82  usbdl_usbacm_adap.obj(i.USBDL_CheckStartCmd)
    USBDL_CheckUARTSendEnd                   0x00001b00   Thumb Code     2  usbdl_usbacm_adap.obj(i.USBDL_CheckUARTSendEnd)
    USBDL_GetUARTByte                        0x00001b04   Thumb Code    10  usbdl_usbacm_adap.obj(i.USBDL_GetUARTByte)
    USBDL_GetUARTByte_Ext                    0x00001b10   Thumb Code    70  usbdl_usbacm_adap.obj(i.USBDL_GetUARTByte_Ext)
    USBDL_Is_USB_Download_Mode               0x00001b60   Thumb Code     6  usbdl_usbacm_adap.obj(i.USBDL_Is_USB_Download_Mode)
    USBDL_PutUARTByte                        0x00001b6c   Thumb Code    10  usbdl_usbacm_adap.obj(i.USBDL_PutUARTByte)
    USBDL_PutUARTByte_Complete               0x00001b78   Thumb Code    10  usbdl_usbacm_adap.obj(i.USBDL_PutUARTByte_Complete)
    USBDL_PutUARTByte_Complete_Ext           0x00001b84   Thumb Code    90  usbdl_usbacm_adap.obj(i.USBDL_PutUARTByte_Complete_Ext)
    USBDL_PutUARTByte_Ext                    0x00001bf0   Thumb Code   116  usbdl_usbacm_adap.obj(i.USBDL_PutUARTByte_Ext)
    USBDL_Release                            0x00001c74   Thumb Code    34  usbdl_usbacm_adap.obj(i.USBDL_Release)
    USBDL_UART_Init                          0x00001c9c   Thumb Code   144  usbdl_usbacm_adap.obj(i.USBDL_UART_Init)
    USBDL_USBPowerON                         0x00001d48   Thumb Code   234  usbdl_usb_drv.obj(i.USBDL_USBPowerON)
    USBDL_Update_USB_Download_Mode           0x00001e4c   Thumb Code    40  usbdl_usbacm_adap.obj(i.USBDL_Update_USB_Download_Mode)
    USBDL_hwInit                             0x00001e7c   Thumb Code    26  usbdl_usbacm_adap.obj(i.USBDL_hwInit)
    USB_Acm_CommIf_Create                    0x00001f0c   Thumb Code   204  usbdl_usbacm_drv.obj(i.USB_Acm_CommIf_Create)
    USB_Acm_CommIf_Reset                     0x00001fe0   Thumb Code    10  usbdl_usbacm_drv.obj(i.USB_Acm_CommIf_Reset)
    USB_Acm_CommIf_Speed_Reset               0x00001ff0   Thumb Code    14  usbdl_usbacm_drv.obj(i.USB_Acm_CommIf_Speed_Reset)
    USB_Acm_DataIf_Create                    0x00002004   Thumb Code   194  usbdl_usbacm_drv.obj(i.USB_Acm_DataIf_Create)
    USB_Acm_DataIf_Reset                     0x000020dc   Thumb Code    50  usbdl_usbacm_drv.obj(i.USB_Acm_DataIf_Reset)
    USB_Acm_DataIf_Speed_Reset               0x00002114   Thumb Code    46  usbdl_usbacm_drv.obj(i.USB_Acm_DataIf_Speed_Reset)
    USB_CtrlEPStall                          0x00002320   Thumb Code    92  usbdl_usb_drv.obj(i.USB_CtrlEPStall)
    USB_Dbg_Trace                            0x00002384   Thumb Code     2  usbdl_debug_tool.obj(i.USB_Dbg_Trace)
    USB_DeRegister_CreateFunc                0x00002388   Thumb Code     8  usbdl_usb_resource.obj(i.USB_DeRegister_CreateFunc)
    USB_DeRegister_Device_Code               0x00002394   Thumb Code     8  usbdl_usb_resource.obj(i.USB_DeRegister_Device_Code)
    USB_EP0En                                0x000023a0   Thumb Code    14  usbdl_usb_drv.obj(i.USB_EP0En)
    USB_EP0_Pkt_Len                          0x000023b0   Thumb Code    22  usbdl_usb_drv.obj(i.USB_EP0_Pkt_Len)
    USB_EPFIFORead                           0x000023cc   Thumb Code    10  usbdl_usb_drv.obj(i.USB_EPFIFORead)
    USB_EPFIFORead_Shift                     0x000023d8   Thumb Code    70  usbdl_usb_drv.obj(i.USB_EPFIFORead_Shift)
    USB_EPFIFOWrite                          0x0000242c   Thumb Code    70  usbdl_usb_drv.obj(i.USB_EPFIFOWrite)
    USB_EP_Bulk_Rx_Ready                     0x00002480   Thumb Code    28  usbdl_usb_drv.obj(i.USB_EP_Bulk_Rx_Ready)
    USB_EP_Bulk_Tx_Ready                     0x000024a0   Thumb Code    60  usbdl_usb_drv.obj(i.USB_EP_Bulk_Tx_Ready)
    USB_EP_Rx_Pkt_Len                        0x00002520   Thumb Code    32  usbdl_usb_drv.obj(i.USB_EP_Rx_Pkt_Len)
    USB_EnSysIntr                            0x00002544   Thumb Code    18  usbdl_usb_drv.obj(i.USB_EnSysIntr)
    USB_Generate_EP0Data                     0x000026d4   Thumb Code    20  usbdl_usb.obj(i.USB_Generate_EP0Data)
    USB_GetAcmParam                          0x000026ec   Thumb Code     4  usb_custom.obj(i.USB_GetAcmParam)
    USB_GetCustomFunc                        0x000026f4   Thumb Code     4  usb_custom.obj(i.USB_GetCustomFunc)
    USB_GetDeviceParam                       0x000026fc   Thumb Code     4  usb_custom.obj(i.USB_GetDeviceParam)
    USB_GetMsParam                           0x00002704   Thumb Code     4  usb_custom.obj(i.USB_GetMsParam)
    USB_GetVideoParam                        0x0000270c   Thumb Code     4  usb_custom.obj(i.USB_GetVideoParam)
    USB_Get_Bulk_Rx_Ep                       0x00002714   Thumb Code    70  usbdl_usb_resource.obj(i.USB_Get_Bulk_Rx_Ep)
    USB_Get_Bulk_Tx_Ep                       0x00002764   Thumb Code    70  usbdl_usb_resource.obj(i.USB_Get_Bulk_Tx_Ep)
    USB_Get_EP0_Status                       0x000027b4   Thumb Code    38  usbdl_usb_drv.obj(i.USB_Get_EP0_Status)
    USB_Get_EP_Stall_Status                  0x000027dc   Thumb Code    32  usbdl_usb_drv.obj(i.USB_Get_EP_Stall_Status)
    USB_Get_Interface_Number                 0x00002804   Thumb Code    74  usbdl_usb_resource.obj(i.USB_Get_Interface_Number)
    USB_Get_Intr_Ep                          0x00002858   Thumb Code    64  usbdl_usb_resource.obj(i.USB_Get_Intr_Ep)
    USB_Get_String_Number                    0x000028a0   Thumb Code    76  usbdl_usb_resource.obj(i.USB_Get_String_Number)
    USB_HISR                                 0x000028f4   Thumb Code   332  usbdl_usb_drv.obj(i.USB_HISR)
    USB_High_Speed_Enable                    0x00002a4c   Thumb Code    26  usbdl_usb_drv.obj(i.USB_High_Speed_Enable)
    USB_Init                                 0x00002a68   Thumb Code    78  usbdl_usb.obj(i.USB_Init)
    USB_Init_Acm_Status                      0x00002ac4   Thumb Code    16  usbdl_usbacm_drv.obj(i.USB_Init_Acm_Status)
    USB_Init_Device_Status                   0x00002ad8   Thumb Code   180  usbdl_usb.obj(i.USB_Init_Device_Status)
    USB_Init_Drv_Info                        0x00002b90   Thumb Code    62  usbdl_usb_drv.obj(i.USB_Init_Drv_Info)
    USB_Initialize_Drv                       0x00002cc0   Thumb Code    32  usbdl_usb_drv.obj(i.USB_Initialize_Drv)
    USB_Is_High_Speed                        0x00002ce4   Thumb Code    18  usbdl_usb_drv.obj(i.USB_Is_High_Speed)
    USB_PDNDisable                           0x00002cf8   Thumb Code    44  usbdl_usb_drv.obj(i.USB_PDNDisable)
    USB_PowerControl                         0x00002d2c   Thumb Code     8  usb_custom.obj(i.USB_PowerControl)
    USB_Register_CreateFunc                  0x00002d34   Thumb Code    74  usbdl_usb_resource.obj(i.USB_Register_CreateFunc)
    USB_Register_Device_Code                 0x00002d88   Thumb Code    62  usbdl_usb_resource.obj(i.USB_Register_Device_Code)
    USB_Register_Drv_Info                    0x00002dd0   Thumb Code    70  usbdl_usb_drv.obj(i.USB_Register_Drv_Info)
    USB_Register_EP0_RxHdlr                  0x00002e1c   Thumb Code     6  usbdl_usb.obj(i.USB_Register_EP0_RxHdlr)
    USB_Release_Acm_Status                   0x00002e28   Thumb Code    16  usbdl_usbacm_drv.obj(i.USB_Release_Acm_Status)
    USB_ResetDrv_Info                        0x00002eb8   Thumb Code    40  usbdl_usb_drv.obj(i.USB_ResetDrv_Info)
    USB_Reset_Drv                            0x00002ee8   Thumb Code    34  usbdl_usb_drv.obj(i.USB_Reset_Drv)
    USB_Reset_FIFO                           0x00002f10   Thumb Code     8  usbdl_usb_drv.obj(i.USB_Reset_FIFO)
    USB_RxEPEn                               0x00002f1c   Thumb Code    76  usbdl_usb_drv.obj(i.USB_RxEPEn)
    USB_RxEPInit                             0x00002f6c   Thumb Code   152  usbdl_usb_drv.obj(i.USB_RxEPInit)
    USB_SetAddress                           0x00003014   Thumb Code    12  usbdl_usb_drv.obj(i.USB_SetAddress)
    USB_Set_DP_Pull_High                     0x00003020   Thumb Code    26  usbdl_usb_drv.obj(i.USB_Set_DP_Pull_High)
    USB_Software_Create                      0x0000303c   Thumb Code   392  usbdl_usb_resource.obj(i.USB_Software_Create)
    USB_Software_Init                        0x000031d4   Thumb Code   110  usbdl_usb_resource.obj(i.USB_Software_Init)
    USB_Software_Speed_Init                  0x0000324c   Thumb Code   226  usbdl_usb_resource.obj(i.USB_Software_Speed_Init)
    USB_TxEPEn                               0x00003508   Thumb Code    78  usbdl_usb_drv.obj(i.USB_TxEPEn)
    USB_TxEPInit                             0x0000355c   Thumb Code   140  usbdl_usb_drv.obj(i.USB_TxEPInit)
    USB_UART_Share                           0x000035f8   Thumb Code    24  usbdl_usb_drv.obj(i.USB_UART_Share)
    USB_Update_EP0_State                     0x00003614   Thumb Code    64  usbdl_usb_drv.obj(i.USB_Update_EP0_State)
    VerifyExtBootloader                      0x00003654   Thumb Code     4  bl_Main.obj(i.VerifyExtBootloader)
    WacthDogRestart                          0x00003658   Thumb Code     8  bl_Init.obj(i.WacthDogRestart)
    WaitFor32KStable                         0x00003668   Thumb Code    24  bl_Init.obj(i.WaitFor32KStable)
    WatchDogResetAll                         0x00003680   Thumb Code     8  bl_Init.obj(i.WatchDogResetAll)
    checksumCMD                              0x00003690   Thumb Code    60  bl_FactoryConn.obj(i.checksumCMD)
    custom_InitDRAM                          0x000036cc   Thumb Code     6  custom_emi.obj(i.custom_InitDRAM)
    custom_RAM_baseaddr                      0x000036d4   Thumb Code     6  custom_blconfig.obj(i.custom_RAM_baseaddr)
    custom_ROM_baseaddr                      0x000036dc   Thumb Code     4  custom_blconfig.obj(i.custom_ROM_baseaddr)
    custom_check_valid_secro                 0x000036e4   Thumb Code     4  custom_blconfig.obj(i.custom_check_valid_secro)
    custom_get_software_version              0x000036e8   Thumb Code     4  custom_blconfig.obj(i.custom_get_software_version)
    drv_get_current_time                     0x000036ec   Thumb Code     6  usbdl_debug_tool.obj(i.drv_get_current_time)
    getBlRegionCMD                           0x000036f8   Thumb Code    58  bl_FactoryConn.obj(i.getBlRegionCMD)
    getGPTTImer3Value                        0x00003734   Thumb Code    10  bl_Init.obj(i.getGPTTImer3Value)
    getSWVersionCMD                          0x00003744   Thumb Code    56  bl_FactoryConn.obj(i.getSWVersionCMD)
    isGPTTImer3Started                       0x0000377c   Thumb Code    14  bl_Init.obj(i.isGPTTImer3Started)
    jump_cmd2                                0x00003790   Thumb Code   222  bl_FactoryConn.obj(i.jump_cmd2)
    keypad_GetFunc                           0x00003880   Thumb Code     4  keypad_def.obj(i.keypad_GetFunc)
    keypad_Get_Data                          0x00003888   Thumb Code     4  keypad_def.obj(i.keypad_Get_Data)
    pmu6253_vusb_enable                      0x00003890   Thumb Code    18  usbdl_pmu.obj(i.pmu6253_vusb_enable)
    readCMD                                  0x000038a8   Thumb Code    54  bl_FactoryConn.obj(i.readCMD)
    readCMD_32                               0x000038e0   Thumb Code    54  bl_FactoryConn.obj(i.readCMD_32)
    startGPTTImer3                           0x00003918   Thumb Code    16  bl_Init.obj(i.startGPTTImer3)
    waitBlReadyCMD                           0x0000392c   Thumb Code    72  bl_FactoryConn.obj(i.waitBlReadyCMD)
    writeCMD                                 0x00003980   Thumb Code    60  bl_FactoryConn.obj(i.writeCMD)
    writeCMD_32                              0x000039bc   Thumb Code    60  bl_FactoryConn.obj(i.writeCMD_32)
    writeCMD_noecho                          0x000039f8   Thumb Code    54  bl_FactoryConn.obj(i.writeCMD_noecho)
    __16__fpl_dcheck_NaN2                    0x00003a30   Thumb Code    68  dcheck.o(x$fpl$dcheck)
    __fpl_dcheck_NaN2                        0x00003a34   ARM Code       0  dcheck.o(x$fpl$dcheck)
    __16__fpl_dcmp_InfNaN                    0x00003a74   Thumb Code   108  dcmpin.o(x$fpl$dcmpinfnan)
    __fpl_dcmp_InfNaN                        0x00003a78   ARM Code       0  dcmpin.o(x$fpl$dcmpinfnan)
    __fpl_inf_dcmp                           0x00003a9c   ARM Code       0  dcmpin.o(x$fpl$dcmpinfnan)
    __16_ll_uto_d                            0x00003ae0   Thumb Code    12  dfltll_clz.o(x$fpl$dfltll)
    _ll_uto_d                                0x00003ae4   ARM Code       0  dfltll_clz.o(x$fpl$dfltll)
    __16_ll_sto_d                            0x00003aec   Thumb Code   120  dfltll_clz.o(x$fpl$dfltll)
    _ll_sto_d                                0x00003af0   ARM Code       0  dfltll_clz.o(x$fpl$dfltll)
    __16_dcmpge                              0x00003b64   Thumb Code   128  dgeqf.o(x$fpl$dgeqf)
    _dcmpge                                  0x00003b68   ARM Code       0  dgeqf.o(x$fpl$dgeqf)
    __16__fpl_exception                      0x00003be8   Thumb Code   324  except.o(x$fpl$exception)
    __fpl_exception                          0x00003bec   ARM Code       0  except.o(x$fpl$exception)
    __16_fp_init                             0x00003d50   Thumb Code    28  fpinit.o(x$fpl$fpinit)
    _fp_init                                 0x00003d54   ARM Code       0  fpinit.o(x$fpl$fpinit)
    __fplib_config_pureend_doubles           0x00003d64   ARM Code       0  fpinit.o(x$fpl$fpinit)
    __16__fpl_return_NaN                     0x00003d6c   Thumb Code   148  retnan.o(x$fpl$retnan)
    __fpl_return_NaN                         0x00003d70   ARM Code       0  retnan.o(x$fpl$retnan)
    __16_fp_trapveneer                       0x00003e08   Thumb Code    40  trapv.o(x$fpl$trapveneer)
    _fp_trapveneer                           0x00003e0c   ARM Code       0  trapv.o(x$fpl$trapveneer)
    __16__fpl_cmpreturn                      0x00003e30   Thumb Code   132  trapv.o(x$fpl$trapveneer)
    __fpl_cmpreturn                          0x00003e34   ARM Code       0  trapv.o(x$fpl$trapveneer)
    g_SST_SecurePlatform                     0x00003eb4   Data           1  SSS_interface.obj(.constdata)
    g_SST_USBDownload4EndUser                0x00003eb5   Data           1  SSS_interface.obj(.constdata)
    g_SST_REMAPPING_ADDR                     0x00003eb8   Data           4  SSS_interface.obj(.constdata)
    g_SST_BootROM_version                    0x00003ebc   Data           4  SSS_interface.obj(.constdata)
    g_SST_CONFIG_base                        0x00003ec0   Data           4  SSS_interface.obj(.constdata)
    g_SST_EFUSE_base                         0x00003ec4   Data           4  SSS_interface.obj(.constdata)
    g_EFUSE_VER                              0x00003ec8   Data           4  SSS_interface.obj(.constdata)
    BootLDVerno                              0x00003fcc   Data           5  bl_verno.obj(.constdata)
    usbdlkey_position                        0x000041d0   Data           1  custom_blconfig.obj(.constdata)
    usbdlauto_timeout                        0x000041d2   Data           2  custom_blconfig.obj(.constdata)
    EMI_CSConfiguration                      0x000041d4   Data           4  custom_emi.obj(.constdata)
    EMI_SettingOnCS                          0x000041dc   Data          16  custom_emi.obj(.constdata)
    gpio_usbdl_pin                           0x000041ec   Data           1  gpio_var.obj(.constdata)
    keypad_custom_func                       0x000041f0   Data           4  keypad_def.obj(.constdata)
    keypad_custom_def                        0x000041f4   Data          80  keypad_def.obj(.constdata)
    INQUIRE_DATA                             0x000042f8   Data          36  usb_custom.obj(.constdata)
    const_g_mtk_secinfo_str                  0x000045c4   Data          12  SSS_secure_shared.obj(.constdata)
    const_g_mtk_rominfo_str                  0x000045d0   Data          12  SSS_secure_shared.obj(.constdata)
    Image$$READ_ONLY_TAIL$$Length            0x0000468c   Number         0  anon$$obj.o ABSOLUTE
    CUST_MEM_INFO                            0x000049a4   Data         232  custom_emi.obj(SECOND_PART)
    Load$$EMIINIT_CODE$$Base                 0x00004a8c   Number         0  anon$$obj.o ABSOLUTE
    Load$$FAST_ALGORITHM$$Base               0x00004d48   Number         0  anon$$obj.o ABSOLUTE
    Load$$FAST_CODE$$Base                    0x000050a8   Number         0  anon$$obj.o ABSOLUTE
    Load$$EXT_READ_WRITE$$Base               0x000052d4   Number         0  anon$$obj.o ABSOLUTE
    Load$$READ_WRITE$$Base                   0x000052d4   Number         0  anon$$obj.o ABSOLUTE
    Image$$EXT_READ_WRITE$$Base              0x08000000   Number         0  anon$$obj.o ABSOLUTE
    UART_Baud_Table                          0x08000002   Data          20  bl_UART.obj(.data)
    psram_compare_pattern                    0x08000018   Data           4  custom_emi.obj(.data)
    gpio_check_for_write                     0x0800001c   Data          12  gpio_setting.obj(.data)
    gpio_check_for_read                      0x08000028   Data          12  gpio_setting.obj(.data)
    Image$$EXT_READ_WRITE$$ZI$$Base          0x08000040   Number         0  anon$$obj.o ABSOLUTE
    g_bootupDisabled                         0x08000040   Data           1  bl_Main.obj(.bss)
    g_usbdlDisabled                          0x08000041   Data           1  bl_Main.obj(.bss)
    g_mauiFeatureCombination                 0x08000048   Data           4  bl_Main.obj(.bss)
    g_randomSeed                             0x0800004c   Data           4  bl_Main.obj(.bss)
    gpio_debug_enable                        0x08000054   Data           1  gpio_drv.obj(.bss)
    gUsbDevice                               0x0800005c   Data         340  usbdl_usb.obj(.bss)
    g_UsbDrvInfo                             0x080001b4   Data         100  usbdl_usb_drv.obj(.bss)
    keypadCustomFunc                         0x08000290   Data           4  usbdl_usbacm_adap.obj(.bss)
    keypad_comm_def                          0x08000294   Data           4  usbdl_usbacm_adap.obj(.bss)
    usbacm_tx_buf                            0x08000298   Data         516  usbdl_usbacm_adap.obj(.bss)
    usbacm_rx_buf                            0x0800049c   Data         516  usbdl_usbacm_adap.obj(.bss)
    gUSBAcm_IsInEPComplete                   0x080006a0   Data           1  usbdl_usbacm_drv.obj(.bss)
    USB2UARTPort                             0x080006a4   Data         100  usbdl_usbacm_drv.obj(.bss)
    g_UsbACM                                 0x08000708   Data          48  usbdl_usbacm_drv.obj(.bss)
    g_BlFirstDownload                        0x08000738   Data           1  bl_Secure.obj(.bss)
    g_Bl_Secure_Test                         0x0800073c   Data           4  bl_Secure.obj(.bss)
    BL_Shared_info                           0x40000000   Data          64  bl_ImageLoader.obj(BL_INFO_NOR)
    INT_SetPLL                               0x40000080   Thumb Code   154  bl_Init.obj(EMIINITCODE)
    Image$$EMIINIT_CODE$$Base                0x40000080   Number         0  anon$$obj.o ABSOLUTE
    Image$$FAST_ALGORITHM$$Base              0x40000080   Number         0  anon$$obj.o ABSOLUTE
    $Ven$AA$L$$_ll_cmpge                     0x40000080   ARM Code       0  anon$$obj.o(Veneer$$Code)
    $Ven$AA$L$$_ll_neg                       0x40000088   ARM Code       0  anon$$obj.o(Veneer$$Code)
    $Ven$AA$L$$_ll_sto_d                     0x40000090   ARM Code       0  anon$$obj.o(Veneer$$Code)
    $Ven$AA$L$$_dcmpge                       0x40000098   ARM Code       0  anon$$obj.o(Veneer$$Code)
    $Ven$AA$L$$_ll_subls                     0x400000a0   ARM Code       0  anon$$obj.o(Veneer$$Code)
    $Ven$AA$L$$_ll_mullu                     0x400000a8   ARM Code       0  anon$$obj.o(Veneer$$Code)
    $Ven$AA$L$$__rt_sdiv                     0x400000b0   ARM Code       0  anon$$obj.o(Veneer$$Code)
    $Ven$AA$L$$__rt_sdiv10                   0x400000b8   ARM Code       0  anon$$obj.o(Veneer$$Code)
    CheckUARTSendEnd                         0x400000c0 * Thumb Code    28  bl_UART.obj(i.CheckUARTSendEnd)
    INT_DisableCacheOnEMI                    0x400000e4 * Thumb Code     8  bl_portingfunc.obj(i.INT_DisableCacheOnEMI)
    PutUARTByte                              0x400000f0   Thumb Code    16  bl_UART.obj(i.PutUARTByte)
    RestoreIRQMask                           0x40000104 * Thumb Code     2  bl_portingfunc.obj(i.RestoreIRQMask)
    SaveAndSetIRQMask                        0x40000108 * Thumb Code     4  bl_portingfunc.obj(i.SaveAndSetIRQMask)
    dbg_print                                0x4000010c * Thumb Code   352  bl_DBGPRINT.obj(i.dbg_print)
    SetPLLEMI                                0x4000013c * Thumb Code    38  bl_Init.obj(EMIINITCODE)
    custom_setEMI                            0x40000168   Thumb Code    82  custom_emi.obj(EMIINITCODE)
    custom_setAdvEMI                         0x400001cc   Thumb Code   312  custom_emi.obj(EMIINITCODE)
    itof                                     0x400002ec   Thumb Code    56  bl_DBGPRINT.obj(i.itof)
    kal_assert_fail                          0x40000328 * Thumb Code    36  bl_portingfunc.obj(i.kal_assert_fail)
    $Ven$AT$L$$WacthDogRestart               0x40000330   ARM Code       0  anon$$obj.o(Veneer$$Code)
    Image$$EMIINIT_CODE$$ZI$$Base            0x4000033c   Number         0  anon$$obj.o ABSOLUTE
    uart_init                                0x40000354 * Thumb Code    64  bl_UART.obj(i.uart_init)
    Image$$FAST_ALGORITHM$$ZI$$Base          0x400003e0   Number         0  anon$$obj.o ABSOLUTE
    buf                                      0x4000040a   Data         512  bl_DBGPRINT.obj(.bss)
    Image$$FAST_CODE$$Base                   0x4000060c   Number         0  anon$$obj.o ABSOLUTE
    jump_cmd                                 0x4000060c   Thumb Code    22  bl_Main.obj(INTERNCODE)
    BootAndHandOver                          0x40000628   Thumb Code    66  bl_Main.obj(INTERNCODE)
    CodeCacheConfig                          0x40000678   Thumb Code    76  cache.obj(INTERNCODE)
    CodeCacheSetting                         0x400006c4   Thumb Code   182  cache.obj(INTERNCODE)
    CodeCacheClearAllSetting                 0x40000788   Thumb Code    44  cache.obj(INTERNCODE)
    MPUClearAllSetting                       0x400007bc   Thumb Code    44  cache.obj(INTERNCODE)
    JumpCmd                                  0x400007f4   ARM Code       0  bl_BOOTARM.obj(SHARECODE)
    RemapCmd                                 0x400007f8   ARM Code       0  bl_BOOTARM.obj(SHARECODE)
    $Ven$AT$L$$NorFlashBooting               0x40000808   ARM Code       0  anon$$obj.o(Veneer$$Code)
    $Ven$AT$L$$custom_ROM_baseaddr           0x40000814   ARM Code       0  anon$$obj.o(Veneer$$Code)
    $Ven$AT$L$$custom_RAM_baseaddr           0x40000820   ARM Code       0  anon$$obj.o(Veneer$$Code)
    $Ven$AT$L$$CacheDeinit                   0x4000082c   ARM Code       0  anon$$obj.o(Veneer$$Code)
    Image$$FAST_CODE$$ZI$$Base               0x40000838   Number         0  anon$$obj.o ABSOLUTE
    Image$$READ_WRITE$$Base                  0x4001cc00   Number         0  anon$$obj.o ABSOLUTE
    Image$$READ_WRITE$$ZI$$Base              0x4001cc00   Number         0  anon$$obj.o ABSOLUTE
    __SIG_IGN                                0xfffffffd   Number         0  sigdefs.o ABSOLUTE
    __SIG_ERR                                0xfffffffe   Number         0  sigdefs.o ABSOLUTE
    __SIG_DFL                                0xffffffff   Number         0  sigdefs.o ABSOLUTE


================================================================================

Memory Map of the image

  Image Entry point : 0x00000000

  Load Region READ_ONLY (Base: 0x00000000, Size: 0x00005314, Max: 0x00010000, ABSOLUTE)

    Execution Region READ_ONLY (Base: 0x00000000, Size: 0x000000fc, Max: 0x00000400, ABSOLUTE)

    Base Addr    Size         Type   Attr  Idx  E Section Name        Object

    0x00000000   0x000000a4   Code   RO    42   * C$$code             bl_BOOTARM.obj(bootloader.lib)
    0x000000a4   0x0000000c   Code   RO  1689     Veneer$$Code        anon$$obj.o
    0x000000b0   0x0000000c   Code   RO  1690     Veneer$$Code        anon$$obj.o
    0x000000bc   0x00000040   Data   RO   136     HEAD_BL             bl_Main.obj(bootloader.lib)


    Execution Region BL_ALG_TABLE (Base: 0x00000400, Size: 0x00000000, Max: 0xffffffff, ABSOLUTE, FIXED)

    **** No section assigned to this execution region ****


    Execution Region BL_SECINFO (Base: 0x00000400, Size: 0x00000000, Max: 0xffffffff, ABSOLUTE)

    **** No section assigned to this execution region ****


    Execution Region READ_ONLY_TAIL (Base: 0x00000400, Size: 0x0000468c, Max: 0xffffffff, ABSOLUTE)

    Base Addr    Size         Type   Attr  Idx  E Section Name        Object

    0x00000400   0x000000b8   Code   RO  1608     .text               lib_init.o(c_t__un.l)
    0x000004b8   0x00000010   Code   RO  1610     .text               llcmpge.o(c_t__un.l)
    0x000004c8   0x0000000c   Code   RO  1612     .text               llmullu.o(c_t__un.l)
    0x000004d4   0x00000010   Code   RO  1614     .text               llneg.o(c_t__un.l)
    0x000004e4   0x00000010   Code   RO  1618     .text               llsubls.o(c_t__un.l)
    0x000004f4   0x00000014   Code   RO  1624     .text               memcpy.o(c_t__un.l)
    0x00000508   0x00000024   Code   RO  1626     .text               memset.o(c_t__un.l)
    0x0000052c   0x0000005c   Code   RO  1628     .text               rt_memclr_w.o(c_t__un.l)
    0x00000588   0x000000b8   Code   RO  1630     .text               rt_memcpy.o(c_t__un.l)
    0x00000640   0x00000070   Code   RO  1632     .text               rt_memcpy_w.o(c_t__un.l)
    0x000006b0   0x000000d8   Code   RO  1634     .text               rt_sdiv.o(c_t__un.l)
    0x00000788   0x00000044   Code   RO  1638     .text               rtsdiv10.o(c_t__un.l)
    0x000007cc   0x00000010   Code   RO  1648     .text               libspace.o(c_t__un.l)
    0x000007dc   0x00000020   Code   RO  1651     .text               llmul3m.o(c_t__un.l)
    0x000007fc   0x00000010   Code   RO  1653     .text               rt_div0.o(c_t__un.l)
    0x0000080c   0x00000018   Code   RO  1655     .text               rt_fp_status_addr.o(c_t__un.l)
    0x00000824   0x00000048   Code   RO  1657     .text               rt_memclr.o(c_t__un.l)
    0x0000086c   0x00000020   Code   RO  1665     .text               rt_raise.o(c_t__un.l)
    0x0000088c   0x00000044   Code   RO  1673     .text               __raise.o(c_t__un.l)
    0x000008d0   0x00000044   Code   RO  1675     .text               _fptrap.o(c_t__un.l)
    0x00000914   0x0000001c   Code   RO  1677     .text               sys_exit.o(c_t__un.l)
    0x00000930   0x00000010   Code   RO  1679     .text               callvia.o(c_t__un.l)
    0x00000940   0x00000118   Code   RO  1680     .text               defsig.o(c_t__un.l)
    0x00000a58   0x00000008   Code   RO  1684     .text               use_semi.o(c_t__un.l)
    0x00000a60   0x00000014   Code   RO  1686     .text               sys_wrch.o(c_t__un.l)
    0x00000a74   0x00000004   Code   RO    35     BL_ALGORITHM        bl_Alg.obj(bootloader.lib)
    0x00000a78   0x00000004   Code   RO    36     BL_ALGORITHM        bl_Alg.obj(bootloader.lib)
    0x00000a7c   0x000000d0   Code   RO   813     COMMON_CODE         SSS_secure_shared.obj(sss.lib)
    0x00000b4c   0x0000004c   Code   RO   831     COMMON_CODE         SSS_secure_shared.obj(sss.lib)
    0x00000b98   0x00000020   Code   RO   833     COMMON_CODE         SSS_secure_shared.obj(sss.lib)
    0x00000bb8   0x00000018   Code   RO   834     COMMON_CODE         SSS_secure_shared.obj(sss.lib)
    0x00000bd0   0x00000014   Code   RO    48     EXT_BOOTLOADER_CODE  bl_Cache.obj(bootloader.lib)
    0x00000be4   0x00000030   Code   RO    49     EXT_BOOTLOADER_CODE  bl_Cache.obj(bootloader.lib)
    0x00000c14   0x00000004   Code   RO    66     EXT_BOOTLOADER_CODE  bl_ImageLoader.obj(bootloader.lib)
    0x00000c18   0x00000030   Code   RO    88     EXT_BOOTLOADER_CODE  bl_Init.obj(bootloader.lib)
    0x00000c48   0x00000008   Code   RO    89     EXT_BOOTLOADER_CODE  bl_Init.obj(bootloader.lib)
    0x00000c50   0x00000020   Code   RO    90     EXT_BOOTLOADER_CODE  bl_Init.obj(bootloader.lib)
    0x00000c70   0x0000003c   Code   RO    91     EXT_BOOTLOADER_CODE  bl_Init.obj(bootloader.lib)
    0x00000cac   0x0000001c   Code   RO   122     EXT_BOOTLOADER_CODE  bl_Main.obj(bootloader.lib)
    0x00000cc8   0x00000038   Code   RO   123     EXT_BOOTLOADER_CODE  bl_Main.obj(bootloader.lib)
    0x00000d00   0x00000018   Code   RO   124     EXT_BOOTLOADER_CODE  bl_Main.obj(bootloader.lib)
    0x00000d18   0x00000050   Code   RO   125     EXT_BOOTLOADER_CODE  bl_Main.obj(bootloader.lib)
    0x00000d68   0x0000006c   Code   RO   126     EXT_BOOTLOADER_CODE  bl_Main.obj(bootloader.lib)
    0x00000dd4   0x0000005c   Code   RO   127     EXT_BOOTLOADER_CODE  bl_Main.obj(bootloader.lib)
    0x00000e30   0x00000030   Code   RO   128     EXT_BOOTLOADER_CODE  bl_Main.obj(bootloader.lib)
    0x00000e60   0x00000068   Code   RO   131     EXT_BOOTLOADER_CODE  bl_Main.obj(bootloader.lib)
    0x00000ec8   0x00000004   Code   RO   132     EXT_BOOTLOADER_CODE  bl_Main.obj(bootloader.lib)
    0x00000ecc   0x00000008   Code   RO   178     EXT_BOOTLOADER_CODE  bl_regioninit.obj(bootloader.lib)
    0x00000ed4   0x000002f4   Code   RO   177     RegionInit          bl_regioninit.obj(bootloader.lib)
    0x000011c8   0x0000000c   Code   RO  1691     Veneer$$Code        anon$$obj.o
    0x000011d4   0x0000000c   Code   RO  1692     Veneer$$Code        anon$$obj.o
    0x000011e0   0x0000000c   Code   RO  1693     Veneer$$Code        anon$$obj.o
    0x000011ec   0x0000000c   Code   RO  1694     Veneer$$Code        anon$$obj.o
    0x000011f8   0x0000000c   Code   RO  1695     Veneer$$Code        anon$$obj.o
    0x00001204   0x0000000c   Code   RO  1696     Veneer$$Code        anon$$obj.o
    0x00001210   0x0000000c   Code   RO  1697     Veneer$$Code        anon$$obj.o
    0x0000121c   0x0000000c   Code   RO  1698     Veneer$$Code        anon$$obj.o
    0x00001228   0x0000000c   Code   RO  1699     Veneer$$Code        anon$$obj.o
    0x00001234   0x0000000c   Code   RO  1700     Veneer$$Code        anon$$obj.o
    0x00001240   0x0000000c   Code   RO  1701     Veneer$$Code        anon$$obj.o
    0x0000124c   0x00000008   Code   RO  1702     Veneer$$Code        anon$$obj.o
    0x00001254   0x00000048   Code   RO   186     i.CodeCacheGetChannel  cache.obj(bootloader.lib)
    0x0000129c   0x000000e0   Code   RO  1179     i.Connect_FactoryTool  bl_FactoryConn.obj(sss.lib)
    0x0000137c   0x0000000c   Code   RO    84     i.DriverInit        bl_Init.obj(bootloader.lib)
    0x00001388   0x00000078   Code   RO   265     i.GPIO_InitIO       gpio.obj(bootloader.lib)
    0x00001400   0x00000074   Code   RO   259     i.GPIO_ModeSetup    gpio.obj(bootloader.lib)
    0x00001474   0x00000048   Code   RO   264     i.GPIO_PullSelSetup  gpio.obj(bootloader.lib)
    0x000014bc   0x00000048   Code   RO   262     i.GPIO_PullenSetup  gpio.obj(bootloader.lib)
    0x00001504   0x0000005c   Code   RO   266     i.GPIO_ReadIO       gpio.obj(bootloader.lib)
    0x00001560   0x00000008   Code   RO   310     i.GPIO_init         gpio_drv.obj(bootloader.lib)
    0x00001568   0x00000138   Code   RO   313     i.GPIO_setting_init  gpio_setting.obj(bootloader.lib)
    0x000016a0   0x00000020   Code   RO    93     i.GenerateRandomSeed  bl_Init.obj(bootloader.lib)
    0x000016c0   0x00000028   Code   RO  1166     i.Get16Data         bl_FactoryConn.obj(sss.lib)
    0x000016e8   0x00000024   Code   RO  1164     i.GetData           bl_FactoryConn.obj(sss.lib)
    0x0000170c   0x0000000c   Code   RO   378     i.HW_TDMA_Start     l1_interface.obj(bootloader.lib)
    0x00001718   0x00000058   Code   RO   380     i.HW_wait_32k_start  l1_interface.obj(bootloader.lib)
    0x00001770   0x0000013c   Code   RO   120     i.INT_Version_Check  bl_Main.obj(bootloader.lib)
    0x000018ac   0x00000014   Code   RO   119     i.INT_Version_Check_PutUARTByte  bl_Main.obj(bootloader.lib)
    0x000018c0   0x0000003c   Code   RO    87     i.Init              bl_Init.obj(bootloader.lib)
    0x000018fc   0x00000004   Code   RO    92     i.Init_DTLB         bl_Init.obj(bootloader.lib)
    0x00001900   0x00000004   Code   RO    65     i.LoadExtBootloader  bl_ImageLoader.obj(bootloader.lib)
    0x00001904   0x00000004   Code   RO    64     i.PreserveExtBootloaderHeader  bl_ImageLoader.obj(bootloader.lib)
    0x00001908   0x00000024   Code   RO  1167     i.Put16Data         bl_FactoryConn.obj(sss.lib)
    0x0000192c   0x00000024   Code   RO  1165     i.PutData           bl_FactoryConn.obj(sss.lib)
    0x00001950   0x00000014   Code   RO   778     i.USB2UART_LineCoding2DCB  usbdl_usbacm_drv.obj(bootloader.lib)
    0x00001964   0x000000c0   Code   RO   740     i.USBDLKey_Pressed  usbdl_usbacm_adap.obj(bootloader.lib)
    0x00001a24   0x0000007c   Code   RO   744     i.USBDL_ACMInit     usbdl_usbacm_adap.obj(bootloader.lib)
    0x00001aa0   0x00000004   Code   RO   599     i.USBDL_Cable_IN    usbdl_pmu.obj(bootloader.lib)
    0x00001aa4   0x0000005c   Code   RO   754     i.USBDL_CheckStartCmd  usbdl_usbacm_adap.obj(bootloader.lib)
    0x00001b00   0x00000004   Code   RO   755     i.USBDL_CheckUARTSendEnd  usbdl_usbacm_adap.obj(bootloader.lib)
    0x00001b04   0x0000000c   Code   RO   753     i.USBDL_GetUARTByte  usbdl_usbacm_adap.obj(bootloader.lib)
    0x00001b10   0x00000050   Code   RO   752     i.USBDL_GetUARTByte_Ext  usbdl_usbacm_adap.obj(bootloader.lib)
    0x00001b60   0x0000000c   Code   RO   742     i.USBDL_Is_USB_Download_Mode  usbdl_usbacm_adap.obj(bootloader.lib)
    0x00001b6c   0x0000000c   Code   RO   749     i.USBDL_PutUARTByte  usbdl_usbacm_adap.obj(bootloader.lib)
    0x00001b78   0x0000000c   Code   RO   751     i.USBDL_PutUARTByte_Complete  usbdl_usbacm_adap.obj(bootloader.lib)
    0x00001b84   0x0000006c   Code   RO   750     i.USBDL_PutUARTByte_Complete_Ext  usbdl_usbacm_adap.obj(bootloader.lib)
    0x00001bf0   0x00000084   Code   RO   748     i.USBDL_PutUARTByte_Ext  usbdl_usbacm_adap.obj(bootloader.lib)
    0x00001c74   0x00000028   Code   RO   746     i.USBDL_Release     usbdl_usbacm_adap.obj(bootloader.lib)
    0x00001c9c   0x000000ac   Code   RO   745     i.USBDL_UART_Init   usbdl_usbacm_adap.obj(bootloader.lib)
    0x00001d48   0x00000104   Code   RO   637     i.USBDL_USBPowerON  usbdl_usb_drv.obj(bootloader.lib)
    0x00001e4c   0x00000030   Code   RO   741     i.USBDL_Update_USB_Download_Mode  usbdl_usbacm_adap.obj(bootloader.lib)
    0x00001e7c   0x0000001c   Code   RO   743     i.USBDL_hwInit      usbdl_usbacm_adap.obj(bootloader.lib)
    0x00001e98   0x0000000c   Code   RO   792     i.USB_Acm_BulkIn_Hdr  usbdl_usbacm_drv.obj(bootloader.lib)
    0x00001ea4   0x00000018   Code   RO   791     i.USB_Acm_BulkIn_Reset  usbdl_usbacm_drv.obj(bootloader.lib)
    0x00001ebc   0x00000038   Code   RO   790     i.USB_Acm_BulkOut_Hdr  usbdl_usbacm_drv.obj(bootloader.lib)
    0x00001ef4   0x00000018   Code   RO   789     i.USB_Acm_BulkOut_Reset  usbdl_usbacm_drv.obj(bootloader.lib)
    0x00001f0c   0x000000d4   Code   RO   780     i.USB_Acm_CommIf_Create  usbdl_usbacm_drv.obj(bootloader.lib)
    0x00001fe0   0x00000010   Code   RO   781     i.USB_Acm_CommIf_Reset  usbdl_usbacm_drv.obj(bootloader.lib)
    0x00001ff0   0x00000014   Code   RO   782     i.USB_Acm_CommIf_Speed_Reset  usbdl_usbacm_drv.obj(bootloader.lib)
    0x00002004   0x000000d8   Code   RO   783     i.USB_Acm_DataIf_Create  usbdl_usbacm_drv.obj(bootloader.lib)
    0x000020dc   0x00000038   Code   RO   784     i.USB_Acm_DataIf_Reset  usbdl_usbacm_drv.obj(bootloader.lib)
    0x00002114   0x00000034   Code   RO   785     i.USB_Acm_DataIf_Speed_Reset  usbdl_usbacm_drv.obj(bootloader.lib)
    0x00002148   0x0000005c   Code   RO   788     i.USB_Acm_Ep0_Command  usbdl_usbacm_drv.obj(bootloader.lib)
    0x000021a4   0x0000003c   Code   RO   793     i.USB_Acm_Ep0_SetLineCoding  usbdl_usbacm_drv.obj(bootloader.lib)
    0x000021e0   0x00000080   Code   RO   614     i.USB_Cmd_GetDescriptor  usbdl_usb.obj(bootloader.lib)
    0x00002260   0x0000005c   Code   RO   612     i.USB_Cmd_GetStatus  usbdl_usb.obj(bootloader.lib)
    0x000022bc   0x00000064   Code   RO   613     i.USB_Cmd_SetFeature  usbdl_usb.obj(bootloader.lib)
    0x00002320   0x00000064   Code   RO   653     i.USB_CtrlEPStall   usbdl_usb_drv.obj(bootloader.lib)
    0x00002384   0x00000004   Code   RO   595     i.USB_Dbg_Trace     usbdl_debug_tool.obj(bootloader.lib)
    0x00002388   0x0000000c   Code   RO   715     i.USB_DeRegister_CreateFunc  usbdl_usb_resource.obj(bootloader.lib)
    0x00002394   0x0000000c   Code   RO   716     i.USB_DeRegister_Device_Code  usbdl_usb_resource.obj(bootloader.lib)
    0x000023a0   0x00000010   Code   RO   641     i.USB_EP0En         usbdl_usb_drv.obj(bootloader.lib)
    0x000023b0   0x0000001c   Code   RO   656     i.USB_EP0_Pkt_Len   usbdl_usb_drv.obj(bootloader.lib)
    0x000023cc   0x0000000c   Code   RO   651     i.USB_EPFIFORead    usbdl_usb_drv.obj(bootloader.lib)
    0x000023d8   0x00000054   Code   RO   650     i.USB_EPFIFORead_Shift  usbdl_usb_drv.obj(bootloader.lib)
    0x0000242c   0x00000054   Code   RO   652     i.USB_EPFIFOWrite   usbdl_usb_drv.obj(bootloader.lib)
    0x00002480   0x00000020   Code   RO   659     i.USB_EP_Bulk_Rx_Ready  usbdl_usb_drv.obj(bootloader.lib)
    0x000024a0   0x00000044   Code   RO   657     i.USB_EP_Bulk_Tx_Ready  usbdl_usb_drv.obj(bootloader.lib)
    0x000024e4   0x0000003c   Code   RO   669     i.USB_EP_Check      usbdl_usb_drv.obj(bootloader.lib)
    0x00002520   0x00000024   Code   RO   658     i.USB_EP_Rx_Pkt_Len  usbdl_usb_drv.obj(bootloader.lib)
    0x00002544   0x00000014   Code   RO   642     i.USB_EnSysIntr     usbdl_usb_drv.obj(bootloader.lib)
    0x00002558   0x000000c4   Code   RO   607     i.USB_Endpoint0_Hdlr  usbdl_usb.obj(bootloader.lib)
    0x0000261c   0x00000068   Code   RO   610     i.USB_Endpoint0_Idle  usbdl_usb.obj(bootloader.lib)
    0x00002684   0x00000050   Code   RO   609     i.USB_Endpoint0_Tx  usbdl_usb.obj(bootloader.lib)
    0x000026d4   0x00000018   Code   RO   604     i.USB_Generate_EP0Data  usbdl_usb.obj(bootloader.lib)
    0x000026ec   0x00000008   Code   RO   572     i.USB_GetAcmParam   usb_custom.obj(bootloader.lib)
    0x000026f4   0x00000008   Code   RO   574     i.USB_GetCustomFunc  usb_custom.obj(bootloader.lib)
    0x000026fc   0x00000008   Code   RO   570     i.USB_GetDeviceParam  usb_custom.obj(bootloader.lib)
    0x00002704   0x00000008   Code   RO   571     i.USB_GetMsParam    usb_custom.obj(bootloader.lib)
    0x0000270c   0x00000008   Code   RO   573     i.USB_GetVideoParam  usb_custom.obj(bootloader.lib)
    0x00002714   0x00000050   Code   RO   719     i.USB_Get_Bulk_Rx_Ep  usbdl_usb_resource.obj(bootloader.lib)
    0x00002764   0x00000050   Code   RO   718     i.USB_Get_Bulk_Tx_Ep  usbdl_usb_resource.obj(bootloader.lib)
    0x000027b4   0x00000028   Code   RO   654     i.USB_Get_EP0_Status  usbdl_usb_drv.obj(bootloader.lib)
    0x000027dc   0x00000028   Code   RO   633     i.USB_Get_EP_Stall_Status  usbdl_usb_drv.obj(bootloader.lib)
    0x00002804   0x00000054   Code   RO   720     i.USB_Get_Interface_Number  usbdl_usb_resource.obj(bootloader.lib)
    0x00002858   0x00000048   Code   RO   717     i.USB_Get_Intr_Ep   usbdl_usb_resource.obj(bootloader.lib)
    0x000028a0   0x00000054   Code   RO   721     i.USB_Get_String_Number  usbdl_usb_resource.obj(bootloader.lib)
    0x000028f4   0x00000158   Code   RO   668     i.USB_HISR          usbdl_usb_drv.obj(bootloader.lib)
    0x00002a4c   0x0000001c   Code   RO   639     i.USB_High_Speed_Enable  usbdl_usb_drv.obj(bootloader.lib)
    0x00002a68   0x0000005c   Code   RO   605     i.USB_Init          usbdl_usb.obj(bootloader.lib)
    0x00002ac4   0x00000014   Code   RO   786     i.USB_Init_Acm_Status  usbdl_usbacm_drv.obj(bootloader.lib)
    0x00002ad8   0x000000b8   Code   RO   602     i.USB_Init_Device_Status  usbdl_usb.obj(bootloader.lib)
    0x00002b90   0x00000044   Code   RO   630     i.USB_Init_Drv_Info  usbdl_usb_drv.obj(bootloader.lib)
    0x00002bd4   0x000000ec   Code   RO   606     i.USB_Initialize    usbdl_usb.obj(bootloader.lib)
    0x00002cc0   0x00000024   Code   RO   643     i.USB_Initialize_Drv  usbdl_usb_drv.obj(bootloader.lib)
    0x00002ce4   0x00000014   Code   RO   663     i.USB_Is_High_Speed  usbdl_usb_drv.obj(bootloader.lib)
    0x00002cf8   0x00000034   Code   RO   635     i.USB_PDNDisable    usbdl_usb_drv.obj(bootloader.lib)
    0x00002d2c   0x00000008   Code   RO   575     i.USB_PowerControl  usb_custom.obj(bootloader.lib)
    0x00002d34   0x00000054   Code   RO   713     i.USB_Register_CreateFunc  usbdl_usb_resource.obj(bootloader.lib)
    0x00002d88   0x00000048   Code   RO   714     i.USB_Register_Device_Code  usbdl_usb_resource.obj(bootloader.lib)
    0x00002dd0   0x0000004c   Code   RO   632     i.USB_Register_Drv_Info  usbdl_usb_drv.obj(bootloader.lib)
    0x00002e1c   0x0000000c   Code   RO   603     i.USB_Register_EP0_RxHdlr  usbdl_usb.obj(bootloader.lib)
    0x00002e28   0x00000014   Code   RO   787     i.USB_Release_Acm_Status  usbdl_usbacm_drv.obj(bootloader.lib)
    0x00002e3c   0x0000007c   Code   RO   608     i.USB_Reset         usbdl_usb.obj(bootloader.lib)
    0x00002eb8   0x00000030   Code   RO   631     i.USB_ResetDrv_Info  usbdl_usb_drv.obj(bootloader.lib)
    0x00002ee8   0x00000028   Code   RO   640     i.USB_Reset_Drv     usbdl_usb_drv.obj(bootloader.lib)
    0x00002f10   0x0000000c   Code   RO   667     i.USB_Reset_FIFO    usbdl_usb_drv.obj(bootloader.lib)
    0x00002f1c   0x00000050   Code   RO   649     i.USB_RxEPEn        usbdl_usb_drv.obj(bootloader.lib)
    0x00002f6c   0x000000a8   Code   RO   647     i.USB_RxEPInit      usbdl_usb_drv.obj(bootloader.lib)
    0x00003014   0x0000000c   Code   RO   644     i.USB_SetAddress    usbdl_usb_drv.obj(bootloader.lib)
    0x00003020   0x0000001c   Code   RO   638     i.USB_Set_DP_Pull_High  usbdl_usb_drv.obj(bootloader.lib)
    0x0000303c   0x00000198   Code   RO   723     i.USB_Software_Create  usbdl_usb_resource.obj(bootloader.lib)
    0x000031d4   0x00000078   Code   RO   724     i.USB_Software_Init  usbdl_usb_resource.obj(bootloader.lib)
    0x0000324c   0x000000f4   Code   RO   722     i.USB_Software_Speed_Init  usbdl_usb_resource.obj(bootloader.lib)
    0x00003340   0x000001c8   Code   RO   611     i.USB_Stdcmd        usbdl_usb.obj(bootloader.lib)
    0x00003508   0x00000054   Code   RO   648     i.USB_TxEPEn        usbdl_usb_drv.obj(bootloader.lib)
    0x0000355c   0x0000009c   Code   RO   646     i.USB_TxEPInit      usbdl_usb_drv.obj(bootloader.lib)
    0x000035f8   0x0000001c   Code   RO   636     i.USB_UART_Share    usbdl_usb_drv.obj(bootloader.lib)
    0x00003614   0x00000040   Code   RO   655     i.USB_Update_EP0_State  usbdl_usb_drv.obj(bootloader.lib)
    0x00003654   0x00000004   Code   RO   121     i.VerifyExtBootloader  bl_Main.obj(bootloader.lib)
    0x00003658   0x00000010   Code   RO    75     i.WacthDogRestart   bl_Init.obj(bootloader.lib)
    0x00003668   0x00000018   Code   RO    78     i.WaitFor32KStable  bl_Init.obj(bootloader.lib)
    0x00003680   0x00000010   Code   RO    77     i.WatchDogResetAll  bl_Init.obj(bootloader.lib)
    0x00003690   0x0000003c   Code   RO  1173     i.checksumCMD       bl_FactoryConn.obj(sss.lib)
    0x000036cc   0x00000008   Code   RO   233     i.custom_InitDRAM   custom_emi.obj(bootloader.lib)
    0x000036d4   0x00000008   Code   RO   222     i.custom_RAM_baseaddr  custom_blconfig.obj(bootloader.lib)
    0x000036dc   0x00000008   Code   RO   221     i.custom_ROM_baseaddr  custom_blconfig.obj(bootloader.lib)
    0x000036e4   0x00000004   Code   RO   224     i.custom_check_valid_secro  custom_blconfig.obj(bootloader.lib)
    0x000036e8   0x00000004   Code   RO   223     i.custom_get_software_version  custom_blconfig.obj(bootloader.lib)
    0x000036ec   0x0000000c   Code   RO   594     i.drv_get_current_time  usbdl_debug_tool.obj(bootloader.lib)
    0x000036f8   0x0000003c   Code   RO  1175     i.getBlRegionCMD    bl_FactoryConn.obj(sss.lib)
    0x00003734   0x00000010   Code   RO    82     i.getGPTTImer3Value  bl_Init.obj(bootloader.lib)
    0x00003744   0x00000038   Code   RO  1174     i.getSWVersionCMD   bl_FactoryConn.obj(sss.lib)
    0x0000377c   0x00000014   Code   RO    79     i.isGPTTImer3Started  bl_Init.obj(bootloader.lib)
    0x00003790   0x000000f0   Code   RO  1176     i.jump_cmd2         bl_FactoryConn.obj(sss.lib)
    0x00003880   0x00000008   Code   RO   370     i.keypad_GetFunc    keypad_def.obj(bootloader.lib)
    0x00003888   0x00000008   Code   RO   371     i.keypad_Get_Data   keypad_def.obj(bootloader.lib)
    0x00003890   0x00000018   Code   RO   598     i.pmu6253_vusb_enable  usbdl_pmu.obj(bootloader.lib)
    0x000038a8   0x00000038   Code   RO  1169     i.readCMD           bl_FactoryConn.obj(sss.lib)
    0x000038e0   0x00000038   Code   RO  1172     i.readCMD_32        bl_FactoryConn.obj(sss.lib)
    0x00003918   0x00000014   Code   RO    80     i.startGPTTImer3    bl_Init.obj(bootloader.lib)
    0x0000392c   0x00000054   Code   RO  1177     i.waitBlReadyCMD    bl_FactoryConn.obj(sss.lib)
    0x00003980   0x0000003c   Code   RO  1168     i.writeCMD          bl_FactoryConn.obj(sss.lib)
    0x000039bc   0x0000003c   Code   RO  1171     i.writeCMD_32       bl_FactoryConn.obj(sss.lib)
    0x000039f8   0x00000038   Code   RO  1170     i.writeCMD_noecho   bl_FactoryConn.obj(sss.lib)
    0x00003a30   0x00000044   Code   RO  1667     x$fpl$dcheck        dcheck.o(f_t_p.l)
    0x00003a74   0x0000006c   Code   RO  1661     x$fpl$dcmpinfnan    dcmpin.o(f_t_p.l)
    0x00003ae0   0x00000084   Code   RO  1644     x$fpl$dfltll        dfltll_clz.o(f_t_p.l)
    0x00003b64   0x00000084   Code   RO  1646     x$fpl$dgeqf         dgeqf.o(f_t_p.l)
    0x00003be8   0x00000168   Code   RO  1663     x$fpl$exception     except.o(f_t_p.l)
    0x00003d50   0x0000001c   Code   RO  1659     x$fpl$fpinit        fpinit.o(f_t_p.l)
    0x00003d6c   0x0000009c   Code   RO  1669     x$fpl$retnan        retnan.o(f_t_p.l)
    0x00003e08   0x000000ac   Code   RO  1671     x$fpl$trapveneer    trapv.o(f_t_p.l)
    0x00003eb4   0x00000001   Data   RO    12     .constdata          SSS_interface.obj(bootloader.lib)
    0x00003eb5   0x00000001   Data   RO    14     .constdata          SSS_interface.obj(bootloader.lib)
    0x00003eb6   0x00000002   PAD
    0x00003eb8   0x00000004   Data   RO    25     .constdata          SSS_interface.obj(bootloader.lib)
    0x00003ebc   0x00000004   Data   RO    26     .constdata          SSS_interface.obj(bootloader.lib)
    0x00003ec0   0x00000004   Data   RO    28     .constdata          SSS_interface.obj(bootloader.lib)
    0x00003ec4   0x00000004   Data   RO    31     .constdata          SSS_interface.obj(bootloader.lib)
    0x00003ec8   0x00000004   Data   RO    34     .constdata          SSS_interface.obj(bootloader.lib)
    0x00003ecc   0x00000034   Data   RO    95     .constdata          bl_Init.obj(bootloader.lib)
    0x00003f00   0x000000cc   Data   RO   134     .constdata          bl_Main.obj(bootloader.lib)
    0x00003fcc   0x00000005   Data   RO   183     .constdata          bl_verno.obj(bootloader.lib)
    0x00003fd1   0x00000003   PAD
    0x00003fd4   0x000001fc   Data   RO   200     .constdata          cache.obj(bootloader.lib)
    0x000041d0   0x00000001   Data   RO   225     .constdata          custom_blconfig.obj(bootloader.lib)
    0x000041d1   0x00000001   PAD
    0x000041d2   0x00000002   Data   RO   226     .constdata          custom_blconfig.obj(bootloader.lib)
    0x000041d4   0x00000018   Data   RO   239     .constdata          custom_emi.obj(bootloader.lib)
    0x000041ec   0x00000001   Data   RO   342     .constdata          gpio_var.obj(bootloader.lib)
    0x000041ed   0x00000003   PAD
    0x000041f0   0x00000054   Data   RO   373     .constdata          keypad_def.obj(bootloader.lib)
    0x00004244   0x00000088   Data   RO   576     .constdata          usb_custom.obj(bootloader.lib)
    0x000042cc   0x0000001a   Data   RO   577     .constdata          usb_custom.obj(bootloader.lib)
    0x000042e6   0x00000010   Data   RO   578     .constdata          usb_custom.obj(bootloader.lib)
    0x000042f6   0x00000002   PAD
    0x000042f8   0x00000024   Data   RO   579     .constdata          usb_custom.obj(bootloader.lib)
    0x0000431c   0x0000001c   Data   RO   580     .constdata          usb_custom.obj(bootloader.lib)
    0x00004338   0x00000026   Data   RO   581     .constdata          usb_custom.obj(bootloader.lib)
    0x0000435e   0x00000026   Data   RO   582     .constdata          usb_custom.obj(bootloader.lib)
    0x00004384   0x00000026   Data   RO   583     .constdata          usb_custom.obj(bootloader.lib)
    0x000043aa   0x00000026   Data   RO   584     .constdata          usb_custom.obj(bootloader.lib)
    0x000043d0   0x0000002e   Data   RO   585     .constdata          usb_custom.obj(bootloader.lib)
    0x000043fe   0x00000026   Data   RO   586     .constdata          usb_custom.obj(bootloader.lib)
    0x00004424   0x00000026   Data   RO   587     .constdata          usb_custom.obj(bootloader.lib)
    0x0000444a   0x00000002   PAD
    0x0000444c   0x00000020   Data   RO   615     .constdata          usbdl_usb.obj(bootloader.lib)
    0x0000446c   0x00000024   Data   RO   671     .constdata          usbdl_usb_drv.obj(bootloader.lib)
    0x00004490   0x000000ec   Data   RO   725     .constdata          usbdl_usb_resource.obj(bootloader.lib)
    0x0000457c   0x00000048   Data   RO   758     .constdata          usbdl_usbacm_adap.obj(bootloader.lib)
    0x000045c4   0x00000278   Data   RO   841     .constdata          SSS_secure_shared.obj(sss.lib)
    0x0000483c   0x0000003c   Data   RO  1180     .constdata          bl_FactoryConn.obj(sss.lib)
    0x00004878   0x0000012b   Data   RO  1681     .constdata          defsig.o(c_t__un.l)
    0x000049a3   0x00000001   PAD
    0x000049a4   0x000000e8   Data   RO   242     SECOND_PART         custom_emi.obj(bootloader.lib)


    Execution Region BL_INFO_NOR (Base: 0x40000000, Size: 0x00000040, Max: 0x00000080, ABSOLUTE)

    Base Addr    Size         Type   Attr  Idx  E Section Name        Object

    0x40000000   0x00000040   Zero   RW    68     BL_INFO_NOR         bl_ImageLoader.obj(bootloader.lib)


    Execution Region EMIINIT_CODE (Base: 0x40000080, Size: 0x000002bc, Max: 0xffffffff, OVERLAY)

    Base Addr    Size         Type   Attr  Idx  E Section Name        Object

    0x40000080   0x000000bc   Code   RO    73     EMIINITCODE         bl_Init.obj(bootloader.lib)
    0x4000013c   0x0000002c   Code   RO    85     EMIINITCODE         bl_Init.obj(bootloader.lib)
    0x40000168   0x00000064   Code   RO   232     EMIINITCODE         custom_emi.obj(bootloader.lib)
    0x400001cc   0x00000164   Code   RO   234     EMIINITCODE         custom_emi.obj(bootloader.lib)
    0x40000330   0x0000000c   Code   RO  1703     Veneer$$Code        anon$$obj.o


    Execution Region FAST_ALGORITHM (Base: 0x40000080, Size: 0x0000058c, Max: 0x00001600, OVERLAY)

    Base Addr    Size         Type   Attr  Idx  E Section Name        Object

    0x40000080   0x00000008   Code   RO  1704     Veneer$$Code        anon$$obj.o
    0x40000088   0x00000008   Code   RO  1705     Veneer$$Code        anon$$obj.o
    0x40000090   0x00000008   Code   RO  1706     Veneer$$Code        anon$$obj.o
    0x40000098   0x00000008   Code   RO  1707     Veneer$$Code        anon$$obj.o
    0x400000a0   0x00000008   Code   RO  1708     Veneer$$Code        anon$$obj.o
    0x400000a8   0x00000008   Code   RO  1709     Veneer$$Code        anon$$obj.o
    0x400000b0   0x00000008   Code   RO  1710     Veneer$$Code        anon$$obj.o
    0x400000b8   0x00000008   Code   RO  1711     Veneer$$Code        anon$$obj.o
    0x400000c0   0x00000024   Code   RO   156     i.CheckUARTSendEnd  bl_UART.obj(bootloader.lib)
    0x400000e4   0x0000000c   Code   RO   164     i.INT_DisableCacheOnEMI  bl_portingfunc.obj(bootloader.lib)
    0x400000f0   0x00000014   Code   RO   155     i.PutUARTByte       bl_UART.obj(bootloader.lib)
    0x40000104   0x00000004   Code   RO   166     i.RestoreIRQMask    bl_portingfunc.obj(bootloader.lib)
    0x40000108   0x00000004   Code   RO   165     i.SaveAndSetIRQMask  bl_portingfunc.obj(bootloader.lib)
    0x4000010c   0x00000178   Code   RO    57     i.dbg_print         bl_DBGPRINT.obj(bootloader.lib)
    0x40000284   0x00000068   Code   RO    58     i.itoa              bl_DBGPRINT.obj(bootloader.lib)
    0x400002ec   0x0000003c   Code   RO    56     i.itof              bl_DBGPRINT.obj(bootloader.lib)
    0x40000328   0x0000002c   Code   RO   168     i.kal_assert_fail   bl_portingfunc.obj(bootloader.lib)
    0x40000354   0x00000048   Code   RO   157     i.uart_init         bl_UART.obj(bootloader.lib)
    0x4000039c   0x00000008   Data   RO    59     .constdata          bl_DBGPRINT.obj(bootloader.lib)
    0x400003a4   0x0000003c   Data   RO   170     .constdata          bl_portingfunc.obj(bootloader.lib)
    0x400003e0   0x0000022a   Zero   RW    60     .bss                bl_DBGPRINT.obj(bootloader.lib)


    Execution Region FAST_CODE (Base: 0x4000060c, Size: 0x0000022c, Max: 0xffffffff, ABSOLUTE)

    Base Addr    Size         Type   Attr  Idx  E Section Name        Object

    0x4000060c   0x0000001c   Code   RO   129     INTERNCODE          bl_Main.obj(bootloader.lib)
    0x40000628   0x00000050   Code   RO   130     INTERNCODE          bl_Main.obj(bootloader.lib)
    0x40000678   0x0000004c   Code   RO   188     INTERNCODE          cache.obj(bootloader.lib)
    0x400006c4   0x000000c4   Code   RO   189     INTERNCODE          cache.obj(bootloader.lib)
    0x40000788   0x00000034   Code   RO   190     INTERNCODE          cache.obj(bootloader.lib)
    0x400007bc   0x00000034   Code   RO   192     INTERNCODE          cache.obj(bootloader.lib)
    0x400007f0   0x00000018   Code   RO    43     SHARECODE           bl_BOOTARM.obj(bootloader.lib)
    0x40000808   0x0000000c   Code   RO  1712     Veneer$$Code        anon$$obj.o
    0x40000814   0x0000000c   Code   RO  1713     Veneer$$Code        anon$$obj.o
    0x40000820   0x0000000c   Code   RO  1714     Veneer$$Code        anon$$obj.o
    0x4000082c   0x0000000c   Code   RO  1715     Veneer$$Code        anon$$obj.o


    Execution Region READ_WRITE (Base: 0x4001cc00, Size: 0x00001000, Max: 0xffffffff, ABSOLUTE)

    Base Addr    Size         Type   Attr  Idx  E Section Name        Object

    0x4001cc00   0x00001000   Zero   RW    40     STACK_POOL_INTSRAM  bl_BOOTARM.obj(bootloader.lib)


    Execution Region EXT_READ_WRITE (Base: 0x08000000, Size: 0x000007a0, Max: 0x00020000, ABSOLUTE)

    Base Addr    Size         Type   Attr  Idx  E Section Name        Object

    0x08000000   0x00000002   Data   RW   133     .data               bl_Main.obj(bootloader.lib)
    0x08000002   0x00000014   Data   RW   158     .data               bl_UART.obj(bootloader.lib)
    0x08000016   0x00000002   PAD
    0x08000018   0x00000004   Data   RW   238     .data               custom_emi.obj(bootloader.lib)
    0x0800001c   0x0000000c   Data   RW   315     .data               gpio_setting.obj(bootloader.lib)
    0x08000028   0x0000000c   Data   RW   316     .data               gpio_setting.obj(bootloader.lib)
    0x08000034   0x00000004   Data   RW   670     .data               usbdl_usb_drv.obj(bootloader.lib)
    0x08000038   0x00000001   Data   RW   757     .data               usbdl_usbacm_adap.obj(bootloader.lib)
    0x08000039   0x00000003   PAD
    0x0800003c   0x00000004   Data   RW    41     DUMMY_POOL          bl_BOOTARM.obj(bootloader.lib)
    0x08000040   0x00000010   Zero   RW   135     .bss                bl_Main.obj(bootloader.lib)
    0x08000050   0x00000004   Zero   RW   201     .bss                cache.obj(bootloader.lib)
    0x08000054   0x00000001   Zero   RW   311     .bss                gpio_drv.obj(bootloader.lib)
    0x08000055   0x00000003   PAD
    0x08000058   0x00000158   Zero   RW   616     .bss                usbdl_usb.obj(bootloader.lib)
    0x080001b0   0x00000068   Zero   RW   672     .bss                usbdl_usb_drv.obj(bootloader.lib)
    0x08000218   0x00000070   Zero   RW   726     .bss                usbdl_usb_resource.obj(bootloader.lib)
    0x08000288   0x00000418   Zero   RW   759     .bss                usbdl_usbacm_adap.obj(bootloader.lib)
    0x080006a0   0x00000098   Zero   RW   794     .bss                usbdl_usbacm_drv.obj(bootloader.lib)
    0x08000738   0x00000001   Zero   RW  1350     .bss                bl_Secure.obj(sss.lib)
    0x08000739   0x00000003   PAD
    0x0800073c   0x00000004   Zero   RW  1352     .bss                bl_Secure.obj(sss.lib)
    0x08000740   0x00000060   Zero   RW  1649     .bss                libspace.o(c_t__un.l)



  Load Region __HIDDEN_BL_SECURE_MAC (Base: 0x00005314, Size: 0x00000000, Max: 0xffffffff, ABSOLUTE)

    Execution Region __HIDDEN_BL_SECURE_MAC (Base: 0x00005314, Size: 0x00000000, Max: 0xffffffff, ABSOLUTE)

    **** No section assigned to this execution region ****


    Execution Region __HIDDEN_BL_SECURE_MAC_CONTENT (Base: 0x00005314, Size: 0x00000000, Max: 0xffffffff, ABSOLUTE)

    **** No section assigned to this execution region ****


    Execution Region __HIDDEN_SECURE_MAC (Base: 0x00005314, Size: 0x00000000, Max: 0xffffffff, ABSOLUTE)

    **** No section assigned to this execution region ****



  Load Region LR$$Debug (Base: 0x00000000, Size: 0x00000000, Max: 0xffffffff, ABSOLUTE)

    Execution Region ER$$Debug (Base: 0x00000000, Size: 0x00000000, Max: 0xffffffff, ABSOLUTE)

    Base Addr    Size         Type   Attr  Idx  E Section Name        Object

    0x00000000   0x0000000c   Dbug   RW    47     .debug_abbrev       bl_BOOTARM.obj(bootloader.lib)
    0x0000000c   0x0000000c   Dbug   RW   181     .debug_abbrev       bl_regioninit.obj(bootloader.lib)
    0x00000018   0x000003ec   Dbug   RW  1084     .debug_abbrev       SSS_secure_shared.obj(sss.lib)
    0x00000000   0x0000003c   Dbug   RW    38     .debug_frame        bl_Alg.obj(bootloader.lib)
    0x0000003c   0x0000003c   Dbug   RW    39     .debug_frame        bl_Alg.obj(bootloader.lib)
    0x00000078   0x0000004c   Dbug   RW    52     .debug_frame        bl_Cache.obj(bootloader.lib)
    0x000000c4   0x00000048   Dbug   RW    53     .debug_frame        bl_Cache.obj(bootloader.lib)
    0x0000010c   0x00000050   Dbug   RW    61     .debug_frame        bl_DBGPRINT.obj(bootloader.lib)
    0x0000015c   0x00000060   Dbug   RW    62     .debug_frame        bl_DBGPRINT.obj(bootloader.lib)
    0x000001bc   0x00000054   Dbug   RW    63     .debug_frame        bl_DBGPRINT.obj(bootloader.lib)
    0x00000210   0x0000003c   Dbug   RW    69     .debug_frame        bl_ImageLoader.obj(bootloader.lib)
    0x0000024c   0x0000003c   Dbug   RW    70     .debug_frame        bl_ImageLoader.obj(bootloader.lib)
    0x00000288   0x0000003c   Dbug   RW    71     .debug_frame        bl_ImageLoader.obj(bootloader.lib)
    0x000002c4   0x00000050   Dbug   RW    96     .debug_frame        bl_Init.obj(bootloader.lib)
    0x00000314   0x0000003c   Dbug   RW    98     .debug_frame        bl_Init.obj(bootloader.lib)
    0x00000350   0x0000003c   Dbug   RW   100     .debug_frame        bl_Init.obj(bootloader.lib)
    0x0000038c   0x0000004c   Dbug   RW   101     .debug_frame        bl_Init.obj(bootloader.lib)
    0x000003d8   0x0000003c   Dbug   RW   102     .debug_frame        bl_Init.obj(bootloader.lib)
    0x00000414   0x0000003c   Dbug   RW   103     .debug_frame        bl_Init.obj(bootloader.lib)
    0x00000450   0x0000003c   Dbug   RW   105     .debug_frame        bl_Init.obj(bootloader.lib)
    0x0000048c   0x0000003c   Dbug   RW   107     .debug_frame        bl_Init.obj(bootloader.lib)
    0x000004c8   0x00000050   Dbug   RW   108     .debug_frame        bl_Init.obj(bootloader.lib)
    0x00000518   0x0000004c   Dbug   RW   110     .debug_frame        bl_Init.obj(bootloader.lib)
    0x00000564   0x0000004c   Dbug   RW   111     .debug_frame        bl_Init.obj(bootloader.lib)
    0x000005b0   0x0000004c   Dbug   RW   112     .debug_frame        bl_Init.obj(bootloader.lib)
    0x000005fc   0x0000004c   Dbug   RW   113     .debug_frame        bl_Init.obj(bootloader.lib)
    0x00000648   0x00000050   Dbug   RW   114     .debug_frame        bl_Init.obj(bootloader.lib)
    0x00000698   0x0000003c   Dbug   RW   115     .debug_frame        bl_Init.obj(bootloader.lib)
    0x000006d4   0x0000004c   Dbug   RW   116     .debug_frame        bl_Init.obj(bootloader.lib)
    0x00000720   0x0000003c   Dbug   RW   139     .debug_frame        bl_Main.obj(bootloader.lib)
    0x0000075c   0x00000054   Dbug   RW   140     .debug_frame        bl_Main.obj(bootloader.lib)
    0x000007b0   0x0000003c   Dbug   RW   141     .debug_frame        bl_Main.obj(bootloader.lib)
    0x000007ec   0x00000050   Dbug   RW   142     .debug_frame        bl_Main.obj(bootloader.lib)
    0x0000083c   0x0000004c   Dbug   RW   143     .debug_frame        bl_Main.obj(bootloader.lib)
    0x00000888   0x0000003c   Dbug   RW   144     .debug_frame        bl_Main.obj(bootloader.lib)
    0x000008c4   0x00000058   Dbug   RW   145     .debug_frame        bl_Main.obj(bootloader.lib)
    0x0000091c   0x00000050   Dbug   RW   146     .debug_frame        bl_Main.obj(bootloader.lib)
    0x0000096c   0x00000058   Dbug   RW   147     .debug_frame        bl_Main.obj(bootloader.lib)
    0x000009c4   0x0000004c   Dbug   RW   148     .debug_frame        bl_Main.obj(bootloader.lib)
    0x00000a10   0x0000004c   Dbug   RW   149     .debug_frame        bl_Main.obj(bootloader.lib)
    0x00000a5c   0x0000004c   Dbug   RW   150     .debug_frame        bl_Main.obj(bootloader.lib)
    0x00000aa8   0x0000004c   Dbug   RW   151     .debug_frame        bl_Main.obj(bootloader.lib)
    0x00000af4   0x0000003c   Dbug   RW   152     .debug_frame        bl_Main.obj(bootloader.lib)
    0x00000b30   0x0000003c   Dbug   RW   161     .debug_frame        bl_UART.obj(bootloader.lib)
    0x00000b6c   0x0000003c   Dbug   RW   162     .debug_frame        bl_UART.obj(bootloader.lib)
    0x00000ba8   0x0000003c   Dbug   RW   163     .debug_frame        bl_UART.obj(bootloader.lib)
    0x00000be4   0x0000003c   Dbug   RW   171     .debug_frame        bl_portingfunc.obj(bootloader.lib)
    0x00000c20   0x0000003c   Dbug   RW   172     .debug_frame        bl_portingfunc.obj(bootloader.lib)
    0x00000c5c   0x0000003c   Dbug   RW   173     .debug_frame        bl_portingfunc.obj(bootloader.lib)
    0x00000c98   0x0000004c   Dbug   RW   175     .debug_frame        bl_portingfunc.obj(bootloader.lib)
    0x00000ce4   0x00000058   Dbug   RW   204     .debug_frame        cache.obj(bootloader.lib)
    0x00000d3c   0x00000050   Dbug   RW   206     .debug_frame        cache.obj(bootloader.lib)
    0x00000d8c   0x0000005c   Dbug   RW   207     .debug_frame        cache.obj(bootloader.lib)
    0x00000de8   0x0000004c   Dbug   RW   208     .debug_frame        cache.obj(bootloader.lib)
    0x00000e34   0x0000004c   Dbug   RW   210     .debug_frame        cache.obj(bootloader.lib)
    0x00000e80   0x0000003c   Dbug   RW   228     .debug_frame        custom_blconfig.obj(bootloader.lib)
    0x00000ebc   0x0000003c   Dbug   RW   229     .debug_frame        custom_blconfig.obj(bootloader.lib)
    0x00000ef8   0x0000003c   Dbug   RW   230     .debug_frame        custom_blconfig.obj(bootloader.lib)
    0x00000f34   0x0000003c   Dbug   RW   231     .debug_frame        custom_blconfig.obj(bootloader.lib)
    0x00000f70   0x0000004c   Dbug   RW   243     .debug_frame        custom_emi.obj(bootloader.lib)
    0x00000fbc   0x0000003c   Dbug   RW   244     .debug_frame        custom_emi.obj(bootloader.lib)
    0x00000ff8   0x00000054   Dbug   RW   245     .debug_frame        custom_emi.obj(bootloader.lib)
    0x0000104c   0x00000050   Dbug   RW   285     .debug_frame        gpio.obj(bootloader.lib)
    0x0000109c   0x0000003c   Dbug   RW   288     .debug_frame        gpio.obj(bootloader.lib)
    0x000010d8   0x0000003c   Dbug   RW   290     .debug_frame        gpio.obj(bootloader.lib)
    0x00001114   0x00000054   Dbug   RW   291     .debug_frame        gpio.obj(bootloader.lib)
    0x00001168   0x00000050   Dbug   RW   292     .debug_frame        gpio.obj(bootloader.lib)
    0x000011b8   0x0000004c   Dbug   RW   312     .debug_frame        gpio_drv.obj(bootloader.lib)
    0x00001204   0x0000003c   Dbug   RW   319     .debug_frame        gpio_setting.obj(bootloader.lib)
    0x00001240   0x0000003c   Dbug   RW   375     .debug_frame        keypad_def.obj(bootloader.lib)
    0x0000127c   0x0000003c   Dbug   RW   376     .debug_frame        keypad_def.obj(bootloader.lib)
    0x000012b8   0x0000003c   Dbug   RW   381     .debug_frame        l1_interface.obj(bootloader.lib)
    0x000012f4   0x00000054   Dbug   RW   383     .debug_frame        l1_interface.obj(bootloader.lib)
    0x00001348   0x0000003c   Dbug   RW   588     .debug_frame        usb_custom.obj(bootloader.lib)
    0x00001384   0x0000003c   Dbug   RW   589     .debug_frame        usb_custom.obj(bootloader.lib)
    0x000013c0   0x0000003c   Dbug   RW   590     .debug_frame        usb_custom.obj(bootloader.lib)
    0x000013fc   0x0000003c   Dbug   RW   591     .debug_frame        usb_custom.obj(bootloader.lib)
    0x00001438   0x0000003c   Dbug   RW   592     .debug_frame        usb_custom.obj(bootloader.lib)
    0x00001474   0x0000004c   Dbug   RW   593     .debug_frame        usb_custom.obj(bootloader.lib)
    0x000014c0   0x0000003c   Dbug   RW   596     .debug_frame        usbdl_debug_tool.obj(bootloader.lib)
    0x000014fc   0x0000003c   Dbug   RW   597     .debug_frame        usbdl_debug_tool.obj(bootloader.lib)
    0x00001538   0x0000003c   Dbug   RW   600     .debug_frame        usbdl_pmu.obj(bootloader.lib)
    0x00001574   0x0000003c   Dbug   RW   601     .debug_frame        usbdl_pmu.obj(bootloader.lib)
    0x000015b0   0x00000050   Dbug   RW   617     .debug_frame        usbdl_usb.obj(bootloader.lib)
    0x00001600   0x0000003c   Dbug   RW   618     .debug_frame        usbdl_usb.obj(bootloader.lib)
    0x0000163c   0x0000003c   Dbug   RW   619     .debug_frame        usbdl_usb.obj(bootloader.lib)
    0x00001678   0x00000050   Dbug   RW   620     .debug_frame        usbdl_usb.obj(bootloader.lib)
    0x000016c8   0x00000054   Dbug   RW   621     .debug_frame        usbdl_usb.obj(bootloader.lib)
    0x0000171c   0x00000058   Dbug   RW   622     .debug_frame        usbdl_usb.obj(bootloader.lib)
    0x00001774   0x00000050   Dbug   RW   623     .debug_frame        usbdl_usb.obj(bootloader.lib)
    0x000017c4   0x00000054   Dbug   RW   624     .debug_frame        usbdl_usb.obj(bootloader.lib)
    0x00001818   0x00000060   Dbug   RW   625     .debug_frame        usbdl_usb.obj(bootloader.lib)
    0x00001878   0x00000054   Dbug   RW   626     .debug_frame        usbdl_usb.obj(bootloader.lib)
    0x000018cc   0x00000054   Dbug   RW   627     .debug_frame        usbdl_usb.obj(bootloader.lib)
    0x00001920   0x0000004c   Dbug   RW   628     .debug_frame        usbdl_usb.obj(bootloader.lib)
    0x0000196c   0x00000054   Dbug   RW   629     .debug_frame        usbdl_usb.obj(bootloader.lib)
    0x000019c0   0x0000004c   Dbug   RW   673     .debug_frame        usbdl_usb_drv.obj(bootloader.lib)
    0x00001a0c   0x0000003c   Dbug   RW   674     .debug_frame        usbdl_usb_drv.obj(bootloader.lib)
    0x00001a48   0x00000068   Dbug   RW   675     .debug_frame        usbdl_usb_drv.obj(bootloader.lib)
    0x00001ab0   0x00000058   Dbug   RW   676     .debug_frame        usbdl_usb_drv.obj(bootloader.lib)
    0x00001b08   0x00000050   Dbug   RW   678     .debug_frame        usbdl_usb_drv.obj(bootloader.lib)
    0x00001b58   0x0000003c   Dbug   RW   679     .debug_frame        usbdl_usb_drv.obj(bootloader.lib)
    0x00001b94   0x00000054   Dbug   RW   680     .debug_frame        usbdl_usb_drv.obj(bootloader.lib)
    0x00001be8   0x0000003c   Dbug   RW   681     .debug_frame        usbdl_usb_drv.obj(bootloader.lib)
    0x00001c24   0x0000003c   Dbug   RW   682     .debug_frame        usbdl_usb_drv.obj(bootloader.lib)
    0x00001c60   0x00000048   Dbug   RW   683     .debug_frame        usbdl_usb_drv.obj(bootloader.lib)
    0x00001ca8   0x0000003c   Dbug   RW   684     .debug_frame        usbdl_usb_drv.obj(bootloader.lib)
    0x00001ce4   0x0000003c   Dbug   RW   685     .debug_frame        usbdl_usb_drv.obj(bootloader.lib)
    0x00001d20   0x00000048   Dbug   RW   686     .debug_frame        usbdl_usb_drv.obj(bootloader.lib)
    0x00001d68   0x0000003c   Dbug   RW   687     .debug_frame        usbdl_usb_drv.obj(bootloader.lib)
    0x00001da4   0x0000005c   Dbug   RW   689     .debug_frame        usbdl_usb_drv.obj(bootloader.lib)
    0x00001e00   0x0000005c   Dbug   RW   690     .debug_frame        usbdl_usb_drv.obj(bootloader.lib)
    0x00001e5c   0x00000050   Dbug   RW   691     .debug_frame        usbdl_usb_drv.obj(bootloader.lib)
    0x00001eac   0x00000050   Dbug   RW   692     .debug_frame        usbdl_usb_drv.obj(bootloader.lib)
    0x00001efc   0x00000050   Dbug   RW   693     .debug_frame        usbdl_usb_drv.obj(bootloader.lib)
    0x00001f4c   0x0000004c   Dbug   RW   694     .debug_frame        usbdl_usb_drv.obj(bootloader.lib)
    0x00001f98   0x00000050   Dbug   RW   695     .debug_frame        usbdl_usb_drv.obj(bootloader.lib)
    0x00001fe8   0x00000058   Dbug   RW   696     .debug_frame        usbdl_usb_drv.obj(bootloader.lib)
    0x00002040   0x00000054   Dbug   RW   697     .debug_frame        usbdl_usb_drv.obj(bootloader.lib)
    0x00002094   0x0000004c   Dbug   RW   698     .debug_frame        usbdl_usb_drv.obj(bootloader.lib)
    0x000020e0   0x0000003c   Dbug   RW   699     .debug_frame        usbdl_usb_drv.obj(bootloader.lib)
    0x0000211c   0x00000050   Dbug   RW   700     .debug_frame        usbdl_usb_drv.obj(bootloader.lib)
    0x0000216c   0x00000050   Dbug   RW   701     .debug_frame        usbdl_usb_drv.obj(bootloader.lib)
    0x000021bc   0x0000004c   Dbug   RW   702     .debug_frame        usbdl_usb_drv.obj(bootloader.lib)
    0x00002208   0x0000003c   Dbug   RW   706     .debug_frame        usbdl_usb_drv.obj(bootloader.lib)
    0x00002244   0x0000003c   Dbug   RW   710     .debug_frame        usbdl_usb_drv.obj(bootloader.lib)
    0x00002280   0x0000005c   Dbug   RW   711     .debug_frame        usbdl_usb_drv.obj(bootloader.lib)
    0x000022dc   0x0000004c   Dbug   RW   712     .debug_frame        usbdl_usb_drv.obj(bootloader.lib)
    0x00002328   0x0000005c   Dbug   RW   727     .debug_frame        usbdl_usb_resource.obj(bootloader.lib)
    0x00002384   0x0000005c   Dbug   RW   728     .debug_frame        usbdl_usb_resource.obj(bootloader.lib)
    0x000023e0   0x0000003c   Dbug   RW   729     .debug_frame        usbdl_usb_resource.obj(bootloader.lib)
    0x0000241c   0x0000003c   Dbug   RW   730     .debug_frame        usbdl_usb_resource.obj(bootloader.lib)
    0x00002458   0x00000054   Dbug   RW   731     .debug_frame        usbdl_usb_resource.obj(bootloader.lib)
    0x000024ac   0x00000054   Dbug   RW   732     .debug_frame        usbdl_usb_resource.obj(bootloader.lib)
    0x00002500   0x00000054   Dbug   RW   733     .debug_frame        usbdl_usb_resource.obj(bootloader.lib)
    0x00002554   0x00000054   Dbug   RW   734     .debug_frame        usbdl_usb_resource.obj(bootloader.lib)
    0x000025a8   0x00000054   Dbug   RW   735     .debug_frame        usbdl_usb_resource.obj(bootloader.lib)
    0x000025fc   0x0000005c   Dbug   RW   736     .debug_frame        usbdl_usb_resource.obj(bootloader.lib)
    0x00002658   0x0000005c   Dbug   RW   737     .debug_frame        usbdl_usb_resource.obj(bootloader.lib)
    0x000026b4   0x0000005c   Dbug   RW   738     .debug_frame        usbdl_usb_resource.obj(bootloader.lib)
    0x00002710   0x0000005c   Dbug   RW   761     .debug_frame        usbdl_usbacm_adap.obj(bootloader.lib)
    0x0000276c   0x00000050   Dbug   RW   762     .debug_frame        usbdl_usbacm_adap.obj(bootloader.lib)
    0x000027bc   0x0000003c   Dbug   RW   763     .debug_frame        usbdl_usbacm_adap.obj(bootloader.lib)
    0x000027f8   0x0000004c   Dbug   RW   764     .debug_frame        usbdl_usbacm_adap.obj(bootloader.lib)
    0x00002844   0x00000050   Dbug   RW   765     .debug_frame        usbdl_usbacm_adap.obj(bootloader.lib)
    0x00002894   0x00000054   Dbug   RW   766     .debug_frame        usbdl_usbacm_adap.obj(bootloader.lib)
    0x000028e8   0x0000004c   Dbug   RW   767     .debug_frame        usbdl_usbacm_adap.obj(bootloader.lib)
    0x00002934   0x00000054   Dbug   RW   769     .debug_frame        usbdl_usbacm_adap.obj(bootloader.lib)
    0x00002988   0x0000004c   Dbug   RW   770     .debug_frame        usbdl_usbacm_adap.obj(bootloader.lib)
    0x000029d4   0x00000054   Dbug   RW   771     .debug_frame        usbdl_usbacm_adap.obj(bootloader.lib)
    0x00002a28   0x0000004c   Dbug   RW   772     .debug_frame        usbdl_usbacm_adap.obj(bootloader.lib)
    0x00002a74   0x00000058   Dbug   RW   773     .debug_frame        usbdl_usbacm_adap.obj(bootloader.lib)
    0x00002acc   0x0000004c   Dbug   RW   774     .debug_frame        usbdl_usbacm_adap.obj(bootloader.lib)
    0x00002b18   0x00000054   Dbug   RW   775     .debug_frame        usbdl_usbacm_adap.obj(bootloader.lib)
    0x00002b6c   0x0000003c   Dbug   RW   776     .debug_frame        usbdl_usbacm_adap.obj(bootloader.lib)
    0x00002ba8   0x0000003c   Dbug   RW   795     .debug_frame        usbdl_usbacm_drv.obj(bootloader.lib)
    0x00002be4   0x00000054   Dbug   RW   797     .debug_frame        usbdl_usbacm_drv.obj(bootloader.lib)
    0x00002c38   0x0000003c   Dbug   RW   798     .debug_frame        usbdl_usbacm_drv.obj(bootloader.lib)
    0x00002c74   0x0000003c   Dbug   RW   799     .debug_frame        usbdl_usbacm_drv.obj(bootloader.lib)
    0x00002cb0   0x00000054   Dbug   RW   800     .debug_frame        usbdl_usbacm_drv.obj(bootloader.lib)
    0x00002d04   0x0000004c   Dbug   RW   801     .debug_frame        usbdl_usbacm_drv.obj(bootloader.lib)
    0x00002d50   0x00000050   Dbug   RW   802     .debug_frame        usbdl_usbacm_drv.obj(bootloader.lib)
    0x00002da0   0x0000003c   Dbug   RW   803     .debug_frame        usbdl_usbacm_drv.obj(bootloader.lib)
    0x00002ddc   0x0000003c   Dbug   RW   804     .debug_frame        usbdl_usbacm_drv.obj(bootloader.lib)
    0x00002e18   0x00000050   Dbug   RW   805     .debug_frame        usbdl_usbacm_drv.obj(bootloader.lib)
    0x00002e68   0x0000003c   Dbug   RW   806     .debug_frame        usbdl_usbacm_drv.obj(bootloader.lib)
    0x00002ea4   0x00000050   Dbug   RW   807     .debug_frame        usbdl_usbacm_drv.obj(bootloader.lib)
    0x00002ef4   0x0000003c   Dbug   RW   808     .debug_frame        usbdl_usbacm_drv.obj(bootloader.lib)
    0x00002f30   0x0000003c   Dbug   RW   809     .debug_frame        usbdl_usbacm_drv.obj(bootloader.lib)
    0x00002f6c   0x0000004c   Dbug   RW   810     .debug_frame        usbdl_usbacm_drv.obj(bootloader.lib)
    0x00002fb8   0x00000054   Dbug   RW   948     .debug_frame        SSS_secure_shared.obj(sss.lib)
    0x0000300c   0x0000004c   Dbug   RW  1038     .debug_frame        SSS_secure_shared.obj(sss.lib)
    0x00003058   0x00000050   Dbug   RW  1048     .debug_frame        SSS_secure_shared.obj(sss.lib)
    0x000030a8   0x0000004c   Dbug   RW  1053     .debug_frame        SSS_secure_shared.obj(sss.lib)
    0x000030f4   0x00000050   Dbug   RW  1233     .debug_frame        bl_FactoryConn.obj(sss.lib)
    0x00003144   0x00000050   Dbug   RW  1238     .debug_frame        bl_FactoryConn.obj(sss.lib)
    0x00003194   0x00000050   Dbug   RW  1243     .debug_frame        bl_FactoryConn.obj(sss.lib)
    0x000031e4   0x00000050   Dbug   RW  1248     .debug_frame        bl_FactoryConn.obj(sss.lib)
    0x00003234   0x00000054   Dbug   RW  1253     .debug_frame        bl_FactoryConn.obj(sss.lib)
    0x00003288   0x00000050   Dbug   RW  1258     .debug_frame        bl_FactoryConn.obj(sss.lib)
    0x000032d8   0x00000050   Dbug   RW  1263     .debug_frame        bl_FactoryConn.obj(sss.lib)
    0x00003328   0x00000054   Dbug   RW  1268     .debug_frame        bl_FactoryConn.obj(sss.lib)
    0x0000337c   0x00000050   Dbug   RW  1273     .debug_frame        bl_FactoryConn.obj(sss.lib)
    0x000033cc   0x00000050   Dbug   RW  1278     .debug_frame        bl_FactoryConn.obj(sss.lib)
    0x0000341c   0x00000058   Dbug   RW  1283     .debug_frame        bl_FactoryConn.obj(sss.lib)
    0x00003474   0x00000054   Dbug   RW  1288     .debug_frame        bl_FactoryConn.obj(sss.lib)
    0x000034c8   0x0000005c   Dbug   RW  1293     .debug_frame        bl_FactoryConn.obj(sss.lib)
    0x00003524   0x0000004c   Dbug   RW  1298     .debug_frame        bl_FactoryConn.obj(sss.lib)
    0x00003570   0x00000054   Dbug   RW  1308     .debug_frame        bl_FactoryConn.obj(sss.lib)
    0x000035c4   0x00000088   Dbug   RW  1609     .debug_frame        lib_init.o(c_t__un.l)
    0x0000364c   0x00000044   Dbug   RW  1611     .debug_frame        llcmpge.o(c_t__un.l)
    0x00003690   0x0000003c   Dbug   RW  1613     .debug_frame        llmullu.o(c_t__un.l)
    0x000036cc   0x00000044   Dbug   RW  1615     .debug_frame        llneg.o(c_t__un.l)
    0x00003710   0x00000044   Dbug   RW  1619     .debug_frame        llsubls.o(c_t__un.l)
    0x00003754   0x0000004c   Dbug   RW  1625     .debug_frame        memcpy.o(c_t__un.l)
    0x000037a0   0x0000004c   Dbug   RW  1627     .debug_frame        memset.o(c_t__un.l)
    0x000037ec   0x00000054   Dbug   RW  1629     .debug_frame        rt_memclr_w.o(c_t__un.l)
    0x00003840   0x0000003c   Dbug   RW  1631     .debug_frame        rt_memcpy.o(c_t__un.l)
    0x0000387c   0x00000054   Dbug   RW  1633     .debug_frame        rt_memcpy_w.o(c_t__un.l)
    0x000038d0   0x00000044   Dbug   RW  1635     .debug_frame        rt_sdiv.o(c_t__un.l)
    0x00003914   0x00000044   Dbug   RW  1639     .debug_frame        rtsdiv10.o(c_t__un.l)
    0x00003958   0x0000005c   Dbug   RW  1645     .debug_frame        dfltll_clz.o(f_t_p.l)
    0x000039b4   0x00000060   Dbug   RW  1647     .debug_frame        dgeqf.o(f_t_p.l)
    0x00003a14   0x00000044   Dbug   RW  1650     .debug_frame        libspace.o(c_t__un.l)
    0x00003a58   0x00000054   Dbug   RW  1652     .debug_frame        llmul3m.o(c_t__un.l)
    0x00003aac   0x0000003c   Dbug   RW  1654     .debug_frame        rt_div0.o(c_t__un.l)
    0x00003ae8   0x00000050   Dbug   RW  1656     .debug_frame        rt_fp_status_addr.o(c_t__un.l)
    0x00003b38   0x00000044   Dbug   RW  1658     .debug_frame        rt_memclr.o(c_t__un.l)
    0x00003b7c   0x00000050   Dbug   RW  1660     .debug_frame        fpinit.o(f_t_p.l)
    0x00003bcc   0x00000060   Dbug   RW  1662     .debug_frame        dcmpin.o(f_t_p.l)
    0x00003c2c   0x00000078   Dbug   RW  1664     .debug_frame        except.o(f_t_p.l)
    0x00003ca4   0x00000054   Dbug   RW  1666     .debug_frame        rt_raise.o(c_t__un.l)
    0x00003cf8   0x00000054   Dbug   RW  1668     .debug_frame        dcheck.o(f_t_p.l)
    0x00003d4c   0x0000005c   Dbug   RW  1670     .debug_frame        retnan.o(f_t_p.l)
    0x00003da8   0x00000084   Dbug   RW  1672     .debug_frame        trapv.o(f_t_p.l)
    0x00003e2c   0x00000058   Dbug   RW  1674     .debug_frame        __raise.o(c_t__un.l)
    0x00003e84   0x00000060   Dbug   RW  1676     .debug_frame        _fptrap.o(c_t__un.l)
    0x00003ee4   0x00000044   Dbug   RW  1678     .debug_frame        sys_exit.o(c_t__un.l)
    0x00003f28   0x00000054   Dbug   RW  1682     .debug_frame        defsig.o(c_t__un.l)
    0x00003f7c   0x00000044   Dbug   RW  1685     .debug_frame        use_semi.o(c_t__un.l)
    0x00003fc0   0x00000050   Dbug   RW  1687     .debug_frame        sys_wrch.o(c_t__un.l)
    0x00000000   0x00000060   Dbug   RW    45     .debug_info         bl_BOOTARM.obj(bootloader.lib)
    0x00000060   0x00000064   Dbug   RW   179     .debug_info         bl_regioninit.obj(bootloader.lib)
    0x000000c4   0x000001bc   Dbug   RW  1109     .debug_info         SSS_secure_shared.obj(sss.lib)
    0x00000280   0x000000f4   Dbug   RW   851     .debug_info         SSS_secure_shared.obj(sss.lib)
    0x00000374   0x000002c8   Dbug   RW  1162     .debug_info         SSS_secure_shared.obj(sss.lib)
    0x0000063c   0x000000fc   Dbug   RW   914     .debug_info         SSS_secure_shared.obj(sss.lib)
    0x00000738   0x00000f9c   Dbug   RW  1155     .debug_info         SSS_secure_shared.obj(sss.lib)
    0x000016d4   0x0000011c   Dbug   RW   920     .debug_info         SSS_secure_shared.obj(sss.lib)
    0x000017f0   0x000000f8   Dbug   RW   923     .debug_info         SSS_secure_shared.obj(sss.lib)
    0x000018e8   0x00000154   Dbug   RW   945     .debug_info         SSS_secure_shared.obj(sss.lib)
    0x00001a3c   0x0000014c   Dbug   RW  1035     .debug_info         SSS_secure_shared.obj(sss.lib)
    0x00001b88   0x000000c8   Dbug   RW  1045     .debug_info         SSS_secure_shared.obj(sss.lib)
    0x00001c50   0x000000bc   Dbug   RW  1050     .debug_info         SSS_secure_shared.obj(sss.lib)
    0x00001d0c   0x000000e4   Dbug   RW  1182     .debug_info         bl_FactoryConn.obj(sss.lib)
    0x00001df0   0x000000a4   Dbug   RW  1185     .debug_info         bl_FactoryConn.obj(sss.lib)
    0x00001e94   0x000000e8   Dbug   RW  1188     .debug_info         bl_FactoryConn.obj(sss.lib)
    0x00001f7c   0x000000a4   Dbug   RW  1191     .debug_info         bl_FactoryConn.obj(sss.lib)
    0x00002020   0x0000010c   Dbug   RW  1194     .debug_info         bl_FactoryConn.obj(sss.lib)
    0x0000212c   0x000000e0   Dbug   RW  1197     .debug_info         bl_FactoryConn.obj(sss.lib)
    0x0000220c   0x0000010c   Dbug   RW  1200     .debug_info         bl_FactoryConn.obj(sss.lib)
    0x00002318   0x00000108   Dbug   RW  1203     .debug_info         bl_FactoryConn.obj(sss.lib)
    0x00002420   0x000000e4   Dbug   RW  1206     .debug_info         bl_FactoryConn.obj(sss.lib)
    0x00002504   0x000000f4   Dbug   RW  1209     .debug_info         bl_FactoryConn.obj(sss.lib)
    0x000025f8   0x000000dc   Dbug   RW  1212     .debug_info         bl_FactoryConn.obj(sss.lib)
    0x000026d4   0x0000011c   Dbug   RW  1215     .debug_info         bl_FactoryConn.obj(sss.lib)
    0x000027f0   0x000001f0   Dbug   RW  1218     .debug_info         bl_FactoryConn.obj(sss.lib)
    0x000029e0   0x000000c4   Dbug   RW  1221     .debug_info         bl_FactoryConn.obj(sss.lib)
    0x00002aa4   0x00000174   Dbug   RW  1227     .debug_info         bl_FactoryConn.obj(sss.lib)
    0x00002c18   0x000000dc   Dbug   RW  1230     .debug_info         bl_FactoryConn.obj(sss.lib)
    0x00002cf4   0x000000b8   Dbug   RW  1235     .debug_info         bl_FactoryConn.obj(sss.lib)
    0x00002dac   0x000000dc   Dbug   RW  1240     .debug_info         bl_FactoryConn.obj(sss.lib)
    0x00002e88   0x000000b8   Dbug   RW  1245     .debug_info         bl_FactoryConn.obj(sss.lib)
    0x00002f40   0x000000f4   Dbug   RW  1250     .debug_info         bl_FactoryConn.obj(sss.lib)
    0x00003034   0x000000cc   Dbug   RW  1255     .debug_info         bl_FactoryConn.obj(sss.lib)
    0x00003100   0x000000e8   Dbug   RW  1260     .debug_info         bl_FactoryConn.obj(sss.lib)
    0x000031e8   0x000000e8   Dbug   RW  1265     .debug_info         bl_FactoryConn.obj(sss.lib)
    0x000032d0   0x000000cc   Dbug   RW  1270     .debug_info         bl_FactoryConn.obj(sss.lib)
    0x0000339c   0x000000d8   Dbug   RW  1275     .debug_info         bl_FactoryConn.obj(sss.lib)
    0x00003474   0x000000c4   Dbug   RW  1280     .debug_info         bl_FactoryConn.obj(sss.lib)
    0x00003538   0x000000e0   Dbug   RW  1285     .debug_info         bl_FactoryConn.obj(sss.lib)
    0x00003618   0x000001a8   Dbug   RW  1290     .debug_info         bl_FactoryConn.obj(sss.lib)
    0x000037c0   0x000000e0   Dbug   RW  1295     .debug_info         bl_FactoryConn.obj(sss.lib)
    0x000038a0   0x00000188   Dbug   RW  1305     .debug_info         bl_FactoryConn.obj(sss.lib)
    0x00003a28   0x00000118   Dbug   RW  1362     .debug_info         bl_Secure.obj(sss.lib)
    0x00000000   0x000000b0   Dbug   RW    46     .debug_line         bl_BOOTARM.obj(bootloader.lib)
    0x000000b0   0x000000ac   Dbug   RW   180     .debug_line         bl_regioninit.obj(bootloader.lib)
    0x0000015c   0x00000088   Dbug   RW   944     .debug_line         SSS_secure_shared.obj(sss.lib)
    0x000001e4   0x00000080   Dbug   RW  1034     .debug_line         SSS_secure_shared.obj(sss.lib)
    0x00000264   0x0000006c   Dbug   RW  1044     .debug_line         SSS_secure_shared.obj(sss.lib)
    0x000002d0   0x00000068   Dbug   RW  1049     .debug_line         SSS_secure_shared.obj(sss.lib)
    0x00000338   0x00000078   Dbug   RW  1229     .debug_line         bl_FactoryConn.obj(sss.lib)
    0x000003b0   0x0000006c   Dbug   RW  1234     .debug_line         bl_FactoryConn.obj(sss.lib)
    0x0000041c   0x00000078   Dbug   RW  1239     .debug_line         bl_FactoryConn.obj(sss.lib)
    0x00000494   0x00000068   Dbug   RW  1244     .debug_line         bl_FactoryConn.obj(sss.lib)
    0x000004fc   0x0000007c   Dbug   RW  1249     .debug_line         bl_FactoryConn.obj(sss.lib)
    0x00000578   0x00000078   Dbug   RW  1254     .debug_line         bl_FactoryConn.obj(sss.lib)
    0x000005f0   0x0000007c   Dbug   RW  1259     .debug_line         bl_FactoryConn.obj(sss.lib)
    0x0000066c   0x0000007c   Dbug   RW  1264     .debug_line         bl_FactoryConn.obj(sss.lib)
    0x000006e8   0x00000078   Dbug   RW  1269     .debug_line         bl_FactoryConn.obj(sss.lib)
    0x00000760   0x00000078   Dbug   RW  1274     .debug_line         bl_FactoryConn.obj(sss.lib)
    0x000007d8   0x00000078   Dbug   RW  1279     .debug_line         bl_FactoryConn.obj(sss.lib)
    0x00000850   0x00000070   Dbug   RW  1284     .debug_line         bl_FactoryConn.obj(sss.lib)
    0x000008c0   0x000000b8   Dbug   RW  1289     .debug_line         bl_FactoryConn.obj(sss.lib)
    0x00000978   0x00000068   Dbug   RW  1294     .debug_line         bl_FactoryConn.obj(sss.lib)
    0x000009e0   0x000000c8   Dbug   RW  1304     .debug_line         bl_FactoryConn.obj(sss.lib)
    0x00000000   0x00000060   Dbug   RW   947     .debug_loc          SSS_secure_shared.obj(sss.lib)
    0x00000060   0x000000c4   Dbug   RW  1037     .debug_loc          SSS_secure_shared.obj(sss.lib)
    0x00000124   0x000000ac   Dbug   RW  1047     .debug_loc          SSS_secure_shared.obj(sss.lib)
    0x000001d0   0x00000090   Dbug   RW  1052     .debug_loc          SSS_secure_shared.obj(sss.lib)
    0x00000260   0x0000008c   Dbug   RW  1232     .debug_loc          bl_FactoryConn.obj(sss.lib)
    0x000002ec   0x00000070   Dbug   RW  1237     .debug_loc          bl_FactoryConn.obj(sss.lib)
    0x0000035c   0x0000008c   Dbug   RW  1242     .debug_loc          bl_FactoryConn.obj(sss.lib)
    0x000003e8   0x00000070   Dbug   RW  1247     .debug_loc          bl_FactoryConn.obj(sss.lib)
    0x00000458   0x000000a8   Dbug   RW  1252     .debug_loc          bl_FactoryConn.obj(sss.lib)
    0x00000500   0x00000080   Dbug   RW  1257     .debug_loc          bl_FactoryConn.obj(sss.lib)
    0x00000580   0x000000a8   Dbug   RW  1262     .debug_loc          bl_FactoryConn.obj(sss.lib)
    0x00000628   0x000000a8   Dbug   RW  1267     .debug_loc          bl_FactoryConn.obj(sss.lib)
    0x000006d0   0x00000080   Dbug   RW  1272     .debug_loc          bl_FactoryConn.obj(sss.lib)
    0x00000750   0x000000a8   Dbug   RW  1277     .debug_loc          bl_FactoryConn.obj(sss.lib)
    0x000007f8   0x00000090   Dbug   RW  1282     .debug_loc          bl_FactoryConn.obj(sss.lib)
    0x00000888   0x00000074   Dbug   RW  1287     .debug_loc          bl_FactoryConn.obj(sss.lib)
    0x000008fc   0x000001d4   Dbug   RW  1292     .debug_loc          bl_FactoryConn.obj(sss.lib)
    0x00000ad0   0x00000034   Dbug   RW  1297     .debug_loc          bl_FactoryConn.obj(sss.lib)
    0x00000b04   0x0000008c   Dbug   RW  1307     .debug_loc          bl_FactoryConn.obj(sss.lib)
    0x00000000   0x00000028   Dbug   RW   852     .debug_pubnames     SSS_secure_shared.obj(sss.lib)
    0x00000028   0x0000002c   Dbug   RW   915     .debug_pubnames     SSS_secure_shared.obj(sss.lib)
    0x00000054   0x00000038   Dbug   RW   921     .debug_pubnames     SSS_secure_shared.obj(sss.lib)
    0x0000008c   0x00000034   Dbug   RW   924     .debug_pubnames     SSS_secure_shared.obj(sss.lib)
    0x000000c0   0x00000028   Dbug   RW   946     .debug_pubnames     SSS_secure_shared.obj(sss.lib)
    0x000000e8   0x0000002c   Dbug   RW  1036     .debug_pubnames     SSS_secure_shared.obj(sss.lib)
    0x00000114   0x00000038   Dbug   RW  1046     .debug_pubnames     SSS_secure_shared.obj(sss.lib)
    0x0000014c   0x00000034   Dbug   RW  1051     .debug_pubnames     SSS_secure_shared.obj(sss.lib)
    0x00000180   0x000000e8   Dbug   RW  1110     .debug_pubnames     SSS_secure_shared.obj(sss.lib)
    0x00000268   0x000003d4   Dbug   RW  1156     .debug_pubnames     SSS_secure_shared.obj(sss.lib)
    0x0000063c   0x00000130   Dbug   RW  1163     .debug_pubnames     SSS_secure_shared.obj(sss.lib)
    0x0000076c   0x00000020   Dbug   RW  1183     .debug_pubnames     bl_FactoryConn.obj(sss.lib)
    0x0000078c   0x00000020   Dbug   RW  1186     .debug_pubnames     bl_FactoryConn.obj(sss.lib)
    0x000007ac   0x00000020   Dbug   RW  1189     .debug_pubnames     bl_FactoryConn.obj(sss.lib)
    0x000007cc   0x00000020   Dbug   RW  1192     .debug_pubnames     bl_FactoryConn.obj(sss.lib)
    0x000007ec   0x00000020   Dbug   RW  1195     .debug_pubnames     bl_FactoryConn.obj(sss.lib)
    0x0000080c   0x00000020   Dbug   RW  1198     .debug_pubnames     bl_FactoryConn.obj(sss.lib)
    0x0000082c   0x00000028   Dbug   RW  1201     .debug_pubnames     bl_FactoryConn.obj(sss.lib)
    0x00000854   0x00000024   Dbug   RW  1204     .debug_pubnames     bl_FactoryConn.obj(sss.lib)
    0x00000878   0x00000024   Dbug   RW  1207     .debug_pubnames     bl_FactoryConn.obj(sss.lib)
    0x0000089c   0x00000024   Dbug   RW  1210     .debug_pubnames     bl_FactoryConn.obj(sss.lib)
    0x000008c0   0x00000028   Dbug   RW  1213     .debug_pubnames     bl_FactoryConn.obj(sss.lib)
    0x000008e8   0x00000028   Dbug   RW  1216     .debug_pubnames     bl_FactoryConn.obj(sss.lib)
    0x00000910   0x00000020   Dbug   RW  1219     .debug_pubnames     bl_FactoryConn.obj(sss.lib)
    0x00000930   0x00000028   Dbug   RW  1222     .debug_pubnames     bl_FactoryConn.obj(sss.lib)
    0x00000958   0x0000002c   Dbug   RW  1228     .debug_pubnames     bl_FactoryConn.obj(sss.lib)
    0x00000984   0x00000020   Dbug   RW  1231     .debug_pubnames     bl_FactoryConn.obj(sss.lib)
    0x000009a4   0x00000020   Dbug   RW  1236     .debug_pubnames     bl_FactoryConn.obj(sss.lib)
    0x000009c4   0x00000020   Dbug   RW  1241     .debug_pubnames     bl_FactoryConn.obj(sss.lib)
    0x000009e4   0x00000020   Dbug   RW  1246     .debug_pubnames     bl_FactoryConn.obj(sss.lib)
    0x00000a04   0x00000020   Dbug   RW  1251     .debug_pubnames     bl_FactoryConn.obj(sss.lib)
    0x00000a24   0x00000020   Dbug   RW  1256     .debug_pubnames     bl_FactoryConn.obj(sss.lib)
    0x00000a44   0x00000028   Dbug   RW  1261     .debug_pubnames     bl_FactoryConn.obj(sss.lib)
    0x00000a6c   0x00000024   Dbug   RW  1266     .debug_pubnames     bl_FactoryConn.obj(sss.lib)
    0x00000a90   0x00000024   Dbug   RW  1271     .debug_pubnames     bl_FactoryConn.obj(sss.lib)
    0x00000ab4   0x00000024   Dbug   RW  1276     .debug_pubnames     bl_FactoryConn.obj(sss.lib)
    0x00000ad8   0x00000028   Dbug   RW  1281     .debug_pubnames     bl_FactoryConn.obj(sss.lib)
    0x00000b00   0x00000028   Dbug   RW  1286     .debug_pubnames     bl_FactoryConn.obj(sss.lib)
    0x00000b28   0x00000020   Dbug   RW  1291     .debug_pubnames     bl_FactoryConn.obj(sss.lib)
    0x00000b48   0x00000028   Dbug   RW  1296     .debug_pubnames     bl_FactoryConn.obj(sss.lib)
    0x00000b70   0x0000002c   Dbug   RW  1306     .debug_pubnames     bl_FactoryConn.obj(sss.lib)
    0x00000b9c   0x00000090   Dbug   RW  1363     .debug_pubnames     bl_Secure.obj(sss.lib)


================================================================================

Image component sizes


      Code    RO Data    RW Data    ZI Data      Debug   Object Name

       288          0          0          0          0   anon$$obj.o

    ------------------------------------------------------------------------
       288          0          0          0          0   Object Totals

    ------------------------------------------------------------------------

      Code    RO Data    RW Data    ZI Data      Debug   Library Member Name

        32          0          0          0         84   llmul3m.o
       540          8          0        554        260   bl_DBGPRINT.obj
       992        268          2         16       1040   bl_Main.obj
      1160         60          0          0      14012   bl_FactoryConn.obj
        28          0          0          0        120   usbdl_pmu.obj
        36          0          0          0         76   memset.o
        72          0          0          0         68   rt_memclr.o
         8          0          0          0        120   bl_Alg.obj
        92          0          0          0         84   rt_memclr_w.o
        68          0          0          0         96   _fptrap.o
        16          0          0          0          0   callvia.o
         8          0          0          0         68   use_semi.o
       312          0         24          0         60   gpio_setting.obj
       764          0          0          0        284   bl_regioninit.obj
       156          0          0          0         92   retnan.o
        16         84          0          0        120   keypad_def.obj
        16          0          0          0         68   llneg.o
        16          0          0          0         68   llcmpge.o
      2224         36          4        104       2408   usbdl_usb_drv.obj
        68          0          0          0         84   dcheck.o
        28          0          0          0         68   sys_exit.o
        68          0          0          0         68   rtsdiv10.o
        16          0          0         96         68   libspace.o
        20          0          0          0         80   sys_wrch.o
      1068         72          1       1048       1176   usbdl_usbacm_adap.obj
        32          0          0          0         84   rt_raise.o
       132          0          0          0         92   dfltll_clz.o
       184          0          0          0         60   rt_memcpy.o
       100          0          0          0        144   l1_interface.obj
       128          0         20          0        180   bl_UART.obj
       172          0          0          0        132   trapv.o
       900          0          0        152       1040   usbdl_usbacm_drv.obj
       280        299          0          0         84   defsig.o
        16          0          0          0         60   rt_div0.o
        12          0          0          0         60   llmullu.o
       112          0          0          0         84   rt_memcpy_w.o
        24          0          0          0         80   rt_fp_status_addr.o
        24          3          0          0        240   custom_blconfig.obj
        20          0          0          0         76   memcpy.o
      1352        236          0        112       1000   usbdl_usb_resource.obj
        16          0          0          0         68   llsubls.o
        12          0          0         64        180   bl_ImageLoader.obj
         0          5          0          0          0   bl_verno.obj
       188          0          4       4096        284   bl_BOOTARM.obj
       340        632          0          0      11544   SSS_secure_shared.obj
       472          0          0          0        364   gpio.obj
        64         60          0          0        256   bl_portingfunc.obj
       360          0          0          0        120   except.o
       600         52          0          0       1116   bl_Init.obj
        68          0          0          0         88   __raise.o
        16          0          0          0        120   usbdl_debug_tool.obj
      1828         32          0        344       1040   usbdl_usb.obj
       448        508          0          4        412   cache.obj
       464        256          4          0        220   custom_emi.obj
       184          0          0          0        136   lib_init.o
         0         22          0          0          0   SSS_interface.obj
         0          0          0          5        424   bl_Secure.obj
         8          0          0          1         76   gpio_drv.obj
        68          0          0          0        148   bl_Cache.obj
       132          0          0          0         96   dgeqf.o
       108          0          0          0         96   dcmpin.o
        28          0          0          0         80   fpinit.o
         0          1          0          0          0   gpio_var.obj
       216          0          0          0         68   rt_sdiv.o
        48        516          0          0        376   usb_custom.obj

    ------------------------------------------------------------------------
     16980       3150         59       6596      41400   Library Totals

    ------------------------------------------------------------------------

      Code    RO Data    RW Data    ZI Data      Debug   Library Name

      1156          0          0          0        792   f_t_p.l
      1500        692          0          5      25980   sss.lib
      1652        299          0         96       1844   c_t__un.l
     12672       2159         59       6495      12784   bootloader.lib

    ------------------------------------------------------------------------
     16980       3150         59       6596      41400   Library Totals

    ------------------------------------------------------------------------

================================================================================


      Code    RO Data    RW Data    ZI Data      Debug   

     17268       3150         59       6596      41400   Grand Totals

================================================================================

    Total RO  Size(Code + RO Data)                20418 (  19.94kB)
    Total RW  Size(RW Data + ZI Data)              6655 (   6.50kB)
    Total ROM Size(Code + RO Data + RW Data)      20477 (  20.00kB)

================================================================================

